 SDKRIL

 Timestamp is 54004908 (Fri Aug 29 17:34:00 2014)

 Preferred load address is 10000000

 Start         Length     Name                   Class
 0001:00000000 0002413cH .text                   CODE
 0001:0002413c 000000a4H .text$yc                CODE
 0001:000241e0 000000ccH .text$yd                CODE
 0002:00000000 0000d1f4H .rdata                  DATA
 0002:0000d1f4 00000075H .rdata$debug            DATA
 0002:0000d26c 0000016cH .rdata$r                DATA
 0002:0000d3d8 00000090H .xdata                  DATA
 0002:0000d468 000000e8H .xdata$x                DATA
 0002:0000d550 0000003cH .idata$2                DATA
 0002:0000d58c 00000014H .idata$3                DATA
 0002:0000d5a0 00000168H .idata$4                DATA
 0002:0000d708 0000014cH .idata$6                DATA
 0002:0000d860 000059bdH .edata                  DATA
 0003:00000000 00000168H .idata$5                DATA
 0003:00000168 00000004H .CRT$XCA                DATA
 0003:0000016c 00000004H .CRT$XCAA               DATA
 0003:00000170 00000010H .CRT$XCU                DATA
 0003:00000180 00000004H .CRT$XCZ                DATA
 0003:00000184 00000004H .CRT$XIA                DATA
 0003:00000188 00000004H .CRT$XIZ                DATA
 0003:0000018c 00000004H .CRT$XPA                DATA
 0003:00000190 00000004H .CRT$XPZ                DATA
 0003:00000194 00000004H .CRT$XTA                DATA
 0003:00000198 00000004H .CRT$XTZ                DATA
 0003:000001a0 00000974H .data                   DATA
 0003:00000b18 00006428H .bss                    DATA
 0004:00000000 00001410H .pdata                  DATA
 0005:00000000 00000058H .rsrc$01                DATA
 0005:00000060 000003a0H .rsrc$02                DATA

  Address         Publics by Value              Rva+Base       Lib:Object

 0000:00000000       ___safe_se_handler_count   00000000     <absolute>
 0000:00000000       ___safe_se_handler_table   00000000     <absolute>
 0001:00000000       ?Parse@BerTlv@@QAAHPBEI@Z  10001000 f   parse.obj
 0001:000000a0       ?MatchStringBeginning@@YAHQBD0AAPBD@Z 100010a0 f   parse.obj
 0001:000000f0       ?ParseUInt@@YAHQBDHAAIAAPBD@Z 100010f0 f   parse.obj
 0001:00000190       ?ParseString@@YAHQBDQADIAAPBD@Z 10001190 f   parse.obj
 0001:0000021c       ?ParseUnlimitedString@@YAHQBDAAPADAAIAAPBD@Z 1000121c f   parse.obj
 0001:000002d8       ??_ECriticalSection@@UAAPAXI@Z 100012d8 f i  CIL library: CIL module
 0001:000002d8       ??_GCriticalSection@@UAAPAXI@Z 100012d8 f i SDKRIL.obj
 0001:00000308       ??1SWISYNCBLOCK@@QAA@XZ    10001308 f i SDKRIL.obj
 0001:00000314       ?DeviceRemoval@@YAXK@Z     10001314 f   SDKRIL.obj
 0001:000003b8       DllMain                    100013b8 f   SDKRIL.obj
 0001:000003d4       SwiApiStartup              100013d4 f   SDKRIL.obj
 0001:00000400       SwiApiShutdown             10001400 f   SDKRIL.obj
 0001:000004b4       ?SwiGetAudioMode@@YA?AW4SWI_RCODE@@PAGK@Z 100014b4 f   SDKRIL.obj
 0001:000004b4       ?SwiSetAudioMode@@YA?AW4SWI_RCODE@@GK@Z 100014b4 f   SDKRIL.obj
 0001:000004c4       SwiGetAvailAirServers      100014c4 f   SDKRIL.obj
 0001:000006d0       SwiSelectAirServer         100016d0 f   SDKRIL.obj
 0001:00000c68       SwiGetAirServerInfo        10001c68 f   SDKRIL.obj
 0001:00000ee4       SwiSetNetworkPreferenceGobi 10001ee4 f   SDKRIL.obj
 0001:00000f60       SwiRegisterCallback        10001f60 f   SDKRIL.obj
 0001:00001018       SwiDeRegisterCallback      10002018 f   SDKRIL.obj
 0001:0000105c       SwiNotify                  1000205c f   SDKRIL.obj
 0001:00001094       SwiStopNotify              10002094 f   SDKRIL.obj
 0001:000010cc       SwiGetHardwareVersion      100020cc f   SDKRIL.obj
 0001:0000132c       SwiGetFirmwareVersion      1000232c f   SDKRIL.obj
 0001:000013bc       SwiGetBootVersion          100023bc f   SDKRIL.obj
 0001:0000144c       SwiGetRadioPower           1000244c f   SDKRIL.obj
 0001:000014bc       SwiSetRadioPower           100024bc f   SDKRIL.obj
 0001:000014f8       SwiGetPriInfo              100024f8 f   SDKRIL.obj
 0001:00001578       SwiGetPriVersion           10002578 f   SDKRIL.obj
 0001:000015f4       SwiStartDataSession        100025f4 f   SDKRIL.obj
 0001:000016d8       SwiStopDataSession         100026d8 f   SDKRIL.obj
 0001:000017a8       SwiGetIPConfigurationGobi  100027a8 f   SDKRIL.obj
 0001:000018e4       SwiGetServingNetworkGobi   100028e4 f   SDKRIL.obj
 0001:00001a7c       SwiGetImagePreference      10002a7c f   SDKRIL.obj
 0001:00001abc       SwiSetImagePreference      10002abc f   SDKRIL.obj
 0001:00001b1c       SwiUpgradeFirmware         10002b1c f   SDKRIL.obj
 0001:00001b5c       SwiDialCall                10002b5c f   SDKRIL.obj
 0001:00001bb4       SwiGetModelID              10002bb4 f   SDKRIL.obj
 0001:00001bf4       SwiEndCall                 10002bf4 f   SDKRIL.obj
 0001:00001c34       SwiAnserCall               10002c34 f   SDKRIL.obj
 0001:00001c74       SwiManageCalls             10002c74 f   SDKRIL.obj
 0001:00001cb4       SwiATSetCLIP               10002cb4 f   SDKRIL.obj
 0001:00001e98       SwiATGetCLIP               10002e98 f   SDKRIL.obj
 0001:000023a4       SwiATSetCLIR               100033a4 f   SDKRIL.obj
 0001:00002588       SwiATGetCLIR               10003588 f   SDKRIL.obj
 0001:00002920       SwiATSetCOLP               10003920 f   SDKRIL.obj
 0001:000029b4       SwiATReleaseCall           100039b4 f   SDKRIL.obj
 0001:00002b04       SwiATGetCOLP               10003b04 f   SDKRIL.obj
 0001:00002f0c       SwiATSetCOLR               10003f0c f   SDKRIL.obj
 0001:00002fa0       SwiATGetCOLR               10003fa0 f   SDKRIL.obj
 0001:00003320       SwiATSetEnum               10004320 f   SDKRIL.obj
 0001:000036b0       SwiATSetSideToneGain       100046b0 f   SDKRIL.obj
 0001:000039a8       SwiATReset                 100049a8 f   SDKRIL.obj
 0001:00003c14       SwiATRtnReset              10004c14 f   SDKRIL.obj
 0001:00003ec0       SwiATGetProvisionStatus    10004ec0 f   SDKRIL.obj
 0001:000041f0       SwiHandleSuspend           100051f0 f   SDKRIL.obj
 0001:00004270       ?HandlingResume@@YAXPAX@Z  10005270 f   SDKRIL.obj
 0001:0000427c       SwiHandleResume            1000527c f   SDKRIL.obj
 0001:00004320       ?IsInitialized@CSwiGobiDll@@QAA_NXZ 10005320 f i SDKRIL.obj
 0001:00004328       ?SendSMSNotify@@YAXPAX@Z   10005328 f   SDKRILCdma.obj
 0001:000044d8       SwiGetCDMANetworkParameters 100054d8 f   SDKRILCdma.obj
 0001:0000456c       SwiIsModemReady            1000556c f   SDKRILCdma.obj
 0001:00004638       SwiGetESN                  10005638 f   SDKRILCdma.obj
 0001:00004648       SwiGetESNGobi              10005648 f   SDKRILCdma.obj
 0001:00004760       SwiGetRssi                 10005760 f   SDKRILCdma.obj
 0001:00004848       SwiGetChannelNumber        10005848 f   SDKRILCdma.obj
 0001:0000492c       SwiGetMEIDESN              1000592c f   SDKRILCdma.obj
 0001:00004b10       SwiGetServiceIndication    10005b10 f   SDKRILCdma.obj
 0001:00004c74       SwiGetRoamingStatus        10005c74 f   SDKRILCdma.obj
 0001:00004dd8       SwiGetByteCounter          10005dd8 f   SDKRILCdma.obj
 0001:00004efc       SwiGetActivationStatus     10005efc f   SDKRILCdma.obj
 0001:00004f80       SwiSetCallOriginateCmd     10005f80 f   SDKRILCdma.obj
 0001:000050c0       SwiGetCallConnectionState  100060c0 f   SDKRILCdma.obj
 0001:000051a4       SwiSetCallDisconnectCmd    100061a4 f   SDKRILCdma.obj
 0001:0000523c       SwiGetCdmaSMSMessageStatus 1000623c f   SDKRILCdma.obj
 0001:000052e0       SwiRetrieveCdmaSMSMessage  100062e0 f   SDKRILCdma.obj
 0001:0000574c       SwiStoreCdmaSMSMessage     1000674c f   SDKRILCdma.obj
 0001:00005988       SwiSendCdmaSMS             10006988 f   SDKRILCdma.obj
 0001:00005b84       SwiGetEFileInfo            10006b84 f   SDKRILCdma.obj
 0001:00005d20       SwiGetEFile                10006d20 f   SDKRILCdma.obj
 0001:00005e70       SwiGetPhoneNumber          10006e70 f   SDKRILCdma.obj
 0001:00005f40       SwiGetPRLVersion           10006f40 f   SDKRILCdma.obj
 0001:00005fdc       SwiModemReset              10006fdc f   SDKRIL.obj
 0001:00005fdc       SwiResetModem              10006fdc f   SDKRILCdma.obj
 0001:00006010       SwiSetMobileDirNum         10007010 f   SDKRILCdma.obj
 0001:00006184       SwiSetIMSI                 10007184 f   SDKRILCdma.obj
 0001:000063a4       SwiGetCdmaIMSI             100073a4 f   SDKRILCdma.obj
 0001:00006580       SwiGetCurrentBaseStation   10007580 f   SDKRILCdma.obj
 0001:00006658       SwiGetTechPowersaveMode    10007658 f   SDKRILCdma.obj
 0001:00006658       SwiGetActiveNam            10007658 f   SDKRILCdma.obj
 0001:00006658       SwiGetECIO                 10007658 f   SDKRILCdma.obj
 0001:0000669c       SwiSetPowerDown            1000769c f   SDKRILCdma.obj
 0001:000066ec       SwiGetTechSID              100076ec f   SDKRILCdma.obj
 0001:00006780       SwiGetTechNID              10007780 f   SDKRILCdma.obj
 0001:0000680c       SwiGetTechBandClass        1000780c f   SDKRILCdma.obj
 0001:00006930       SwiGetCarrierID            10007930 f   SDKRILCdma.obj
 0001:00006cd0       SwiGetSystemTime           10007cd0 f   SDKRILCdma.obj
 0001:00006d34       SwiPstUnlock               10007d34 f   SDKRILCdma.obj
 0001:00006e2c       SwiPstLock                 10007e2c f   SDKRILCdma.obj
 0001:000070b0       SwiPstGetSci               100080b0 f   SDKRILCdma.obj
 0001:00007134       SwiPstSetSci               10008134 f   SDKRILCdma.obj
 0001:000071b4       SwiPstGetPrefMode          100081b4 f   SDKRILCdma.obj
 0001:000072d4       SwiPstSetPrefMode          100082d4 f   SDKRILCdma.obj
 0001:00007364       SwiPstGetTermHome          10008364 f   SDKRILCdma.obj
 0001:000073e4       SwiPstGetTermSid           100083e4 f   SDKRILCdma.obj
 0001:00007468       SwiPstGetTermNid           10008468 f   SDKRILCdma.obj
 0001:000074ec       SwiPstGetAccolc            100084ec f   SDKRILCdma.obj
 0001:00007588       SwiPstSetAccolc            10008588 f   SDKRILCdma.obj
 0001:0000764c       SwiPstSetCurrentNam        1000864c f   SDKRILCdma.obj
 0001:000076dc       SwiPstGetImsiMcc           100086dc f   SDKRILCdma.obj
 0001:000077e8       SwiPstSetImsiMcc           100087e8 f   SDKRILCdma.obj
 0001:00007870       SwiPstGetImsi1112          10008870 f   SDKRILCdma.obj
 0001:0000797c       SwiPstSetImsi1112          1000897c f   SDKRILCdma.obj
 0001:000079fc       SwiPstGetSystemPref        100089fc f   SDKRILCdma.obj
 0001:00007b88       SwiPstGetHomeSidNid        10008b88 f   SDKRILCdma.obj
 0001:00007cc8       SwiPstSetHomeSidNid        10008cc8 f   SDKRILCdma.obj
 0001:00007d9c       SwiGetTechHardwareVersion  10008d9c f   SDKRILCdma.obj
 0001:00007da0       SwiPriGetActivationMask    10008da0 f   SDKRILCdma.obj
 0001:00007de8       SwiPriGetMDNLength         10008de8 f   SDKRILCdma.obj
 0001:00007e30       SwiPriGetMaxMosmsLen       10008e30 f   SDKRILCdma.obj
 0001:00007e74       SwiPstSetDsQcMip           10008e74 f   SDKRILCdma.obj
 0001:00007ec8       SwiPstGetDsQcMip           10008ec8 f   SDKRILCdma.obj
 0001:00007f1c       SwiPstSetDsMipActiveProf   10008f1c f   SDKRILCdma.obj
 0001:00007fc0       SwiPstGetDsMipActiveProf   10008fc0 f   SDKRILCdma.obj
 0001:0000805c       SwiPstSetDsMipGenUser      1000905c f   SDKRILCdma.obj
 0001:000081b0       SwiPstGetDsMipGenUser      100091b0 f   SDKRILCdma.obj
 0001:00008408       SwiPstSetDsMipSsUserProf   10009408 f   SDKRILCdma.obj
 0001:00008564       SwiPstGetDsMipSsUserProf   10009564 f   SDKRILCdma.obj
 0001:00008600       SwiPstGetDsMipEnableProf   10009600 f   SDKRILCdma.obj
 0001:00008780       SwiGetMipErrCode           10009780 f   SDKRILCdma.obj
 0001:00008838       SwiSetAKey                 10009838 f   SDKRILCdma.obj
 0001:00008838       SwiResetByteCounter        10009838 f   SDKRILCdma.obj
 0001:00008870       SwiSetDormant              10009870 f   SDKRILCdma.obj
 0001:000088b0       SwiGetRssiEcio             100098b0 f   SDKRILCdma.obj
 0001:000089b8       SwiGetHdrRoamStatus        100099b8 f   SDKRILCdma.obj
 0001:00008b1c       SwiGetHdrSrvState          10009b1c f   SDKRILCdma.obj
 0001:00008c78       SwiGetHdrHybrPref          10009c78 f   SDKRILCdma.obj
 0001:00008cbc       SwiSetHdrHybrPref          10009cbc f   SDKRILCdma.obj
 0001:00008d44       SwiSetTempModePref         10009d44 f   SDKRILCdma.obj
 0001:00008fa8       SwiPstGetHdrUserId         10009fa8 f   SDKRILCdma.obj
 0001:0000903c       SwiPstSetHdrUserId         1000a03c f   SDKRILCdma.obj
 0001:000090e0       SwiPstGetHdrPassword       1000a0e0 f   SDKRILCdma.obj
 0001:00009174       SwiPstSetHdrPassword       1000a174 f   SDKRILCdma.obj
 0001:00009218       SwiPowerSaveExit           1000a218 f   SDKRILCdma.obj
 0001:0000925c       SwiSetPower                1000a25c f   SDKRILCdma.obj
 0001:000092e0       SwiGetPower                1000a2e0 f   SDKRILCdma.obj
 0001:00009368       SwiRtnReset                1000a368 f   SDKRILCdma.obj
 0001:00009410       SwiGetNDISMode             1000a410 f   SDKRILCdma.obj
 0001:00009424       SwiSetNDISPrefMode         1000a424 f   SDKRILCdma.obj
 0001:00009468       SwiGetIOTADisable          1000a468 f   SDKRILCdma.obj
 0001:000094ac       SwiGetOMADMConfig          1000a4ac f   SDKRILCdma.obj
 0001:00009570       SwiSetOMADMConfig          1000a570 f   SDKRILCdma.obj
 0001:00009700       SwiStartOMADMSession       1000a700 f   SDKRILCdma.obj
 0001:000097d8       SwiCancelOMADMSession      1000a7d8 f   SDKRILCdma.obj
 0001:0000989c       SwiGetOMADMSessionState    1000a89c f   SDKRILCdma.obj
 0001:00009a30       SwiGetOMADMNIAlert         1000aa30 f   SDKRILCdma.obj
 0001:00009bd8       SwiSetOMADMNIAlertResponse 1000abd8 f   SDKRILCdma.obj
 0001:00009db0       SwiGetGeneralFeatureSupport 1000adb0 f   SDKRILCdma.obj
 0001:00009df4       SwiActivateAutomatic       1000adf4 f   SDKRILCdma.obj
 0001:00009eb0       SwiSetMobileIPProfile      1000aeb0 f   SDKRILCdma.obj
 0001:00009fcc       SwiGetMobileIPProfile      1000afcc f   SDKRILCdma.obj
 0001:0000a0f4       SwiPstGetDisplayBannerName 1000b0f4 f   SDKRILCdma.obj
 0001:0000a540       SwiSetOMAEXEventReport     1000b540 f   SDKRILCdma.obj
 0001:0000a59c       SwiOMAEXSessionStart       1000b59c f   SDKRILCdma.obj
 0001:0000a5fc       SwiOMAEXSessionCancel      1000b5fc f   SDKRILCdma.obj
 0001:0000a658       SwiOMAEXSelection          1000b658 f   SDKRILCdma.obj
 0001:0000a6b8       SwiOMAEXGetSettings        1000b6b8 f   SDKRILCdma.obj
 0001:0000a740       SwiOMAEXSetSettings        1000b740 f   SDKRILCdma.obj
 0001:0000a7c8       SwiOMAEXGetSessionInfo     1000b7c8 f   SDKRILCdma.obj
 0001:0000a828       SwiOMAEXInit               1000b828 f   SDKRILCdma.obj
 0001:0000a884       SwiOMAEXShutdown           1000b884 f   SDKRILCdma.obj
 0001:0000a8e8       SwiGetNetworkProviderID    1000b8e8 f   SDKRILGsm.obj
 0001:0000aa70       SwiGetGsmIMSI              1000ba70 f   SDKRILGsm.obj
 0001:0000abd0       SwiGetImei                 1000bbd0 f   SDKRILGsm.obj
 0001:0000acac       SwiGetPLMNMode             1000bcac f   SDKRILGsm.obj
 0001:0000acf4       SwiSetPLMNMode             1000bcf4 f   SDKRILGsm.obj
 0001:0000b1e0       ?GobiPerformNetworkScan@@YAXPAX@Z 1000c1e0 f   SDKRILGsm.obj
 0001:0000b544       SwiStartPLMNSearch         1000c544 f   SDKRILGsm.obj
 0001:0000b600       SwiGetPLMNSelection        1000c600 f   SDKRILGsm.obj
 0001:0000b7cc       ParseGetUsimRecordStatus   1000c7cc f   SDKRILGsm.obj
 0001:0000bc94       SwiSendRestrictedSIMCmd    1000cc94 f   SDKRILGsm.obj
 0001:0000c284       SwiGetSIMRecordStatus      1000d284 f   SDKRILGsm.obj
 0001:0000c70c       SwiSendGenericSimCommand   1000d70c f   SDKRILGsm.obj
 0001:0000cd78       SwiGetGsmProfileBasic      1000dd78 f   SDKRILGsm.obj
 0001:0000cfc8       SwiSetGsmProfileBasic      1000dfc8 f   SDKRILGsm.obj
 0001:0000d38c       SwiGetGsmProfileSummary    1000e38c f   SDKRILGsm.obj
 0001:0000d3c4       SwiActivateProfile         1000e3c4 f   SDKRILGsm.obj
 0001:0000d56c       SwiGetPhonebookEntry       1000e56c f   SDKRILGsm.obj
 0001:0000d780       SwiGetPktSessionStatusEx   1000e780 f   SDKRILGsm.obj
 0001:0000d800       SwiGetIPAddress            1000e800 f   SDKRILGsm.obj
 0001:0000d914       SwiGetPinStatus            1000e914 f   SDKRILGsm.obj
 0001:0000da38       SwiGetSimLockGobi          1000ea38 f   SDKRILGsm.obj
 0001:0000db20       SwiGetProfileSummary       1000eb20 f   SDKRILGsm.obj
 0001:0000db20       SwiGetSimLock              1000eb20 f   SDKRILGsm.obj
 0001:0000db20       SwiGetProfile              1000eb20 f   SDKRILGsm.obj
 0001:0000db20       SwiGetPktSessionStatus     1000eb20 f   SDKRILGsm.obj
 0001:0000db20       SwiSetSimLock              1000eb20 f   SDKRILGsm.obj
 0001:0000db20       SwiSetSimPassword          1000eb20 f   SDKRILGsm.obj
 0001:0000db20       SwiSetProfile              1000eb20 f   SDKRILGsm.obj
 0001:0000db54       SwiSetSimLockGobi          1000eb54 f   SDKRILGsm.obj
 0001:0000dc40       SwiSetSimPasswordGobi      1000ec40 f   SDKRILGsm.obj
 0001:0000deb8       SwiGetSimVerifyGobi        1000eeb8 f   SDKRILGsm.obj
 0001:0000e008       SwiSetSimVerifyGobi        1000f008 f   SDKRILGsm.obj
 0001:0000e194       SwiGetTrafficStatistics    1000f194 f   SDKRILGsm.obj
 0001:0000e260       SwiGetSMSMessageStatus     1000f260 f   SDKRILGsm.obj
 0001:0000e474       SwiRetrieveSMSMessageGobi  1000f474 f   SDKRILGsm.obj
 0001:0000e8ac       SwiRetrieveCBSMSMessageGobi 1000f8ac f   SDKRILGsm.obj
 0001:0000ea34       SwiStoreSMSMessageGobi     1000fa34 f   SDKRILGsm.obj
 0001:0000eba4       SwiSendSMS                 1000fba4 f   SDKRILGsm.obj
 0001:0000ee78       SwiGetGsmSMSCAddr          1000fe78 f   SDKRILGsm.obj
 0001:0000f00c       SwiSetGsmSMSCAddr          1001000c f   SDKRILGsm.obj
 0001:0000f110       SwiGetPreferredOperatorListGobi 10010110 f   SDKRILGsm.obj
 0001:0000f934       SwiRemovePreferredOperatorGobi 10010934 f   SDKRILGsm.obj
 0001:0000fb28       SwiAddPreferredOperatorGobi 10010b28 f   SDKRILGsm.obj
 0001:0001004c       SwiSetHostStartup          1001104c f   SDKRILGsm.obj
 0001:00010164       ?SwiGetGsmSystemStatusWithPSAttachedState@@YA?AW4SWI_RCODE@@PAUSWI_STRUCT_GsmSystemStatus@@PAH@Z 10011164 f   SDKRILGsm.obj
 0001:000107c8       SwiGetGsmSystemStatus      100117c8 f   SDKRILGsm.obj
 0001:00010820       ?EncodeDestAddrHdr@@YA?AW4SWI_RCODE@@PAEPADEPAKE@Z 10011820 f   sms.obj
 0001:0001096c       ?EncodeCallbackNumber@@YA?AW4SWI_RCODE@@PAEPADEPAKE@Z 1001196c f   sms.obj
 0001:00010ab8       ?EncodeUserDataHdr@@YA?AW4SWI_RCODE@@PAEW4SWI_TYPE_SMS_DataEncodeType@@PADEPAK@Z 10011ab8 f   sms.obj
 0001:00010c50       ?EncodeMsgIdenfier@@YA?AW4SWI_RCODE@@PAEEGPAK@Z 10011c50 f   sms.obj
 0001:00010d1c       ?SplitParamMTSms@@YA?AW4SWI_RCODE@@PAEKPAGPAPAE020@Z 10011d1c f   sms.obj
 0001:00011024       ?DecodeBearerData@@YA?AW4SWI_RCODE@@PAEEPAG000000PAPAE002020@Z 10012024 f   sms.obj
 0001:00011594       ?DecodeOriginAddr@@YA?AW4SWI_RCODE@@PAE00PAG0@Z 10012594 f   sms.obj
 0001:000116f4       ?DecodeCallbackAddr@@YA?AW4SWI_RCODE@@PAE0PAG0@Z 100126f4 f   sms.obj
 0001:00011898       ?DecodeUserData@@YA?AW4SWI_RCODE@@PAEE00PAPAE@Z 10012898 f   sms.obj
 0001:00011b2c       ?DecodeCompleteMTSms@@YA?AW4SWI_RCODE@@PAEKPAUSWI_STRUCT_CDMA_SMS_RetrieveSms@@@Z 10012b2c f   sms.obj
 0001:000120d8       ?EncodeCompleteMoSms@@YA?AW4SWI_RCODE@@PAPAEPAKPADE2EW4SWI_TYPE_SMS_DataEncodeType@@2EEGE@Z 100130d8 f   sms.obj
 0001:000127d0       ?EncodeMOPDU@@YA?AW4SWI_RCODE@@PAUSWI_STRUCT_GSM_SMS_StoreSmsGobi@@PAEPAG@Z 100137d0 f   sms.obj
 0001:00012cf4       ?DecodeTypeofAddr@@YA?AW4SWI_RCODE@@PAW4SWI_TYPE_SMS_Address@@PAW4SWI_TYPE_SMS_AddressNumbering@@E@Z 10013cf4 f   sms.obj
 0001:00012dac       ?DecodeCompletePDU@@YA?AW4SWI_RCODE@@PAEKPAUSWI_STRUCT_GSM_SMS_RetrieveSmsGobi@@@Z 10013dac f   sms.obj
 0001:000132d8       ?PackByteToBits@@YAXEQAEGG@Z 100142d8 f   sms.obj
 0001:000133b8       ?UnpackBitsToAByte@@YAEPAEHH@Z 100143b8 f   sms.obj
 0001:0001347c       ??4CSwiGobiDll@@QAAAAV0@ABV0@@Z 1001447c f i stdafx.obj
 0001:0001349c       ?Initialize@CSwiATPort@@QAA?AW4SWI_RCODE@@PBGJDJJHHHHH@Z 1001449c f   SwiAtPort.obj
 0001:0001383c       ?Shutdown@CSwiATPort@@QAA?AW4SWI_RCODE@@XZ 1001483c f   SwiAtPort.obj
 0001:000138cc       ?WaitForResponseTimeout@CSwiATPort@@AAAHPAD0K@Z 100148cc f   SwiAtPort.obj
 0001:00013b84       ?WaitForResponse@CSwiATPort@@AAAHPAD0@Z 10014b84 f   SwiAtPort.obj
 0001:00013d88       ?ParseNotification@CSwiATPort@@AAAXQBDAAPBDPAH@Z 10014d88 f   SwiAtPort.obj
 0001:00013eb4       ?SendATCommand@CSwiATPort@@QAAHPAD0@Z 10014eb4 f   SwiAtPort.obj
 0001:00014094       ?SendATCommandTimeout@CSwiATPort@@QAAHPAD0K@Z 10015094 f   SwiAtPort.obj
 0001:00014268       ?ConvertGobiError@@YA?AW4SWI_RCODE@@K@Z 10015268 f   SwiError.obj
 0001:00014310       ?ExtractOMADMSessionTypeAndInitiator@@YAXKPAW4SWI_TYPE_OMADM_SESSION_TYPE@@PAW4SWI_TYPE_OMADM_SESSION_INITIATOR@@@Z 10015310 f   SwiError.obj
 0001:000143e4       ?ConvertGobi2OMADMError@@YA?AW4SWI_TYPE_OMADM_SESSION_RESULT@@W4SWI_TYPE_OMADM_SESSION_INITIATOR@@K@Z 100153e4 f   SwiError.obj
 0001:000144b8       ?ConvertGobi2SwiPowerMode@@YA?AW4SWI_TYPE_Power@@K@Z 100154b8 f   SwiError.obj
 0001:00014520       ?ConvertGobi2SwiNvPrefOpMode@@YA?AW4SWI_TYPE_NvPrefOpMode@@KPAH@Z 10015520 f   SwiError.obj
 0001:00014670       ?ConvertSwi2GobiNvPrefOpMode@@YAKW4SWI_TYPE_NvPrefOpMode@@PAH@Z 10015670 f   SwiError.obj
 0001:0001474c       ?ExtractErrorCode@@YAHPBD0PAK@Z 1001574c f   SwiError.obj
 0001:0001487c       ?FindRIfaceIndex@@YAHW4eRadioTech@@EPAE1@Z 1001587c f   SwiGobiDll.obj
 0001:000148c0       ??0CSwiGobiDll@@QAA@XZ     100158c0 f   SwiGobiDll.obj
 0001:000148e4       ??1CSwiGobiDll@@QAA@XZ     100158e4 f   SwiGobiDll.obj
 0001:000148e8       ?Cleanup@CSwiGobiDll@@IAAXXZ 100158e8 f   SwiGobiDll.obj
 0001:00014cd0       ?Initialize@CSwiGobiDll@@QAA_NXZ 10015cd0 f   SwiGobiDll.obj
 0001:00015fe8       ?GetDLLVersion@CSwiGobiDll@@QAAKXZ 10016fe8 f   SwiGobiDll.obj
 0001:00015ff0       ?Connect@CSwiGobiDll@@QAAKXZ 10016ff0 f   SwiGobiDll.obj
 0001:00016058       ?Disconnect@CSwiGobiDll@@QAAKXZ 10017058 f   SwiGobiDll.obj
 0001:0001607c       ?GetWirelessTech@CSwiGobiDll@@QAA?AW4SWI_TYPE_WirelessTech@@XZ 1001707c f   SwiGobiDll.obj
 0001:000163a8       ?GetConnectedDeviceID@CSwiGobiDll@@QAAKKPAD@Z 100173a8 f   SwiGobiDll.obj
 0001:000163d0       ?GetFirmwareInfo@CSwiGobiDll@@QAAKPAK0000@Z 100173d0 f   SwiGobiDll.obj
 0001:00016424       ?GetCwePkgsInfo@CSwiGobiDll@@QAAKPAGPAE010101010101@Z 10017424 f   SwiGobiDll.obj
 0001:000164c8       ?GetSessionState@CSwiGobiDll@@QAAKPAK@Z 100174c8 f   SwiGobiDll.obj
 0001:000164e8       ?GetDormancyState@CSwiGobiDll@@QAAKPAK@Z 100174e8 f   SwiGobiDll.obj
 0001:00016508       ?GetDunCallInfo@CSwiGobiDll@@QAAKPAKPAE101111PA_KPAG221100002221@Z 10017508 f   SwiGobiDll.obj
 0001:000165ec       ?StartDataSession@CSwiGobiDll@@QAAKPAD00PAK1@Z 100175ec f   SwiGobiDll.obj
 0001:00016664       ?StopDataSession@CSwiGobiDll@@QAAKK@Z 10017664 f   SwiGobiDll.obj
 0001:00016684       ?GetIPAddress@CSwiGobiDll@@QAAKPAK@Z 10017684 f   SwiGobiDll.obj
 0001:000166a4       ?GetPacketStatus@CSwiGobiDll@@QAAKPAK00000@Z 100176a4 f   SwiGobiDll.obj
 0001:00016700       ?SetMobileIP@CSwiGobiDll@@QAAKK@Z 10017700 f   SwiGobiDll.obj
 0001:00016720       ?GetMobileIP@CSwiGobiDll@@QAAKPAK@Z 10017720 f   SwiGobiDll.obj
 0001:00016740       ?SetActiveMobileIPProfile@CSwiGobiDll@@QAAKPADE@Z 10017740 f   SwiGobiDll.obj
 0001:00016768       ?GetActiveMobileIPProfile@CSwiGobiDll@@QAAKPAE@Z 10017768 f   SwiGobiDll.obj
 0001:00016788       ?SetMobileIPProfile@CSwiGobiDll@@QAAKPADEPAEPAK22102200@Z 10017788 f   SwiGobiDll.obj
 0001:0001681c       ?GetMobileIPProfile@CSwiGobiDll@@QAAKEPAEPAK110EPAD11@Z 1001781c f   SwiGobiDll.obj
 0001:00016898       ?SetMobileIPParameters@CSwiGobiDll@@QAAKPADPAKPAE22222@Z 10017898 f   SwiGobiDll.obj
 0001:00016904       ?GetMobileIPParameters@CSwiGobiDll@@QAAKPAKPAE11111@Z 10017904 f   SwiGobiDll.obj
 0001:00016968       ?GetLastMobileIPError@CSwiGobiDll@@QAAKPAK@Z 10017968 f   SwiGobiDll.obj
 0001:00016988       ?GetAutoconnect@CSwiGobiDll@@QAAKPAK@Z 10017988 f   SwiGobiDll.obj
 0001:000169a8       ?SetAutoconnect@CSwiGobiDll@@QAAKK@Z 100179a8 f   SwiGobiDll.obj
 0001:000169c8       ?SetDefaultProfile@CSwiGobiDll@@QAAKKPAK0000PAD111@Z 100179c8 f   SwiGobiDll.obj
 0001:00016a84       ?GetDefaultProfile@CSwiGobiDll@@QAAKKPAK0000EPADE1E1@Z 10017a84 f   SwiGobiDll.obj
 0001:00016b58       ?GetByteTotals@CSwiGobiDll@@QAAKPAK0@Z 10017b58 f   SwiGobiDll.obj
 0001:00016b80       ?GetRFInfo@CSwiGobiDll@@QAAKPAE0@Z 10017b80 f   SwiGobiDll.obj
 0001:00016ba8       ?PerformNetworkScan@CSwiGobiDll@@QAAKPAE0@Z 10017ba8 f   SwiGobiDll.obj
 0001:00016bd0       ?PerformNetworkRATScan@CSwiGobiDll@@QAAKPAE000@Z 10017bd0 f   SwiGobiDll.obj
 0001:00016c14       ?InitiateNetworkRegistration@CSwiGobiDll@@QAAKKGGK@Z 10017c14 f   SwiGobiDll.obj
 0001:00016c58       ?InitiateDomainAttach@CSwiGobiDll@@QAAKK@Z 10017c58 f   SwiGobiDll.obj
 0001:00016c78       ?GetNetworkPreference@CSwiGobiDll@@QAAKPAK00@Z 10017c78 f   SwiGobiDll.obj
 0001:00016cb4       ?SetNetworkPreference@CSwiGobiDll@@QAAKKK@Z 10017cb4 f   SwiGobiDll.obj
 0001:00016cdc       ?SetCDMANetworkParameters@CSwiGobiDll@@QAAKPADPAE1PAK222@Z 10017cdc f   SwiGobiDll.obj
 0001:00016d40       ?GetCDMANetworkParameters@CSwiGobiDll@@QAAKPAE000000PAK111@Z 10017d40 f   SwiGobiDll.obj
 0001:00016dcc       ?GetACCOLC@CSwiGobiDll@@QAAKPAE@Z 10017dcc f   SwiGobiDll.obj
 0001:00016dec       ?SetACCOLC@CSwiGobiDll@@QAAKPADE@Z 10017dec f   SwiGobiDll.obj
 0001:00016e14       ?GetANAAAAuthenticationStatus@CSwiGobiDll@@QAAKPAK@Z 10017e14 f   SwiGobiDll.obj
 0001:00016e34       ?GetDeviceCapabilities@CSwiGobiDll@@QAAKPAK0000PAE@Z 10017e34 f   SwiGobiDll.obj
 0001:00016e90       ?GetFirmwareRevisions@CSwiGobiDll@@QAAKEPADE0E0@Z 10017e90 f   SwiGobiDll.obj
 0001:00016eec       ?GetPRLVersion@CSwiGobiDll@@QAAKPAG@Z 10017eec f   SwiGobiDll.obj
 0001:00016f0c       ?Set3Gpp2SubscriptionInfo@CSwiGobiDll@@QAAKPAEPAUMinBasedImsi@@PAUTrueImsi@@00@Z 10017f0c f   SwiGobiDll.obj
 0001:00016f60       ?Get3Gpp2SubscriptionInfo@CSwiGobiDll@@QAAKPAEPAUMinBasedImsi@@PAUTrueImsi@@00@Z 10017f60 f   SwiGobiDll.obj
 0001:00016fb4       ?GetERIFile@CSwiGobiDll@@QAAKPAKPAE@Z 10017fb4 f   SwiGobiDll.obj
 0001:00016fdc       ?ActivateManual@CSwiGobiDll@@QAAKPADG00KPAE00@Z 10017fdc f   SwiGobiDll.obj
 0001:00017048       ?GetPower@CSwiGobiDll@@QAAKPAK@Z 10018048 f   SwiGobiDll.obj
 0001:00017068       ?GetOfflineReason@CSwiGobiDll@@QAAKPAK0@Z 10018068 f   SwiGobiDll.obj
 0001:00017090       ?GetNetworkTime@CSwiGobiDll@@QAAKPA_KPAK@Z 10018090 f   SwiGobiDll.obj
 0001:000170b8       ?ValidateSPC@CSwiGobiDll@@QAAKPAD@Z 100180b8 f   SwiGobiDll.obj
 0001:000170d8       ?DeleteSMS@CSwiGobiDll@@QAAKKPAK0@Z 100180d8 f   SwiGobiDll.obj
 0001:00017158       ?GetSMSList@CSwiGobiDll@@QAAKKPAK0PAE@Z 10018158 f   SwiGobiDll.obj
 0001:000171dc       ?GetSMS@CSwiGobiDll@@QAAKKKPAK00PAE@Z 100181dc f   SwiGobiDll.obj
 0001:00017278       ?ModifySMSStatus@CSwiGobiDll@@QAAKKKK@Z 10018278 f   SwiGobiDll.obj
 0001:000172f8       ?SaveSMS@CSwiGobiDll@@QAAKKKKPAEPAK@Z 100182f8 f   SwiGobiDll.obj
 0001:0001738c       ?SendSMS@CSwiGobiDll@@QAAKKKPAEEPAK@Z 1001838c f   SwiGobiDll.obj
 0001:00017420       ?GetSMSCAddress@CSwiGobiDll@@QAAKEPADE0@Z 10018420 f   SwiGobiDll.obj
 0001:000174a4       ?SetSMSCAddress@CSwiGobiDll@@QAAKPAD0@Z 100184a4 f   SwiGobiDll.obj
 0001:00017518       ?SetSMSProtocol@CSwiGobiDll@@QAAKE@Z 10018518 f   SwiGobiDll.obj
 0001:00017584       ?SetSMSRoute@CSwiGobiDll@@QAAKKPAE@Z 10018584 f   SwiGobiDll.obj
 0001:000175f8       ?SetSMSBroadcastActivation@CSwiGobiDll@@QAAKEE@Z 100185f8 f   SwiGobiDll.obj
 0001:0001766c       ?DMSUIMSetPINProtection@CSwiGobiDll@@QAAKKKPADPAK1@Z 1001866c f   SwiGobiDll.obj
 0001:000176c0       ?UIMGetCardStatus@CSwiGobiDll@@QAAKPAHPAUQMI_UIM_GET_CARD_STATUS_RESP@@@Z 100186c0 f   SwiGobiDll.obj
 0001:000176e8       ?UIMVerifyPIN@CSwiGobiDll@@QAAKPAUQMI_UIM_VERIFY_PIN_REQ_SESSION_INFORMATION@@PAUQMI_UIM_VERIFY_PIN_REQ_VERIFY_PIN@@PAUQMI_UIM_VERIFY_PIN_RESP_RETRIES_REMAINING@@@Z 100186e8 f   SwiGobiDll.obj
 0001:00017724       ?UIMUnblockPIN@CSwiGobiDll@@QAAKPAUQMI_UIM_UNBLOCK_PIN_REQ_SESSION_INFORMATION@@PAUQMI_UIM_UNBLOCK_PIN_REQ_UNBLOCK_PIN@@PAUQMI_UIM_UNBLOCK_PIN_RESP_RETRIES_REMAINING@@@Z 10018724 f   SwiGobiDll.obj
 0001:00017760       ?UIMSetPINProtection@CSwiGobiDll@@QAAKPAUQMI_UIM_SET_PIN_PROTECTION_REQ_SESSION_INFORMATION@@PAUQMI_UIM_SET_PIN_PROTECTION_REQ_SET_PIN_PROTECTION@@PAUQMI_UIM_SET_PIN_PROTECTION_RESP_RETRIES_REMAINING@@@Z 10018760 f   SwiGobiDll.obj
 0001:0001779c       ?UIMChangePIN@CSwiGobiDll@@QAAKPAUQMI_UIM_CHANGE_PIN_REQ_SESSION_INFORMATION@@PAUQMI_UIM_CHANGE_PIN_REQ_CHANGE_PIN@@PAUQMI_UIM_CHANGE_PIN_RESP_RETRIES_REMAINING@@@Z 1001879c f   SwiGobiDll.obj
 0001:000177d8       ?DMSUIMVerifyPIN@CSwiGobiDll@@QAAKKPADPAK1@Z 100187d8 f   SwiGobiDll.obj
 0001:0001781c       ?DMSUIMUnblockPIN@CSwiGobiDll@@QAAKKPAD0PAK1@Z 1001881c f   SwiGobiDll.obj
 0001:00017870       ?DMSUIMChangePIN@CSwiGobiDll@@QAAKKPAD0PAK1@Z 10018870 f   SwiGobiDll.obj
 0001:000178c4       ?DMSUIMGetPINStatus@CSwiGobiDll@@QAAKKPAK00@Z 100188c4 f   SwiGobiDll.obj
 0001:00017908       ?DMSUIMGetICCID@CSwiGobiDll@@QAAKEPAD@Z 10018908 f   SwiGobiDll.obj
 0001:00017930       ?DMSUIMGetControlKeyStatus@CSwiGobiDll@@QAAKKPAK00@Z 10018930 f   SwiGobiDll.obj
 0001:00017974       ?DMSUIMSetControlKeyProtection@CSwiGobiDll@@QAAKKKPADPAK@Z 10018974 f   SwiGobiDll.obj
 0001:000179ac       ?DMSUIMUnblockControlKey@CSwiGobiDll@@QAAKKPADPAK@Z 100189ac f   SwiGobiDll.obj
 0001:000179e8       ?ResetToFactoryDefaults@CSwiGobiDll@@QAAKPAD@Z 100189e8 f   SwiGobiDll.obj
 0001:00017a08       ?GetPDSState@CSwiGobiDll@@QAAKPAK0@Z 10018a08 f   SwiGobiDll.obj
 0001:00017a30       ?SetPDSState@CSwiGobiDll@@QAAKK@Z 10018a30 f   SwiGobiDll.obj
 0001:00017a50       ?PDSInjectTimeReference@CSwiGobiDll@@QAAK_KG@Z 10018a50 f   SwiGobiDll.obj
 0001:00017a88       ?GetPDSDefaults@CSwiGobiDll@@QAAKPAKPAE00@Z 10018a88 f   SwiGobiDll.obj
 0001:00017acc       ?SetPDSDefaults@CSwiGobiDll@@QAAKKEKK@Z 10018acc f   SwiGobiDll.obj
 0001:00017b10       ?GetXTRAAutomaticDownload@CSwiGobiDll@@QAAKPAKPAG@Z 10018b10 f   SwiGobiDll.obj
 0001:00017b38       ?SetXTRAAutomaticDownload@CSwiGobiDll@@QAAKKG@Z 10018b38 f   SwiGobiDll.obj
 0001:00017b60       ?GetXTRANetwork@CSwiGobiDll@@QAAKPAK@Z 10018b60 f   SwiGobiDll.obj
 0001:00017b80       ?SetXTRANetwork@CSwiGobiDll@@QAAKK@Z 10018b80 f   SwiGobiDll.obj
 0001:00017ba0       ?GetXTRAValidity@CSwiGobiDll@@QAAKPAG00@Z 10018ba0 f   SwiGobiDll.obj
 0001:00017bdc       ?SetXTRAValidity@CSwiGobiDll@@QAAKGGG@Z 10018bdc f   SwiGobiDll.obj
 0001:00017c18       ?SetXTRAEmbeddedClient@CSwiGobiDll@@QAAKEE@Z 10018c18 f   SwiGobiDll.obj
 0001:00017c40       ?SetNMEAConfig@CSwiGobiDll@@QAAKEEEPAG@Z 10018c40 f   SwiGobiDll.obj
 0001:00017c84       ?GetNMEAConfig@CSwiGobiDll@@QAAKPAE00PAG@Z 10018c84 f   SwiGobiDll.obj
 0001:00017cc8       ?ForceXTRADownload@CSwiGobiDll@@QAAKXZ 10018cc8 f   SwiGobiDll.obj
 0001:00017ce4       ?GetAGPSConfig@CSwiGobiDll@@QAAKPAK0@Z 10018ce4 f   SwiGobiDll.obj
 0001:00017d0c       ?SetAGPSConfig@CSwiGobiDll@@QAAKKK@Z 10018d0c f   SwiGobiDll.obj
 0001:00017d34       ?GetServiceAutomaticTracking@CSwiGobiDll@@QAAKPAK@Z 10018d34 f   SwiGobiDll.obj
 0001:00017d54       ?SetServiceAutomaticTracking@CSwiGobiDll@@QAAKK@Z 10018d54 f   SwiGobiDll.obj
 0001:00017d74       ?GetPortAutomaticTracking@CSwiGobiDll@@QAAKPAK@Z 10018d74 f   SwiGobiDll.obj
 0001:00017d94       ?SetPortAutomaticTracking@CSwiGobiDll@@QAAKK@Z 10018d94 f   SwiGobiDll.obj
 0001:00017db4       ?ResetPDSData@CSwiGobiDll@@QAAKPAK0@Z 10018db4 f   SwiGobiDll.obj
 0001:00017ddc       ?GetDataBearerTechnology@CSwiGobiDll@@QAAKPAK@Z 10018ddc f   SwiGobiDll.obj
 0001:00017dfc       ?GetSessionDuration@CSwiGobiDll@@QAAKPA_K@Z 10018dfc f   SwiGobiDll.obj
 0001:00017e1c       ?GetSignalStrengths@CSwiGobiDll@@QAAKPAKPAC0@Z 10018e1c f   SwiGobiDll.obj
 0001:00017e98       ?GetServingNetworkCaps@CSwiGobiDll@@QAAKPAE0@Z 10018e98 f   SwiGobiDll.obj
 0001:00017ec0       ?GetConnectionRate@CSwiGobiDll@@QAAKPAK000@Z 10018ec0 f   SwiGobiDll.obj
 0001:00017f04       ?GetServingNetwork@CSwiGobiDll@@QAAKPAK000PAE10PAG2EPAD@Z 10018f04 f   SwiGobiDll.obj
 0001:00017f90       ?GetHomeNetwork@CSwiGobiDll@@QAAKPAG0EPAD00@Z 10018f90 f   SwiGobiDll.obj
 0001:00017fec       ?GetManufacturer@CSwiGobiDll@@QAAKEPAD@Z 10018fec f   SwiGobiDll.obj
 0001:00018014       ?GetModelID@CSwiGobiDll@@QAAKEPAD@Z 10019014 f   SwiGobiDll.obj
 0001:0001803c       ?GetFirmwareRevision@CSwiGobiDll@@QAAKEPAD@Z 1001903c f   SwiGobiDll.obj
 0001:00018064       ?GetHardwareRevision@CSwiGobiDll@@QAAKEPAD@Z 10019064 f   SwiGobiDll.obj
 0001:0001808c       ?GetVoiceNumber@CSwiGobiDll@@QAAKEPADE0@Z 1001908c f   SwiGobiDll.obj
 0001:000180d0       ?GetSerialNumbers@CSwiGobiDll@@QAAKEPADE0E0@Z 100190d0 f   SwiGobiDll.obj
 0001:0001812c       ?GetIMSI@CSwiGobiDll@@QAAKEPAD@Z 1001912c f   SwiGobiDll.obj
 0001:00018154       ?UpgradeFirmwareW@CSwiGobiDll@@QAAKPAG@Z 10019154 f   SwiGobiDll.obj
 0001:00018174       ?GetImageStoreW@CSwiGobiDll@@QAAKGPAG@Z 10019174 f   SwiGobiDll.obj
 0001:0001819c       ?GetImageInfoW@CSwiGobiDll@@QAAKPBGPAK1111@Z 1001919c f   SwiGobiDll.obj
 0001:000181f8       ?DisableCallbacks@CSwiGobiDll@@QAAXXZ 100191f8 f   SwiGobiDll.obj
 0001:00018408       ?SetSessionStateCB@CSwiGobiDll@@SAKP6AXKK@Z@Z 10019408 f   SwiGobiDll.obj
 0001:0001847c       ?SetDataCapsCB@CSwiGobiDll@@SAKP6AXEPAE@Z@Z 1001947c f   SwiGobiDll.obj
 0001:000184a8       ?SetByteTotalsCB@CSwiGobiDll@@SAKP6AX_K0@ZE@Z 100194a8 f   SwiGobiDll.obj
 0001:000184d4       ?SetDataBearerCB@CSwiGobiDll@@SAKP6AXK@Z@Z 100194d4 f   SwiGobiDll.obj
 0001:00018500       ?SetDormancyStatusCB@CSwiGobiDll@@SAKP6AXK@Z@Z 10019500 f   SwiGobiDll.obj
 0001:0001852c       ?SetMobileIPStatusCB@CSwiGobiDll@@SAKP6AXK@Z@Z 1001952c f   SwiGobiDll.obj
 0001:00018558       ?SetActivationStatusCB@CSwiGobiDll@@SAKP6AXK@Z@Z 10019558 f   SwiGobiDll.obj
 0001:00018584       ?SetPowerCB@CSwiGobiDll@@SAKP6AXK@Z@Z 10019584 f   SwiGobiDll.obj
 0001:000185b0       ?SetRoamingIndicatorCB@CSwiGobiDll@@SAKP6AXK@Z@Z 100195b0 f   SwiGobiDll.obj
 0001:000185dc       ?SetSignalStrengthCB@CSwiGobiDll@@SAKP6AXCK@ZEPAC@Z 100195dc f   SwiGobiDll.obj
 0001:00018608       ?SetRFInfoCB@CSwiGobiDll@@SAKP6AXKKK@Z@Z 10019608 f   SwiGobiDll.obj
 0001:00018634       ?SetNewSMSCB@CSwiGobiDll@@SAKP6AXKK@Z@Z 10019634 f   SwiGobiDll.obj
 0001:00018660       ?SetNewSMSCBCB@CSwiGobiDll@@SAKP6AXEKEGPAE@Z@Z 10019660 f   SwiGobiDll.obj
 0001:0001868c       ?SetVoiceMessageCB@CSwiGobiDll@@SAKP6AXEPAE00@Z@Z 1001968c f   SwiGobiDll.obj
 0001:000186f8       ?SetPhonebookRecordReadCB@CSwiGobiDll@@SAKP6AXEGPAUarrPBInfo@@@Z@Z 100196f8 f   SwiGobiDll.obj
 0001:00018724       ?SetNITZCB@CSwiGobiDll@@SAKP6AXGEEEEEEEE@Z@Z 10019724 f   SwiGobiDll.obj
 0001:00018750       ?SetEmergencyModeCB@CSwiGobiDll@@SAKP6AXPAE@Z@Z 10019750 f   SwiGobiDll.obj
 0001:0001877c       ?SetOMADMStateCB@CSwiGobiDll@@SAKP6AXKK@Z@Z 1001977c f   SwiGobiDll.obj
 0001:000187a8       ?SetOMADMAlertCB@CSwiGobiDll@@SAKP6AXKG@Z@Z 100197a8 f   SwiGobiDll.obj
 0001:000187d4       ?SetDeviceRemovalCallback@CSwiGobiDll@@QAAKP6AXK@Z@Z 100197d4 f   SwiGobiDll.obj
 0001:00018840       ?SetPower@CSwiGobiDll@@QAAKK@Z 10019840 f   SwiGobiDll.obj
 0001:000188bc       ?ActivateAutomatic@CSwiGobiDll@@QAAKPAD@Z 100198bc f   SwiGobiDll.obj
 0001:00018974       ?GetActivationState@CSwiGobiDll@@QAAKPAK@Z 10019974 f   SwiGobiDll.obj
 0001:000189e0       ?OMADMGetFeatureSettings@CSwiGobiDll@@QAAKPAK0@Z 100199e0 f   SwiGobiDll.obj
 0001:00018a54       ?OMADMGetSessionInfo@CSwiGobiDll@@QAAKPAK00PAEPAG2@Z 10019a54 f   SwiGobiDll.obj
 0001:00018af0       ?OMADMSetProvisioningFeature@CSwiGobiDll@@QAAKK@Z 10019af0 f   SwiGobiDll.obj
 0001:00018b5c       ?OMADMSetPRLUpdateFeature@CSwiGobiDll@@QAAKK@Z 10019b5c f   SwiGobiDll.obj
 0001:00018bc8       ?OMADMStartSession@CSwiGobiDll@@QAAKK@Z 10019bc8 f   SwiGobiDll.obj
 0001:00018c34       ?OMADMCancelSession@CSwiGobiDll@@QAAKXZ 10019c34 f   SwiGobiDll.obj
 0001:00018c9c       ?OMADMGetPendingNIA@CSwiGobiDll@@QAAKPAKPAG@Z 10019c9c f   SwiGobiDll.obj
 0001:00018d10       ?OMADMSendSelection@CSwiGobiDll@@QAAKKG@Z 10019d10 f   SwiGobiDll.obj
 0001:00018d84       ?GetIPConfiguration@CSwiGobiDll@@QAAKPAK0000@Z 10019d84 f   SwiGobiDll.obj
 0001:00018e18       ?OMAEXSetEventReport@CSwiGobiDll@@QAAKXZ 10019e18 f   SwiGobiDll.obj
 0001:00018e80       ?OMAEXSessionStart@CSwiGobiDll@@QAAKPAE@Z 10019e80 f   SwiGobiDll.obj
 0001:00018eec       ?OMAEXSessionCancel@CSwiGobiDll@@QAAKXZ 10019eec f   SwiGobiDll.obj
 0001:00018f54       ?OMAEXSelection@CSwiGobiDll@@QAAKPAE@Z 10019f54 f   SwiGobiDll.obj
 0001:00018fc0       ?OMAEXGetSettings@CSwiGobiDll@@QAAKPAE00000@Z 10019fc0 f   SwiGobiDll.obj
 0001:0001905c       ?OMAEXSetSettings@CSwiGobiDll@@QAAKPAE00000@Z 1001a05c f   SwiGobiDll.obj
 0001:000190f8       ?OMAEXSessionGetInfo@CSwiGobiDll@@QAAKPAUomaSessionInfo@@@Z 1001a0f8 f   SwiGobiDll.obj
 0001:00019164       ?OMAEXInit@CSwiGobiDll@@QAAKXZ 1001a164 f   SwiGobiDll.obj
 0001:000191cc       ?OMAEXShutdown@CSwiGobiDll@@QAAKXZ 1001a1cc f   SwiGobiDll.obj
 0001:00019234       ?GetImagePreference@CSwiGobiDll@@QAAKPAKPAE@Z 1001a234 f   SwiGobiDll.obj
 0001:0001925c       ?SetImagePreference@CSwiGobiDll@@QAAKKPAEKEPAK0@Z 1001a25c f   SwiGobiDll.obj
 0001:000192b8       ?GetAudioProfile@CSwiGobiDll@@QAAKPAE@Z 1001a2b8 f   SwiGobiDll.obj
 0001:00019358       ?SetAudioProfile@CSwiGobiDll@@QAAKPAE@Z 1001a358 f   SwiGobiDll.obj
 0001:00019444       ?SetMICMuteStatus@CSwiGobiDll@@QAAKPAE@Z 1001a444 f   SwiGobiDll.obj
 0001:00019530       ?SetSpeakerMuteStatus@CSwiGobiDll@@QAAKPAE@Z 1001a530 f   SwiGobiDll.obj
 0001:0001961c       ?SetReceiverVolume@CSwiGobiDll@@QAAKPAE@Z 1001a61c f   SwiGobiDll.obj
 0001:00019700       ?SetMicVolume@CSwiGobiDll@@QAAKPAG@Z 1001a700 f   SwiGobiDll.obj
 0001:000197f4       ?GetMicVolume@CSwiGobiDll@@QAAKPAG@Z 1001a7f4 f   SwiGobiDll.obj
 0001:000198c0       ?SetEchoCancelMode@CSwiGobiDll@@QAAKPAE@Z 1001a8c0 f   SwiGobiDll.obj
 0001:000199b4       ?GetEchoCancelMode@CSwiGobiDll@@QAAKPAE@Z 1001a9b4 f   SwiGobiDll.obj
 0001:00019a80       ?SetNoiseSuppression@CSwiGobiDll@@QAAKPAE@Z 1001aa80 f   SwiGobiDll.obj
 0001:00019b74       ?GetNoiseSuppression@CSwiGobiDll@@QAAKPAE@Z 1001ab74 f   SwiGobiDll.obj
 0001:00019c40       ?SetAutoOutputGain@CSwiGobiDll@@QAAKPAE@Z 1001ac40 f   SwiGobiDll.obj
 0001:00019d34       ?GetAutoOutputGain@CSwiGobiDll@@QAAKPAE@Z 1001ad34 f   SwiGobiDll.obj
 0001:00019e00       ?SetAutoInputGain@CSwiGobiDll@@QAAKPAE@Z 1001ae00 f   SwiGobiDll.obj
 0001:00019ef4       ?GetAutoInputGain@CSwiGobiDll@@QAAKPAE@Z 1001aef4 f   SwiGobiDll.obj
 0001:00019fc0       ?SetTXPCMFilter@CSwiGobiDll@@QAAKPAG0PAK0@Z 1001afc0 f   SwiGobiDll.obj
 0001:0001a0c0       ?GetTXPCMFilter@CSwiGobiDll@@QAAKPAG0PAK0@Z 1001b0c0 f   SwiGobiDll.obj
 0001:0001a1a4       ?SetRXPCMFilter@CSwiGobiDll@@QAAKPAG0PAK0@Z 1001b1a4 f   SwiGobiDll.obj
 0001:0001a2a4       ?GetRXPCMFilter@CSwiGobiDll@@QAAKPAG0PAK0@Z 1001b2a4 f   SwiGobiDll.obj
 0001:0001a388       ?SetRXGainLevel@CSwiGobiDll@@QAAKPAEPAG1@Z 1001b388 f   SwiGobiDll.obj
 0001:0001a480       ?SetSideToneGain@CSwiGobiDll@@QAAKPAG@Z 1001b480 f   SwiGobiDll.obj
 0001:0001a574       ?GetSideToneGain@CSwiGobiDll@@QAAKPAG@Z 1001b574 f   SwiGobiDll.obj
 0001:0001a640       ?PlayAudioTone@CSwiGobiDll@@QAAKPAE@Z 1001b640 f   SwiGobiDll.obj
 0001:0001a704       ?OrigUSSD@CSwiGobiDll@@QAAKPAUUSSInfo@@PAGPAUalphaIDInfo@@0PAE3PAUccSUPSType@@@Z 1001b704 f   SwiGobiDll.obj
 0001:0001a768       ?AnswerUSSD@CSwiGobiDll@@QAAKPAUUSSInfo@@@Z 1001b768 f   SwiGobiDll.obj
 0001:0001a788       ?CancelUSSD@CSwiGobiDll@@QAAKXZ 1001b788 f   SwiGobiDll.obj
 0001:0001a7a4       ?ChangeBarringPwd@CSwiGobiDll@@QAAKPAUcallBarringPwd@@PAGPAUalphaIDInfo@@PAE3PAUccSUPSType@@@Z 1001b7a4 f   SwiGobiDll.obj
 0001:0001a800       ?DialCall@CSwiGobiDll@@QAAKPAUtDialReqParam@@PAEPAUalphaIDInfo@@1PAUccSUPSType@@@Z 1001b800 f   SwiGobiDll.obj
 0001:0001a854       ?EndCall@CSwiGobiDll@@QAAKPAE0@Z 1001b854 f   SwiGobiDll.obj
 0001:0001a87c       ?AnserCall@CSwiGobiDll@@QAAKPAE0@Z 1001b87c f   SwiGobiDll.obj
 0001:0001a8a4       ?SetCallInfoCB@CSwiGobiDll@@SAKP6AXPAUarrCallInfo@@PAUarrRemotePartyNum@@PAUarrRemotePartyName@@PAUarrAlertingType@@PAUarrSvcOption@@PAUarrCallEndReason@@PAUarrAlphaIDInfo@@PAUarrPeerNumInfo@@PAUarrDiagInfo@@77PAUarrAlertingPattern@@@Z@Z 1001b8a4 f   SwiGobiDll.obj
 0001:0001a8d0       ?SetInfoRecCB@CSwiGobiDll@@SAKP6AXPAEPAUsignalInfo@@PAUcallerIDInfo@@PAD330PAUpeerNumInfo@@44PAUredirectNumInfo@@0000PAUlineCtlInfo@@PAUextDisplayInfo@@@Z@Z 1001b8d0 f   SwiGobiDll.obj
 0001:0001a8fc       ?SetUSSDInfoCB@CSwiGobiDll@@SAKP6AXPAEPAUUSSInfo@@@Z@Z 1001b8fc f   SwiGobiDll.obj
 0001:0001a928       ?SetAllPbInitDoneCB@CSwiGobiDll@@SAKP6AXEPAEPAG@Z@Z 1001b928 f   SwiGobiDll.obj
 0001:0001a994       ?SetEmergencyListCB@CSwiGobiDll@@SAKP6AXEPAUemergencyNumberEntry@@@Z@Z 1001b994 f   SwiGobiDll.obj
 0001:0001aa00       ?SetOMAEXEventCB@CSwiGobiDll@@SAKP6AXPAUFUMOInfo@@PAUOMAInfo@@@Z@Z 1001ba00 f   SwiGobiDll.obj
 0001:0001aa6c       ?ManageCalls@CSwiGobiDll@@QAAKPAE0PAG@Z 1001ba6c f   SwiGobiDll.obj
 0001:0001aaa8       ?GetCLIR@CSwiGobiDll@@QAAKPAUstatusResp@@PAGPAUalphaIDInfo@@PAE3PAUccSUPSType@@@Z 1001baa8 f   SwiGobiDll.obj
 0001:0001ab04       ?GetCallWaiting@CSwiGobiDll@@QAAKPAE0PAGPAUalphaIDInfo@@00PAUccSUPSType@@@Z 1001bb04 f   SwiGobiDll.obj
 0001:0001ab68       ?SetSUPS@CSwiGobiDll@@QAAKPAUvoiceSetSUPSServiceReq@@PAGPAUalphaIDInfo@@PAE3PAUccSUPSType@@@Z 1001bb68 f   SwiGobiDll.obj
 0001:0001abc4       ?GetCallBarring@CSwiGobiDll@@QAAKPAE00PAGPAUalphaIDInfo@@00PAUccSUPSType@@@Z 1001bbc4 f   SwiGobiDll.obj
 0001:0001ac30       ?GetCallForwarding@CSwiGobiDll@@QAAKPAE0PAUgetCallFWInfo@@0PAUalphaIDInfo@@00PAUccSUPSType@@PAUgetExtCallFWInfo@@@Z 1001bc30 f   SwiGobiDll.obj
 0001:0001aca4       ?GetAllCallInfo@CSwiGobiDll@@QAAKPAUarrCallInfo@@PAUarrRemotePartyNum@@PAUarrRemotePartyName@@PAUarrAlertingType@@PAUarrUUSInfo@@PAUarrSvcOption@@PAE6PAUarrCallEndReason@@PAUarrAlphaIDInfo@@PAUarrPeerNumInfo@@PAUarrDiagInfo@@99PAUarrAlertingPattern@@@Z 1001bca4 f   SwiGobiDll.obj
 0001:0001ad50       ?SendFlash@CSwiGobiDll@@QAAKPAEPAD00@Z 1001bd50 f   SwiGobiDll.obj
 0001:0001ad94       ?StartDTMF@CSwiGobiDll@@QAAKPAE00@Z 1001bd94 f   SwiGobiDll.obj
 0001:0001add0       ?StopDTMF@CSwiGobiDll@@QAAKPAE0@Z 1001bdd0 f   SwiGobiDll.obj
 0001:0001adf8       ?GetPhonebookCapabilities@CSwiGobiDll@@QAAKPAEPAG1100@Z 1001bdf8 f   SwiGobiDll.obj
 0001:0001ae54       ?ReadPhonebookRecords@CSwiGobiDll@@QAAKPAEPAG111@Z 1001be54 f   SwiGobiDll.obj
 0001:0001aea8       ?WritePhonebookRecord@CSwiGobiDll@@QAAKPAEPAG1000000@Z 1001bea8 f   SwiGobiDll.obj
 0001:0001af1c       ?DeletePhonebookRecord@CSwiGobiDll@@QAAKPAEPAG1@Z 1001bf1c f   SwiGobiDll.obj
 0001:0001af58       ?GetCellLocationInfo@CSwiGobiDll@@QAAKPAUgeranCellInfo@@PAUumtsCellInfo@@PAUcdmaCellInfo@@PAK@Z 1001bf58 f   SwiGobiDll.obj
 0001:0001afd8       ?GetWaitingMessage@CSwiGobiDll@@QAAKPAUwaitingMsgInfo@@@Z 1001bfd8 f   SwiGobiDll.obj
 0001:0001b040       ?GetRTREConfig@CSwiGobiDll@@QAAKPAE0@Z 1001c040 f   SwiGobiDll.obj
 0001:0001b0b0       ?SwiM2MAV_AudioGetProfile@CSwiGobiDll@@QAAKPAE000000@Z 1001c0b0 f   SwiGobiDll.obj
 0001:0001b114       ?SwiM2MAV_AudioSetProfile@CSwiGobiDll@@QAAKPAE00000@Z 1001c114 f   SwiGobiDll.obj
 0001:0001b170       ?SwiM2MAV_AudioGetVolume@CSwiGobiDll@@QAAKPAE00@Z 1001c170 f   SwiGobiDll.obj
 0001:0001b1ac       ?SwiM2MAV_AudioSetVolume@CSwiGobiDll@@QAAKPAE00@Z 1001c1ac f   SwiGobiDll.obj
 0001:0001b1e8       ?SwiM2MAV_AudioGetAVMute@CSwiGobiDll@@QAAKPAE000@Z 1001c1e8 f   SwiGobiDll.obj
 0001:0001b22c       ?SwiM2MAV_AudioSetAVMute@CSwiGobiDll@@QAAKPAE000@Z 1001c22c f   SwiGobiDll.obj
 0001:0001b270       ?SwiM2MAV_AudioGetAVCFG@CSwiGobiDll@@QAAKPAUAudioConfig@@PAE@Z 1001c270 f   SwiGobiDll.obj
 0001:0001b298       ?SwiM2MAV_AudioSetAVCFG@CSwiGobiDll@@QAAKPAE00PAUPIFACETable@@@Z 1001c298 f   SwiGobiDll.obj
 0001:0001b2dc       ?SwiM2MAV_AudioNVDef@CSwiGobiDll@@QAAKXZ 1001c2dc f   SwiGobiDll.obj
 0001:0001b2f8       ?SwiM2MAV_AudioSetLPBK@CSwiGobiDll@@QAAKPAE@Z 1001c2f8 f   SwiGobiDll.obj
 0001:0001b318       ?SwiM2MAV_AudioGetSpeakerGain@CSwiGobiDll@@QAAKPAEPAG@Z 1001c318 f   SwiGobiDll.obj
 0001:0001b340       ?SwiM2MAV_AudioSetSpeakerGain@CSwiGobiDll@@QAAKPAEPAG@Z 1001c340 f   SwiGobiDll.obj
 0001:0001b368       ?SwiM2MAV_AudioGetSTG@CSwiGobiDll@@QAAKPAEPAG@Z 1001c368 f   SwiGobiDll.obj
 0001:0001b390       ?SwiM2MAV_AudioSetSTG@CSwiGobiDll@@QAAKPAEPAG@Z 1001c390 f   SwiGobiDll.obj
 0001:0001b3b8       ?SwiM2MAV_AudioGetTxVolume@CSwiGobiDll@@QAAKPAEPAG@Z 1001c3b8 f   SwiGobiDll.obj
 0001:0001b3e0       ?SwiM2MAV_AudioSetTxVolume@CSwiGobiDll@@QAAKPAEPAG@Z 1001c3e0 f   SwiGobiDll.obj
 0001:0001b408       ?SwiM2MAV_AudioGetMicGain@CSwiGobiDll@@QAAKPAEPAG@Z 1001c408 f   SwiGobiDll.obj
 0001:0001b430       ?SwiM2MAV_AudioSetMicGain@CSwiGobiDll@@QAAKPAEPAG@Z 1001c430 f   SwiGobiDll.obj
 0001:0001b458       ?SwiM2MAV_AudioGetVolDB@CSwiGobiDll@@QAAKPAE00PAG@Z 1001c458 f   SwiGobiDll.obj
 0001:0001b49c       ?SwiM2MAV_AudioSetVolDB@CSwiGobiDll@@QAAKPAE00PAG@Z 1001c49c f   SwiGobiDll.obj
 0001:0001b4e0       ?SwiM2MAV_AudioGetAVTXG@CSwiGobiDll@@QAAKPAEPAG@Z 1001c4e0 f   SwiGobiDll.obj
 0001:0001b508       ?SwiM2MAV_AudioSetAVTXG@CSwiGobiDll@@QAAKPAEPAG@Z 1001c508 f   SwiGobiDll.obj
 0001:0001b530       ?SwiM2MAV_AudioGetAVRXG@CSwiGobiDll@@QAAKPAEPAG@Z 1001c530 f   SwiGobiDll.obj
 0001:0001b558       ?SwiM2MAV_AudioSetAVRXG@CSwiGobiDll@@QAAKPAEPAG@Z 1001c558 f   SwiGobiDll.obj
 0001:0001b580       ?SwiM2MAV_AudioGetAVEC@CSwiGobiDll@@QAAKPAE0@Z 1001c580 f   SwiGobiDll.obj
 0001:0001b5a8       ?SwiM2MAV_AudioSetAVEC@CSwiGobiDll@@QAAKPAE0@Z 1001c5a8 f   SwiGobiDll.obj
 0001:0001b5d0       ?SwiM2MAV_AudioGetAVNS@CSwiGobiDll@@QAAKPAE0@Z 1001c5d0 f   SwiGobiDll.obj
 0001:0001b5f8       ?SwiM2MAV_AudioSetAVNS@CSwiGobiDll@@QAAKPAE0@Z 1001c5f8 f   SwiGobiDll.obj
 0001:0001b620       ?SwiM2MAV_AudioPlayTone@CSwiGobiDll@@QAAKPAE0PAG@Z 1001c620 f   SwiGobiDll.obj
 0001:0001b65c       ??1bad_alloc@std@@UAA@XZ   1001c65c f i SwiNotify.obj
 0001:0001b670       ??_Gbad_alloc@std@@UAAPAXI@Z 1001c670 f i SwiNotify.obj
 0001:0001b670       ??_Ebad_alloc@std@@UAAPAXI@Z 1001c670 f i  CIL library: CIL module
 0001:0001b6a0       ?GenericCallStateChanged@@YAXXZ 1001c6a0 f i SwiNotify.obj
 0001:0001b6a0       ?DormancyStatusCallback@@YAXK@Z 1001c6a0 f i SwiNotify.obj
 0001:0001b6a0       ?GenericSmsSendStatusChanged@@YAXXZ 1001c6a0 f i SwiNotify.obj
 0001:0001b6a0       ??3@YAXPAX0@Z              1001c6a0 f i SwiNotify.obj
 0001:0001b6a0       ?GenericPlmnModeChanged@@YAXXZ 1001c6a0 f i SwiNotify.obj
 0001:0001b6a0       ?GenericPhonebookReadyChanged@@YAXXZ 1001c6a0 f i SwiNotify.obj
 0001:0001b6a0       ?GenericPlmnReadyChanged@@YAXXZ 1001c6a0 f i SwiNotify.obj
 0001:0001b6a0       ?GenericPlmnAvailableChanged@@YAXXZ 1001c6a0 f i SwiNotify.obj
 0001:0001b6ac       ??0logic_error@std@@QAA@ABV?$basic_string@DU?$char_traits@D@std@@V?$allocator@D@2@@1@@Z 1001c6ac f i SwiNotify.obj
 0001:0001b724       ?what@logic_error@std@@UBAPBDXZ 1001c724 f i SwiNotify.obj
 0001:0001b73c       ??1logic_error@std@@UAA@XZ 1001c73c f i SwiNotify.obj
 0001:0001b73c       ??1length_error@std@@UAA@XZ 1001c73c f i SwiNotify.obj
 0001:0001b768       ??_Elength_error@std@@UAAPAXI@Z 1001c768 f i  CIL library: CIL module
 0001:0001b768       ??_Glength_error@std@@UAAPAXI@Z 1001c768 f i SwiNotify.obj
 0001:0001b768       ??_Elogic_error@std@@UAAPAXI@Z 1001c768 f i  CIL library: CIL module
 0001:0001b768       ??_Glogic_error@std@@UAAPAXI@Z 1001c768 f i SwiNotify.obj
 0001:0001b7a8       ?OMAEXEventCallback@CSwiNotify@@SAXPAUFUMOInfo@@PAUOMAInfo@@@Z 1001c7a8 f   SwiNotify.obj
 0001:0001b89c       ?CallInfoCallback@CSwiNotify@@SAXPAUarrCallInfo@@PAUarrRemotePartyNum@@PAUarrRemotePartyName@@PAUarrAlertingType@@PAUarrSvcOption@@PAUarrCallEndReason@@PAUarrAlphaIDInfo@@PAUarrPeerNumInfo@@PAUarrDiagInfo@@77PAUarrAlertingPattern@@@Z 1001c89c f   SwiNotify.obj
 0001:0001be34       ?InfoRecCallback@CSwiNotify@@SAXPAEPAUsignalInfo@@PAUcallerIDInfo@@PAD330PAUpeerNumInfo@@44PAUredirectNumInfo@@0000PAUlineCtlInfo@@PAUextDisplayInfo@@@Z 1001ce34 f   SwiNotify.obj
 0001:0001c124       ?USSDCallback@CSwiNotify@@SAXPAEPAUUSSInfo@@@Z 1001d124 f   SwiNotify.obj
 0001:0001c280       ?ReadSIMPhoneBookCallback@CSwiNotify@@SAXEGPAUarrPBInfo@@@Z 1001d280 f   SwiNotify.obj
 0001:0001c448       ?AllSIMPhonebookInitDoneCallback@CSwiNotify@@SAXEPAEPAG@Z 1001d448 f   SwiNotify.obj
 0001:0001c4ec       ?EmergencyListCallback@CSwiNotify@@SAXEPAUemergencyNumberEntry@@@Z 1001d4ec f   SwiNotify.obj
 0001:0001c6b0       ?NetworkIdentityAndTimeZoneCallback@@YAXGEEEEEEEE@Z 1001d6b0 f   SwiNotify.obj
 0001:0001c76c       ?EmergencyModeCallback@@YAXPAE@Z 1001d76c f   SwiNotify.obj
 0001:0001c824       ?SessionStateCallback@CSwiNotify@@SAXKK@Z 1001d824 f   SwiNotify.obj
 0001:0001c8b4       ?ActivationStatusCallback@CSwiNotify@@SAXK@Z 1001d8b4 f   SwiNotify.obj
 0001:0001c934       ?GobiAPIPowerCallback@@YAXK@Z 1001d934 f   SwiNotify.obj
 0001:0001c978       ?PowerCallback@CSwiNotify@@SAXPAX@Z 1001d978 f   SwiNotify.obj
 0001:0001c9f8       ?GobiAPIRoamingIndicatorCallback@@YAXK@Z 1001d9f8 f   SwiNotify.obj
 0001:0001ca3c       ?RoamingIndicatorCallback@CSwiNotify@@SAXPAX@Z 1001da3c f   SwiNotify.obj
 0001:0001cabc       ?GobiAPISignalStrengthCallback@@YAXCK@Z 1001dabc f   SwiNotify.obj
 0001:0001cb18       ?SignalStrengthCallback@CSwiNotify@@SAXPAX@Z 1001db18 f   SwiNotify.obj
 0001:0001cba0       ?GobiAPIRFinfoCallback@@YAXKKK@Z 1001dba0 f   SwiNotify.obj
 0001:0001cbe4       ?RFinfoCallback@CSwiNotify@@SAXK@Z 1001dbe4 f   SwiNotify.obj
 0001:0001cc64       ?NewSMSCallback@@YAXKK@Z   1001dc64 f   SwiNotify.obj
 0001:0001cd98       ?NewSMSCBCallback@@YAXEKEGPAE@Z 1001dd98 f   SwiNotify.obj
 0001:0001ce20       ?VoiceMessageCallback@@YAXEPAE00@Z 1001de20 f   SwiNotify.obj
 0001:0001cfa8       ?GobiAPIDataCapabilities@@YAXEPAE@Z 1001dfa8 f   SwiNotify.obj
 0001:0001d06c       ?ByteTotalsCallback@CSwiNotify@@SAX_K0@Z 1001e06c f   SwiNotify.obj
 0001:0001d10c       ?GobiAPIOMADMStateCallback@@YAXKK@Z 1001e10c f   SwiNotify.obj
 0001:0001d148       ?GobiAPIOMADMAlertCallback@@YAXKG@Z 1001e148 f   SwiNotify.obj
 0001:0001d1e8       ?OMADMStateCallback@CSwiNotify@@SAXK@Z 1001e1e8 f   SwiNotify.obj
 0001:0001d270       ?OMADMAlertCallback@CSwiNotify@@SAXPAX@Z 1001e270 f   SwiNotify.obj
 0001:0001d2f0       ?RemoveAll@CSwiNotify@@QAAXXZ 1001e2f0 f   SwiNotify.obj
 0001:0001d418       ?LocateCallbackFn@CSwiNotify@@QAAHW4SWI_TYPE_Notify@@W4eCBAdminOperation@@PAHPAK@Z 1001e418 f   SwiNotify.obj
 0001:0001da88       ??1szCallbackItem@@QAA@XZ  1001ea88 f i SwiNotify.obj
 0001:0001dad8       ?Add@CSwiNotify@@QAA?AW4SWI_RCODE@@W4SWI_TYPE_Notify@@K@Z 1001ead8 f   SwiNotify.obj
 0001:0001e150       ?Remove@CSwiNotify@@QAA?AW4SWI_RCODE@@W4SWI_TYPE_Notify@@K@Z 1001f150 f   SwiNotify.obj
 0001:0001e590       ?HandleSignalStrengthCallback@CSwiNotify@@QAAHPAXCK@Z 1001f590 f   SwiNotify.obj
 0001:0001ef5c       ?HandleSessionStateCallback@CSwiNotify@@QAAHPAXKK@Z 1001ff5c f   SwiNotify.obj
 0001:0001f2b4       ?HandleRoamingIndicatorCallback@CSwiNotify@@QAAHPAXK@Z 100202b4 f   SwiNotify.obj
 0001:0001f7ec       ?HandlePowerCallback@CSwiNotify@@QAAHPAXK@Z 100207ec f   SwiNotify.obj
 0001:0001fa64       ?HandleActivationStatusCallback@CSwiNotify@@QAAHPAXK@Z 10020a64 f   SwiNotify.obj
 0001:0001fc68       ?HandleOMADMStateCallback@CSwiNotify@@QAAHPAXK@Z 10020c68 f   SwiNotify.obj
 0001:0001fe5c       ?HandleOMADMAlertCallback@CSwiNotify@@QAAHPAX@Z 10020e5c f   SwiNotify.obj
 0001:00020088       ?HandleByteTotalsCallback@CSwiNotify@@QAAHPAX_K1@Z 10021088 f   SwiNotify.obj
 0001:000202bc       ?HandleRFinfoCallback@CSwiNotify@@QAAHPAXK@Z 100212bc f   SwiNotify.obj
 0001:00020470       ?HandleSuspend@CSwiNotify@@QAAXXZ 10021470 f   SwiNotify.obj
 0001:000205f4       ?HandleResume@CSwiNotify@@QAAXXZ 100215f4 f   SwiNotify.obj
 0001:00020728       ??1?$basic_string@DU?$char_traits@D@std@@V?$allocator@D@2@@std@@QAA@XZ 10021728 f i SwiNotify.obj
 0001:00020734       ??1?$list@UszCallbackItem@@V?$allocator@UszCallbackItem@@@std@@@std@@QAA@XZ 10021734 f i SwiNotify.obj
 0001:000207dc       ?erase@?$list@UszCallbackItem@@V?$allocator@UszCallbackItem@@@std@@@std@@QAA?AV?$_Iterator@$00@12@V312@@Z 100217dc f i SwiNotify.obj
 0001:000208a8       ??E?$_Iterator@$00@?$list@UszNotifyItem@@V?$allocator@UszNotifyItem@@@std@@@std@@QAA?AV012@H@Z 100218a8 f i SwiNotify.obj
 0001:000208a8       ??E?$_Iterator@$00@?$list@UszCallbackItem@@V?$allocator@UszCallbackItem@@@std@@@std@@QAA?AV012@H@Z 100218a8 f i SwiNotify.obj
 0001:000208f8       ??9?$_Const_iterator@$00@?$list@UszNotifyItem@@V?$allocator@UszNotifyItem@@@std@@@std@@QBA_NABV012@@Z 100218f8 f i SwiNotify.obj
 0001:000208f8       ??9?$_Const_iterator@$00@?$list@UszCallbackItem@@V?$allocator@UszCallbackItem@@@std@@@std@@QBA_NABV012@@Z 100218f8 f i SwiNotify.obj
 0001:0002094c       ?assign@?$basic_string@DU?$char_traits@D@std@@V?$allocator@D@2@@std@@QAAAAV12@ABV12@II@Z 1002194c f i SwiNotify.obj
 0001:00020a10       ?_Tidy@?$basic_string@DU?$char_traits@D@std@@V?$allocator@D@2@@std@@IAAX_NI@Z 10021a10 f i SwiNotify.obj
 0001:00020a78       ?_Insert@?$list@UszNotifyItem@@V?$allocator@UszNotifyItem@@@std@@@std@@QAAXV?$_Iterator@$00@12@ABUszNotifyItem@@@Z 10021a78 f i SwiNotify.obj
 0001:00020b44       ?_Buynode@?$list@UszNotifyItem@@V?$allocator@UszNotifyItem@@@std@@@std@@IAAPAU_Node@?$_List_nod@UszNotifyItem@@V?$allocator@UszNotifyItem@@@std@@@2@XZ 10021b44 f i SwiNotify.obj
 0001:00020b64       ?_Buynode@?$list@UszCallbackItem@@V?$allocator@UszCallbackItem@@@std@@@std@@IAAPAU_Node@?$_List_nod@UszCallbackItem@@V?$allocator@UszCallbackItem@@@std@@@2@XZ 10021b64 f i SwiNotify.obj
 0001:00020b84       ?erase@?$basic_string@DU?$char_traits@D@std@@V?$allocator@D@2@@std@@QAAAAV12@II@Z 10021b84 f i SwiNotify.obj
 0001:00020c18       ?_Grow@?$basic_string@DU?$char_traits@D@std@@V?$allocator@D@2@@std@@IAA_NI_N@Z 10021c18 f i SwiNotify.obj
 0001:00020cbc       ?_Buynode@?$list@UszNotifyItem@@V?$allocator@UszNotifyItem@@@std@@@std@@IAAPAU_Node@?$_List_nod@UszNotifyItem@@V?$allocator@UszNotifyItem@@@std@@@2@PAU342@0ABUszNotifyItem@@@Z 10021cbc f i SwiNotify.obj
 0001:00020d04       ?_Buynode@?$list@UszCallbackItem@@V?$allocator@UszCallbackItem@@@std@@@std@@IAAPAU_Node@?$_List_nod@UszCallbackItem@@V?$allocator@UszCallbackItem@@@std@@@2@PAU342@0ABUszCallbackItem@@@Z 10021d04 f i SwiNotify.obj
 0001:00020da0       ??0length_error@std@@QAA@ABV01@@Z 10021da0 f i SwiNotify.obj
 0001:00020dc8       ??0logic_error@std@@QAA@ABV01@@Z 10021dc8 f i SwiNotify.obj
 0001:00020e40       ??0?$basic_string@DU?$char_traits@D@std@@V?$allocator@D@2@@std@@QAA@PBD@Z 10021e40 f i SwiNotify.obj
 0001:00020e80       ?_Copy@?$basic_string@DU?$char_traits@D@std@@V?$allocator@D@2@@std@@IAAXII@Z 10021e80 f i SwiNotify.obj
 0001:00020fc8       ?assign@?$basic_string@DU?$char_traits@D@std@@V?$allocator@D@2@@std@@QAAAAV12@PBDI@Z 10021fc8 f i SwiNotify.obj
 0001:00021068       ?_Inside@?$basic_string@DU?$char_traits@D@std@@V?$allocator@D@2@@std@@IAA_NPBD@Z 10022068 f i SwiNotify.obj
 0001:000210a8       ??$_Allocate@D@std@@YAPADIPAD@Z 100220a8 f i SwiNotify.obj
 0001:00021114       ??0bad_alloc@std@@QAA@ABV01@@Z 10022114 f i SwiNotify.obj
 0001:0002113c       ??0?$list@UszNotifyItem@@V?$allocator@UszNotifyItem@@@std@@@std@@QAA@ABV01@@Z 1002213c f i SwiNotify.obj
 0001:00021220       ??$_Insert@V?$_Const_iterator@$00@?$list@UszNotifyItem@@V?$allocator@UszNotifyItem@@@std@@@std@@@?$list@UszNotifyItem@@V?$allocator@UszNotifyItem@@@std@@@std@@QAAXV?$_Iterator@$00@01@V?$_Const_iterator@$00@01@1Uforward_iterator_tag@1@@Z 10022220 f i SwiNotify.obj
 0001:000213a4       ?SemiByteToChar@@YADEH@Z   100223a4 f   util.obj
 0001:00021410       ?SemiByteCharsToByte@@YAEDD@Z 10022410 f   util.obj
 0001:00021454       ?ComposeCmdWithByteArray@@YAHQBDQBEI0AAPAD@Z 10022454 f   util.obj
 0001:00021660       ?AllocateOrReallocateStorage@@YAHQAPAEIIQAII@Z 10022660 f   util.obj
 0001:0002176c       ?DumpMem@@YAXPAXH@Z        1002276c f   util.obj
 0001:00022028       __security_check_cookie    10023028     corelibc:armsecgs.obj
 0001:0002203c       __gsfailure                1002303c     corelibc:armsecgs.obj
 0001:00022080       _onexit                    10023080 f   corelibc:onexit.obj
 0001:0002212c       atexit                     1002312c f   corelibc:onexit.obj
 0001:0002214c       _DllMainCRTStartup         1002314c f   corelibc:pegdmain.obj
 0001:000221e4       _cinit                     100231e4 f   corelibc:crt0dat.obj
 0001:00022354       _cexit                     10023354 f   corelibc:crt0dat.obj
 0001:00022370       __security_init_cookie     10023370 f   corelibc:seccinit.obj
 0001:000223c0       ntohl                      100233c0 f   ws2:WS2.dll
 0001:000223d0       inet_ntoa                  100233d0 f   ws2:WS2.dll
 0001:000223e0       ?strncpyz@@YAPADQADQBDI@Z  100233e0 f   toolbox:toolbox_i.obj
 0001:00022438       strspn                     10023438 f   coredll:COREDLL.dll
 0001:00022448       ??3@YAXPAX@Z               10023448 f   coredll:COREDLL.dll
 0001:00022458       strstr                     10023458 f   coredll:COREDLL.dll
 0001:00022468       LocalAlloc                 10023468 f   coredll:COREDLL.dll
 0001:00022478       LocalFree                  10023478 f   coredll:COREDLL.dll
 0001:00022488       strchr                     10023488 f   coredll:COREDLL.dll
 0001:00022498       ??2@YAPAXI@Z               10023498 f   coredll:COREDLL.dll
 0001:000224a8       InitializeCriticalSection  100234a8 f   coredll:COREDLL.dll
 0001:000224b8       DeleteCriticalSection      100234b8 f   coredll:COREDLL.dll
 0001:000224c8       EnterCriticalSection       100234c8 f   coredll:COREDLL.dll
 0001:000224d8       LeaveCriticalSection       100234d8 f   coredll:COREDLL.dll
 0001:000224e8       NKDbgPrintfW               100234e8 f   coredll:COREDLL.dll
 0001:000224f8       swscanf                    100234f8 f   coredll:COREDLL.dll
 0001:00022508       GetLastError               10023508 f   coredll:COREDLL.dll
 0001:00022518       _snprintf                  10023518 f   coredll:COREDLL.dll
 0001:00022528       ??_U@YAPAXI@Z              10023528 f   coredll:COREDLL.dll
 0001:00022538       ??_V@YAXPAX@Z              10023538 f   coredll:COREDLL.dll
 0001:00022548       sscanf                     10023548 f   coredll:COREDLL.dll
 0001:00022558       malloc                     10023558 f   coredll:COREDLL.dll
 0001:00022568       free                       10023568 f   coredll:COREDLL.dll
 0001:00022578       CloseHandle                10023578 f   coredll:COREDLL.dll
 0001:00022588       CreateThread               10023588 f   coredll:COREDLL.dll
 0001:00022598       wcsstr                     10023598 f   coredll:COREDLL.dll
 0001:000225a8       Sleep                      100235a8 f   coredll:COREDLL.dll
 0001:000225b8       strtoul                    100235b8 f   coredll:COREDLL.dll
 0001:000225c8       MultiByteToWideChar        100235c8 f   coredll:COREDLL.dll
 0001:000225d8       sprintf                    100235d8 f   coredll:COREDLL.dll
 0001:000225e8       atol                       100235e8 f   coredll:COREDLL.dll
 0001:000225f8       swprintf                   100235f8 f   coredll:COREDLL.dll
 0001:00022608       _wtol                      10023608 f   coredll:COREDLL.dll
 0001:00022618       CreateFileW                10023618 f   coredll:COREDLL.dll
 0001:00022628       SetLastError               10023628 f   coredll:COREDLL.dll
 0001:00022638       GetCommState               10023638 f   coredll:COREDLL.dll
 0001:00022648       SetCommTimeouts            10023648 f   coredll:COREDLL.dll
 0001:00022658       SetupComm                  10023658 f   coredll:COREDLL.dll
 0001:00022668       toupper                    10023668 f   coredll:COREDLL.dll
 0001:00022678       SetCommState               10023678 f   coredll:COREDLL.dll
 0001:00022688       PurgeComm                  10023688 f   coredll:COREDLL.dll
 0001:00022698       GetTickCount               10023698 f   coredll:COREDLL.dll
 0001:000226a8       ReadFile                   100236a8 f   coredll:COREDLL.dll
 0001:000226b8       WriteFile                  100236b8 f   coredll:COREDLL.dll
 0001:000226c8       GetProcAddressW            100236c8 f   coredll:COREDLL.dll
 0001:000226d8       FreeLibrary                100236d8 f   coredll:COREDLL.dll
 0001:000226e8       LoadLibraryW               100236e8 f   coredll:COREDLL.dll
 0001:000226f8       ??1exception@std@@UAA@XZ   100236f8 f   coredll:COREDLL.dll
 0001:00022708       ??0exception@std@@QAA@PBD@Z 10023708 f   coredll:COREDLL.dll
 0001:00022718       ??0exception@std@@QAA@XZ   10023718 f   coredll:COREDLL.dll
 0001:00022728       ??_7type_info@@6B@         10023728 f   coredll:COREDLL.dll
 0001:00022738       ??0exception@std@@QAA@ABV01@@Z 10023738 f   coredll:COREDLL.dll
 0001:00022748       ?what@exception@std@@UBAPBDXZ 10023748 f   coredll:COREDLL.dll
 0001:00022758       __report_gsfailure         10023758 f   coredll:COREDLL.dll
 0001:00022768       LocalReAlloc               10023768 f   coredll:COREDLL.dll
 0001:00022778       LocalSize                  10023778 f   coredll:COREDLL.dll
 0001:00022788       __security_gen_cookie      10023788 f   coredll:COREDLL.dll
 0001:00022798       wcsncpy                    10023798 f   coredll:COREDLL.dll
 0001:000227a8       wcslen                     100237a8 f   coredll:COREDLL.dll
 0001:000227b8       strncpy                    100237b8 f   coredll:COREDLL.dll
 0001:000227c8       strlen                     100237c8 f   coredll:COREDLL.dll
 0001:000227d8       wcscpy                     100237d8 f   coredll:COREDLL.dll
 0001:000227e8       __C_specific_handler       100237e8 f   coredll:COREDLL.dll
 0001:000227f8       memmove                    100237f8 f   coredll:COREDLL.dll
 0001:00022808       memcpy                     10023808 f   coredll:COREDLL.dll
 0001:00022818       wcscmp                     10023818 f   coredll:COREDLL.dll
 0001:00022828       strcpy_s                   10023828 f   LIBCMT:strcpy_s.obj
 0001:000228e8       memcpy_s                   100238e8 f   LIBCMT:memcpy_s.obj
 0001:000229d0       memmove_s                  100239d0 f   LIBCMT:memmove_s.obj
 0001:00022a88       _invalid_parameter_noinfo  10023a88 f   LIBCMT:invarg.obj
 0001:00022ac4       _invoke_watson             10023ac4 f   LIBCMT:invarg.obj
 0001:00022af0       _invalid_parameter         10023af0 f   LIBCMT:invarginternal.obj
 0001:00022b1c       ??1out_of_range@std@@UAA@XZ 10023b1c f i libcpmt:string.obj
 0001:00022b48       ??_Gout_of_range@std@@UAAPAXI@Z 10023b48 f i libcpmt:string.obj
 0001:00022b48       ??_Eout_of_range@std@@UAAPAXI@Z 10023b48 f i libcpmt:string.obj
 0001:00022b9c       ?_Xlen@_String_base@std@@SAXXZ 10023b9c f   libcpmt:string.obj
 0001:00022c2c       ?_Xran@_String_base@std@@SAXXZ 10023c2c f   libcpmt:string.obj
 0001:00022cb4       ??0out_of_range@std@@QAA@ABV01@@Z 10023cb4 f i libcpmt:string.obj
 0001:00022ce4       memset                     10023ce4 f   coredll:COREDLL.dll
 0001:00022cf4       RaiseException             10023cf4 f   coredll:COREDLL.dll
 0001:00022d04       __CxxThrowException        10023d04 f   coredll:COREDLL.dll
 0001:00022d1c       __FrameUnwindToState       10023d1c f   LIBCMT:frame_ce.obj
 0001:00023094       ?_DestructExceptionObject@@YAXPAUEHExceptionRecord@@E@Z 10024094 f   LIBCMT:frame_ce.obj
 0001:00023100       ?_OffsetToAddress@@YAPAXHPAKK@Z 10024100 f   LIBCMT:frame_ce.obj
 0001:0002314c       ?FindFrameInfo@@YAPAU_FrameInfo@@PAK@Z 1002414c f   LIBCMT:frame_ce.obj
 0001:0002318c       ?FindCatchFrameInfo@@YAPAU_FrameInfo@@PAK@Z 1002418c f   LIBCMT:frame_ce.obj
 0001:000231cc       ?_GetRangeOfTrysToCheck@@YAPBU_s_TryBlockMapEntry@@PBU_s_FuncInfo@@HHPAI1@Z 100241cc f   LIBCMT:frame_ce.obj
 0001:00023bd8       __InternalCxxFrameHandler  10024bd8 f   LIBCMT:frame_ce.obj
 0001:00023d30       __CxxFrameHandler3         10024d30 f   LIBCMT:frame_ce.obj
 0001:00023d68       GetCRTStorage              10024d68 f   LIBCMT:corecrt.obj
 0001:00023e34       _CallSettingFrame          10024e34     LIBCMT:handlers_arm.obj
 0001:00023e78       ?FindFrameForUnwind@@YAPAKPAKPBU_s_FuncInfo@@@Z 10024e78 f   LIBCMT:mdframe_arm.obj
 0001:00023ec0       ?FindCatchFrame@@YAPAKPAKK@Z 10024ec0 f   LIBCMT:mdframe_arm.obj
 0001:00023f0c       ?AdjustFrameForCatch@@YAPAKPAKPBU_s_FuncInfo@@@Z 10024f0c f   LIBCMT:mdframe_arm.obj
 0001:00023f44       ?GetCurrentState@@YAHPAKPAU_DISPATCHER_CONTEXT@@PBU_s_FuncInfo@@@Z 10024f44 f   LIBCMT:ehstate_arm_mips.obj
 0001:00023fa0       strcmp                     10024fa0 f   coredll:COREDLL.dll
 0001:00023fb0       ?terminate@std@@YAXXZ      10024fb0 f   coredll:COREDLL.dll
 0001:00023fc0       TlsCall                    10024fc0 f   coredll:COREDLL.dll
 0001:00023fd0       TlsSetValue                10024fd0 f   coredll:COREDLL.dll
 0001:00023fe0       TlsGetValue                10024fe0 f   coredll:COREDLL.dll
 0001:00023ff0       InterlockedCompareExchange 10024ff0 f   coredll:COREDLL.dll
 0001:00024000       strcpy                     10025000 f   coredll:COREDLL.dll
 0001:00024010       strcat                     10025010 f   coredll:COREDLL.dll
 0001:00024020       wcscat                     10025020 f   coredll:COREDLL.dll
 0001:00024030       __GSHandlerCheckCommon     10025030 f   LIBCMT:gshandler.obj
 0001:00024078       __GSHandlerCheck           10025078 f   LIBCMT:gshandler.obj
 0001:000240a8       __GSHandlerCheck_EH        100250a8 f   LIBCMT:gshandlereh.obj
 0002:00000020       ??_7bad_alloc@std@@6B@     10026020     libcpmt:string.obj
 0002:0000002c       ??_7logic_error@std@@6B@   1002602c     libcpmt:string.obj
 0002:00000038       ??_7length_error@std@@6B@  10026038     libcpmt:string.obj
 0002:00000044       ??_7out_of_range@std@@6B@  10026044     libcpmt:string.obj
 0002:00000098       ??_C@_0BA@JFNIOLAK@string?5too?5long?$AA@ 10026098     libcpmt:string.obj
 0002:000000f4       ??_C@_0BI@CFPLBAOH@invalid?5string?5position?$AA@ 100260f4     libcpmt:string.obj
 0002:0000010c       ??_C@_01CLKCMJKC@?5?$AA@   1002610c     parse.obj
 0002:00000110       ??_C@_02PCIJFNDE@?$AN?6?$AA@ 10026110     parse.obj
 0002:00000114       ??_C@_0P@GHFPNOJB@bad?5allocation?$AA@ 10026114     SDKRIL.obj
 0002:00000124       ??_C@_1BK@MLJBIMDO@?$AA?4?$AA?2?$AAS?$AAD?$AAK?$AAR?$AAI?$AAL?$AA?4?$AAc?$AAp?$AAp?$AA?$AA@ 10026124     SDKRIL.obj
 0002:00000140       ??_C@_1DI@NBJEIDEF@?$AAD?$AAe?$AAv?$AAi?$AAc?$AAe?$AAR?$AAe?$AAm?$AAo?$AAv?$AAa?$AAl?$AA?0?$AA?5?$AAn?$AAS?$AAt?$AAa?$AAt?$AAu?$AAs?$AA?5?$AA?$DN?$AA?5?$AA?$CF?$AAd?$AA?$AA@ 10026140     SDKRIL.obj
 0002:00000178       ??_C@_1EM@BCCGAMIL@?$AAS?$AAD?$AAK?$AAR?$AAI?$AAL?$AA?5?$AAd?$AAl?$AAl?$AA?5?$AAi?$AAs?$AA?5?$AAa?$AAt?$AAt?$AAa?$AAc?$AAh?$AAe?$AAd?$AA?5?$AAt?$AAo?$AA?5?$AAa?$AA?5?$AAp?$AAr?$AAo?$AAc@ 10026178     SDKRIL.obj
 0002:000001c8       ??_C@_1EK@HIJMKGAB@?$AAS?$AAw?$AAi?$AAA?$AAp?$AAi?$AAS?$AAh?$AAu?$AAt?$AAd?$AAo?$AAw?$AAn?$AA?3?$AA?3?$AAI?$AAn?$AAs?$AAi?$AAd?$AAe?$AA?5?$AA?5?$AAS?$AAW?$AAI?$AAS?$AAY?$AAN?$AAC?$AAB@ 100261c8     SDKRIL.obj
 0002:00000214       ??_C@_1BC@FDHFOMEN@?$AAD?$AAe?$AAv?$AAi?$AAc?$AAe?$AAI?$AAD?$AA?$AA@ 10026214     SDKRIL.obj
 0002:00000228       ??_C@_1DK@DFOPCCDF@?$AAS?$AAo?$AAf?$AAt?$AAw?$AAa?$AAr?$AAe?$AA?2?$AAS?$AAi?$AAe?$AAr?$AAr?$AAa?$AA?5?$AAW?$AAi?$AAr?$AAe?$AAl?$AAe?$AAs?$AAs?$AA?5?$AAI?$AAn?$AAc?$AA?$AA@ 10026228     SDKRIL.obj
 0002:00000264       ??_C@_1BM@EJJJFNJP@?$AAV?$AAI?$AAD?$AA_?$AA?$CF?$AAx?$AA?$CG?$AAP?$AAI?$AAD?$AA_?$AA?$CF?$AAx?$AA?$AA@ 10026264     SDKRIL.obj
 0002:00000280       ??_C@_1HI@HMEJCFGL@?$AAD?$AAE?$AAB?$AAU?$AAG?$AA?3?$AA?5?$AAv?$AAi?$AAd?$AAp?$AAi?$AAd?$AAS?$AAt?$AAr?$AA?5?$AAd?$AAe?$AAt?$AAe?$AAc?$AAt?$AAe?$AAd?$AA?5?$AAi?$AAs?$AA?5?$AA?$CF?$AAs?$AA?0@ 10026280     SDKRIL.obj
 0002:000002f8       ??_C@_1EI@PINDODPK@?$AAV?$AAi?$AAd?$AA?5?$AA?$DN?$AA?5?$AA?$CF?$AAd?$AA?5?$AAa?$AAn?$AAd?$AA?5?$AAP?$AAi?$AAd?$AA?5?$AA?$DN?$AA?5?$AA?$CF?$AAd?$AA?0?$AA?5?$AAd?$AAo?$AA?5?$AAn?$AAo?$AAt?$AA?5?$AAm?$AAa@ 100262f8     SDKRIL.obj
 0002:00000340       ??_C@_1EK@DEJGFAAH@?$AAF?$AAa?$AAi?$AAl?$AAe?$AAd?$AA?5?$AAt?$AAo?$AA?5?$AAr?$AAe?$AAa?$AAd?$AA?5?$AAD?$AAe?$AAv?$AAi?$AAc?$AAe?$AA?5?$AAI?$AAD?$AA?0?$AA?5?$AAe?$AAr?$AAr?$AAo?$AAr?$AA?5@ 10026340     SDKRIL.obj
 0002:0000038c       ??_C@_1CI@CEFCOHFP@?$AAA?$AAP?$AAI?$AA?5?$AAn?$AAo?$AAt?$AA?5?$AAi?$AAn?$AAi?$AAt?$AAi?$AAa?$AAl?$AAi?$AAz?$AAe?$AAd?$AA?$AA@ 1002638c     SDKRIL.obj
 0002:000003b4       ??_C@_1BM@LGIGLBBH@?$AAD?$AAe?$AAv?$AAi?$AAc?$AAe?$AA?5?$AAI?$AAD?$AA?3?$AA?5?$AA?$CF?$AAi?$AA?$AA@ 100263b4     SDKRIL.obj
 0002:000003d0       ??_C@_1EO@HHOKFBLA@?$AAS?$AAD?$AAK?$AAR?$AAI?$AAL?$AA?5?$AAd?$AAo?$AA?5?$AAn?$AAo?$AAt?$AA?5?$AAh?$AAa?$AAn?$AAd?$AAl?$AAe?$AA?5?$AAd?$AAe?$AAv?$AAi?$AAc?$AAe?$AAI?$AAD?$AA?5?$AA?$DN?$AA?5@ 100263d0     SDKRIL.obj
 0002:00000420       ??_C@_1EC@INGBEEGE@?$AAS?$AAw?$AAi?$AAS?$AAe?$AAl?$AAe?$AAc?$AAt?$AAA?$AAi?$AAr?$AAS?$AAe?$AAr?$AAv?$AAe?$AAr?$AA?5?$AAr?$AAe?$AAt?$AAu?$AAr?$AAn?$AAi?$AAn?$AAg?$AA?3?$AA?5?$AA?$CF?$AAd@ 10026420     SDKRIL.obj
 0002:00000468       ??_C@_1GE@JLHEEOOA@?$AA?$CK?$AA?$CK?$AA?$CK?$AA?$CK?$AA?$CK?$AAC?$AAo?$AAu?$AAl?$AAd?$AA?5?$AAn?$AAo?$AAt?$AA?5?$AAd?$AAe?$AAt?$AAe?$AAr?$AAm?$AAi?$AAn?$AAe?$AA?5?$AAw?$AAi?$AAr?$AAe?$AAl?$AAe?$AAs@ 10026468     SDKRIL.obj
 0002:000004cc       ??_C@_1CI@PFNIEBMJ@?$AAP?$AAR?$AAI?$AA?5?$AAv?$AAe?$AAr?$AAs?$AAi?$AAo?$AAn?$AA?5?$AAi?$AAs?$AA?5?$AA?$DN?$AA?5?$AA?$CF?$AAs?$AA?$AA@ 100264cc     SDKRIL.obj
 0002:000004f4       ??_C@_1BA@GKCOAPMF@?$AAC?$AAo?$AAm?$AAP?$AAo?$AAr?$AAt?$AA?$AA@ 100264f4     SDKRIL.obj
 0002:00000504       ??_C@_1CO@PFFMHNAH@?$AAS?$AAo?$AAf?$AAt?$AAw?$AAa?$AAr?$AAe?$AA?2?$AAM?$AAi?$AAc?$AAr?$AAo?$AAs?$AAo?$AAf?$AAt?$AA?2?$AAR?$AAI?$AAL?$AA?$AA@ 10026504     SDKRIL.obj
 0002:00000534       ??_C@_09PGLNONHM@AT?$CLCMEE?$DN1?$AA@ 10026534     SDKRIL.obj
 0002:00000540       ??_C@_1EG@GCNCAOG@?$AAA?$AAT?$AA?$CL?$AAC?$AAM?$AAE?$AAE?$AA?$DN?$AA1?$AA?5?$AAA?$AAT?$AA?5?$AAc?$AAm?$AAd?$AA?5?$AAe?$AAr?$AAr?$AAo?$AAr?$AA?5?$AAs?$AAt?$AAr?$AAi?$AAn?$AAg?$AA?5?$AA?$DN?$AA?5@ 10026540     SDKRIL.obj
 0002:00000588       ??_C@_1FO@PAMEOBJK@?$AAM?$AAo?$AAb?$AAi?$AAl?$AAe?$AA?5?$AAT?$AAe?$AAr?$AAm?$AAi?$AAn?$AAa?$AAt?$AAi?$AAo?$AAn?$AA?5?$AAE?$AAr?$AAr?$AAo?$AAr?$AA?5?$AAV?$AAa?$AAl?$AAu?$AAe?$AAs?$AA?5@ 10026588     SDKRIL.obj
 0002:000005e8       ??_C@_1HC@NPPPPNDG@?$AAF?$AAa?$AAi?$AAl?$AAe?$AAd?$AA?5?$AAt?$AAo?$AA?5?$AAs?$AAe?$AAt?$AA?5?$AAM?$AAo?$AAb?$AAi?$AAl?$AAe?$AA?5?$AAT?$AAe?$AAr?$AAm?$AAi?$AAn?$AAa?$AAt?$AAi?$AAo?$AAn@ 100265e8     SDKRIL.obj
 0002:0000065c       ??_C@_1DE@LJFKPKJL@?$AAA?$AAT?$AA?5?$AAP?$AAo?$AAr?$AAt?$AA?5?$AAI?$AAn?$AAi?$AAt?$AAi?$AAa?$AAl?$AAi?$AAz?$AAe?$AA?5?$AAf?$AAa?$AAi?$AAl?$AAe?$AAd?$AA?$AA@ 1002665c     SDKRIL.obj
 0002:00000690       ??_C@_1EC@FHIHNHOA@?$AAC?$AAa?$AAn?$AAn?$AAo?$AAt?$AA?5?$AAo?$AAp?$AAe?$AAn?$AA?5?$AAR?$AAe?$AAg?$AAi?$AAs?$AAt?$AAr?$AAy?$AA?5?$AAf?$AAo?$AAr?$AA?5?$AAA?$AAT?$AA?5?$AAp?$AAo?$AAr?$AAt@ 10026690     SDKRIL.obj
 0002:000006d8       ??_C@_1GM@OKHAADI@?$AAN?$AAa?$AAm?$AAe?$AA?3?$AA?5?$AA?$CF?$AAs?$AA?5?$AA?9?$AA?5?$AAC?$AAl?$AAa?$AAs?$AAs?$AA?3?$AA?5?$AA?$CF?$AAi?$AA?5?$AA?9?$AA?5?$AAI?$AAn?$AAt?$AAe?$AAr?$AAf?$AAa?$AAc?$AAe@ 100266d8     SDKRIL.obj
 0002:00000748       ??_C@_1HA@PBCNNPOG@?$AAF?$AAa?$AAi?$AAl?$AAe?$AAd?$AA?5?$AAt?$AAo?$AA?5?$AAg?$AAe?$AAt?$AA?5?$AAa?$AAd?$AAd?$AAi?$AAt?$AAi?$AAo?$AAn?$AAa?$AAl?$AA?5?$AAd?$AAe?$AAv?$AAi?$AAc?$AAe?$AA?5@ 10026748     SDKRIL.obj
 0002:000007b8       ??_C@_1GI@DHLBJFON@?$AAS?$AAe?$AAt?$AAN?$AAe?$AAt?$AAw?$AAo?$AAr?$AAk?$AAP?$AAr?$AAe?$AAf?$AAe?$AAr?$AAe?$AAn?$AAc?$AAe?$AA?5?$AAf?$AAa?$AAi?$AAl?$AAe?$AAd?$AA?0?$AA?5?$AAT?$AAe?$AAc@ 100267b8     SDKRIL.obj
 0002:00000820       ??_C@_1EE@EFFBFFPO@?$AAh?$AAa?$AAn?$AAd?$AAl?$AAe?$AA?3?$AA?5?$AA0?$AAx?$AA?$CF?$AAx?$AA?5?$AAf?$AAi?$AAl?$AAt?$AAe?$AAr?$AA?3?$AA?5?$AA0?$AAx?$AA?$CF?$AA8?$AA?4?$AA8?$AAx?$AA?$CF?$AA8?$AA?4?$AA8@ 10026820     SDKRIL.obj
 0002:00000868       ??_C@_1EG@DHJBFBEC@?$AAG?$AAe?$AAt?$AAH?$AAa?$AAr?$AAd?$AAw?$AAa?$AAr?$AAe?$AAR?$AAe?$AAv?$AAi?$AAs?$AAi?$AAo?$AAn?$AA?5?$AAy?$AAi?$AAe?$AAl?$AAd?$AAs?$AA?5?$AAr?$AAc?$AA?5?$AA?$DN?$AA?5@ 10026868     SDKRIL.obj
 0002:000008b0       ??_C@_1FM@CAAEOAPB@?$AAG?$AAe?$AAt?$AAM?$AAo?$AAd?$AAe?$AAl?$AAI?$AAD?$AA?5?$AAy?$AAi?$AAe?$AAl?$AAd?$AAs?$AA?5?$AAr?$AAc?$AA?5?$AA?$DN?$AA?5?$AA?$CF?$AAd?$AA?0?$AA?5?$AAr?$AAe?$AAm?$AAa?$AAi@ 100268b0     SDKRIL.obj
 0002:00000910       ??_C@_1GG@LHDJALIJ@?$AAG?$AAe?$AAt?$AAM?$AAa?$AAn?$AAu?$AAf?$AAa?$AAc?$AAt?$AAu?$AAr?$AAe?$AAr?$AA?5?$AAy?$AAi?$AAe?$AAl?$AAd?$AAs?$AA?5?$AAr?$AAc?$AA?5?$AA?$DN?$AA?5?$AA?$CF?$AAd?$AA?0?$AA?5@ 10026910     SDKRIL.obj
 0002:00000978       ??_C@_09DOCJFLFE@?$CF2d?$CF4d?$CF2d?$AA@ 10026978     SDKRIL.obj
 0002:00000988       ??_C@_1GO@DLHMCICL@?$AAS?$AAw?$AAi?$AAS?$AAt?$AAa?$AAr?$AAt?$AAD?$AAa?$AAt?$AAa?$AAS?$AAe?$AAs?$AAs?$AAi?$AAo?$AAn?$AA?5?$AAr?$AAe?$AAt?$AAu?$AAr?$AAn?$AAi?$AAn?$AAg?$AA?3?$AA?5?$AA?$CF@ 10026988     SDKRIL.obj
 0002:000009f8       ??_C@_1EC@JOBMIAJ@?$AAS?$AAw?$AAi?$AAS?$AAt?$AAo?$AAp?$AAD?$AAa?$AAt?$AAa?$AAS?$AAe?$AAs?$AAs?$AAi?$AAo?$AAn?$AA?5?$AAr?$AAe?$AAt?$AAu?$AAr?$AAn?$AAi?$AAn?$AAg?$AA?3?$AA?5?$AA?$CF?$AAd@ 100269f8     SDKRIL.obj
 0002:00000a40       ??_C@_1FA@HHFCPODO@?$AAS?$AAw?$AAi?$AAG?$AAe?$AAt?$AAI?$AAP?$AAC?$AAo?$AAn?$AAf?$AAi?$AAg?$AAu?$AAr?$AAa?$AAt?$AAi?$AAo?$AAn?$AAG?$AAo?$AAb?$AAi?$AA?5?$AAr?$AAe?$AAt?$AAu?$AAr?$AAn@ 10026a40     SDKRIL.obj
 0002:00000a90       ??_C@_1DC@BGFGLNND@?$AAG?$AAo?$AAb?$AAi?$AA?5?$AAA?$AAP?$AAI?$AA?5?$AAn?$AAo?$AAt?$AA?5?$AAi?$AAn?$AAi?$AAt?$AAi?$AAa?$AAl?$AAi?$AAz?$AAe?$AAd?$AA?$AA@ 10026a90     SDKRIL.obj
 0002:00000ac4       ??_C@_0M@DNMPLDHO@AT?$CLCLIP?$DN?$CFu?$AN?$AA@ 10026ac4     SDKRIL.obj
 0002:00000ad0       ??_C@_1KA@KOOMEPME@?$AAC?$AAM?$AAE?$AA?5?$AAE?$AAr?$AAr?$AAo?$AAr?$AA?5?$AAv?$AAa?$AAl?$AAu?$AAe?$AAs?$AA?5?$AAf?$AAr?$AAo?$AAm?$AA?5?$AAm?$AAo?$AAd?$AAe?$AAm?$AA?5?$AAa?$AAr?$AAe?$AA?5@ 10026ad0     SDKRIL.obj
 0002:00000b70       ??_C@_1FK@EKNODHPB@?$AAS?$AAw?$AAi?$AAA?$AAT?$AAS?$AAe?$AAt?$AAC?$AAL?$AAI?$AAP?$AA?3?$AA?3?$AAE?$AAx?$AAt?$AAr?$AAa?$AAc?$AAt?$AAe?$AAd?$AA?5?$AAC?$AAM?$AAE?$AA?5?$AAE?$AAr?$AAr?$AAo@ 10026b70     SDKRIL.obj
 0002:00000bd0       ??_C@_1FE@BNGDGGCG@?$AAS?$AAw?$AAi?$AAA?$AAT?$AAS?$AAe?$AAt?$AAC?$AAL?$AAI?$AAP?$AA?3?$AA?5?$AAF?$AAa?$AAi?$AAl?$AAe?$AAd?$AA?5?$AAt?$AAo?$AA?5?$AAe?$AAx?$AAt?$AAr?$AAa?$AAc?$AAt?$AA?5@ 10026bd0     SDKRIL.obj
 0002:00000c24       ??_C@_1CK@FLMLKAMO@?$AAI?$AAs?$AAI?$AAn?$AAi?$AAt?$AAi?$AAa?$AAl?$AAi?$AAz?$AAe?$AAd?$AA?5?$AAf?$AAa?$AAi?$AAl?$AAe?$AAd?$AA?$AA@ 10026c24     SDKRIL.obj
 0002:00000c50       ??_C@_1DK@PMBFKPGH@?$AAS?$AAW?$AAI?$AA_?$AAW?$AAI?$AAR?$AAE?$AAL?$AAE?$AAS?$AAS?$AAT?$AAE?$AAC?$AAH?$AA_?$AAG?$AAs?$AAm?$AA?5?$AAn?$AAo?$AAt?$AA?5?$AAg?$AAs?$AAm?$AA?$AA@ 10026c50     SDKRIL.obj
 0002:00000c8c       ??_C@_1DE@BDLJKCPP@?$AAg?$AA_?$AAA?$AAT?$AAP?$AAo?$AAr?$AAt?$AAI?$AAn?$AAs?$AAt?$AAa?$AAn?$AAc?$AAe?$AA?5?$AAn?$AAo?$AAt?$AA?5?$AAi?$AAn?$AAi?$AAt?$AA?$AA@ 10026c8c     SDKRIL.obj
 0002:00000cc0       ??_C@_09OPKBNJOE@AT?$CLCLIP?$DP?$AN?$AA@ 10026cc0     SDKRIL.obj
 0002:00000cd0       ??_C@_1FK@CDEINALE@?$AAS?$AAw?$AAi?$AAA?$AAT?$AAG?$AAe?$AAt?$AAC?$AAL?$AAI?$AAP?$AA?3?$AA?3?$AAE?$AAx?$AAt?$AAr?$AAa?$AAc?$AAt?$AAe?$AAd?$AA?5?$AAC?$AAM?$AAE?$AA?5?$AAE?$AAr?$AAr?$AAo@ 10026cd0     SDKRIL.obj
 0002:00000d30       ??_C@_1FE@JJMIMIHA@?$AAS?$AAw?$AAi?$AAA?$AAT?$AAG?$AAe?$AAt?$AAC?$AAL?$AAI?$AAP?$AA?3?$AA?5?$AAF?$AAa?$AAi?$AAl?$AAe?$AAd?$AA?5?$AAt?$AAo?$AA?5?$AAe?$AAx?$AAt?$AAr?$AAa?$AAc?$AAt?$AA?5@ 10026d30     SDKRIL.obj
 0002:00000d84       ??_C@_13JGCMLPCH@?$AA1?$AA?$AA@ 10026d84     SDKRIL.obj
 0002:00000d88       ??_C@_1EK@JJCNHCCC@?$AAM?$AAa?$AAt?$AAc?$AAh?$AAS?$AAt?$AAr?$AAi?$AAn?$AAg?$AAB?$AAe?$AAg?$AAi?$AAn?$AAn?$AAi?$AAn?$AAg?$AA?5?$AAf?$AAa?$AAi?$AAl?$AAe?$AAd?$AA?5?$AA?$CI?$AAe?$AAc?$AAh@ 10026d88     SDKRIL.obj
 0002:00000dd4       ??_C@_13IEJJBAMJ@?$AA2?$AA?$AA@ 10026dd4     SDKRIL.obj
 0002:00000dd8       ??_C@_1CO@HIEALLFP@?$AAP?$AAa?$AAr?$AAs?$AAe?$AAR?$AAs?$AAp?$AAP?$AAr?$AAe?$AAf?$AAi?$AAx?$AA?5?$AAf?$AAa?$AAi?$AAl?$AAe?$AAd?$AA?5?$AA?$AA@ 10026dd8     SDKRIL.obj
 0002:00000e08       ??_C@_13DMCFHHKM@?$AA3?$AA?$AA@ 10026e08     SDKRIL.obj
 0002:00000e0c       ??_C@_07BBCOIKBL@?$CLCLIP?3?5?$AA@ 10026e0c     SDKRIL.obj
 0002:00000e14       ??_C@_1DK@IJKEKHNB@?$AAM?$AAa?$AAt?$AAc?$AAh?$AAS?$AAt?$AAr?$AAi?$AAn?$AAg?$AAB?$AAe?$AAg?$AAi?$AAn?$AAn?$AAi?$AAn?$AAg?$AA?5?$AAf?$AAa?$AAi?$AAl?$AAe?$AAd?$AA?5?$AA?$AA@ 10026e14     SDKRIL.obj
 0002:00000e50       ??_C@_13KBPCEPBF@?$AA4?$AA?$AA@ 10026e50     SDKRIL.obj
 0002:00000e54       ??_C@_1CI@KOEGPPLE@?$AAP?$AAa?$AAr?$AAs?$AAe?$AAU?$AAI?$AAn?$AAt?$AA?5?$AA1?$AA?5?$AAf?$AAa?$AAi?$AAl?$AAe?$AAd?$AA?5?$AA?$AA@ 10026e54     SDKRIL.obj
 0002:00000e7c       ??_C@_13BJEOCIHA@?$AA5?$AA?$AA@ 10026e7c     SDKRIL.obj
 0002:00000e80       ??_C@_01IHBHIGKO@?0?$AA@   10026e80     SDKRIL.obj
 0002:00000e84       ??_C@_0M@HAAHBCHF@AT?$CLCLIR?$DN?$CFu?$AN?$AA@ 10026e84     SDKRIL.obj
 0002:00000e90       ??_C@_1FK@IAKFAHLF@?$AAS?$AAw?$AAi?$AAA?$AAT?$AAS?$AAe?$AAt?$AAC?$AAL?$AAI?$AAR?$AA?3?$AA?3?$AAE?$AAx?$AAt?$AAr?$AAa?$AAc?$AAt?$AAe?$AAd?$AA?5?$AAC?$AAM?$AAE?$AA?5?$AAE?$AAr?$AAr?$AAo@ 10026e90     SDKRIL.obj
 0002:00000ef0       ??_C@_1FE@KKCFKAIH@?$AAS?$AAw?$AAi?$AAA?$AAT?$AAS?$AAe?$AAt?$AAC?$AAL?$AAI?$AAR?$AA?3?$AA?5?$AAF?$AAa?$AAi?$AAl?$AAe?$AAd?$AA?5?$AAt?$AAo?$AA?5?$AAe?$AAx?$AAt?$AAr?$AAa?$AAc?$AAt?$AA?5@ 10026ef0     SDKRIL.obj
 0002:00000f44       ??_C@_09EFKIBBGP@AT?$CLCLIR?$DP?$AN?$AA@ 10026f44     SDKRIL.obj
 0002:00000f50       ??_C@_1FK@OJDDOAPA@?$AAS?$AAw?$AAi?$AAA?$AAT?$AAG?$AAe?$AAt?$AAC?$AAL?$AAI?$AAR?$AA?3?$AA?3?$AAE?$AAx?$AAt?$AAr?$AAa?$AAc?$AAt?$AAe?$AAd?$AA?5?$AAC?$AAM?$AAE?$AA?5?$AAE?$AAr?$AAr?$AAo@ 10026f50     SDKRIL.obj
 0002:00000fb0       ??_C@_1FE@COIOAONB@?$AAS?$AAw?$AAi?$AAA?$AAT?$AAG?$AAe?$AAt?$AAC?$AAL?$AAI?$AAR?$AA?3?$AA?5?$AAF?$AAa?$AAi?$AAl?$AAe?$AAd?$AA?5?$AAt?$AAo?$AA?5?$AAe?$AAx?$AAt?$AAr?$AAa?$AAc?$AAt?$AA?5@ 10026fb0     SDKRIL.obj
 0002:00001004       ??_C@_07LLCHECJA@?$CLCLIR?3?5?$AA@ 10027004     SDKRIL.obj
 0002:0000100c       ??_C@_1BK@IBBCMBAP@?$AAS?$AAw?$AAi?$AAA?$AAT?$AAS?$AAe?$AAt?$AAC?$AAO?$AAL?$AAP?$AA?$AA@ 1002700c     SDKRIL.obj
 0002:00001028       ??_C@_1CC@PPKPAHLI@?$AAS?$AAw?$AAi?$AAA?$AAT?$AAR?$AAe?$AAl?$AAe?$AAa?$AAs?$AAe?$AAC?$AAa?$AAl?$AAl?$AA?$AA@ 10027028     SDKRIL.obj
 0002:0000104c       ??_C@_0N@IADMANHI@AT?$CLCHLD?$DN1?$CFu?$AN?$AA@ 1002704c     SDKRIL.obj
 0002:0000105c       ??_C@_1BK@LDAELDBG@?$AAS?$AAw?$AAi?$AAA?$AAT?$AAG?$AAe?$AAt?$AAC?$AAO?$AAL?$AAP?$AA?$AA@ 1002705c     SDKRIL.obj
 0002:00001078       ??_C@_09KBNFCEDK@AT?$CLCOLP?$DP?$AN?$AA@ 10027078     SDKRIL.obj
 0002:00001084       ??_C@_07FPFKHHMF@?$CLCOLP?3?5?$AA@ 10027084     SDKRIL.obj
 0002:0000108c       ??_C@_1BK@CLBLAJIE@?$AAS?$AAw?$AAi?$AAA?$AAT?$AAS?$AAe?$AAt?$AAC?$AAO?$AAL?$AAR?$AA?$AA@ 1002708c     SDKRIL.obj
 0002:000010a8       ??_C@_1BK@BJANHLJN@?$AAS?$AAw?$AAi?$AAA?$AAT?$AAG?$AAe?$AAt?$AAC?$AAO?$AAL?$AAR?$AA?$AA@ 100270a8     SDKRIL.obj
 0002:000010c4       ??_C@_09LNMOMLB@AT?$CLCOLR?$DP?$AN?$AA@ 100270c4     SDKRIL.obj
 0002:000010d0       ??_C@_07PFFDLPEO@?$CLCOLR?3?5?$AA@ 100270d0     SDKRIL.obj
 0002:000010d8       ??_C@_0BC@ELFMDCBL@AT?$CBUNLOCK?$DN?$CCA710?$CC?$AN?$AA@ 100270d8     SDKRIL.obj
 0002:000010f0       ??_C@_1EI@KLLNKDNC@?$AAS?$AAw?$AAi?$AAA?$AAT?$AAS?$AAe?$AAt?$AAE?$AAn?$AAu?$AAm?$AA?5?$AAf?$AAa?$AAi?$AAl?$AAe?$AAd?$AA?5?$AAt?$AAo?$AA?5?$AAu?$AAn?$AAl?$AAo?$AAc?$AAk?$AA?5?$AAm?$AAo@ 100270f0     SDKRIL.obj
 0002:00001138       ??_C@_1FK@NANKOFGF@?$AAS?$AAw?$AAi?$AAA?$AAT?$AAS?$AAe?$AAt?$AAE?$AAn?$AAu?$AAm?$AA?3?$AA?3?$AAE?$AAx?$AAt?$AAr?$AAa?$AAc?$AAt?$AAe?$AAd?$AA?5?$AAC?$AAM?$AAE?$AA?5?$AAE?$AAr?$AAr?$AAo@ 10027138     SDKRIL.obj
 0002:00001198       ??_C@_1FE@KMIBCLIC@?$AAS?$AAw?$AAi?$AAA?$AAT?$AAS?$AAe?$AAt?$AAE?$AAn?$AAu?$AAm?$AA?3?$AA?5?$AAF?$AAa?$AAi?$AAl?$AAe?$AAd?$AA?5?$AAt?$AAo?$AA?5?$AAe?$AAx?$AAt?$AAr?$AAa?$AAc?$AAt?$AA?5@ 10027198     SDKRIL.obj
 0002:000011ec       ??_C@_0O@MPBMFMGD@AT?$CBNVENUM?$DN?$CFs?$AN?$AA@ 100271ec     SDKRIL.obj
 0002:00001200       ??_C@_1FI@CJPAPDEL@?$AAS?$AAw?$AAi?$AAA?$AAT?$AAS?$AAe?$AAt?$AAS?$AAi?$AAd?$AAe?$AAT?$AAo?$AAn?$AAe?$AAG?$AAa?$AAi?$AAn?$AA?5?$AAf?$AAa?$AAi?$AAl?$AAe?$AAd?$AA?5?$AAt?$AAo?$AA?5?$AAu@ 10027200     SDKRIL.obj
 0002:00001258       ??_C@_1GK@CDDDEOBB@?$AAS?$AAw?$AAi?$AAA?$AAT?$AAS?$AAe?$AAt?$AAS?$AAi?$AAd?$AAe?$AAT?$AAo?$AAn?$AAe?$AAG?$AAa?$AAi?$AAn?$AA?3?$AA?3?$AAE?$AAx?$AAt?$AAr?$AAa?$AAc?$AAt?$AAe?$AAd?$AA?5@ 10027258     SDKRIL.obj
 0002:000012c8       ??_C@_1GE@GKOOKPC@?$AAS?$AAw?$AAi?$AAA?$AAT?$AAS?$AAe?$AAt?$AAS?$AAi?$AAd?$AAe?$AAT?$AAo?$AAn?$AAe?$AAG?$AAa?$AAi?$AAn?$AA?3?$AA?5?$AAF?$AAa?$AAi?$AAl?$AAe?$AAd?$AA?5?$AAt?$AAo?$AA?5@ 100272c8     SDKRIL.obj
 0002:0000132c       ??_C@_0BF@KGOPJOCJ@AT?$CBAVCODECSTG?$DN?$CFd?0?$CFx?$AN?$AA@ 1002732c     SDKRIL.obj
 0002:00001344       ??_C@_09JBNCAPNB@AT?$CBRESET?$AN?$AA@ 10027344     SDKRIL.obj
 0002:00001350       ??_C@_1FG@PPPDFGMI@?$AAS?$AAw?$AAi?$AAA?$AAT?$AAR?$AAe?$AAs?$AAe?$AAt?$AA?3?$AA?3?$AAE?$AAx?$AAt?$AAr?$AAa?$AAc?$AAt?$AAe?$AAd?$AA?5?$AAC?$AAM?$AAE?$AA?5?$AAE?$AAr?$AAr?$AAo?$AAr?$AA?5@ 10027350     SDKRIL.obj
 0002:000013a8       ??_C@_1FA@OHKPOOOM@?$AAS?$AAw?$AAi?$AAA?$AAT?$AAR?$AAe?$AAs?$AAe?$AAt?$AA?3?$AA?5?$AAF?$AAa?$AAi?$AAl?$AAe?$AAd?$AA?5?$AAt?$AAo?$AA?5?$AAe?$AAx?$AAt?$AAr?$AAa?$AAc?$AAt?$AA?5?$AAC?$AAM@ 100273a8     SDKRIL.obj
 0002:000013f8       ??_C@_1CK@OOEJNDAF@?$AAS?$AAw?$AAi?$AAA?$AAT?$AAR?$AAe?$AAs?$AAe?$AAt?$AA?3?$AA?3?$AAn?$AAo?$AA?5?$AAE?$AAr?$AAr?$AAo?$AAr?$AA?$AA@ 100273f8     SDKRIL.obj
 0002:00001424       ??_C@_0L@DENDKENN@AT$RTN?$DN?$CFs?$AN?$AA@ 10027424     SDKRIL.obj
 0002:00001430       ??_C@_1FM@NHDKICMM@?$AAS?$AAw?$AAi?$AAA?$AAT?$AAR?$AAt?$AAn?$AAR?$AAe?$AAs?$AAe?$AAt?$AA?3?$AA?3?$AAE?$AAx?$AAt?$AAr?$AAa?$AAc?$AAt?$AAe?$AAd?$AA?5?$AAC?$AAM?$AAE?$AA?5?$AAE?$AAr?$AAr@ 10027430     SDKRIL.obj
 0002:00001490       ??_C@_1FG@KKJNCEBB@?$AAS?$AAw?$AAi?$AAA?$AAT?$AAR?$AAt?$AAn?$AAR?$AAe?$AAs?$AAe?$AAt?$AA?3?$AA?5?$AAF?$AAa?$AAi?$AAl?$AAe?$AAd?$AA?5?$AAt?$AAo?$AA?5?$AAe?$AAx?$AAt?$AAr?$AAa?$AAc?$AAt@ 10027490     SDKRIL.obj
 0002:000014e8       ??_C@_1DA@NEKCNPBG@?$AAS?$AAw?$AAi?$AAA?$AAT?$AAR?$AAt?$AAn?$AAR?$AAe?$AAs?$AAe?$AAt?$AA?3?$AA?3?$AAn?$AAo?$AA?5?$AAE?$AAr?$AAr?$AAo?$AAr?$AA?$AA@ 100274e8     SDKRIL.obj
 0002:00001518       ??_C@_07LOKEFHKB@AT?$CLMDN?$AN?$AA@ 10027518     SDKRIL.obj
 0002:00001520       ??_C@_1FC@NONJAMJG@?$AAS?$AAw?$AAi?$AAH?$AAa?$AAn?$AAd?$AAl?$AAe?$AAS?$AAu?$AAs?$AAp?$AAe?$AAn?$AAd?$AA?5?$AAN?$AAO?$AAO?$AAP?$AA?5?$AAf?$AAo?$AAr?$AA?5?$AAt?$AAa?$AAr?$AAg?$AAe?$AAt@ 10027520     SDKRIL.obj
 0002:00001578       ??_C@_1FA@MEAICPMI@?$AAS?$AAw?$AAi?$AAH?$AAa?$AAn?$AAd?$AAl?$AAe?$AAR?$AAe?$AAs?$AAu?$AAm?$AAe?$AA?5?$AAN?$AAO?$AAO?$AAP?$AA?5?$AAf?$AAo?$AAr?$AA?5?$AAt?$AAa?$AAr?$AAg?$AAe?$AAt?$AAD@ 10027578     SDKRIL.obj
 0002:000015c8       ??_7CriticalSection@@6B@   100275c8     SDKRIL.obj
 0002:000015cc       ??_C@_1BG@FEIGEILE@?$AAO?$AAM?$AA?5?$AAH?$AAa?$AAn?$AAd?$AAs?$AAe?$AAt?$AA?$AA@ 100275cc     SDKRILCdma.obj
 0002:000015e4       ??_C@_1BM@HLGGGPPF@?$AAC?$AAh?$AAi?$AAn?$AAa?$AA?5?$AAT?$AAe?$AAl?$AAe?$AAc?$AAo?$AAm?$AA?$AA@ 100275e4     SDKRILCdma.obj
 0002:00001600       ??_C@_1BC@PGLBBGPP@?$AAI?$AAu?$AAs?$AAa?$AAc?$AAe?$AAl?$AAl?$AA?$AA@ 10027600     SDKRILCdma.obj
 0002:00001614       ??_C@_19KFCNPIAE@?$AAK?$AAD?$AAD?$AAI?$AA?$AA@ 10027614     SDKRILCdma.obj
 0002:00001620       ??_C@_1BM@LKNNANDO@?$AAL?$AAe?$AAa?$AAp?$AA?5?$AAW?$AAi?$AAr?$AAe?$AAl?$AAe?$AAs?$AAs?$AA?$AA@ 10027620     SDKRILCdma.obj
 0002:0000163c       ??_C@_1BK@PJLKCLFI@?$AAM?$AAe?$AAt?$AAr?$AAo?$AAP?$AAC?$AAS?$AA?5?$AAC?$AAo?$AAm?$AA?$AA@ 1002763c     SDKRILCdma.obj
 0002:00001658       ??_C@_1BC@INOJPGM@?$AAT?$AAa?$AAt?$AAa?$AA?5?$AAC?$AAo?$AAm?$AA?$AA@ 10027658     SDKRILCdma.obj
 0002:0000166c       ??_C@_1BK@OCMFDAFL@?$AAR?$AAe?$AAl?$AAi?$AAa?$AAn?$AAc?$AAe?$AA?5?$AAC?$AAo?$AAm?$AA?$AA@ 1002766c     SDKRILCdma.obj
 0002:00001688       ??_C@_1BG@DHNBLHJE@?$AAS?$AAK?$AA?5?$AAT?$AAe?$AAl?$AAe?$AAc?$AAo?$AAm?$AA?$AA@ 10027688     SDKRILCdma.obj
 0002:000016a0       ??_C@_17NKFDFJHA@?$AAT?$AAN?$AAZ?$AA?$AA@ 100276a0     SDKRILCdma.obj
 0002:000016a8       ??_C@_1BK@IIMKLOEA@?$AAC?$AAh?$AAi?$AAn?$AAa?$AA?5?$AAU?$AAn?$AAi?$AAc?$AAo?$AAm?$AA?$AA@ 100276a8     SDKRILCdma.obj
 0002:000016c4       ??_C@_1BA@NKBOGNNJ@?$AAT?$AAe?$AAl?$AAs?$AAt?$AAr?$AAa?$AA?$AA@ 100276c4     SDKRILCdma.obj
 0002:000016d4       ??_C@_1BI@KAEOFCDM@?$AAU?$AAS?$AA?5?$AAC?$AAe?$AAl?$AAl?$AAu?$AAl?$AAa?$AAr?$AA?$AA@ 100276d4     SDKRILCdma.obj
 0002:000016ec       ??_C@_1M@CJLILBCD@?$AAT?$AAe?$AAl?$AAu?$AAs?$AA?$AA@ 100276ec     SDKRILCdma.obj
 0002:000016f8       ??_C@_19BAPHGJFB@?$AAB?$AAe?$AAl?$AAl?$AA?$AA@ 100276f8     SDKRILCdma.obj
 0002:00001704       ??_C@_1O@BFKCBMPA@?$AAA?$AAl?$AAl?$AAt?$AAe?$AAl?$AA?$AA@ 10027704     SDKRILCdma.obj
 0002:00001714       ??_C@_1O@LKNPFOFO@?$AAS?$AAp?$AAr?$AAi?$AAn?$AAt?$AA?$AA@ 10027714     SDKRILCdma.obj
 0002:00001724       ??_C@_1BA@HKLKHEFI@?$AAV?$AAe?$AAr?$AAi?$AAz?$AAo?$AAn?$AA?$AA@ 10027724     SDKRILCdma.obj
 0002:00001734       ??_C@_1CC@FHIPPGOJ@?$AA?4?$AA?2?$AAS?$AAD?$AAK?$AAR?$AAI?$AAL?$AAC?$AAd?$AAm?$AAa?$AA?4?$AAc?$AAp?$AAp?$AA?$AA@ 10027734     SDKRILCdma.obj
 0002:00001758       ??_C@_1DK@JHBFFPFP@?$AAS?$AAe?$AAn?$AAd?$AA?5?$AAS?$AAM?$AAS?$AA?5?$AAN?$AAo?$AAt?$AAi?$AAf?$AAi?$AAc?$AAa?$AAt?$AAi?$AAo?$AAn?$AA?5?$AAT?$AAh?$AAr?$AAe?$AAa?$AAd?$AA?$AA@ 10027758     SDKRILCdma.obj
 0002:00001794       ??_C@_1DM@FDCOJPGH@?$AAG?$AAl?$AAo?$AAb?$AAa?$AAl?$AA?5?$AAf?$AAl?$AAa?$AAg?$AA?5?$AAs?$AAa?$AAy?$AAs?$AA?5?$AAm?$AAs?$AAg?$AA?5?$AAn?$AAo?$AAt?$AA?5?$AAs?$AAe?$AAn?$AAt?$AA?$AA@ 10027794     SDKRILCdma.obj
 0002:000017d0       ??_C@_1EO@BCDBNNPB@?$AAG?$AAl?$AAo?$AAb?$AAa?$AAl?$AA?5?$AAf?$AAl?$AAa?$AAg?$AA?5?$AAs?$AAa?$AAy?$AAs?$AA?5?$AAm?$AAs?$AAg?$AA?5?$AAs?$AAe?$AAn?$AAt?$AA?5?$AAs?$AAu?$AAc?$AAc?$AAe?$AAs@ 100277d0     SDKRILCdma.obj
 0002:00001820       ??_C@_1FA@BBMINECN@?$AAs?$AAt?$AAr?$AAt?$AAo?$AAu?$AAl?$AA?5?$AAf?$AAa?$AAi?$AAl?$AAe?$AAd?$AA?5?$AAa?$AAn?$AAd?$AA?5?$AAr?$AAe?$AAt?$AAu?$AAr?$AAn?$AAe?$AAd?$AA?5?$AAv?$AAa?$AAl?$AAu@ 10027820     SDKRILCdma.obj
 0002:00001870       ??_C@_1EK@DGKHAHBG@?$AAs?$AAt?$AAr?$AAt?$AAo?$AAu?$AAl?$AA?5?$AAf?$AAa?$AAi?$AAl?$AAe?$AAd?$AA?5?$AAo?$AAn?$AA?5?$AAe?$AAi?$AAt?$AAh?$AAe?$AAr?$AA?5?$AAm?$AAe?$AAi?$AAd?$AA?5?$AAo?$AAr@ 10027870     SDKRILCdma.obj
 0002:000018c0       ??_C@_1FA@OBOELMMH@?$AAM?$AAe?$AAi?$AAd?$AA_?$AAH?$AAi?$AAg?$AAh?$AA?5?$AA?$DN?$AA?5?$AA?$CF?$AAX?$AA?5?$AA?5?$AAM?$AAe?$AAi?$AAd?$AA_?$AAL?$AAo?$AAw?$AA?5?$AA?$DN?$AA?5?$AA?$CF?$AAX?$AA?5?$AAP?$AAE@ 100278c0     SDKRILCdma.obj
 0002:00001910       ??_C@_1II@OBBDAENM@?$AAS?$AAw?$AAi?$AAG?$AAe?$AAt?$AAS?$AAe?$AAr?$AAv?$AAi?$AAc?$AAe?$AAI?$AAn?$AAd?$AAi?$AAc?$AAa?$AAt?$AAi?$AAo?$AAn?$AA?5?$AAd?$AAe?$AAt?$AAe?$AAc?$AAt?$AAs?$AA?5@ 10027910     SDKRILCdma.obj
 0002:00001998       ??_C@_1IA@NPLOEDI@?$AAS?$AAw?$AAi?$AAG?$AAe?$AAt?$AAR?$AAo?$AAa?$AAm?$AAi?$AAn?$AAg?$AAS?$AAt?$AAa?$AAt?$AAu?$AAs?$AA?5?$AAd?$AAe?$AAt?$AAe?$AAc?$AAt?$AAs?$AA?5?$AAi?$AAn?$AAc?$AAo@ 10027998     SDKRILCdma.obj
 0002:00001a18       ??_C@_1KI@NAEGBMC@?$AAS?$AAw?$AAi?$AAS?$AAe?$AAt?$AAC?$AAa?$AAl?$AAl?$AAO?$AAr?$AAi?$AAg?$AAi?$AAn?$AAa?$AAt?$AAe?$AAC?$AAm?$AAd?$AA?5?$AAn?$AAo?$AAt?$AA?5?$AAo?$AAf?$AAf?$AAi?$AAc@ 10027a18     SDKRILCdma.obj
 0002:00001ac0       ??_C@_00CNPNBAHC@?$AA@     10027ac0     SDKRILCdma.obj
 0002:00001ac8       ??_C@_1HO@IIBJDAOD@?$AAS?$AAw?$AAi?$AAS?$AAe?$AAt?$AAC?$AAa?$AAl?$AAl?$AAO?$AAr?$AAi?$AAg?$AAi?$AAn?$AAa?$AAt?$AAe?$AAC?$AAm?$AAd?$AA?5?$AAu?$AAn?$AAh?$AAa?$AAn?$AAd?$AAl?$AAe?$AA?5@ 10027ac8     SDKRILCdma.obj
 0002:00001b48       ??_C@_1HI@HEHGIHA@?$AAS?$AAw?$AAi?$AAG?$AAe?$AAt?$AAC?$AAa?$AAl?$AAl?$AAC?$AAo?$AAn?$AAn?$AAe?$AAc?$AAt?$AAi?$AAo?$AAn?$AAS?$AAt?$AAa?$AAt?$AAe?$AA?5?$AAr?$AAe?$AAt?$AAu?$AAr?$AAn@ 10027b48     SDKRILCdma.obj
 0002:00001bc0       ??_C@_1KI@BJLAKOIO@?$AAS?$AAw?$AAi?$AAS?$AAe?$AAt?$AAC?$AAa?$AAl?$AAl?$AAD?$AAi?$AAs?$AAc?$AAo?$AAn?$AAn?$AAe?$AAc?$AAt?$AAC?$AAm?$AAd?$AA?5?$AAn?$AAo?$AAt?$AA?5?$AAo?$AAf?$AAf?$AAi@ 10027bc0     SDKRILCdma.obj
 0002:00001c68       ??_C@_1FG@OACMAIPJ@?$AAG?$AAo?$AAb?$AAi?$AA?5?$AAA?$AAp?$AAi?$AA?5?$AAG?$AAe?$AAt?$AAS?$AAM?$AAS?$AAL?$AAi?$AAs?$AAt?$AA?5?$AAf?$AAa?$AAi?$AAl?$AAe?$AAd?$AA?5?$AAw?$AAi?$AAt?$AAh?$AA?5@ 10027c68     SDKRILCdma.obj
 0002:00001cc0       ??_C@_1FC@LPFKGFCF@?$AAG?$AAo?$AAb?$AAi?$AA?5?$AAS?$AAM?$AAS?$AA?5?$AAL?$AAi?$AAs?$AAt?$AA?5?$AAs?$AAi?$AAz?$AAe?$AA?5?$AAf?$AAo?$AAr?$AA?5?$AAU?$AAN?$AAR?$AAE?$AAA?$AAD?$AA?5?$AAm?$AAs@ 10027cc0     SDKRILCdma.obj
 0002:00001d18       ??_C@_1IC@GLDIOAJP@?$AAG?$AAo?$AAb?$AAi?$AA?5?$AAG?$AAe?$AAt?$AAS?$AAM?$AAS?$AA?5?$AAL?$AAo?$AAo?$AAp?$AA?5?$AAL?$AAo?$AAo?$AAp?$AA?5?$AAi?$AAn?$AAd?$AAe?$AAx?$AA?5?$AAi?$AA?5?$AA?$DN?$AA?5@ 10027d18     SDKRILCdma.obj
 0002:00001da0       ??_C@_1EO@MNIHNLHB@?$AAG?$AAo?$AAb?$AAi?$AA?5?$AAA?$AAp?$AAi?$AA?5?$AAG?$AAe?$AAt?$AAS?$AAM?$AAS?$AA?5?$AAf?$AAa?$AAi?$AAl?$AAe?$AAd?$AA?5?$AAw?$AAi?$AAt?$AAh?$AA?5?$AAe?$AAr?$AAr?$AAo@ 10027da0     SDKRILCdma.obj
 0002:00001df0       ??_C@_1FG@PBHEHFMI@?$AAD?$AAe?$AAc?$AAo?$AAd?$AAe?$AAC?$AAo?$AAm?$AAp?$AAl?$AAe?$AAt?$AAe?$AAM?$AAT?$AAS?$AAm?$AAs?$AA?5?$AAf?$AAa?$AAi?$AAl?$AAe?$AAd?$AA?5?$AAw?$AAi?$AAt?$AAh?$AA?5@ 10027df0     SDKRILCdma.obj
 0002:00001e48       ??_C@_1FE@LFCMJEHJ@?$AAG?$AAo?$AAb?$AAi?$AA?5?$AAA?$AAp?$AAi?$AA?5?$AAD?$AAe?$AAl?$AAe?$AAt?$AAe?$AAS?$AAM?$AAS?$AA?5?$AAf?$AAa?$AAi?$AAl?$AAe?$AAd?$AA?5?$AAw?$AAi?$AAt?$AAh?$AA?5?$AAe@ 10027e48     SDKRILCdma.obj
 0002:00001e9c       ??_C@_1DO@DNAFGMEP@?$AAU?$AAn?$AAe?$AAx?$AAp?$AAe?$AAc?$AAt?$AAe?$AAd?$AA?5?$AAd?$AAa?$AAt?$AAa?$AA?5?$AAl?$AAe?$AAn?$AAg?$AAh?$AAt?$AA?5?$AAf?$AAo?$AAr?$AA?5?$AAM?$AAW?$AAI?$AA?$AA@ 10027e9c     SDKRILCdma.obj
 0002:00001ee0       ??_C@_1HA@BJHJAOAE@?$AAM?$AAs?$AAg?$AA?5?$AAF?$AAo?$AAr?$AAm?$AAa?$AAt?$AA?5?$AA?$DN?$AA?5?$AA?$CF?$AAd?$AA?0?$AA?5?$AAM?$AAs?$AAg?$AA?5?$AAT?$AAa?$AAg?$AA?5?$AA?$DN?$AA?5?$AA?$CF?$AAd?$AA?4?$AA?5?$AAO@ 10027ee0     SDKRILCdma.obj
 0002:00001f50       ??_C@_1GI@BDDCKNC@?$AAO?$AAn?$AAe?$AA?5?$AAM?$AAs?$AAg?$AA?5?$AAa?$AAl?$AAr?$AAe?$AAa?$AAd?$AAy?$AA?5?$AAs?$AAt?$AAo?$AAr?$AAe?$AAd?$AA?5?$AAi?$AAn?$AA?5?$AAt?$AAh?$AAe?$AA?5?$AAm?$AAo@ 10027f50     SDKRILCdma.obj
 0002:00001fb8       ??_C@_1FG@CKBLAIDF@?$AAS?$AAM?$AAS?$AA?5?$AAM?$AAS?$AAg?$AA?5?$AAb?$AAo?$AAd?$AAy?$AA?5?$AAi?$AAs?$AA?5?$AAl?$AAo?$AAn?$AAg?$AAe?$AAr?$AA?5?$AAt?$AAh?$AAa?$AAn?$AA?5?$AA1?$AA6?$AA0?$AA?5@ 10027fb8     SDKRILCdma.obj
 0002:00002010       ??_C@_1DK@FECFOMAH@?$AAE?$AAn?$AAc?$AAo?$AAd?$AAe?$AAC?$AAo?$AAm?$AAp?$AAl?$AAe?$AAt?$AAe?$AAM?$AAo?$AAS?$AAm?$AAs?$AA?5?$AAf?$AAa?$AAi?$AAl?$AAe?$AAd?$AA?5?$AA?6?$AA?$AA@ 10028010     SDKRILCdma.obj
 0002:00002050       ??_C@_1EE@NFBDPPNO@?$AAN?$AAo?$AA?5?$AAS?$AAM?$AAS?$AA?5?$AAM?$AAs?$AAg?$AA?5?$AAi?$AAs?$AA?5?$AAs?$AAt?$AAo?$AAr?$AAe?$AAd?$AA?5?$AAi?$AAn?$AA?5?$AAt?$AAh?$AAe?$AA?5?$AAm?$AAo?$AAd?$AAe@ 10028050     SDKRILCdma.obj
 0002:00002098       ??_C@_1IC@ENFHKFBA@?$AAG?$AAo?$AAb?$AAi?$AA?5?$AAS?$AAe?$AAn?$AAd?$AAS?$AAM?$AAS?$AA?5?$AAf?$AAa?$AAi?$AAl?$AAe?$AAd?$AA?5?$AAw?$AAi?$AAt?$AAh?$AA?5?$AAe?$AAr?$AAr?$AAo?$AAr?$AA?5?$AAc@ 10028098     SDKRILCdma.obj
 0002:00002120       ??_C@_1HI@OKGNLIPL@?$AAP?$AAr?$AAe?$AAv?$AAi?$AAo?$AAu?$AAs?$AA?5?$AAS?$AAm?$AAs?$AAS?$AAe?$AAn?$AAd?$AAN?$AAo?$AAt?$AAi?$AAf?$AAy?$AAT?$AAh?$AAr?$AAe?$AAa?$AAd?$AA?5?$AAH?$AAa?$AAn@ 10028120     SDKRILCdma.obj
 0002:00002198       ??_C@_1GK@HOKHMLFA@?$AAE?$AAr?$AAr?$AAo?$AAr?$AA?5?$AAS?$AAe?$AAn?$AAd?$AAi?$AAn?$AAg?$AA?5?$AAS?$AAM?$AAS?$AA?5?$AAn?$AAo?$AAt?$AAi?$AAf?$AAi?$AAc?$AAa?$AAt?$AAi?$AAo?$AAn?$AA?0?$AA?5@ 10028198     SDKRILCdma.obj
 0002:00002204       ??_C@_1BC@IAOFKNMN@?$AAe?$AAr?$AAi?$AA_?$AAn?$AAa?$AAm?$AA1?$AA?$AA@ 10028204     SDKRILCdma.obj
 0002:00002218       ??_C@_1BC@JCFAACCD@?$AAe?$AAr?$AAi?$AA_?$AAn?$AAa?$AAm?$AA2?$AA?$AA@ 10028218     SDKRILCdma.obj
 0002:00002230       ??_C@_1II@EENOMIII@?$AAG?$AAe?$AAt?$AAE?$AAR?$AAI?$AAF?$AAi?$AAl?$AAe?$AA?5?$AAr?$AAe?$AAt?$AAu?$AAr?$AAn?$AAs?$AA?5?$AAr?$AAc?$AA?5?$AA?$DN?$AA?5?$AA?$CF?$AAd?$AA?0?$AA?5?$AAf?$AAi?$AAl?$AAe@ 10028230     SDKRILCdma.obj
 0002:000022b8       ??_C@_1GC@FELBHPJE@?$AAS?$AAw?$AAi?$AAG?$AAe?$AAt?$AAE?$AAF?$AAi?$AAl?$AAe?$AAI?$AAn?$AAf?$AAo?$AA?5?$AAd?$AAo?$AAe?$AAs?$AAn?$AA?8?$AAt?$AA?5?$AAh?$AAa?$AAn?$AAd?$AAl?$AAe?$AA?5?$AAp@ 100282b8     SDKRILCdma.obj
 0002:00002320       ??_C@_1HM@CHJLOMCF@?$AAG?$AAe?$AAt?$AAE?$AAR?$AAI?$AAF?$AAi?$AAl?$AAe?$AA?5?$AAr?$AAe?$AAt?$AAu?$AAr?$AAn?$AAs?$AA?5?$AAr?$AAc?$AA?5?$AA?$DN?$AA?5?$AA?$CF?$AAd?$AA?0?$AA?5?$AAf?$AAi?$AAl?$AAe@ 10028320     SDKRILCdma.obj
 0002:000023a0       ??_C@_1FK@IIOLNHOO@?$AAS?$AAw?$AAi?$AAG?$AAe?$AAt?$AAE?$AAF?$AAi?$AAl?$AAe?$AA?5?$AAd?$AAo?$AAe?$AAs?$AAn?$AA?8?$AAt?$AA?5?$AAh?$AAa?$AAn?$AAd?$AAl?$AAe?$AA?5?$AAp?$AAs?$AAz?$AAE?$AAF@ 100283a0     SDKRILCdma.obj
 0002:000023fc       ??_C@_1CC@OGBPFNKE@?$AAP?$AAR?$AAL?$AA?5?$AAV?$AAe?$AAr?$AAs?$AAi?$AAo?$AAn?$AA?5?$AA?$DN?$AA?5?$AA?$CF?$AAu?$AA?$AA@ 100283fc     SDKRILCdma.obj
 0002:00002420       ??_C@_1GG@HKLKBAO@?$AAG?$AAo?$AAb?$AAi?$AA?5?$AAo?$AAn?$AAl?$AAy?$AA?5?$AAh?$AAa?$AAn?$AAd?$AAl?$AAe?$AAs?$AA?5?$AAo?$AAn?$AAe?$AA?5?$AAN?$AAa?$AAm?$AA?4?$AA?5?$AAT?$AAr?$AAe?$AAa?$AAt@ 10028420     SDKRILCdma.obj
 0002:00002488       ??_C@_1FE@DOLJBEHB@?$AAS?$AAe?$AAt?$AA3?$AAG?$AAp?$AAp?$AA2?$AAS?$AAu?$AAb?$AAs?$AAc?$AAr?$AAi?$AAp?$AAt?$AAi?$AAo?$AAn?$AAI?$AAn?$AAf?$AAo?$AA?5?$AAf?$AAa?$AAi?$AAl?$AAe?$AAd?$AA?0@ 10028488     SDKRILCdma.obj
 0002:000024e0       ??_C@_1FE@CNKLIODL@?$AAG?$AAe?$AAt?$AA3?$AAG?$AAp?$AAp?$AA2?$AAS?$AAu?$AAb?$AAs?$AAc?$AAr?$AAi?$AAp?$AAt?$AAi?$AAo?$AAn?$AAI?$AAn?$AAf?$AAo?$AA?5?$AAf?$AAa?$AAi?$AAl?$AAe?$AAd?$AA?0@ 100284e0     SDKRILCdma.obj
 0002:00002534       ??_C@_1CK@FENKLOBB@?$AAC?$AAD?$AAM?$AAA?$AA?5?$AAI?$AAM?$AAS?$AAI?$AA?5?$AA?$CI?$AAM?$AAI?$AAN?$AA?$CJ?$AA?5?$AA?$DN?$AA?5?$AA?$CF?$AAs?$AA?$AA@ 10028534     SDKRILCdma.obj
 0002:00002560       ??_C@_1LI@MFBJGAIG@?$AAS?$AAw?$AAi?$AAG?$AAe?$AAt?$AAT?$AAe?$AAc?$AAh?$AAB?$AAa?$AAn?$AAd?$AAC?$AAl?$AAa?$AAs?$AAs?$AA?5?$AAf?$AAa?$AAi?$AAl?$AAe?$AAd?$AA?0?$AA?5?$AAF?$AAi?$AAn?$AAd@ 10028560     SDKRILCdma.obj
 0002:00002618       ??_C@_1DE@JAGGADPL@?$AAG?$AAe?$AAt?$AAC?$AAw?$AAe?$AAP?$AAk?$AAg?$AAs?$AAI?$AAn?$AAf?$AAo?$AA?5?$AAr?$AAe?$AAt?$AAu?$AAr?$AAn?$AAs?$AA?5?$AA?$CF?$AAd?$AA?$AA@ 10028618     SDKRILCdma.obj
 0002:0000264c       ??_C@_1DG@CMFGIOCO@?$AAG?$AAe?$AAt?$AAF?$AAi?$AAr?$AAm?$AAw?$AAa?$AAr?$AAe?$AAI?$AAn?$AAf?$AAo?$AA?5?$AAr?$AAe?$AAt?$AAu?$AAr?$AAn?$AAs?$AA?5?$AA?$CF?$AAd?$AA?$AA@ 1002864c     SDKRILCdma.obj
 0002:00002684       ??_C@_19CLMCLOMN@?$AAM?$AAC?$AA7?$AA3?$AA?$AA@ 10028684     SDKRILCdma.obj
 0002:00002690       ??_C@_17JPFHOLBM@?$AA1?$AA0?$AA1?$AA?$AA@ 10028690     SDKRILCdma.obj
 0002:00002698       ??_C@_15MJIMBFJA@?$AA1?$AA1?$AA?$AA@ 10028698     SDKRILCdma.obj
 0002:000026a0       ??_C@_1FC@JEJODADP@?$AAO?$AAu?$AAt?$AA?5?$AAo?$AAf?$AA?5?$AAr?$AAa?$AAn?$AAg?$AAe?$AA?5?$AAG?$AAo?$AAb?$AAi?$AAC?$AAa?$AAr?$AAr?$AAi?$AAe?$AAr?$AAI?$AAD?$AA?5?$AAf?$AAo?$AAr?$AA?5?$AAC@ 100286a0     SDKRILCdma.obj
 0002:000026f4       ??_C@_04OBKAGHLG@?$CF06d?$AA@ 100286f4     SDKRILCdma.obj
 0002:00002700       ??_C@_1EG@CPCCBEGD@?$AAF?$AAa?$AAi?$AAl?$AA?5?$AAt?$AAo?$AA?5?$AAc?$AAo?$AAn?$AAv?$AAe?$AAr?$AAt?$AA?5?$AAS?$AAu?$AAb?$AAs?$AAi?$AAd?$AAy?$AAL?$AAo?$AAc?$AAk?$AA?5?$AAt?$AAo?$AA?5?$AAS@ 10028700     SDKRILCdma.obj
 0002:00002748       ??_C@_1HM@JINAAJEI@?$AAN?$AAo?$AA?5?$AAp?$AAr?$AAo?$AAv?$AAi?$AAs?$AAi?$AAo?$AAn?$AAn?$AAi?$AAn?$AAg?$AA?5?$AAd?$AAa?$AAt?$AAa?$AA?5?$AAt?$AAo?$AA?5?$AAb?$AAe?$AA?5?$AAc?$AAo?$AAm?$AAm@ 10028748     SDKRILCdma.obj
 0002:000027c8       ??_C@_1GO@MODMKDON@?$AAS?$AAw?$AAi?$AAS?$AAe?$AAt?$AAS?$AAe?$AAc?$AAu?$AAr?$AAe?$AAC?$AAo?$AAm?$AAm?$AAi?$AAt?$AAU?$AAp?$AAd?$AAa?$AAt?$AAe?$AA?3?$AA?5?$AAf?$AAa?$AAi?$AAl?$AAe?$AAd@ 100287c8     SDKRILCdma.obj
 0002:00002838       ??_C@_1GG@BCEHDICE@?$AAS?$AAw?$AAi?$AAS?$AAe?$AAt?$AAS?$AAe?$AAc?$AAu?$AAr?$AAe?$AAC?$AAo?$AAm?$AAm?$AAi?$AAt?$AAU?$AAp?$AAd?$AAa?$AAt?$AAe?$AA?3?$AA?5?$AAf?$AAa?$AAi?$AAl?$AAe?$AAd@ 10028838     SDKRILCdma.obj
 0002:000028a0       ??_C@_1BC@ELCBMMED@?$AAS?$AAc?$AAi?$AA?5?$AA?$DN?$AA?5?$AA?$CF?$AAd?$AA?$AA@ 100288a0     SDKRILCdma.obj
 0002:000028b8       ??_C@_1GE@IBFJMBPJ@?$AAG?$AAo?$AAb?$AAi?$AA?5?$AAm?$AAo?$AAd?$AAu?$AAl?$AAe?$AA?5?$AAd?$AAo?$AAe?$AAs?$AA?5?$AAn?$AAo?$AAt?$AA?5?$AAa?$AAl?$AAl?$AAo?$AA?5?$AAt?$AAo?$AA?5?$AAs?$AAe?$AAt@ 100288b8     SDKRILCdma.obj
 0002:00002920       ??_C@_1KO@NAELGCPN@?$AAG?$AAo?$AAb?$AAi?$AA?5?$AAG?$AAe?$AAt?$AAN?$AAe?$AAt?$AAw?$AAo?$AAr?$AAk?$AAP?$AAr?$AAe?$AAf?$AAe?$AAr?$AAe?$AAn?$AAc?$AAe?$AA?5?$AA?3?$AA?5?$AAu?$AAT?$AAe?$AAc@ 10028920     SDKRILCdma.obj
 0002:000029d0       ??_C@_1CE@PCABOOAL@?$AAS?$AAw?$AAi?$AA?5?$AAP?$AAr?$AAe?$AAf?$AAM?$AAo?$AAd?$AAe?$AA?5?$AA?$DN?$AA?5?$AA?$CF?$AAd?$AA?$AA@ 100289d0     SDKRILCdma.obj
 0002:000029f4       ??_C@_1CI@PHMDOILK@?$AAT?$AAe?$AAr?$AAm?$AAH?$AAo?$AAm?$AAe?$AAE?$AAn?$AAa?$AAb?$AAl?$AAe?$AA?5?$AA?$DN?$AA?5?$AA?$CF?$AAd?$AA?$AA@ 100289f4     SDKRILCdma.obj
 0002:00002a1c       ??_C@_1CG@NEKCMFIE@?$AAT?$AAe?$AAr?$AAm?$AAS?$AAi?$AAd?$AAE?$AAn?$AAa?$AAb?$AAl?$AAe?$AA?5?$AA?$DN?$AA?5?$AA?$CF?$AAd?$AA?$AA@ 10028a1c     SDKRILCdma.obj
 0002:00002a44       ??_C@_1CG@FBNLIIKP@?$AAT?$AAe?$AAr?$AAm?$AAN?$AAi?$AAd?$AAE?$AAn?$AAa?$AAb?$AAl?$AAe?$AA?5?$AA?$DN?$AA?5?$AA?$CF?$AAd?$AA?$AA@ 10028a44     SDKRILCdma.obj
 0002:00002a6c       ??_C@_1BI@OAMHNHKM@?$AAA?$AAc?$AAc?$AAo?$AAl?$AAc?$AA?5?$AA?$DN?$AA?5?$AA?$CF?$AAd?$AA?$AA@ 10028a6c     SDKRILCdma.obj
 0002:00002a88       ??_C@_1GE@EJEHIOK@?$AAG?$AAo?$AAb?$AAi?$AA?5?$AAd?$AAo?$AAe?$AAs?$AAn?$AA?8?$AAt?$AA?5?$AAs?$AAu?$AAp?$AAp?$AAo?$AAr?$AAt?$AA?5?$AAN?$AAA?$AAM?$AA?5?$AA?$DN?$AA?5?$AA?$CF?$AAd?$AA?4?$AA?5?$AAT@ 10028a88     SDKRILCdma.obj
 0002:00002aec       ??_C@_1BK@PHEDENNL@?$AAI?$AAm?$AAs?$AAi?$AAM?$AAc?$AAc?$AA?5?$AA?$DN?$AA?5?$AA?$CF?$AAd?$AA?$AA@ 10028aec     SDKRILCdma.obj
 0002:00002b08       ??_C@_1FA@DHBGCACD@?$AAG?$AAo?$AAb?$AAi?$AA?5?$AAm?$AAo?$AAd?$AAu?$AAl?$AAe?$AA?5?$AAd?$AAo?$AAe?$AAs?$AA?5?$AAn?$AAo?$AAt?$AA?5?$AAs?$AAu?$AAp?$AAp?$AAo?$AAr?$AAt?$AA?5?$AAS?$AAe?$AAt@ 10028b08     SDKRILCdma.obj
 0002:00002b58       ??_C@_1BO@JIHBIHDG@?$AAD?$AAi?$AAg?$AAi?$AAt?$AAs?$AA1?$AA1?$AA2?$AA?5?$AA?$DN?$AA?5?$AA?$CF?$AAd?$AA?$AA@ 10028b58     SDKRILCdma.obj
 0002:00002b78       ??_C@_1FC@KHLPLAJJ@?$AAG?$AAo?$AAb?$AAi?$AA?5?$AAm?$AAo?$AAd?$AAu?$AAl?$AAe?$AA?5?$AAd?$AAo?$AAe?$AAs?$AA?5?$AAn?$AAo?$AAt?$AA?5?$AAs?$AAu?$AAp?$AAp?$AAo?$AAr?$AAt?$AA?5?$AAS?$AAe?$AAt@ 10028b78     SDKRILCdma.obj
 0002:00002bd0       ??_C@_1GG@DJDCNECA@?$AAA?$AAS?$AAS?$AAE?$AAR?$AAT?$AAI?$AAO?$AAN?$AA?5?$AAF?$AAA?$AAI?$AAL?$AAU?$AAR?$AAE?$AA?3?$AA?5?$AA?$DN?$AA?$DN?$AA?$DN?$AA?$DO?$AAg?$AA_?$AAu?$AAl?$AAR?$AAo?$AAa?$AAm?$AAi@ 10028bd0     SDKRILCdma.obj
 0002:00002c38       ??_C@_1HC@EIDCHGAI@?$AAS?$AAw?$AAi?$AAP?$AAs?$AAt?$AAG?$AAe?$AAt?$AAS?$AAy?$AAs?$AAt?$AAe?$AAm?$AAP?$AAr?$AAe?$AAf?$AA?5?$AAf?$AAa?$AAi?$AAl?$AA?3?$AA?5?$AAO?$AAu?$AAt?$AA?5?$AAo?$AAf@ 10028c38     SDKRILCdma.obj
 0002:00002cb0       ??_C@_1FG@KLFIAFHL@?$AAH?$AAo?$AAm?$AAe?$AA?5?$AAS?$AAi?$AAd?$AA?5?$AA?$DN?$AA?5?$AA?$CF?$AAu?$AA?5?$AA?5?$AAa?$AAn?$AAd?$AA?5?$AAH?$AAo?$AAm?$AAe?$AA?5?$AAN?$AAI?$AAD?$AA?5?$AA?$DN?$AA?5?$AA?$CF?$AAu@ 10028cb0     SDKRILCdma.obj
 0002:00002d08       ??_C@_1LI@PMBPJNGH@?$AAT?$AAh?$AAi?$AAs?$AA?5?$AAA?$AAP?$AAI?$AA?5?$AAn?$AAe?$AAe?$AAd?$AAs?$AA?5?$AAt?$AAo?$AA?5?$AAm?$AAo?$AAd?$AAe?$AAm?$AA?5?$AAr?$AAe?$AAs?$AAe?$AAt?$AA?0?$AA?5?$AAi@ 10028d08     SDKRILCdma.obj
 0002:00002dc0       ??_C@_1DM@NALHHHHD@?$AAA?$AAc?$AAt?$AAi?$AAv?$AAe?$AA?5?$AAM?$AAI?$AAP?$AA?5?$AAp?$AAr?$AAo?$AAf?$AAi?$AAl?$AAe?$AA?5?$AAi?$AAn?$AAd?$AAe?$AAx?$AA?5?$AA?$DN?$AA?5?$AA?$CF?$AAu?$AA?$AA@ 10028dc0     SDKRILCdma.obj
 0002:00002e00       ??_C@_1EM@HGEBCHLG@?$AAG?$AAo?$AAb?$AAi?$AA?5?$AAG?$AAe?$AAt?$AAM?$AAo?$AAb?$AAi?$AAl?$AAe?$AAI?$AAP?$AAP?$AAr?$AAo?$AAf?$AAi?$AAl?$AAe?$AA?5?$AAr?$AAe?$AAt?$AAu?$AAr?$AAn?$AAi?$AAn@ 10028e00     SDKRILCdma.obj
 0002:00002e50       ??_C@_1KM@MJOIAPCH@?$AAn?$AAa?$AAi?$AA?5?$AA?$DN?$AA?$CF?$AAs?$AA?0?$AAp?$AAM?$AAn?$AAH?$AAa?$AAS?$AAp?$AAi?$AAE?$AAn?$AAa?$AAb?$AAl?$AAe?$AA?5?$AA?$DN?$AA?5?$AA?$CF?$AAu?$AA?5?$AA?0?$AA?5?$AAp?$AAM@ 10028e50     SDKRILCdma.obj
 0002:00002f00       ??_C@_1MA@MIHOJMFE@?$AAp?$AAR?$AAe?$AAv?$AAe?$AAr?$AAs?$AAe?$AAT?$AAu?$AAn?$AAn?$AAe?$AAl?$AAi?$AAn?$AAg?$AA?5?$AA?$DN?$AA?5?$AA?$CF?$AAu?$AA?0?$AA?5?$AAp?$AAH?$AAo?$AAm?$AAe?$AAA?$AAd?$AAd@ 10028f00     SDKRILCdma.obj
 0002:00002fc0       ??_C@_1II@INLHKAMD@?$AAG?$AAo?$AAb?$AAi?$AA?5?$AAm?$AAo?$AAd?$AAu?$AAl?$AAe?$AA?5?$AAd?$AAo?$AAe?$AAs?$AA?5?$AAn?$AAo?$AAt?$AA?5?$AAa?$AAl?$AAl?$AAo?$AAw?$AA?5?$AAt?$AAo?$AA?5?$AAr?$AAe@ 10028fc0     SDKRILCdma.obj
 0002:00003048       ??_C@_1GI@EJHEIMBK@?$AAS?$AAw?$AAi?$AAG?$AAe?$AAt?$AAM?$AAo?$AAb?$AAi?$AAl?$AAe?$AAI?$AAP?$AAP?$AAr?$AAo?$AAf?$AAi?$AAl?$AAe?$AA?5?$AAr?$AAe?$AAt?$AAu?$AAr?$AAn?$AAi?$AAn?$AAg?$AA?3@ 10029048     SDKRILCdma.obj
 0002:000030b0       ??_C@_1GE@INHEJGHG@?$AAA?$AAs?$AAs?$AAu?$AAm?$AAi?$AAn?$AAg?$AA?5?$AAM?$AAo?$AAb?$AAi?$AAl?$AAe?$AA?5?$AAI?$AAP?$AA?5?$AAp?$AAr?$AAo?$AAf?$AAi?$AAl?$AAe?$AA?5?$AAi?$AAn?$AAd?$AAe?$AAx@ 100290b0     SDKRILCdma.obj
 0002:00003118       ??_C@_1EK@CIGDFJJI@?$AAG?$AAe?$AAt?$AAL?$AAa?$AAs?$AAt?$AAM?$AAo?$AAb?$AAi?$AAl?$AAe?$AAI?$AAP?$AAE?$AAr?$AAr?$AAo?$AAr?$AA?5?$AAg?$AAe?$AAt?$AAs?$AA?5?$AAt?$AAo?$AA?5?$AAr?$AAc?$AA?5@ 10029118     SDKRILCdma.obj
 0002:00003168       ??_C@_1IA@DNCFECGF@?$AAS?$AAw?$AAi?$AAG?$AAe?$AAt?$AAH?$AAd?$AAr?$AAR?$AAo?$AAa?$AAm?$AAS?$AAt?$AAa?$AAt?$AAu?$AAs?$AA?5?$AAd?$AAe?$AAt?$AAe?$AAc?$AAt?$AAs?$AA?5?$AAi?$AAn?$AAc?$AAo@ 10029168     SDKRILCdma.obj
 0002:000031e8       ??_C@_1HM@CALFAEOJ@?$AAS?$AAw?$AAi?$AAG?$AAe?$AAt?$AAH?$AAd?$AAr?$AAS?$AAr?$AAv?$AAS?$AAt?$AAa?$AAt?$AAe?$AA?5?$AAd?$AAe?$AAt?$AAe?$AAc?$AAt?$AAs?$AA?5?$AAi?$AAn?$AAc?$AAo?$AAm?$AAp@ 100291e8     SDKRILCdma.obj
 0002:00003268       ??_C@_1FO@CEFNMKJC@?$AAS?$AAw?$AAi?$AAS?$AAe?$AAt?$AAH?$AAd?$AAr?$AAH?$AAy?$AAb?$AAr?$AAP?$AAr?$AAe?$AAf?$AA?5?$AAd?$AAo?$AAe?$AAs?$AAn?$AA?8?$AAt?$AA?5?$AAa?$AAl?$AAl?$AAo?$AAw?$AA?5@ 10029268     SDKRILCdma.obj
 0002:000032c8       ??_C@_1HG@EIIKEADK@?$AAA?$AAS?$AAS?$AAE?$AAR?$AAT?$AAI?$AAO?$AAN?$AA?5?$AAF?$AAA?$AAI?$AAL?$AAU?$AAR?$AAE?$AA?3?$AA?5?$AA?$DN?$AA?$DN?$AA?$DN?$AA?$DO?$AAn?$AAM?$AAo?$AAd?$AAe?$AAP?$AAr?$AAe?$AAf@ 100292c8     SDKRILCdma.obj
 0002:00003340       ??_C@_1HI@PBCAPDAG@?$AAA?$AAS?$AAS?$AAE?$AAR?$AAT?$AAI?$AAO?$AAN?$AA?5?$AAF?$AAA?$AAI?$AAL?$AAU?$AAR?$AAE?$AA?3?$AA?5?$AA?$DN?$AA?$DN?$AA?$DN?$AA?$DO?$AAn?$AAM?$AAo?$AAd?$AAe?$AAT?$AAe?$AAr?$AAm@ 10029340     SDKRILCdma.obj
 0002:000033b8       ??_C@_1EK@OLINJJAD@?$AAA?$AAS?$AAS?$AAE?$AAR?$AAT?$AAI?$AAO?$AAN?$AA?5?$AAF?$AAA?$AAI?$AAL?$AAU?$AAR?$AAE?$AA?3?$AA?5?$AA?$DN?$AA?$DN?$AA?$DN?$AA?$DO?$AAn?$AAM?$AAo?$AAd?$AAe?$AAD?$AAu?$AAr?$AA?5@ 100293b8     SDKRILCdma.obj
 0002:00003408       ??_C@_1MO@CDMAEDMJ@?$AAT?$AAh?$AAi?$AAs?$AA?5?$AAa?$AAc?$AAt?$AAi?$AAo?$AAn?$AA?5?$AAn?$AAe?$AAe?$AAd?$AAs?$AA?5?$AAm?$AAo?$AAd?$AAe?$AAm?$AA?5?$AAr?$AAe?$AAs?$AAe?$AAt?$AA?4?$AAI?$AAf@ 10029408     SDKRILCdma.obj
 0002:000034d8       ??_C@_1IG@IHJJPLMI@?$AAS?$AAw?$AAi?$AAS?$AAe?$AAt?$AAT?$AAe?$AAm?$AAp?$AAM?$AAo?$AAd?$AAe?$AAP?$AAr?$AAe?$AAf?$AA?5?$AAc?$AAa?$AAn?$AAn?$AAo?$AAt?$AA?5?$AAi?$AAn?$AAt?$AAe?$AAr?$AAp@ 100294d8     SDKRILCdma.obj
 0002:00003560       ??_C@_1GE@KMLGOCOC@?$AAG?$AAo?$AAb?$AAi?$AA?5?$AAd?$AAo?$AAe?$AAs?$AA?5?$AAa?$AAl?$AAl?$AAo?$AAw?$AA?5?$AAt?$AAo?$AA?5?$AAr?$AAe?$AAa?$AAd?$AA?5?$AAH?$AAD?$AAR?$AA?5?$AAU?$AAs?$AAe?$AAr@ 10029560     SDKRILCdma.obj
 0002:000035c4       ??_C@_11LOCGONAA@?$AA?$AA@ 100295c4     SDKRILCdma.obj
 0002:000035c8       ??_C@_1FO@JEENGOBK@?$AAG?$AAo?$AAb?$AAi?$AA?5?$AAd?$AAo?$AAe?$AAs?$AA?5?$AAa?$AAl?$AAl?$AAo?$AAw?$AA?5?$AAt?$AAo?$AA?5?$AAs?$AAe?$AAt?$AA?5?$AAH?$AAD?$AAR?$AA?5?$AAU?$AAs?$AAe?$AAr?$AA?5@ 100295c8     SDKRILCdma.obj
 0002:00003628       ??_C@_1GG@FEGPCNDH@?$AAG?$AAo?$AAb?$AAi?$AA?5?$AAd?$AAo?$AAe?$AAs?$AA?5?$AAa?$AAl?$AAl?$AAo?$AAw?$AA?5?$AAt?$AAo?$AA?5?$AAr?$AAe?$AAa?$AAd?$AA?5?$AAH?$AAD?$AAR?$AA?5?$AAp?$AAa?$AAs?$AAs@ 10029628     SDKRILCdma.obj
 0002:00003690       ??_C@_1GA@EJCCOEHH@?$AAG?$AAo?$AAb?$AAi?$AA?5?$AAd?$AAo?$AAe?$AAs?$AA?5?$AAa?$AAl?$AAl?$AAo?$AAw?$AA?5?$AAt?$AAo?$AA?5?$AAs?$AAe?$AAt?$AA?5?$AAH?$AAD?$AAR?$AA?5?$AAp?$AAa?$AAs?$AAs?$AAw@ 10029690     SDKRILCdma.obj
 0002:000036f0       ??_C@_1FA@KIIEKPCC@?$AAS?$AAw?$AAi?$AAP?$AAo?$AAw?$AAe?$AAr?$AAS?$AAa?$AAv?$AAe?$AAE?$AAx?$AAi?$AAt?$AA?5?$AAn?$AAo?$AAt?$AA?5?$AAs?$AAu?$AAp?$AAp?$AAo?$AAr?$AAt?$AAe?$AAd?$AA?5?$AAb@ 100296f0     SDKRILCdma.obj
 0002:00003740       ??_C@_1FE@IMDCAPOB@?$AAR?$AAT?$AAN?$AA?5?$AAr?$AAe?$AAs?$AAe?$AAt?$AA?5?$AAt?$AAy?$AAp?$AAe?$AA?5?$AA?$DN?$AA?5?$AA?$CF?$AAd?$AA?5?$AAn?$AAo?$AAt?$AA?5?$AAs?$AAu?$AAp?$AAp?$AAo?$AAr?$AAt?$AAe@ 10029740     SDKRILCdma.obj
 0002:00003798       ??_C@_1FE@MDHLBDJL@?$AAS?$AAw?$AAi?$AAS?$AAe?$AAt?$AAN?$AAD?$AAI?$AAS?$AAP?$AAr?$AAe?$AAf?$AAM?$AAo?$AAd?$AAe?$AA?5?$AAn?$AAo?$AAo?$AAp?$AA?4?$AA?5?$AAA?$AAl?$AAw?$AAa?$AAy?$AAs?$AA?5@ 10029798     SDKRILCdma.obj
 0002:000037f0       ??_C@_1MK@OJPNPJGB@?$AAC?$AAa?$AAn?$AAn?$AAo?$AAt?$AA?5?$AAh?$AAa?$AAn?$AAd?$AAl?$AAe?$AA?5?$AAc?$AAo?$AAn?$AAf?$AAu?$AAs?$AAe?$AAd?$AA?5?$AAP?$AAR?$AAL?$AAU?$AAp?$AAd?$AAa?$AAt?$AAe@ 100297f0     SDKRILCdma.obj
 0002:000038c0       ??_C@_1MI@CJKLJFND@?$AAC?$AAa?$AAn?$AAn?$AAo?$AAt?$AA?5?$AAh?$AAa?$AAn?$AAd?$AAl?$AAe?$AA?5?$AAc?$AAo?$AAn?$AAf?$AAu?$AAs?$AAe?$AAd?$AA?5?$AAD?$AAC?$AAU?$AAp?$AAd?$AAa?$AAt?$AAe?$AA?5@ 100298c0     SDKRILCdma.obj
 0002:00003988       ??_C@_1FG@JNCAHCC@?$AAO?$AAM?$AAA?$AAD?$AAM?$AAS?$AAt?$AAa?$AAr?$AAt?$AAS?$AAe?$AAs?$AAs?$AAi?$AAo?$AAn?$AA?5?$AAf?$AAa?$AAi?$AAl?$AAe?$AAd?$AA?5?$AAw?$AAi?$AAt?$AAh?$AA?5?$AAu?$AAS@ 10029988     SDKRILCdma.obj
 0002:000039e0       ??_C@_1FA@HMAMFEIF@?$AAO?$AAM?$AAA?$AAD?$AAM?$AAC?$AAa?$AAn?$AAc?$AAe?$AAl?$AAS?$AAe?$AAs?$AAs?$AAi?$AAo?$AAn?$AA?5?$AAf?$AAa?$AAi?$AAl?$AAe?$AAd?$AA?0?$AA?5?$AAu?$AAS?$AAt?$AAa?$AAt@ 100299e0     SDKRILCdma.obj
 0002:00003a30       ??_C@_1FA@GJCAGEOO@?$AAO?$AAM?$AAA?$AAD?$AAM?$AAG?$AAe?$AAt?$AAS?$AAe?$AAs?$AAs?$AAi?$AAo?$AAn?$AAI?$AAn?$AAf?$AAo?$AA?5?$AAf?$AAa?$AAi?$AAl?$AAe?$AAd?$AA?5?$AAu?$AAS?$AAt?$AAa?$AAt@ 10029a30     SDKRILCdma.obj
 0002:00003a80       ??_C@_1HG@MGFLMOOJ@?$AAO?$AAM?$AAA?$AAD?$AAM?$AAG?$AAe?$AAt?$AAS?$AAe?$AAs?$AAs?$AAi?$AAo?$AAn?$AAI?$AAn?$AAf?$AAo?$AA?3?$AA?3?$AAS?$AAe?$AAs?$AAs?$AAi?$AAo?$AAn?$AAS?$AAt?$AAa?$AAt@ 10029a80     SDKRILCdma.obj
 0002:00003af8       ??_C@_1DC@LKNLJHLE@?$AAO?$AAM?$AAA?$AAD?$AAM?$AA?5?$AAs?$AAe?$AAs?$AAs?$AAi?$AAo?$AAn?$AA?5?$AAe?$AAr?$AAr?$AAo?$AAr?$AA?5?$AA?$DN?$AA?5?$AA?$CF?$AAd?$AA?$AA@ 10029af8     SDKRILCdma.obj
 0002:00003b30       ??_C@_1EE@LFPADMIL@?$AAg?$AA_?$AAO?$AAM?$AAA?$AAD?$AAM?$AAP?$AAR?$AAL?$AAs?$AAe?$AAs?$AAs?$AAi?$AAo?$AAn?$AAI?$AAD?$AA?5?$AAc?$AAh?$AAa?$AAn?$AAg?$AAe?$AAd?$AA?5?$AAt?$AAo?$AA?5?$AA?$CF@ 10029b30     SDKRILCdma.obj
 0002:00003b78       ??_C@_1EC@NNHOHHIB@?$AAg?$AA_?$AAO?$AAM?$AAA?$AAD?$AAM?$AAD?$AAC?$AAs?$AAe?$AAs?$AAs?$AAi?$AAo?$AAn?$AAI?$AAD?$AA?5?$AAc?$AAh?$AAa?$AAn?$AAg?$AAe?$AAd?$AA?5?$AAt?$AAo?$AA?5?$AA?$CF?$AAd@ 10029b78     SDKRILCdma.obj
 0002:00003bbc       ??_C@_1DM@PPAGCKJB@?$AAU?$AAn?$AAh?$AAa?$AAn?$AAd?$AAl?$AAe?$AAd?$AA?5?$AAp?$AAs?$AAA?$AAl?$AAe?$AAr?$AAt?$AA?9?$AA?$DO?$AAn?$AAT?$AAy?$AAp?$AAe?$AA?5?$AA?$DN?$AA?5?$AA?$CF?$AAd?$AA?$AA@ 10029bbc     SDKRILCdma.obj
 0002:00003bf8       ??_C@_1FI@HBAFLLPM@?$AAO?$AAM?$AAA?$AAD?$AAM?$AAS?$AAe?$AAn?$AAd?$AAS?$AAe?$AAl?$AAe?$AAc?$AAt?$AAi?$AAo?$AAn?$AA?5?$AAf?$AAa?$AAi?$AAl?$AAe?$AAd?$AA?5?$AAw?$AAi?$AAt?$AAh?$AA?5?$AAu@ 10029bf8     SDKRILCdma.obj
 0002:00003c50       ??_C@_1CG@JODMLNAP@?$AAA?$AAP?$AAI?$AA?5?$AAn?$AAo?$AAt?$AA?5?$AAi?$AAn?$AAi?$AAt?$AAi?$AAa?$AAl?$AAz?$AAe?$AAd?$AA?$AA@ 10029c50     SDKRILCdma.obj
 0002:00003c78       ??_C@_1EG@NMKIEODM@?$AAS?$AAw?$AAi?$AAA?$AAc?$AAt?$AAi?$AAv?$AAa?$AAt?$AAe?$AAA?$AAu?$AAt?$AAo?$AAm?$AAa?$AAt?$AAi?$AAc?$AA?5?$AAr?$AAe?$AAt?$AAu?$AAr?$AAn?$AAi?$AAn?$AAg?$AA?3?$AA?5@ 10029c78     SDKRILCdma.obj
 0002:00003cc0       ??_C@_1EI@BPKCFDAD@?$AAS?$AAw?$AAi?$AAS?$AAe?$AAt?$AAM?$AAo?$AAb?$AAi?$AAl?$AAe?$AAI?$AAP?$AAP?$AAr?$AAo?$AAf?$AAi?$AAl?$AAe?$AA?5?$AAr?$AAe?$AAt?$AAu?$AAr?$AAn?$AAi?$AAn?$AAg?$AA?3@ 10029cc0     SDKRILCdma.obj
 0002:00003d08       ??_C@_1EI@KGMJCFEI@?$AAS?$AAw?$AAi?$AAG?$AAe?$AAt?$AAM?$AAo?$AAb?$AAi?$AAl?$AAe?$AAI?$AAP?$AAP?$AAr?$AAo?$AAf?$AAi?$AAl?$AAe?$AA?5?$AAr?$AAe?$AAt?$AAu?$AAr?$AAn?$AAi?$AAn?$AAg?$AA?3@ 10029d08     SDKRILCdma.obj
 0002:00003d50       ??_C@_1FM@CGMKCAAA@?$AAD?$AAi?$AAs?$AAp?$AAl?$AAa?$AAy?$AA?5?$AAb?$AAa?$AAn?$AAn?$AAe?$AAr?$AA?5?$AAN?$AAa?$AAm?$AAe?$AA?5?$AA?$DN?$AA?5?$AA?$CF?$AAs?$AA?5?$AAa?$AAn?$AAd?$AA?5?$AAr?$AAe?$AAt@ 10029d50     SDKRILCdma.obj
 0002:00004188       ??_C@_1CA@FLPLCLPH@?$AA?4?$AA?2?$AAS?$AAD?$AAK?$AAR?$AAI?$AAL?$AAG?$AAs?$AAm?$AA?4?$AAc?$AAp?$AAp?$AA?$AA@ 1002a188     SDKRILGsm.obj
 0002:000041a8       ??_C@_1GC@JJGALPCH@?$AAI?$AAn?$AAi?$AAt?$AAi?$AAa?$AAt?$AAe?$AAD?$AAo?$AAm?$AAa?$AAi?$AAn?$AAA?$AAt?$AAt?$AAa?$AAc?$AAh?$AA?5?$AAf?$AAa?$AAi?$AAl?$AAe?$AAd?$AA?5?$AAw?$AAi?$AAt?$AAh@ 1002a1a8     SDKRILGsm.obj
 0002:00004210       ??_C@_1EA@GDLNJGEA@?$AA?5?$AAS?$AAw?$AAi?$AAS?$AAe?$AAt?$AAP?$AAL?$AAM?$AAN?$AAM?$AAo?$AAd?$AAe?$AA?5?$AAe?$AAM?$AAo?$AAd?$AAe?$AA?5?$AAi?$AAs?$AA?5?$AAM?$AAa?$AAn?$AAu?$AAa?$AAl?$AA?$AA@ 1002a210     SDKRILGsm.obj
 0002:00004250       ??_C@_1DI@IAIIDPEC@?$AAA?$AAl?$AAr?$AAe?$AAa?$AAd?$AAy?$AA?5?$AAo?$AAn?$AA?5?$AAt?$AAh?$AAe?$AA?5?$AAs?$AAa?$AAm?$AAe?$AA?5?$AAn?$AAe?$AAt?$AAw?$AAo?$AAr?$AAk?$AA?$AA@ 1002a250     SDKRILGsm.obj
 0002:00004288       ??_C@_1HE@OKBCBGMH@?$AAC?$AAu?$AAr?$AAr?$AAe?$AAn?$AAt?$AAl?$AAy?$AA?5?$AAr?$AAe?$AAg?$AAi?$AAs?$AAt?$AAe?$AAr?$AAe?$AAd?$AA?5?$AAn?$AAe?$AAt?$AAw?$AAo?$AAr?$AAk?$AA?5?$AAi?$AAs?$AA?5@ 1002a288     SDKRILGsm.obj
 0002:00004300       ??_C@_1HM@GHGGNLML@?$AAG?$AAo?$AAb?$AAi?$AA?5?$AAA?$AAP?$AAI?$AA?5?$AAI?$AAn?$AAi?$AAt?$AAi?$AAa?$AAt?$AAe?$AAN?$AAe?$AAt?$AAw?$AAo?$AAr?$AAk?$AAR?$AAe?$AAg?$AAi?$AAs?$AAt?$AAr?$AAa@ 1002a300     SDKRILGsm.obj
 0002:00004380       ??_C@_1GE@LGKLGHEA@?$AAG?$AAo?$AAb?$AAi?$AA?5?$AAA?$AAP?$AAI?$AA?5?$AAG?$AAe?$AAt?$AAS?$AAe?$AAr?$AAv?$AAi?$AAn?$AAg?$AAN?$AAe?$AAt?$AAw?$AAo?$AAr?$AAk?$AA?5?$AAf?$AAa?$AAi?$AAl?$AAe@ 1002a380     SDKRILGsm.obj
 0002:000043e8       ??_C@_1EG@HKDNLAHG@?$AA?5?$AAS?$AAw?$AAi?$AAS?$AAe?$AAt?$AAP?$AAL?$AAM?$AAN?$AAM?$AAo?$AAd?$AAe?$AA?5?$AAe?$AAM?$AAo?$AAd?$AAe?$AA?5?$AAi?$AAs?$AA?5?$AAA?$AAu?$AAt?$AAo?$AAm?$AAa?$AAt@ 1002a3e8     SDKRILGsm.obj
 0002:00004430       ??_C@_1EM@KMPPOPAO@?$AAS?$AAw?$AAi?$AAS?$AAe?$AAt?$AAP?$AAL?$AAM?$AAN?$AAM?$AAo?$AAd?$AAe?$AA?5?$AAf?$AAa?$AAi?$AAl?$AAe?$AAd?$AA?5?$AAG?$AAo?$AAb?$AAi?$AA?5?$AAe?$AAr?$AAr?$AAo?$AAr@ 1002a430     SDKRILGsm.obj
 0002:00004480       ??_C@_1EG@OJEFPGCO@?$AAE?$AAn?$AAt?$AAe?$AAr?$AAi?$AAn?$AAg?$AA?5?$AAP?$AAe?$AAr?$AAf?$AAo?$AAr?$AAm?$AAN?$AAe?$AAt?$AAw?$AAo?$AAr?$AAk?$AAS?$AAc?$AAa?$AAn?$AA?5?$AAt?$AAh?$AAr?$AAe@ 1002a480     SDKRILGsm.obj
 0002:000044c8       ??_C@_1HM@LDBPCPFI@?$AAP?$AAe?$AAr?$AAf?$AAo?$AAr?$AAm?$AAN?$AAe?$AAt?$AAw?$AAo?$AAr?$AAk?$AAS?$AAc?$AAa?$AAn?$AA?5?$AAf?$AAa?$AAi?$AAl?$AAe?$AAd?$AA?0?$AA?5?$AAe?$AAr?$AAr?$AAo?$AAr@ 1002a4c8     SDKRILGsm.obj
 0002:00004548       ??_C@_1FC@DCICJBKN@?$AAP?$AAe?$AAr?$AAf?$AAo?$AAr?$AAm?$AAN?$AAe?$AAt?$AAw?$AAo?$AAr?$AAk?$AAR?$AAA?$AAT?$AAS?$AAc?$AAa?$AAn?$AA?5?$AAf?$AAa?$AAi?$AAl?$AAe?$AAd?$AA?0?$AA?5?$AAe?$AAr@ 1002a548     SDKRILGsm.obj
 0002:000045a0       ??_C@_1NI@KJECMBKI@?$AAg?$AA_?$AAP?$AAl?$AAm?$AAn?$AAL?$AAi?$AAs?$AAt?$AA?4?$AAs?$AAN?$AAw?$AAI?$AAn?$AAf?$AAo?$AA?$FL?$AAC?$AAo?$AAu?$AAn?$AAt?$AAe?$AAr?$AA?$FN?$AA?4?$AAM?$AAC?$AAC?$AA?5@ 1002a5a0     SDKRILGsm.obj
 0002:00004678       ??_C@_1ME@ENNCBDPD@?$AAG?$AAO?$AAB?$AAI?$AA?5?$AAA?$AAP?$AAI?$AA?5?$AAP?$AAe?$AAr?$AAf?$AAo?$AAr?$AAm?$AAN?$AAe?$AAt?$AAw?$AAo?$AAr?$AAk?$AAS?$AAc?$AAa?$AAn?$AA?1?$AAP?$AAe?$AAr?$AAf@ 1002a678     SDKRILGsm.obj
 0002:00004740       ??_C@_1HI@IEIIKPAM@?$AAG?$AAo?$AAb?$AAi?$AAP?$AAe?$AAr?$AAf?$AAo?$AAr?$AAm?$AAN?$AAe?$AAt?$AAw?$AAo?$AAr?$AAk?$AAS?$AAc?$AAa?$AAn?$AA?3?$AA?3?$AA?5?$AAT?$AAh?$AAe?$AAr?$AAe?$AA?5?$AAa@ 1002a740     SDKRILGsm.obj
 0002:000047b8       ??_C@_1EE@OIBLMGPL@?$AAL?$AAe?$AAa?$AAv?$AAi?$AAn?$AAg?$AA?5?$AAP?$AAe?$AAr?$AAf?$AAo?$AAr?$AAm?$AAN?$AAe?$AAt?$AAw?$AAo?$AAr?$AAk?$AAS?$AAc?$AAa?$AAn?$AA?5?$AAt?$AAh?$AAr?$AAe?$AAa@ 1002a7b8     SDKRILGsm.obj
 0002:00004800       ??_C@_1FI@KOHLCFKK@?$AAC?$AAr?$AAe?$AAa?$AAt?$AAe?$AA?5?$AAt?$AAh?$AAr?$AAe?$AAa?$AAd?$AA?5?$AAf?$AAa?$AAi?$AAl?$AAe?$AAd?$AA?5?$AAf?$AAo?$AAr?$AAS?$AAw?$AAi?$AAS?$AAt?$AAa?$AAr?$AAt@ 1002a800     SDKRILGsm.obj
 0002:00004858       ??_C@_13NOLLCAOD@?$AA?$AA?$AA?$AA@ 1002a858     SDKRILGsm.obj
 0002:00004860       ??_C@_1EE@JKALLCLK@?$AAE?$AAx?$AAt?$AAr?$AAa?$AAP?$AAa?$AAy?$AAl?$AAo?$AAa?$AAd?$AAS?$AAi?$AAz?$AAe?$AA?5?$AAi?$AAs?$AA?5?$AAl?$AAe?$AAs?$AAs?$AA?5?$AA2?$AA?5?$AAB?$AAy?$AAt?$AAe?$AAs@ 1002a860     SDKRILGsm.obj
 0002:000048a4       ??_C@_1CA@LGOIEHGE@?$AAT?$AAA?$AAG?$AA?5?$AA?$CB?$AA?$DN?$AA?5?$AAF?$AAC?$AAP?$AA_?$AAT?$AAA?$AAG?$AA?5?$AA?$AA@ 1002a8a4     SDKRILGsm.obj
 0002:000048c8       ??_C@_1IG@BICKINAC@?$AAA?$AAS?$AAS?$AAE?$AAR?$AAT?$AAI?$AAO?$AAN?$AA?5?$AAF?$AAA?$AAI?$AAL?$AAU?$AAR?$AAE?$AA?3?$AA?5?$AA?$DN?$AA?$DN?$AA?$DN?$AA?$DO?$AAc?$AAb?$AAD?$AAa?$AAt?$AAa?$AAR?$AAe?$AAs@ 1002a8c8     SDKRILGsm.obj
 0002:00004950       ??_C@_1DI@EENDBCOM@?$AAF?$AAI?$AAL?$AAE?$AA_?$AAD?$AAE?$AAS?$AAC?$AAR?$AAI?$AAP?$AAT?$AAO?$AAR?$AA_?$AAT?$AAA?$AAG?$AA?5?$AA?$CB?$AA?$DN?$AA?5?$AAT?$AAA?$AAG?$AA?5?$AA?$AA@ 1002a950     SDKRILGsm.obj
 0002:00004988       ??_C@_1DI@EHCECIEJ@?$AAc?$AAb?$AAD?$AAa?$AAt?$AAa?$AAU?$AAs?$AAe?$AAd?$AA?5?$AA?$DO?$AA?5?$AAc?$AAb?$AAF?$AAc?$AAp?$AAD?$AAa?$AAt?$AAa?$AAS?$AAi?$AAz?$AAe?$AA?5?$AA?$AA@ 1002a988     SDKRILGsm.obj
 0002:000049c0       ??_C@_1JE@NKEACB@?$AAA?$AAS?$AAS?$AAE?$AAR?$AAT?$AAI?$AAO?$AAN?$AA?5?$AAF?$AAA?$AAI?$AAL?$AAU?$AAR?$AAE?$AA?3?$AA?5?$AA?$DN?$AA?$DN?$AA?$DN?$AA?$DO?$AA2?$AA?5?$AA?$DN?$AA?$DN?$AA?5?$AAc?$AAb?$AAF?$AAi@ 1002a9c0     SDKRILGsm.obj
 0002:00004a58       ??_C@_1EI@KMMCCKC@?$AAc?$AAb?$AAF?$AAi?$AAl?$AAe?$AAD?$AAe?$AAs?$AAc?$AAD?$AAa?$AAt?$AAa?$AAS?$AAi?$AAz?$AAe?$AA?5?$AAi?$AAs?$AA?5?$AAl?$AAe?$AAs?$AAs?$AA?5?$AA2?$AA?5?$AAB?$AAy?$AAt@ 1002aa58     SDKRILGsm.obj
 0002:00004aa0       ??_C@_1EI@OLOCCIMG@?$AAc?$AAb?$AAF?$AAi?$AAl?$AAe?$AAD?$AAe?$AAs?$AAc?$AAD?$AAa?$AAt?$AAa?$AAS?$AAi?$AAz?$AAe?$AA?5?$AAi?$AAs?$AA?5?$AAl?$AAe?$AAs?$AAs?$AA?5?$AA5?$AA?5?$AAB?$AAy?$AAt@ 1002aaa0     SDKRILGsm.obj
 0002:00004ae8       ??_C@_1DC@KKMNENCG@?$AAt?$AAl?$AAv?$AAC?$AAu?$AAr?$AAr?$AAe?$AAn?$AAt?$AA?4?$AAP?$AAa?$AAr?$AAs?$AAe?$AA?5?$AAf?$AAa?$AAi?$AAl?$AAe?$AAd?$AA?5?$AA?$AA@ 1002aae8     SDKRILGsm.obj
 0002:00004b20       ??_C@_1FA@CGIEIOEM@?$AAt?$AAl?$AAv?$AAC?$AAu?$AAr?$AAr?$AAe?$AAn?$AAt?$AA?4?$AAG?$AAe?$AAt?$AAL?$AAe?$AAn?$AAg?$AAt?$AAh?$AA?$CI?$AA?$CJ?$AA?5?$AAi?$AAs?$AA?5?$AAl?$AAe?$AAs?$AAs?$AA?5?$AA2@ 1002ab20     SDKRILGsm.obj
 0002:00004b70       ??_C@_1EC@DFOJFEFP@?$AAF?$AAI?$AAL?$AAE?$AA_?$AAI?$AAD?$AA_?$AAT?$AAA?$AAG?$AA?5?$AA?$CB?$AA?$DN?$AA?5?$AAt?$AAl?$AAv?$AAF?$AAi?$AAl?$AAe?$AAI?$AAd?$AA?4?$AAG?$AAe?$AAt?$AAT?$AAa?$AAg?$AA?5@ 1002ab70     SDKRILGsm.obj
 0002:00004bb4       ??_C@_1DE@FGBEMBNL@?$AAt?$AAl?$AAv?$AAF?$AAi?$AAl?$AAe?$AAI?$AAd?$AA?4?$AAG?$AAe?$AAt?$AAL?$AAe?$AAn?$AAg?$AAt?$AAh?$AA?5?$AA?$CB?$AA?$DN?$AA?5?$AA2?$AA?5?$AA?$AA@ 1002abb4     SDKRILGsm.obj
 0002:00004be8       ??_C@_1DG@EAAGICAE@?$AAM?$AAA?$AAS?$AAT?$AAE?$AAR?$AA_?$AAF?$AAI?$AAL?$AAE?$AA_?$AAI?$AAD?$AA?5?$AA?$CB?$AA?$DN?$AA?5?$AAu?$AAF?$AAi?$AAl?$AAe?$AAI?$AAd?$AA?5?$AA?$AA@ 1002abe8     SDKRILGsm.obj
 0002:00004c20       ??_C@_0M@NMAJCJKD@AT?$CLCRSM?$DN?$CFlu?$AA@ 1002ac20     SDKRILGsm.obj
 0002:00004c30       ??_C@_1FI@HJDLAGCB@?$AAA?$AAS?$AAS?$AAE?$AAR?$AAT?$AAI?$AAO?$AAN?$AA?5?$AAF?$AAA?$AAI?$AAL?$AAU?$AAR?$AAE?$AA?3?$AA?5?$AA?$DN?$AA?$DN?$AA?$DN?$AA?$DO?$AAN?$AAU?$AAL?$AAL?$AA?5?$AA?$CB?$AA?$DN?$AA?5?$AAs@ 1002ac30     SDKRILGsm.obj
 0002:00004c88       ??_C@_03FIJBDJNN@?0?$CFu?$AA@ 1002ac88     SDKRILGsm.obj
 0002:00004c8c       ??_C@_09INKGJNCD@?0?$CFu?0?$CFu?0?$CFu?$AA@ 1002ac8c     SDKRILGsm.obj
 0002:00004c98       ??_C@_01LIIJDEN@?$AN?$AA@  1002ac98     SDKRILGsm.obj
 0002:00004c9c       ??_C@_07KANBOJJB@?$CLCRSM?3?5?$AA@ 1002ac9c     SDKRILGsm.obj
 0002:00004ca4       ??_C@_1CI@BOPLCHO@?$AAP?$AAa?$AAr?$AAs?$AAe?$AAU?$AAI?$AAn?$AAt?$AA?5?$AA2?$AA?5?$AAf?$AAa?$AAi?$AAl?$AAe?$AAd?$AA?5?$AA?$AA@ 1002aca4     SDKRILGsm.obj
 0002:00004ccc       ??_C@_1DK@KOBPNBHM@?$AAP?$AAa?$AAr?$AAs?$AAe?$AAU?$AAn?$AAl?$AAi?$AAm?$AAi?$AAt?$AAe?$AAd?$AAS?$AAt?$AAr?$AAi?$AAn?$AAg?$AA?5?$AAf?$AAa?$AAi?$AAl?$AAe?$AAd?$AA?5?$AA?$AA@ 1002accc     SDKRILGsm.obj
 0002:00004d08       ??_C@_1GO@LKFJLNHJ@?$AAA?$AAS?$AAS?$AAE?$AAR?$AAT?$AAI?$AAO?$AAN?$AA?5?$AAF?$AAA?$AAI?$AAL?$AAU?$AAR?$AAE?$AA?3?$AA?5?$AA?$DN?$AA?$DN?$AA?$DN?$AA?$DO?$AA0?$AA?5?$AA?$DN?$AA?$DN?$AA?5?$AA?$CI?$AAc?$AAb?$AAR@ 1002ad08     SDKRILGsm.obj
 0002:00004d78       ??_C@_1DA@LGILLIBC@?$AAP?$AAa?$AAr?$AAs?$AAe?$AAR?$AAs?$AAp?$AAP?$AAo?$AAs?$AAt?$AAf?$AAi?$AAx?$AA?5?$AAf?$AAa?$AAi?$AAl?$AAe?$AAd?$AA?5?$AA?$AA@ 1002ad78     SDKRILGsm.obj
 0002:00004da8       ??_C@_1GA@PELHIHIO@?$AAS?$AAw?$AAi?$AAS?$AAe?$AAn?$AAd?$AAR?$AAe?$AAs?$AAt?$AAr?$AAi?$AAc?$AAt?$AAe?$AAd?$AAS?$AAI?$AAM?$AAC?$AAm?$AAd?$AA?5?$AAf?$AAa?$AAi?$AAl?$AAe?$AAd?$AA?5?$AAw@ 1002ada8     SDKRILGsm.obj
 0002:00004e08       ??_C@_1PI@KAKIHNBM@?$AAA?$AAS?$AAS?$AAE?$AAR?$AAT?$AAI?$AAO?$AAN?$AA?5?$AAF?$AAA?$AAI?$AAL?$AAU?$AAR?$AAE?$AA?3?$AA?5?$AA?$DN?$AA?$DN?$AA?$DN?$AA?$DO?$AA?$CI?$AAs?$AAR?$AAs?$AAR?$AAs?$AAp?$AA?4?$AAd@ 1002ae08     SDKRILGsm.obj
 0002:00004f00       ??_C@_1IE@JEBFCNMG@?$AAR?$AAe?$AAs?$AAt?$AAr?$AAi?$AAc?$AAt?$AAe?$AAd?$AAS?$AAi?$AAm?$AA?5?$AAR?$AAs?$AAp?$AA?5?$AAc?$AAo?$AAn?$AAt?$AAa?$AAi?$AAn?$AAs?$AA?5?$AAe?$AAr?$AAr?$AAo?$AAr@ 1002af00     SDKRILGsm.obj
 0002:00004f88       ??_C@_1LC@DKNEACLD@?$AAR?$AAe?$AAs?$AAt?$AAr?$AAi?$AAc?$AAt?$AAe?$AAd?$AAS?$AAi?$AAm?$AA?5?$AAR?$AAs?$AAp?$AA?5?$AAc?$AAo?$AAn?$AAt?$AAa?$AAi?$AAn?$AAs?$AA?5?$AAe?$AAr?$AAr?$AAo?$AAr@ 1002af88     SDKRILGsm.obj
 0002:00005040       ??_C@_1LG@MKFCAPIA@?$AAR?$AAe?$AAs?$AAt?$AAr?$AAi?$AAc?$AAt?$AAe?$AAd?$AAS?$AAi?$AAm?$AA?5?$AAR?$AAs?$AAp?$AA?5?$AAc?$AAo?$AAn?$AAt?$AAa?$AAi?$AAn?$AAs?$AA?5?$AAe?$AAr?$AAr?$AAo?$AAr@ 1002b040     SDKRILGsm.obj
 0002:000050f8       ??_C@_1MI@JOJKIDD@?$AAR?$AAe?$AAs?$AAt?$AAr?$AAi?$AAc?$AAt?$AAe?$AAd?$AAS?$AAi?$AAm?$AA?5?$AAR?$AAs?$AAp?$AA?5?$AAc?$AAo?$AAn?$AAt?$AAa?$AAi?$AAn?$AAs?$AA?5?$AAe?$AAr?$AAr?$AAo?$AAr@ 1002b0f8     SDKRILGsm.obj
 0002:000051c0       ??_C@_1IG@PHINLLKA@?$AAR?$AAe?$AAs?$AAt?$AAr?$AAi?$AAc?$AAt?$AAe?$AAd?$AAS?$AAi?$AAm?$AA?5?$AAR?$AAs?$AAp?$AA?5?$AAc?$AAo?$AAn?$AAt?$AAa?$AAi?$AAn?$AAs?$AA?5?$AAe?$AAr?$AAr?$AAo?$AAr@ 1002b1c0     SDKRILGsm.obj
 0002:00005248       ??_C@_1IK@JCACGHA@?$AAR?$AAe?$AAs?$AAt?$AAr?$AAi?$AAc?$AAt?$AAe?$AAd?$AAS?$AAi?$AAm?$AA?5?$AAR?$AAs?$AAp?$AA?5?$AAc?$AAo?$AAn?$AAt?$AAa?$AAi?$AAn?$AAs?$AA?5?$AAe?$AAr?$AAr?$AAo?$AAr@ 1002b248     SDKRILGsm.obj
 0002:000052d8       ??_C@_1II@NHNONCDM@?$AAR?$AAe?$AAs?$AAt?$AAr?$AAi?$AAc?$AAt?$AAe?$AAd?$AAS?$AAi?$AAm?$AA?5?$AAR?$AAs?$AAp?$AA?5?$AAc?$AAo?$AAn?$AAt?$AAa?$AAi?$AAn?$AAs?$AA?5?$AAe?$AAr?$AAr?$AAo?$AAr@ 1002b2d8     SDKRILGsm.obj
 0002:00005360       ??_C@_1DE@FEKEDOEN@?$AAR?$AAe?$AAs?$AAt?$AA?5?$AAo?$AAf?$AA?5?$AAp?$AAo?$AAs?$AAs?$AAi?$AAb?$AAl?$AAe?$AA?5?$AAf?$AAa?$AAi?$AAl?$AAu?$AAr?$AAe?$AAs?$AA?$AA@ 1002b360     SDKRILGsm.obj
 0002:00005398       ??_C@_1GG@CBEJMOGO@?$AAS?$AAI?$AAM?$AA?5?$AAR?$AAE?$AAS?$AAP?$AAO?$AAN?$AAS?$AAE?$AA?5?$AAd?$AAa?$AAt?$AAa?$AA?5?$AAn?$AAo?$AAt?$AA?5?$AAp?$AAr?$AAe?$AAs?$AAe?$AAn?$AAt?$AA?5?$AAo?$AAr@ 1002b398     SDKRILGsm.obj
 0002:00005400       ??_C@_1GC@HHLMIADG@?$AAA?$AAS?$AAS?$AAE?$AAR?$AAT?$AAI?$AAO?$AAN?$AA?5?$AAF?$AAA?$AAI?$AAL?$AAU?$AAR?$AAE?$AA?3?$AA?5?$AA?$DN?$AA?$DN?$AA?$DN?$AA?$DO?$AAN?$AAU?$AAL?$AAL?$AA?5?$AA?$CB?$AA?$DN?$AA?5?$AAs@ 1002b400     SDKRILGsm.obj
 0002:00005468       ??_C@_1GG@CFNEEFFC@?$AAA?$AAS?$AAS?$AAE?$AAR?$AAT?$AAI?$AAO?$AAN?$AA?5?$AAF?$AAA?$AAI?$AAL?$AAU?$AAR?$AAE?$AA?3?$AA?5?$AA?$DN?$AA?$DN?$AA?$DN?$AA?$DO?$AA0?$AA?5?$AA?$CB?$AA?$DN?$AA?5?$AAs?$AAA?$AAR?$AAe@ 1002b468     SDKRILGsm.obj
 0002:000054d0       ??_C@_0M@KLIDJEFP@AT?$CLCSIM?$DN?$CFu?0?$AA@ 1002b4d0     SDKRILGsm.obj
 0002:000054e0       ??_C@_1EA@MMEJIFOF@?$AAC?$AAo?$AAm?$AAp?$AAo?$AAs?$AAe?$AAC?$AAm?$AAd?$AAW?$AAi?$AAt?$AAh?$AAB?$AAy?$AAt?$AAe?$AAA?$AAr?$AAr?$AAa?$AAy?$AA?5?$AAF?$AAa?$AAi?$AAl?$AAe?$AAd?$AA?5?$AA?$AA@ 1002b4e0     SDKRILGsm.obj
 0002:00005520       ??_C@_1DA@DEEOIGCP@?$AAC?$AAS?$AAI?$AAM?$AA?5?$AAA?$AAT?$AA?5?$AAc?$AAm?$AAd?$AA?5?$AAs?$AAt?$AAr?$AAi?$AAn?$AAg?$AA?5?$AA?$DN?$AA?5?$AA?$CF?$AAs?$AA?$AA@ 1002b520     SDKRILGsm.obj
 0002:00005550       ??_C@_07EBNNLFBH@?$CLCSIM?3?5?$AA@ 1002b550     SDKRILGsm.obj
 0002:00005558       ??_C@_1EO@DGIDCJJO@?$AAA?$AAS?$AAS?$AAE?$AAR?$AAT?$AAI?$AAO?$AAN?$AA?5?$AAF?$AAA?$AAI?$AAL?$AAU?$AAR?$AAE?$AA?3?$AA?5?$AA?$DN?$AA?$DN?$AA?$DN?$AA?$DO?$AA0?$AA?5?$AA?$DN?$AA?$DN?$AA?5?$AAn?$AAV?$AAa?$AAl@ 1002b558     SDKRILGsm.obj
 0002:000055a8       ??_C@_01BJJEKLCA@?$CC?$AA@ 1002b5a8     SDKRILGsm.obj
 0002:000055ac       ??_C@_1DI@BOIFCLKD@?$AAM?$AAa?$AAt?$AAc?$AAh?$AAS?$AAt?$AAr?$AAi?$AAn?$AAg?$AAB?$AAe?$AAg?$AAi?$AAn?$AAn?$AAi?$AAn?$AAg?$AA?5?$AAf?$AAa?$AAi?$AAl?$AAe?$AAd?$AA?$AA@ 1002b5ac     SDKRILGsm.obj
 0002:000055e8       ??_C@_1FI@CHCBFDKG@?$AAF?$AAa?$AAi?$AAl?$AAe?$AAd?$AA?5?$AAt?$AAo?$AA?5?$AAa?$AAl?$AAl?$AAo?$AAc?$AAa?$AAt?$AAe?$AA?5?$AAm?$AAe?$AAm?$AAo?$AAr?$AAy?$AA?5?$AAf?$AAo?$AAr?$AA?5?$AAC?$AAS@ 1002b5e8     SDKRILGsm.obj
 0002:00005640       ??_C@_1DO@MJJPMGLL@?$AAF?$AAi?$AAr?$AAs?$AAt?$AA?5?$AAc?$AAh?$AAa?$AAr?$AA?5?$AAo?$AAf?$AA?5?$AAr?$AAe?$AAs?$AAp?$AAo?$AAn?$AAs?$AAe?$AA?5?$AAi?$AAs?$AA?5?$AAN?$AAU?$AAL?$AAL?$AA?$AA@ 1002b640     SDKRILGsm.obj
 0002:00005680       ??_C@_1CO@LICIDLCC@?$AAP?$AAa?$AAr?$AAs?$AAe?$AAR?$AAs?$AAp?$AAP?$AAo?$AAs?$AAt?$AAf?$AAi?$AAx?$AA?5?$AAf?$AAa?$AAi?$AAl?$AAe?$AAd?$AA?$AA@ 1002b680     SDKRILGsm.obj
 0002:000056b0       ??_C@_1DK@LNPNOLFA@?$AAA?$AAS?$AAS?$AAE?$AAR?$AAT?$AAI?$AAO?$AAN?$AA?5?$AAF?$AAA?$AAI?$AAL?$AAU?$AAR?$AAE?$AA?3?$AA?5?$AA?$DN?$AA?$DN?$AA?$DN?$AA?$DO?$AAF?$AAA?$AAL?$AAS?$AAE?$AA?$AA@ 1002b6b0     SDKRILGsm.obj
 0002:000056ec       ??_C@_1DG@MFLPPEEM@?$AAM?$AAa?$AAt?$AAc?$AAh?$AAS?$AAt?$AAr?$AAi?$AAn?$AAg?$AAA?$AAn?$AAy?$AAw?$AAh?$AAe?$AAr?$AAe?$AA?5?$AAf?$AAa?$AAi?$AAl?$AAe?$AAd?$AA?$AA@ 1002b6ec     SDKRILGsm.obj
 0002:00005728       ??_C@_1HA@KOCKKBAK@?$AAG?$AAo?$AAb?$AAi?$AA?5?$AAA?$AAP?$AAI?$AA?5?$AAG?$AAe?$AAt?$AAD?$AAe?$AAf?$AAa?$AAu?$AAl?$AAt?$AAP?$AAr?$AAo?$AAf?$AAi?$AAl?$AAe?$AA?5?$AAF?$AAa?$AAi?$AAl?$AAe@ 1002b728     SDKRILGsm.obj
 0002:00005798       ??_C@_1FK@JOLKJEEG@?$AAP?$AAD?$AAP?$AA?5?$AAI?$AAP?$AA?5?$AAA?$AAd?$AAd?$AAr?$AAe?$AAs?$AAs?$AA?5?$AAl?$AAe?$AAn?$AAg?$AAt?$AAh?$AA?5?$AAs?$AAh?$AAo?$AAu?$AAl?$AAd?$AA?5?$AAb?$AAe?$AA?5@ 1002b798     SDKRILGsm.obj
 0002:000057f8       ??_C@_1HA@BAKBEOMG@?$AAG?$AAo?$AAb?$AAi?$AA?5?$AAA?$AAP?$AAI?$AA?5?$AAS?$AAe?$AAt?$AAD?$AAe?$AAf?$AAa?$AAu?$AAl?$AAt?$AAP?$AAr?$AAo?$AAf?$AAi?$AAl?$AAe?$AA?5?$AAF?$AAa?$AAi?$AAl?$AAe@ 1002b7f8     SDKRILGsm.obj
 0002:00005868       ??_C@_1GA@KBKDPB@?$AAD?$AAa?$AAt?$AAa?$AA?5?$AAs?$AAe?$AAs?$AAs?$AAi?$AAo?$AAn?$AA?5?$AAa?$AAl?$AAr?$AAe?$AAa?$AAd?$AAy?$AA?5?$AAa?$AAc?$AAt?$AAi?$AAv?$AAe?$AA?0?$AA?5?$AAD?$AAa?$AAt@ 1002b868     SDKRILGsm.obj
 0002:000058c8       ??_C@_1KA@PJKFIHBC@?$AAG?$AAo?$AAb?$AAi?$AA?5?$AAA?$AAP?$AAI?$AA?5?$AAS?$AAt?$AAa?$AAr?$AAt?$AAD?$AAa?$AAt?$AAa?$AAS?$AAe?$AAs?$AAs?$AAi?$AAo?$AAn?$AA?5?$AAF?$AAa?$AAi?$AAl?$AAe?$AAd@ 1002b8c8     SDKRILGsm.obj
 0002:00005968       ??_C@_1FI@NDPJCHOI@?$AAD?$AAa?$AAt?$AAa?$AA?5?$AAs?$AAe?$AAs?$AAs?$AAi?$AAo?$AAn?$AA?5?$AAN?$AAO?$AAT?$AA?5?$AAa?$AAc?$AAt?$AAi?$AAv?$AAe?$AA?0?$AA?5?$AAD?$AAa?$AAt?$AAs?$AAS?$AAe?$AAs@ 1002b968     SDKRILGsm.obj
 0002:000059c0       ??_C@_1GM@GNOCPKBO@?$AAG?$AAo?$AAb?$AAi?$AA?5?$AAA?$AAP?$AAI?$AA?5?$AAS?$AAt?$AAo?$AAp?$AAD?$AAa?$AAt?$AAa?$AAS?$AAe?$AAs?$AAs?$AAi?$AAo?$AAn?$AA?5?$AAF?$AAa?$AAi?$AAl?$AAe?$AAd?$AA?5@ 1002b9c0     SDKRILGsm.obj
 0002:00005a30       ??_C@_1EI@OECGHCKD@?$AAP?$AAh?$AAo?$AAn?$AAe?$AAB?$AAo?$AAo?$AAk?$AAT?$AAy?$AAp?$AAe?$AA?5?$AA?$DN?$AA?5?$AA?$CF?$AAd?$AA?5?$AAi?$AAs?$AA?5?$AAn?$AAo?$AAt?$AA?5?$AAs?$AAu?$AAp?$AAp?$AAo?$AAr@ 1002ba30     SDKRILGsm.obj
 0002:00005a78       ??_C@_01MIFGBAGJ@?$CL?$AA@ 1002ba78     SDKRILGsm.obj
 0002:00005a80       ??_C@_1GM@DLEGADMH@?$AAG?$AAe?$AAt?$AAV?$AAo?$AAi?$AAc?$AAe?$AAN?$AAu?$AAm?$AAb?$AAe?$AAr?$AA?5?$AAr?$AAe?$AAt?$AAu?$AAr?$AAn?$AAs?$AA?5?$AAa?$AAc?$AAc?$AAe?$AAp?$AAt?$AAa?$AAb?$AAl@ 1002ba80     SDKRILGsm.obj
 0002:00005af0       ??_C@_1EA@IOCDIIML@?$AAi?$AAn?$AAe?$AAt?$AA_?$AAn?$AAt?$AAo?$AAa?$AA?5?$AAf?$AAa?$AAi?$AAl?$AAe?$AAd?$AA?0?$AA?5?$AAu?$AAA?$AAd?$AAd?$AAr?$AAe?$AAs?$AAs?$AA?5?$AA?$DN?$AA?5?$AA?$CF?$AAd?$AA?$AA@ 1002baf0     SDKRILGsm.obj
 0002:00005b30       ??_C@_1FO@KFOECAIJ@?$AAS?$AAw?$AAi?$AAG?$AAe?$AAt?$AAP?$AAi?$AAn?$AAS?$AAt?$AAa?$AAt?$AAu?$AAs?$AA?5?$AAf?$AAa?$AAi?$AAl?$AAe?$AAd?$AA?5?$AAw?$AAi?$AAt?$AAh?$AA?5?$AAe?$AAr?$AAr?$AAo@ 1002bb30     SDKRILGsm.obj
 0002:00005b90       ??_C@_1GC@PAJCJILL@?$AAS?$AAw?$AAi?$AAG?$AAe?$AAt?$AAS?$AAi?$AAm?$AAL?$AAo?$AAc?$AAk?$AAG?$AAo?$AAb?$AAi?$AA?5?$AAf?$AAa?$AAi?$AAl?$AAe?$AAd?$AA?5?$AAw?$AAi?$AAt?$AAh?$AA?5?$AAe?$AAr@ 1002bb90     SDKRILGsm.obj
 0002:00005bf8       ??_C@_1GC@GKCJCBCO@?$AAS?$AAw?$AAi?$AAS?$AAe?$AAt?$AAS?$AAi?$AAm?$AAL?$AAo?$AAc?$AAk?$AAG?$AAo?$AAb?$AAi?$AA?5?$AAf?$AAa?$AAi?$AAl?$AAe?$AAd?$AA?5?$AAw?$AAi?$AAt?$AAh?$AA?5?$AAe?$AAr@ 1002bbf8     SDKRILGsm.obj
 0002:00005c60       ??_C@_1KC@FHHMLAJE@?$AAA?$AAS?$AAS?$AAE?$AAR?$AAT?$AAI?$AAO?$AAN?$AA?5?$AAF?$AAA?$AAI?$AAL?$AAU?$AAR?$AAE?$AA?3?$AA?5?$AA?$DN?$AA?$DN?$AA?$DN?$AA?$DO?$AAp?$AAS?$AAi?$AAm?$AA?9?$AA?$DO?$AAd?$AAw?$AAF@ 1002bc60     SDKRILGsm.obj
 0002:00005d08       ??_C@_1FO@INLLPEEI@?$AAS?$AAw?$AAi?$AAS?$AAe?$AAt?$AAS?$AAi?$AAm?$AAP?$AAa?$AAs?$AAs?$AAw?$AAo?$AAr?$AAd?$AAG?$AAo?$AAb?$AAi?$AA?3?$AA?5?$AAP?$AAI?$AAN?$AA?5?$AAT?$AAY?$AAP?$AAE?$AA?5@ 1002bd08     SDKRILGsm.obj
 0002:00005d68       ??_C@_1LE@EGBCPJCM@?$AAS?$AAw?$AAi?$AAG?$AAe?$AAt?$AAS?$AAi?$AAm?$AAV?$AAe?$AAr?$AAi?$AAf?$AAy?$AAG?$AAo?$AAb?$AAi?$AA?3?$AA?5?$AAP?$AAi?$AAn?$AA?5?$AAN?$AAu?$AAm?$AA?5?$AA?$DN?$AA?5?$AA?$CF@ 1002bd68     SDKRILGsm.obj
 0002:00005e20       ??_C@_1MC@BEEDPLOB@?$AAS?$AAw?$AAi?$AAS?$AAe?$AAt?$AAS?$AAi?$AAm?$AAV?$AAe?$AAr?$AAi?$AAf?$AAy?$AAG?$AAo?$AAb?$AAi?$AA?3?$AA?5?$AAP?$AAi?$AAn?$AA?5?$AAN?$AAu?$AAm?$AA?5?$AA?$DN?$AA?5?$AA?$CF@ 1002be20     SDKRILGsm.obj
 0002:00005ee8       ??_C@_1GG@BNCHPDBE@?$AAS?$AAw?$AAi?$AAS?$AAe?$AAt?$AAS?$AAi?$AAm?$AAV?$AAe?$AAr?$AAi?$AAf?$AAy?$AAG?$AAo?$AAb?$AAi?$AA?5?$AAf?$AAa?$AAi?$AAl?$AAe?$AAd?$AA?5?$AAw?$AAi?$AAt?$AAh?$AA?5@ 1002bee8     SDKRILGsm.obj
 0002:00005f50       ??_C@_1FI@KFAHKIEL@?$AAG?$AAo?$AAb?$AAi?$AA?5?$AAA?$AAP?$AAI?$AA?5?$AAG?$AAe?$AAt?$AAB?$AAy?$AAt?$AAe?$AAT?$AAo?$AAt?$AAa?$AAl?$AAs?$AA?5?$AAr?$AAe?$AAt?$AAu?$AAr?$AAn?$AAe?$AAd?$AA?5@ 1002bf50     SDKRILGsm.obj
 0002:00005fa8       ??_C@_1BI@FPEBAIFJ@?$AAS?$AAe?$AAt?$AAS?$AAM?$AAS?$AAR?$AAo?$AAu?$AAt?$AAe?$AA?$AA@ 1002bfa8     SDKRILGsm.obj
 0002:00005fc0       ??_C@_1DO@HDOCPDLL@?$AAS?$AAe?$AAt?$AAS?$AAM?$AAS?$AAR?$AAo?$AAu?$AAt?$AAe?$AA?5?$AAf?$AAa?$AAi?$AAl?$AAe?$AAd?$AA?0?$AA?5?$AAr?$AAe?$AAt?$AA?5?$AA?$DN?$AA?5?$AA0?$AAx?$AA?$CF?$AAx?$AA?$AA@ 1002bfc0     SDKRILGsm.obj
 0002:00006000       ??_C@_1FK@CJIKLLFI@?$AAS?$AAe?$AAt?$AAS?$AAM?$AAS?$AAB?$AAr?$AAo?$AAa?$AAd?$AAc?$AAa?$AAs?$AAt?$AAA?$AAc?$AAt?$AAi?$AAv?$AAa?$AAt?$AAi?$AAo?$AAn?$AA?5?$AAf?$AAa?$AAi?$AAl?$AAe?$AAd@ 1002c000     SDKRILGsm.obj
 0002:0000605c       ??_C@_1DM@FLMOPHIP@?$AAG?$AAo?$AAb?$AAi?$AA?5?$AAS?$AAM?$AAS?$AA?5?$AAS?$AAe?$AAt?$AA?5?$AAP?$AAr?$AAo?$AAt?$AAo?$AAc?$AAo?$AAl?$AA?5?$AAf?$AAa?$AAi?$AAl?$AAe?$AAd?$AA?$CB?$AA?$AA@ 1002c05c     SDKRILGsm.obj
 0002:00006098       ??_C@_1FA@DDJFLNBN@?$AAT?$AAo?$AAt?$AAa?$AAl?$AA?5?$AAU?$AAN?$AAR?$AAE?$AAA?$AAD?$AA?5?$AAm?$AAs?$AAg?$AAs?$AA?5?$AA?$DN?$AA?5?$AA?$CF?$AAl?$AAu?$AA?0?$AA?5?$AAS?$AAi?$AAm?$AA?5?$AAM?$AAs?$AAg@ 1002c098     SDKRILGsm.obj
 0002:000060e8       ??_C@_1JO@OAKEDNKG@?$AAG?$AAo?$AAb?$AAi?$AA?5?$AAG?$AAe?$AAt?$AAS?$AAM?$AAS?$AA?5?$AAL?$AAo?$AAo?$AAp?$AA?5?$AAi?$AAn?$AAd?$AAe?$AAx?$AA?5?$AAi?$AA?5?$AA?$DN?$AA?5?$AA?$CF?$AAd?$AA?0?$AA?5?$AAM@ 1002c0e8     SDKRILGsm.obj
 0002:00006188       ??_C@_1DA@PGEAIOMA@?$AAG?$AAo?$AAb?$AAi?$AA?5?$AAG?$AAe?$AAt?$AAS?$AAM?$AAS?$AA?5?$AAr?$AAc?$AAv?$AAd?$AA?5?$AAi?$AAn?$AAf?$AAo?$AA?3?$AA?5?$AA?$AA@ 1002c188     SDKRILGsm.obj
 0002:000061b8       ??_C@_1HI@BHCOODPA@?$AAu?$AAM?$AAs?$AAg?$AAT?$AAa?$AAg?$AA?5?$AA?$DN?$AA?5?$AA?$CF?$AAd?$AA?0?$AA?5?$AAu?$AAM?$AAs?$AAg?$AAF?$AAo?$AAr?$AAm?$AAa?$AAt?$AA?5?$AA?$DN?$AA?5?$AA?$CF?$AAd?$AA?0?$AA?5?$AAu@ 1002c1b8     SDKRILGsm.obj
 0002:00006230       ??_C@_1FC@OOHMDPLG@?$AAD?$AAe?$AAc?$AAo?$AAd?$AAe?$AAC?$AAo?$AAm?$AAp?$AAl?$AAe?$AAt?$AAe?$AAP?$AAD?$AAU?$AA?5?$AAf?$AAa?$AAi?$AAl?$AAe?$AAd?$AA?5?$AAw?$AAi?$AAt?$AAh?$AA?5?$AAe?$AAr@ 1002c230     SDKRILGsm.obj
 0002:00006284       ??_C@_1DG@KNBLEEJF@?$AA?5?$AAM?$AAs?$AAg?$AA?5?$AAT?$AAa?$AAg?$AA?5?$AA?$DN?$AA?5?$AA?$CF?$AAd?$AA?5?$AAi?$AAs?$AA?5?$AAi?$AAn?$AAc?$AAo?$AAr?$AAr?$AAe?$AAc?$AAt?$AA?$AA@ 1002c284     SDKRILGsm.obj
 0002:000062c0       ??_C@_1FC@JILNKFFD@?$AAE?$AAn?$AAc?$AAo?$AAd?$AAe?$AAM?$AAO?$AAP?$AAD?$AAU?$AA?5?$AAf?$AAu?$AAn?$AAc?$AAt?$AAi?$AAo?$AAn?$AA?5?$AAf?$AAa?$AAi?$AAl?$AAe?$AAd?$AA?5?$AAw?$AAi?$AAt?$AAh@ 1002c2c0     SDKRILGsm.obj
 0002:00006318       ??_C@_1GE@OGOJBMCK@?$AAF?$AAo?$AAr?$AA?5?$AAM?$AAu?$AAl?$AAt?$AAi?$AAp?$AAa?$AAr?$AAt?$AA?5?$AAS?$AAM?$AAS?$AA?0?$AA?5?$AAs?$AAe?$AAt?$AA?5?$AAl?$AAi?$AAn?$AAk?$AA?5?$AAt?$AAi?$AAm?$AAe@ 1002c318     SDKRILGsm.obj
 0002:00006380       ??_C@_1FM@MCIEPCHM@?$AAL?$AAe?$AAn?$AAg?$AAt?$AAh?$AA?5?$AAo?$AAf?$AA?5?$AAS?$AAM?$AAS?$AA?5?$AAM?$AAs?$AAg?$AA?5?$AAs?$AAt?$AAo?$AAr?$AAe?$AAd?$AA?5?$AAi?$AAn?$AA?5?$AAt?$AAh?$AAe?$AA?5@ 1002c380     SDKRILGsm.obj
 0002:000063e0       ??_C@_1GE@IGHIFCFD@?$AAG?$AAo?$AAb?$AAi?$AA?5?$AAG?$AAe?$AAt?$AAS?$AAM?$AAS?$AAC?$AAA?$AAd?$AAd?$AAr?$AAe?$AAs?$AAs?$AA?5?$AAf?$AAa?$AAi?$AAl?$AAe?$AAd?$AA?5?$AAw?$AAi?$AAt?$AAh?$AA?5@ 1002c3e0     SDKRILGsm.obj
 0002:00006448       ??_C@_1FM@EPAKNNDD@?$AAS?$AAw?$AAi?$AAG?$AAe?$AAt?$AAG?$AAs?$AAm?$AAS?$AAM?$AAS?$AAC?$AAA?$AAd?$AAd?$AAr?$AAf?$AAa?$AAi?$AAl?$AAe?$AAd?$AA?5?$AAw?$AAi?$AAt?$AAh?$AA?5?$AAe?$AAr?$AAr@ 1002c448     SDKRILGsm.obj
 0002:000064a4       ??_C@_1DI@JAFPEFLH@?$AAS?$AAw?$AAi?$AAG?$AAe?$AAt?$AAG?$AAs?$AAm?$AAS?$AAM?$AAS?$AAC?$AAA?$AAd?$AAd?$AAr?$AA?5?$AAf?$AAa?$AAk?$AAi?$AAn?$AAg?$AA?5?$AAO?$AAK?$AA?$AA@ 1002c4a4     SDKRILGsm.obj
 0002:000064dc       ??_C@_03BHHPDANN@145?$AA@  1002c4dc     SDKRILGsm.obj
 0002:000064e0       ??_C@_02DKCKIIND@?$CFs?$AA@ 1002c4e0     SDKRILGsm.obj
 0002:000064e4       ??_C@_02KEKBCPNI@?$CL7?$AA@ 1002c4e4     SDKRILGsm.obj
 0002:000064e8       ??_C@_1FO@GJFLFEFO@?$AAS?$AAw?$AAi?$AAS?$AAe?$AAt?$AAG?$AAs?$AAm?$AAS?$AAM?$AAS?$AAC?$AAA?$AAd?$AAd?$AAr?$AA?5?$AAf?$AAa?$AAi?$AAl?$AAe?$AAd?$AA?5?$AAw?$AAi?$AAt?$AAh?$AA?5?$AAe?$AAr@ 1002c4e8     SDKRILGsm.obj
 0002:00006548       ??_C@_0N@LCDEPHKG@AT?$CLCPOL?$DN?0?$CFu?$AN?$AA@ 1002c548     SDKRILGsm.obj
 0002:00006558       ??_C@_1HE@FFAGMDC@?$AAA?$AAT?$AA?5?$AAc?$AAo?$AAm?$AAm?$AAa?$AAn?$AAd?$AA?5?$AAt?$AAo?$AA?5?$AAs?$AAe?$AAt?$AA?5?$AAt?$AAh?$AAe?$AA?5?$AAO?$AAp?$AAe?$AAr?$AAa?$AAt?$AAo?$AAr?$AA?5?$AAf@ 1002c558     SDKRILGsm.obj
 0002:000065d0       ??_C@_1IA@PDGFBFMK@?$AAS?$AAw?$AAi?$AAG?$AAe?$AAt?$AAP?$AAr?$AAe?$AAf?$AAe?$AAr?$AAr?$AAe?$AAd?$AAO?$AAp?$AAe?$AAr?$AAa?$AAt?$AAo?$AAr?$AAL?$AAi?$AAs?$AAt?$AAG?$AAo?$AAb?$AAi?$AA?3@ 1002c5d0     SDKRILGsm.obj
 0002:00006650       ??_C@_1HK@IEKKLAMD@?$AAS?$AAw?$AAi?$AAG?$AAe?$AAt?$AAP?$AAr?$AAe?$AAf?$AAe?$AAr?$AAr?$AAe?$AAd?$AAO?$AAp?$AAe?$AAr?$AAa?$AAt?$AAo?$AAr?$AAL?$AAi?$AAs?$AAt?$AAG?$AAo?$AAb?$AAi?$AA?3@ 1002c650     SDKRILGsm.obj
 0002:000066cc       ??_C@_09ODKAGID@AT?$CLCPOL?$DP?$AN?$AA@ 1002c6cc     SDKRILGsm.obj
 0002:000066d8       ??_C@_07PALFFFHM@?$CLCPOL?3?5?$AA@ 1002c6d8     SDKRILGsm.obj
 0002:000066e0       ??_C@_1HI@DONDEIHO@?$AAS?$AAw?$AAi?$AAG?$AAe?$AAt?$AAP?$AAr?$AAe?$AAf?$AAe?$AAr?$AAr?$AAe?$AAd?$AAO?$AAp?$AAe?$AAr?$AAa?$AAt?$AAo?$AAr?$AAL?$AAi?$AAs?$AAt?$AAG?$AAo?$AAb?$AAi?$AA?3@ 1002c6e0     SDKRILGsm.obj
 0002:00006758       ??_C@_1HK@NPHGJILE@?$AAS?$AAw?$AAi?$AAG?$AAe?$AAt?$AAP?$AAr?$AAe?$AAf?$AAe?$AAr?$AAr?$AAe?$AAd?$AAO?$AAp?$AAe?$AAr?$AAa?$AAt?$AAo?$AAr?$AAL?$AAi?$AAs?$AAt?$AAG?$AAo?$AAb?$AAi?$AA?3@ 1002c758     SDKRILGsm.obj
 0002:000067d8       ??_C@_1HM@CODMFOKG@?$AAS?$AAw?$AAi?$AAG?$AAe?$AAt?$AAP?$AAr?$AAe?$AAf?$AAe?$AAr?$AAr?$AAe?$AAd?$AAO?$AAp?$AAe?$AAr?$AAa?$AAt?$AAo?$AAr?$AAL?$AAi?$AAs?$AAt?$AAG?$AAo?$AAb?$AAi?$AA?3@ 1002c7d8     SDKRILGsm.obj
 0002:00006854       ??_C@_02GMHACPFF@?$CFu?$AA@ 1002c854     SDKRILGsm.obj
 0002:00006858       ??_C@_1HA@MNCLLMHO@?$AAS?$AAw?$AAi?$AAG?$AAe?$AAt?$AAP?$AAr?$AAe?$AAf?$AAe?$AAr?$AAr?$AAe?$AAd?$AAO?$AAp?$AAe?$AAr?$AAa?$AAt?$AAo?$AAr?$AAL?$AAi?$AAs?$AAt?$AAG?$AAo?$AAb?$AAi?$AA?3@ 1002c858     SDKRILGsm.obj
 0002:000068c8       ??_C@_0M@BBPGAMA@AT?$CLCPOL?$DN?$CFu?$AN?$AA@ 1002c8c8     SDKRILGsm.obj
 0002:000068d4       ??_C@_09IBCBMHAO@AT?$CLCPOL?$DN?0?$AA@ 1002c8d4     SDKRILGsm.obj
 0002:000068e0       ??_C@_0M@INIAHFCD@AT?$CLCPOL?$DN?$CFu?0?$AA@ 1002c8e0     SDKRILGsm.obj
 0002:000068f0       ??_C@_1EM@MIOLNEAM@?$AAA?$AAS?$AAS?$AAE?$AAR?$AAT?$AAI?$AAO?$AAN?$AA?5?$AAF?$AAA?$AAI?$AAL?$AAU?$AAR?$AAE?$AA?3?$AA?5?$AA?$DN?$AA?$DN?$AA?$DN?$AA?$DO?$AAN?$AAU?$AAL?$AAL?$AA?5?$AA?$CB?$AA?$DN?$AA?5?$AAs@ 1002c8f0     SDKRILGsm.obj
 0002:0000693c       ??_C@_06PAOJOCPG@2?0?$CC?$CFs?$CC?$AA@ 1002c93c     SDKRILGsm.obj
 0002:00006944       ??_C@_06MBABPIGL@1?0?$CC?$CFs?$CC?$AA@ 1002c944     SDKRILGsm.obj
 0002:0000694c       ??_C@_06GHHGPDNP@0?0?$CC?$CFs?$CC?$AA@ 1002c94c     SDKRILGsm.obj
 0002:00006954       ??_C@_06GNOEPGFG@?00?00?01?$AA@ 1002c954     SDKRILGsm.obj
 0002:0000695c       ??_C@_06MMEDKAHC@?00?01?00?$AA@ 1002c95c     SDKRILGsm.obj
 0002:00006964       ??_C@_06LPKDBELC@?01?00?00?$AA@ 1002c964     SDKRILGsm.obj
 0002:00006970       ??_C@_1HG@JGKMANJI@?$AAS?$AAw?$AAi?$AAR?$AAe?$AAm?$AAo?$AAv?$AAe?$AAP?$AAr?$AAe?$AAf?$AAe?$AAr?$AAr?$AAe?$AAd?$AAO?$AAp?$AAe?$AAr?$AAa?$AAt?$AAo?$AAr?$AA?3?$AA?5?$AAE?$AAx?$AAt?$AAr@ 1002c970     SDKRILGsm.obj
 0002:000069e8       ??_C@_1HA@MANJIMOM@?$AAS?$AAw?$AAi?$AAR?$AAe?$AAm?$AAo?$AAv?$AAe?$AAP?$AAr?$AAe?$AAf?$AAe?$AAr?$AAr?$AAe?$AAd?$AAO?$AAp?$AAe?$AAr?$AAa?$AAt?$AAo?$AAr?$AA?3?$AA?5?$AAF?$AAa?$AAi?$AAl@ 1002c9e8     SDKRILGsm.obj
 0002:00006a58       ??_C@_1JG@OGBAOGIK@?$AAS?$AAo?$AAr?$AAr?$AAy?$AA?0?$AA?5?$AAc?$AAo?$AAu?$AAl?$AAd?$AAn?$AA?8?$AAt?$AA?5?$AAh?$AAe?$AAl?$AAp?$AA?4?$AA?5?$AAI?$AAn?$AAi?$AAt?$AAi?$AAa?$AAt?$AAe?$AAD?$AAo@ 1002ca58     SDKRILGsm.obj
 0002:00006af0       ??_C@_1II@MDGPMINE@?$AAS?$AAw?$AAi?$AAS?$AAe?$AAt?$AAH?$AAo?$AAs?$AAt?$AAS?$AAt?$AAa?$AAr?$AAt?$AAu?$AAp?$AA?9?$AA?$DO?$AAS?$AAe?$AAt?$AAP?$AAo?$AAw?$AAe?$AAr?$AA?$CI?$AAG?$AAo?$AAb?$AAi@ 1002caf0     SDKRILGsm.obj
 0002:00006b78       ??_C@_1HG@BMILBMPA@?$AAF?$AAi?$AAn?$AAd?$AAR?$AAF?$AAI?$AAn?$AAf?$AAo?$AAI?$AAn?$AAd?$AAe?$AAx?$AA?5?$AA?$CI?$AAR?$AAa?$AAd?$AAi?$AAo?$AAT?$AAe?$AAc?$AAh?$AA?5?$AA?$DN?$AA?5?$AA?$CF?$AAd?$AA?$CJ@ 1002cb78     SDKRILGsm.obj
 0002:00006bf0       ??_C@_1GK@NCGGINBB@?$AAS?$AAw?$AAi?$AAG?$AAe?$AAt?$AAG?$AAs?$AAm?$AAS?$AAy?$AAs?$AAt?$AAe?$AAm?$AAS?$AAt?$AAa?$AAt?$AAu?$AAs?$AA?3?$AA?5?$AAG?$AAe?$AAt?$AAR?$AAF?$AAI?$AAn?$AAf?$AAo@ 1002cbf0     SDKRILGsm.obj
 0002:00006c60       ??_C@_1KA@ECBENMPD@?$AAG?$AAe?$AAt?$AAR?$AAF?$AAI?$AAn?$AAf?$AAo?$AA?5?$AAr?$AAe?$AAt?$AAu?$AAr?$AAn?$AAs?$AA?5?$AAe?$AAr?$AAr?$AAo?$AAr?$AA?5?$AAb?$AAu?$AAt?$AA?5?$AAG?$AAe?$AAt?$AAS@ 1002cc60     SDKRILGsm.obj
 0002:00006d00       ??_C@_1BAC@MCKGFELM@?$AAG?$AAe?$AAt?$AAR?$AAF?$AAI?$AAn?$AAf?$AAo?$AA?5?$AAr?$AAe?$AAt?$AAu?$AAr?$AAn?$AAs?$AA?5?$AAe?$AAr?$AAr?$AAo?$AAr?$AA?5?$AAb?$AAu?$AAt?$AA?5?$AAG?$AAe?$AAt?$AAS@ 1002cd00     SDKRILGsm.obj
 0002:00006e04       ??_C@_17JJEPAIJF@?$AAU?$AAK?$AAN?$AA?$AA@ 1002ce04     SDKRILGsm.obj
 0002:00006e10       ??_C@_1HK@HOMEMJDI@?$AAS?$AAw?$AAi?$AAG?$AAe?$AAt?$AAG?$AAs?$AAm?$AAS?$AAy?$AAs?$AAt?$AAe?$AAm?$AAS?$AAt?$AAa?$AAt?$AAu?$AAs?$AA?3?$AA?5?$AAG?$AAe?$AAt?$AAS?$AAe?$AAr?$AAv?$AAi?$AAn@ 1002ce10     SDKRILGsm.obj
 0002:00006e90       ??_C@_1GI@FKGLLKGI@?$AAS?$AAw?$AAi?$AAG?$AAe?$AAt?$AAG?$AAs?$AAm?$AAS?$AAy?$AAs?$AAt?$AAe?$AAm?$AAS?$AAt?$AAa?$AAt?$AAu?$AAs?$AA?3?$AA?5?$AAG?$AAe?$AAt?$AAP?$AAo?$AAw?$AAe?$AAr?$AA?5@ 1002ce90     SDKRILGsm.obj
 0002:00006ef8       ??_C@_1FM@NOCFGHPB@?$AAE?$AAn?$AAc?$AAo?$AAd?$AAe?$AAr?$AAU?$AAs?$AAe?$AAr?$AAD?$AAa?$AAt?$AAa?$AAH?$AAd?$AAr?$AA?3?$AAe?$AAn?$AAc?$AAo?$AAd?$AAi?$AAn?$AAg?$AA?5?$AAt?$AAy?$AAp?$AAe@ 1002cef8     sms.obj
 0002:00006f54       ??_C@_1BE@IKEJLIJH@?$AA?4?$AA?2?$AAs?$AAm?$AAs?$AA?4?$AAc?$AAp?$AAp?$AA?$AA@ 1002cf54     sms.obj
 0002:00006f68       ??_C@_1EG@EFHCBNKG@?$AAM?$AAs?$AAg?$AA?5?$AAT?$AAY?$AAP?$AAE?$AA?5?$AAi?$AAs?$AA?5?$AAN?$AAO?$AAT?$AA?5?$AAP?$AAO?$AAI?$AAN?$AAT?$AA_?$AAT?$AAO?$AA_?$AAP?$AAO?$AAI?$AAN?$AAT?$AA_?$AAM@ 1002cf68     sms.obj
 0002:00006fb0       ??_C@_1EO@LKNCDOLG@?$AAT?$AAE?$AAL?$AAE?$AAS?$AAE?$AAR?$AAV?$AAI?$AAC?$AAE?$AA?5?$AAI?$AAD?$AAE?$AAN?$AAT?$AAI?$AAF?$AAI?$AAE?$AAR?$AA?5?$AAL?$AAE?$AAN?$AA?5?$AAi?$AAs?$AA?5?$AAn?$AAo@ 1002cfb0     sms.obj
 0002:00007000       ??_C@_1EC@GMOLNILJ@?$AAB?$AAE?$AAA?$AAR?$AAE?$AAR?$AA_?$AAR?$AAE?$AAP?$AAL?$AAY?$AA_?$AAH?$AAD?$AAR?$AA_?$AAL?$AAE?$AAN?$AA?5?$AAi?$AAs?$AA?5?$AAn?$AAo?$AAt?$AA?5?$AA?$DN?$AA?5?$AA?$CF?$AAd@ 1002d000     sms.obj
 0002:00007044       ??_C@_1DK@PNOOBAMJ@?$AAO?$AAR?$AAI?$AAG?$AAA?$AAD?$AAD?$AAR?$AA_?$AAH?$AAD?$AAR?$AA_?$AAL?$AAE?$AAN?$AA?5?$AAi?$AAs?$AA?5?$AAn?$AAo?$AAt?$AA?5?$AA?$DN?$AA?5?$AA?$CF?$AAd?$AA?$AA@ 1002d044     sms.obj
 0002:00007080       ??_C@_1DG@HMDOPOON@?$AAF?$AAa?$AAi?$AAl?$AAe?$AAd?$AA?5?$AAt?$AAo?$AA?5?$AAa?$AAl?$AAl?$AAo?$AAc?$AAa?$AAt?$AAe?$AA?5?$AAm?$AAe?$AAm?$AAe?$AAo?$AAr?$AAy?$AA?$AA@ 1002d080     sms.obj
 0002:000070b8       ??_C@_1GO@PEGBKOFG@?$AAU?$AAn?$AAh?$AAa?$AAn?$AAd?$AAl?$AAe?$AAd?$AA?5?$AAI?$AAd?$AAe?$AAn?$AAt?$AAi?$AAf?$AAi?$AAe?$AAr?$AA?5?$AA?$DN?$AA?5?$AA?$CF?$AAd?$AA?5?$AAo?$AAf?$AA?5?$AAL?$AAe?$AAn@ 1002d0b8     sms.obj
 0002:00007128       ??_C@_1EO@GCPOABEA@?$AAU?$AAn?$AAk?$AAn?$AAo?$AAw?$AAn?$AA?5?$AAI?$AAD?$AAE?$AAN?$AAT?$AAI?$AAF?$AAI?$AAE?$AAR?$AA?5?$AAi?$AAn?$AA?5?$AAM?$AAT?$AA?5?$AAS?$AAM?$AAS?$AA?5?$AAd?$AAa?$AAt@ 1002d128     sms.obj
 0002:00007178       ??_C@_1EO@CCKCOLMG@?$AAM?$AAS?$AAG?$AA_?$AAS?$AAU?$AAB?$AA_?$AAI?$AAD?$AAE?$AAN?$AAT?$AAI?$AAF?$AAI?$AAE?$AAR?$AA_?$AAH?$AAD?$AAR?$AA_?$AAL?$AAE?$AAN?$AA?5?$AAi?$AAs?$AA?5?$AAn?$AAo@ 1002d178     sms.obj
 0002:000071c8       ??_C@_1CO@IOEKGKGG@?$AAM?$AAS?$AAG?$AA?5?$AAT?$AAY?$AAP?$AAE?$AA?5?$AA?$CB?$AA?$DN?$AA?5?$AAD?$AAE?$AAL?$AAI?$AAV?$AAE?$AAR?$AA_?$AAM?$AAT?$AA?$AA@ 1002d1c8     sms.obj
 0002:000071f8       ??_C@_1FG@INCGAPG@?$AAP?$AAR?$AAI?$AAO?$AAR?$AAI?$AAY?$AA_?$AAS?$AAU?$AAB?$AA_?$AAI?$AAD?$AAE?$AAN?$AAT?$AAI?$AAF?$AAI?$AAE?$AAR?$AA_?$AAH?$AAD?$AAR?$AA_?$AAL?$AAE?$AAN?$AA?5?$AAi@ 1002d1f8     sms.obj
 0002:00007250       ??_C@_1GC@HALFHKFI@?$AAM?$AAS?$AAG?$AA_?$AAT?$AAI?$AAM?$AAE?$AAS?$AAT?$AAA?$AAM?$AAP?$AA_?$AAS?$AAU?$AAB?$AA_?$AAI?$AAN?$AAD?$AAE?$AAT?$AAI?$AAF?$AAI?$AAE?$AAR?$AA_?$AAH?$AAD?$AAR@ 1002d250     sms.obj
 0002:000072b8       ??_C@_1GM@NOMDIKLI@?$AAL?$AAA?$AAN?$AAG?$AAU?$AAA?$AAG?$AAE?$AA_?$AAI?$AAN?$AAD?$AAI?$AAC?$AAA?$AAT?$AAO?$AAR?$AA_?$AAS?$AAU?$AAB?$AA_?$AAI?$AAN?$AAD?$AAE?$AAT?$AAI?$AAF?$AAI?$AAE@ 1002d2b8     sms.obj
 0002:00007328       ??_C@_1IK@JAKGJCEG@?$AAL?$AAa?$AAn?$AAg?$AAu?$AAa?$AAg?$AAe?$AA?5?$AAI?$AAn?$AAd?$AAi?$AAc?$AAa?$AAt?$AAo?$AAr?$AA?5?$AAs?$AAu?$AAb?$AA?5?$AAi?$AAd?$AAe?$AAn?$AAt?$AAi?$AAf?$AAi?$AAe@ 1002d328     sms.obj
 0002:000073b4       ??_C@_1DC@KLLMIMCM@?$AAC?$AAa?$AAl?$AAl?$AAb?$AAa?$AAc?$AAk?$AA?5?$AAN?$AAu?$AAm?$AAb?$AAe?$AAr?$AA?5?$AAL?$AAe?$AAn?$AA?5?$AA?$DN?$AA?5?$AA?$CF?$AAd?$AA?$AA@ 1002d3b4     sms.obj
 0002:000073e8       ??_C@_1FE@NFJGFBHJ@?$AAU?$AAn?$AAk?$AAn?$AAo?$AAw?$AAn?$AA?5?$AAs?$AAu?$AAb?$AAi?$AAd?$AAe?$AAn?$AAt?$AAi?$AAf?$AAi?$AAe?$AAr?$AA?5?$AAi?$AAn?$AA?5?$AAb?$AAe?$AAa?$AAr?$AAe?$AAr?$AA?5@ 1002d3e8     sms.obj
 0002:00007440       ??_C@_1JM@JMEBKNPG@?$AAN?$AAu?$AAm?$AAb?$AAe?$AAr?$AA?5?$AAm?$AAo?$AAd?$AAe?$AA?5?$AAo?$AAr?$AA?5?$AAD?$AAi?$AAg?$AAi?$AAt?$AA?5?$AAm?$AAo?$AAd?$AAe?$AA?5?$AAi?$AAs?$AA?5?$AAn?$AAo?$AAt@ 1002d440     sms.obj
 0002:000074e0       ??_C@_1FG@FEDOCGOG@?$AAD?$AAe?$AAc?$AAo?$AAd?$AAe?$AAC?$AAa?$AAl?$AAl?$AAb?$AAa?$AAc?$AAk?$AAA?$AAd?$AAd?$AAr?$AA?5?$AAw?$AAi?$AAt?$AAh?$AA?5?$AAD?$AAi?$AAg?$AAi?$AAt?$AAM?$AAo?$AAd@ 1002d4e0     sms.obj
 0002:00007538       ??_C@_1EO@HNMPJHHG@?$AAU?$AAs?$AAe?$AAr?$AA?5?$AAd?$AAa?$AAt?$AAa?$AA?5?$AAe?$AAn?$AAc?$AAo?$AAn?$AAd?$AAi?$AAg?$AA?5?$AA?$CF?$AAd?$AAi?$AAs?$AA?5?$AAn?$AAo?$AAt?$AA?5?$AAs?$AAu?$AAp?$AAp@ 1002d538     sms.obj
 0002:00007588       ??_C@_1CO@OHGDNACG@?$AAS?$AAp?$AAl?$AAi?$AAt?$AAP?$AAa?$AAr?$AAa?$AAm?$AAM?$AAT?$AAS?$AAm?$AAs?$AA?5?$AAf?$AAa?$AAi?$AAl?$AAe?$AAd?$AA?$AA@ 1002d588     sms.obj
 0002:000075b8       ??_C@_1DA@PGOOBPG@?$AAD?$AAe?$AAc?$AAo?$AAd?$AAe?$AAO?$AAr?$AAi?$AAg?$AAi?$AAn?$AAA?$AAd?$AAd?$AAr?$AA?5?$AAf?$AAa?$AAi?$AAl?$AAe?$AAd?$AA?$AA@ 1002d5b8     sms.obj
 0002:000075e8       ??_C@_1DM@OJPOKNKC@?$AAO?$AAr?$AAi?$AAg?$AAi?$AAn?$AAa?$AAt?$AAi?$AAn?$AAg?$AA?5?$AAA?$AAd?$AAd?$AAr?$AAe?$AAs?$AAs?$AA?5?$AAn?$AAo?$AAt?$AA?5?$AAf?$AAo?$AAu?$AAn?$AAd?$AA?$AA@ 1002d5e8     sms.obj
 0002:00007624       ??_C@_1DA@PBCMPOE@?$AAD?$AAe?$AAc?$AAo?$AAd?$AAe?$AAB?$AAe?$AAa?$AAr?$AAe?$AAr?$AAD?$AAa?$AAt?$AAa?$AA?5?$AAf?$AAa?$AAi?$AAl?$AAe?$AAd?$AA?$AA@ 1002d624     sms.obj
 0002:00007654       ??_C@_1CM@FKFFJDCL@?$AAD?$AAe?$AAc?$AAo?$AAd?$AAe?$AAU?$AAs?$AAe?$AAr?$AAD?$AAa?$AAt?$AAa?$AA?5?$AAf?$AAa?$AAi?$AAl?$AAe?$AAd?$AA?$AA@ 1002d654     sms.obj
 0002:00007680       ??_C@_1CI@NAJJLCHB@?$AAU?$AAs?$AAe?$AAr?$AA?5?$AAD?$AAa?$AAt?$AAa?$AA?5?$AAN?$AAo?$AAt?$AA?5?$AAf?$AAo?$AAu?$AAn?$AAd?$AA?$AA@ 1002d680     sms.obj
 0002:000076a8       ??_C@_1DO@IDHMDBI@?$AAD?$AAe?$AAc?$AAo?$AAd?$AAe?$AAC?$AAa?$AAl?$AAl?$AAb?$AAa?$AAc?$AAk?$AAA?$AAd?$AAd?$AAr?$AA?5?$AAf?$AAa?$AAi?$AAl?$AAe?$AAd?$AA?5?$AAf?$AAo?$AAr?$AA?5?$AA?$AA@ 1002d6a8     sms.obj
 0002:000076e8       ??_C@_1DE@HFEBCKHD@?$AAC?$AAa?$AAl?$AAl?$AAb?$AAa?$AAc?$AAk?$AA?5?$AAN?$AAu?$AAm?$AAb?$AAe?$AAr?$AA?5?$AAN?$AAo?$AAt?$AA?5?$AAf?$AAo?$AAu?$AAn?$AAd?$AA?$AA@ 1002d6e8     sms.obj
 0002:0000771c       ??_C@_1DI@LINGEIIO@?$AAN?$AAu?$AAm?$AAb?$AAe?$AAr?$AA?5?$AAo?$AAf?$AA?5?$AAM?$AAe?$AAs?$AAs?$AAa?$AAg?$AAe?$AA?5?$AAN?$AAo?$AAt?$AA?5?$AAf?$AAo?$AAu?$AAn?$AAd?$AA?$AA@ 1002d71c     sms.obj
 0002:00007754       ??_C@_1CM@NNAJPAJJ@?$AAB?$AAe?$AAa?$AAr?$AAe?$AAr?$AA?5?$AAD?$AAa?$AAt?$AAa?$AA?5?$AAN?$AAo?$AAt?$AA?5?$AAf?$AAo?$AAu?$AAn?$AAd?$AA?$AA@ 1002d754     sms.obj
 0002:00007780       ??_C@_1DE@KOFEJCPK@?$AAF?$AAa?$AAi?$AAl?$AAe?$AAd?$AA?5?$AAt?$AAo?$AA?5?$AAa?$AAl?$AAl?$AAo?$AAc?$AAa?$AAt?$AAe?$AA?5?$AAm?$AAe?$AAm?$AAo?$AAr?$AAy?$AA?$AA@ 1002d780     sms.obj
 0002:000077b8       ??_C@_1EC@GOIJJEHF@?$AAL?$AAe?$AAn?$AA?5?$AAo?$AAf?$AA?5?$AAD?$AAe?$AAs?$AAt?$AAi?$AAn?$AAa?$AAt?$AAi?$AAo?$AAn?$AA?5?$AAH?$AAe?$AAa?$AAd?$AAe?$AAr?$AA?5?$AAi?$AAs?$AA?5?$AA?$CF?$AAl?$AAu@ 1002d7b8     sms.obj
 0002:000077fc       ??_C@_1DC@DLELJBBH@?$AAE?$AAn?$AAc?$AAo?$AAd?$AAe?$AAD?$AAe?$AAs?$AAt?$AAA?$AAd?$AAd?$AAr?$AAH?$AAd?$AAr?$AA?5?$AAf?$AAa?$AAi?$AAl?$AAe?$AAd?$AA?$AA@ 1002d7fc     sms.obj
 0002:00007830       ??_C@_1EO@FOOIINLB@?$AAF?$AAa?$AAi?$AAl?$AAe?$AAd?$AA?5?$AAt?$AAo?$AA?5?$AAa?$AAl?$AAl?$AAo?$AAc?$AAa?$AAt?$AAe?$AA?5?$AAm?$AAe?$AAm?$AAo?$AAr?$AAy?$AA?5?$AAf?$AAo?$AAr?$AA?5?$AAc?$AAa@ 1002d830     sms.obj
 0002:00007880       ??_C@_1DK@OECBOKGO@?$AAE?$AAn?$AAc?$AAo?$AAd?$AAe?$AAC?$AAa?$AAl?$AAl?$AAb?$AAa?$AAc?$AAk?$AAA?$AAd?$AAd?$AAr?$AAH?$AAd?$AAr?$AA?5?$AAf?$AAa?$AAi?$AAl?$AAe?$AAd?$AA?$AA@ 1002d880     sms.obj
 0002:000078c0       ??_C@_1EE@JFFBEHK@?$AAL?$AAe?$AAn?$AAg?$AAt?$AAh?$AA?5?$AAo?$AAf?$AA?5?$AAc?$AAa?$AAl?$AAl?$AAb?$AAa?$AAc?$AAk?$AA?5?$AAn?$AAu?$AAm?$AAb?$AAe?$AAr?$AA?5?$AAi?$AAs?$AA?5?$AAz?$AAe?$AAr@ 1002d8c0     sms.obj
 0002:00007904       ??_C@_1DC@FLGDGGJC@?$AAE?$AAn?$AAc?$AAo?$AAd?$AAe?$AAM?$AAs?$AAg?$AAI?$AAd?$AAe?$AAn?$AAf?$AAi?$AAe?$AAr?$AA?5?$AAf?$AAa?$AAi?$AAl?$AAe?$AAd?$AA?$AA@ 1002d904     sms.obj
 0002:00007938       ??_C@_1DC@NLKCAJDM@?$AAE?$AAn?$AAc?$AAo?$AAd?$AAe?$AAU?$AAs?$AAe?$AAr?$AAD?$AAa?$AAt?$AAa?$AAH?$AAd?$AAr?$AA?5?$AAf?$AAa?$AAi?$AAl?$AAe?$AAd?$AA?$AA@ 1002d938     sms.obj
 0002:0000796c       ??_C@_1DA@PNCMEAJM@?$AAE?$AAn?$AAc?$AAo?$AAd?$AAe?$AAP?$AAr?$AAi?$AAo?$AAr?$AAi?$AAy?$AAH?$AAd?$AAr?$AA?5?$AAf?$AAa?$AAi?$AAl?$AAe?$AAd?$AA?$AA@ 1002d96c     sms.obj
 0002:0000799c       ??_C@_1DO@FBLFONNM@?$AAV?$AAe?$AAr?$AAy?$AA?5?$AAl?$AAa?$AAr?$AAg?$AAe?$AA?5?$AAm?$AAe?$AAs?$AAs?$AAa?$AAg?$AAe?$AA?5?$AAo?$AAf?$AA?5?$AAl?$AAe?$AAn?$AA?5?$AA?$DN?$AA?5?$AA?$CF?$AAd?$AA?$AA@ 1002d99c     sms.obj
 0002:000079dc       ??_C@_1DO@ICBOLLFJ@?$AAD?$AAe?$AAs?$AAt?$AAi?$AAo?$AAn?$AAa?$AAt?$AAi?$AAo?$AAn?$AA?5?$AAa?$AAd?$AAd?$AAr?$AA?5?$AAl?$AAe?$AAn?$AAg?$AAt?$AAh?$AA?5?$AAi?$AAs?$AA?5?$AA?$CF?$AAd?$AA?$AA@ 1002d9dc     sms.obj
 0002:00007a1c       ??_C@_1CO@GDKBCJMM@?$AAD?$AAe?$AAc?$AAo?$AAd?$AAT?$AAy?$AAp?$AAe?$AAo?$AAf?$AAA?$AAd?$AAd?$AAr?$AA?5?$AAf?$AAa?$AAi?$AAl?$AAe?$AAd?$AA?$AA@ 1002da1c     sms.obj
 0002:00007a4c       ??_C@_1CE@FOBFNCPG@?$AAD?$AAe?$AAc?$AAo?$AAd?$AAe?$AAA?$AAd?$AAd?$AAr?$AA?5?$AAf?$AAa?$AAi?$AAl?$AAe?$AAd?$AA?$AA@ 1002da4c     sms.obj
 0002:00007a70       ??_C@_1DK@PKHLKDJB@?$AAS?$AAM?$AAS?$AAC?$AA?5?$AAi?$AAn?$AAf?$AAo?$AAr?$AAm?$AAa?$AAt?$AAi?$AAo?$AAn?$AA?5?$AAn?$AAo?$AAt?$AA?5?$AAp?$AAr?$AAe?$AAs?$AAe?$AAn?$AAt?$AA?$AA@ 1002da70     sms.obj
 0002:00007aac       ??_C@_1DO@MLHHFDH@?$AAM?$AAe?$AAs?$AAs?$AAa?$AAg?$AAe?$AA?5?$AAi?$AAs?$AA?5?$AAn?$AAo?$AAt?$AA?5?$AAo?$AAf?$AA?5?$AAt?$AAy?$AAp?$AAe?$AA?5?$AAd?$AAe?$AAl?$AAi?$AAv?$AAe?$AAr?$AA?$AA@ 1002daac     sms.obj
 0002:00007af0       ??_C@_1FC@JDBKMJBE@?$AAD?$AAe?$AAc?$AAo?$AAd?$AAT?$AAy?$AAp?$AAe?$AAo?$AAf?$AAA?$AAd?$AAd?$AAr?$AA?5?$AAf?$AAa?$AAi?$AAl?$AAe?$AAd?$AA?5?$AAf?$AAo?$AAr?$AA?5?$AAs?$AAe?$AAn?$AAd?$AAe@ 1002daf0     sms.obj
 0002:00007b48       ??_C@_1EI@CFJJJLNK@?$AAD?$AAe?$AAc?$AAo?$AAd?$AAe?$AAA?$AAd?$AAd?$AAr?$AA?5?$AAf?$AAo?$AAr?$AA?5?$AAs?$AAe?$AAn?$AAd?$AAe?$AAr?$AA?5?$AAn?$AAu?$AAm?$AAb?$AAe?$AAr?$AA?5?$AAf?$AAa?$AAi@ 1002db48     sms.obj
 0002:00007b90       ??_C@_1CK@FGJEPGKC@?$AAU?$AAs?$AAe?$AAr?$AA?5?$AAd?$AAa?$AAt?$AAa?$AA?5?$AAc?$AAh?$AAa?$AAr?$AAs?$AA?5?$AA?$DN?$AA?5?$AA?$CF?$AAd?$AA?$AA@ 1002db90     sms.obj
 0002:00007bbc       ??_C@_15BHOFONJE@?$AA?$CF?$AAX?$AA?$AA@ 1002dbbc     sms.obj
 0002:00007bc4       ??_C@_1CO@IHAJILFA@?$AAS?$AAw?$AAi?$AAM?$AA2?$AAM?$AAA?$AAV?$AA_?$AAA?$AAu?$AAd?$AAi?$AAo?$AAP?$AAl?$AAa?$AAy?$AAT?$AAo?$AAn?$AAe?$AA?$AA@ 1002dbc4     stdafx.obj
 0002:00007bf4       ??_C@_1CM@POMOKKD@?$AAS?$AAw?$AAi?$AAM?$AA2?$AAM?$AAA?$AAV?$AA_?$AAA?$AAu?$AAd?$AAi?$AAo?$AAS?$AAe?$AAt?$AAA?$AAV?$AAN?$AAS?$AA?$AA@ 1002dbf4     stdafx.obj
 0002:00007c20       ??_C@_1CM@DNPKJILK@?$AAS?$AAw?$AAi?$AAM?$AA2?$AAM?$AAA?$AAV?$AA_?$AAA?$AAu?$AAd?$AAi?$AAo?$AAG?$AAe?$AAt?$AAA?$AAV?$AAN?$AAS?$AA?$AA@ 1002dc20     stdafx.obj
 0002:00007c4c       ??_C@_1CM@DFDCENPP@?$AAS?$AAw?$AAi?$AAM?$AA2?$AAM?$AAA?$AAV?$AA_?$AAA?$AAu?$AAd?$AAi?$AAo?$AAS?$AAe?$AAt?$AAA?$AAV?$AAE?$AAC?$AA?$AA@ 1002dc4c     stdafx.obj
 0002:00007c78       ??_C@_1CM@HCEDPOG@?$AAS?$AAw?$AAi?$AAM?$AA2?$AAM?$AAA?$AAV?$AA_?$AAA?$AAu?$AAd?$AAi?$AAo?$AAG?$AAe?$AAt?$AAA?$AAV?$AAE?$AAC?$AA?$AA@ 1002dc78     stdafx.obj
 0002:00007ca4       ??_C@_1CO@ICOFFPID@?$AAS?$AAw?$AAi?$AAM?$AA2?$AAM?$AAA?$AAV?$AA_?$AAA?$AAu?$AAd?$AAi?$AAo?$AAS?$AAe?$AAt?$AAA?$AAV?$AAR?$AAX?$AAG?$AA?$AA@ 1002dca4     stdafx.obj
 0002:00007cd4       ??_C@_1CO@KHOONEJN@?$AAS?$AAw?$AAi?$AAM?$AA2?$AAM?$AAA?$AAV?$AA_?$AAA?$AAu?$AAd?$AAi?$AAo?$AAG?$AAe?$AAt?$AAA?$AAV?$AAR?$AAX?$AAG?$AA?$AA@ 1002dcd4     stdafx.obj
 0002:00007d04       ??_C@_1CO@EEIKFGAE@?$AAS?$AAw?$AAi?$AAM?$AA2?$AAM?$AAA?$AAV?$AA_?$AAA?$AAu?$AAd?$AAi?$AAo?$AAS?$AAe?$AAt?$AAA?$AAV?$AAT?$AAX?$AAG?$AA?$AA@ 1002dd04     stdafx.obj
 0002:00007d34       ??_C@_1CO@GBIBNNBK@?$AAS?$AAw?$AAi?$AAM?$AA2?$AAM?$AAA?$AAV?$AA_?$AAA?$AAu?$AAd?$AAi?$AAo?$AAG?$AAe?$AAt?$AAA?$AAV?$AAT?$AAX?$AAG?$AA?$AA@ 1002dd34     stdafx.obj
 0002:00007d64       ??_C@_1CO@LNAOIBJP@?$AAS?$AAw?$AAi?$AAM?$AA2?$AAM?$AAA?$AAV?$AA_?$AAA?$AAu?$AAd?$AAi?$AAo?$AAS?$AAe?$AAt?$AAV?$AAo?$AAl?$AAD?$AAB?$AA?$AA@ 1002dd64     stdafx.obj
 0002:00007d94       ??_C@_1CO@JIAFAKIB@?$AAS?$AAw?$AAi?$AAM?$AA2?$AAM?$AAA?$AAV?$AA_?$AAA?$AAu?$AAd?$AAi?$AAo?$AAG?$AAe?$AAt?$AAV?$AAo?$AAl?$AAD?$AAB?$AA?$AA@ 1002dd94     stdafx.obj
 0002:00007dc4       ??_C@_1DC@HAOBKDAK@?$AAS?$AAw?$AAi?$AAM?$AA2?$AAM?$AAA?$AAV?$AA_?$AAA?$AAu?$AAd?$AAi?$AAo?$AAS?$AAe?$AAt?$AAM?$AAi?$AAc?$AAG?$AAa?$AAi?$AAn?$AA?$AA@ 1002ddc4     stdafx.obj
 0002:00007df8       ??_C@_1DC@IFLHHKEL@?$AAS?$AAw?$AAi?$AAM?$AA2?$AAM?$AAA?$AAV?$AA_?$AAA?$AAu?$AAd?$AAi?$AAo?$AAG?$AAe?$AAt?$AAM?$AAi?$AAc?$AAG?$AAa?$AAi?$AAn?$AA?$AA@ 1002ddf8     stdafx.obj
 0002:00007e2c       ??_C@_1DE@EOBBNMFH@?$AAS?$AAw?$AAi?$AAM?$AA2?$AAM?$AAA?$AAV?$AA_?$AAA?$AAu?$AAd?$AAi?$AAo?$AAS?$AAe?$AAt?$AAT?$AAx?$AAV?$AAo?$AAl?$AAu?$AAm?$AAe?$AA?$AA@ 1002de2c     stdafx.obj
 0002:00007e60       ??_C@_1DE@FIHMDNDF@?$AAS?$AAw?$AAi?$AAM?$AA2?$AAM?$AAA?$AAV?$AA_?$AAA?$AAu?$AAd?$AAi?$AAo?$AAG?$AAe?$AAt?$AAT?$AAx?$AAV?$AAo?$AAl?$AAu?$AAm?$AAe?$AA?$AA@ 1002de60     stdafx.obj
 0002:00007e94       ??_C@_1CM@NOBCNHJP@?$AAS?$AAw?$AAi?$AAM?$AA2?$AAM?$AAA?$AAV?$AA_?$AAA?$AAu?$AAd?$AAi?$AAo?$AAS?$AAe?$AAt?$AAL?$AAP?$AAB?$AAK?$AA?$AA@ 1002de94     stdafx.obj
 0002:00007ec0       ??_C@_1CI@NOFGKEE@?$AAS?$AAw?$AAi?$AAM?$AA2?$AAM?$AAA?$AAV?$AA_?$AAA?$AAu?$AAd?$AAi?$AAo?$AAN?$AAV?$AAD?$AAe?$AAf?$AA?$AA@ 1002dec0     stdafx.obj
 0002:00007ee8       ??_C@_1CO@COCDIGMD@?$AAS?$AAw?$AAi?$AAM?$AA2?$AAM?$AAA?$AAV?$AA_?$AAA?$AAu?$AAd?$AAi?$AAo?$AAG?$AAe?$AAt?$AAA?$AAV?$AAC?$AAF?$AAG?$AA?$AA@ 1002dee8     stdafx.obj
 0002:00007f18       ??_C@_1CO@LCIANNN@?$AAS?$AAw?$AAi?$AAM?$AA2?$AAM?$AAA?$AAV?$AA_?$AAA?$AAu?$AAd?$AAi?$AAo?$AAS?$AAe?$AAt?$AAA?$AAV?$AAC?$AAF?$AAG?$AA?$AA@ 1002df18     stdafx.obj
 0002:00007f48       ??_C@_1DA@HPJBJKKE@?$AAS?$AAw?$AAi?$AAM?$AA2?$AAM?$AAA?$AAV?$AA_?$AAA?$AAu?$AAd?$AAi?$AAo?$AAG?$AAe?$AAt?$AAA?$AAV?$AAM?$AAu?$AAt?$AAe?$AA?$AA@ 1002df48     stdafx.obj
 0002:00007f78       ??_C@_1DA@NBLKNKNI@?$AAS?$AAw?$AAi?$AAM?$AA2?$AAM?$AAA?$AAV?$AA_?$AAA?$AAu?$AAd?$AAi?$AAo?$AAS?$AAe?$AAt?$AAA?$AAV?$AAM?$AAu?$AAt?$AAe?$AA?$AA@ 1002df78     stdafx.obj
 0002:00007fa8       ??_C@_1DA@NPADHLFM@?$AAS?$AAw?$AAi?$AAM?$AA2?$AAM?$AAA?$AAV?$AA_?$AAA?$AAu?$AAd?$AAi?$AAo?$AAS?$AAe?$AAt?$AAV?$AAo?$AAl?$AAu?$AAm?$AAe?$AA?$AA@ 1002dfa8     stdafx.obj
 0002:00007fd8       ??_C@_1DA@HBCIDLCA@?$AAS?$AAw?$AAi?$AAM?$AA2?$AAM?$AAA?$AAV?$AA_?$AAA?$AAu?$AAd?$AAi?$AAo?$AAG?$AAe?$AAt?$AAV?$AAo?$AAl?$AAu?$AAm?$AAe?$AA?$AA@ 1002dfd8     stdafx.obj
 0002:00008008       ??_C@_1DC@EHLKPACE@?$AAS?$AAw?$AAi?$AAM?$AA2?$AAM?$AAA?$AAV?$AA_?$AAA?$AAu?$AAd?$AAi?$AAo?$AAS?$AAe?$AAt?$AAP?$AAr?$AAo?$AAf?$AAi?$AAl?$AAe?$AA?$AA@ 1002e008     stdafx.obj
 0002:0000803c       ??_C@_1DC@LCOMCJGF@?$AAS?$AAw?$AAi?$AAM?$AA2?$AAM?$AAA?$AAV?$AA_?$AAA?$AAu?$AAd?$AAi?$AAo?$AAG?$AAe?$AAt?$AAP?$AAr?$AAo?$AAf?$AAi?$AAl?$AAe?$AA?$AA@ 1002e03c     stdafx.obj
 0002:00008070       ??_C@_1CI@EKPGHNKM@?$AAS?$AAW?$AAI?$AAO?$AAM?$AAA?$AAE?$AAX?$AAS?$AAh?$AAu?$AAt?$AAd?$AAo?$AAw?$AAn?$AAA?$AAp?$AAi?$AA?$AA@ 1002e070     stdafx.obj
 0002:00008098       ??_C@_1CA@LIDENJBL@?$AAS?$AAW?$AAI?$AAO?$AAM?$AAA?$AAE?$AAX?$AAI?$AAn?$AAi?$AAt?$AAA?$AAp?$AAi?$AA?$AA@ 1002e098     stdafx.obj
 0002:000080b8       ??_C@_1CO@LLKDCJKA@?$AAS?$AAW?$AAI?$AAO?$AAM?$AAA?$AAE?$AAX?$AAS?$AAe?$AAs?$AAs?$AAi?$AAo?$AAn?$AAG?$AAe?$AAt?$AAI?$AAn?$AAf?$AAo?$AA?$AA@ 1002e0b8     stdafx.obj
 0002:000080e8       ??_C@_1CI@HCLCIPMF@?$AAS?$AAW?$AAI?$AAO?$AAM?$AAA?$AAE?$AAX?$AAS?$AAe?$AAt?$AAS?$AAe?$AAt?$AAt?$AAi?$AAn?$AAg?$AAs?$AA?$AA@ 1002e0e8     stdafx.obj
 0002:00008110       ??_C@_1CI@GENPGOKH@?$AAS?$AAW?$AAI?$AAO?$AAM?$AAA?$AAE?$AAX?$AAG?$AAe?$AAt?$AAS?$AAe?$AAt?$AAt?$AAi?$AAn?$AAg?$AAs?$AA?$AA@ 1002e110     stdafx.obj
 0002:00008138       ??_C@_1CE@GPIKLGLD@?$AAS?$AAW?$AAI?$AAO?$AAM?$AAA?$AAE?$AAX?$AAS?$AAe?$AAl?$AAe?$AAc?$AAt?$AAi?$AAo?$AAn?$AA?$AA@ 1002e138     stdafx.obj
 0002:0000815c       ??_C@_1CM@KMPDFMLJ@?$AAS?$AAW?$AAI?$AAO?$AAM?$AAA?$AAE?$AAX?$AAS?$AAe?$AAs?$AAs?$AAi?$AAo?$AAn?$AAC?$AAa?$AAn?$AAc?$AAe?$AAl?$AA?$AA@ 1002e15c     stdafx.obj
 0002:00008188       ??_C@_1CK@IHNDAJDA@?$AAS?$AAW?$AAI?$AAO?$AAM?$AAA?$AAE?$AAX?$AAS?$AAe?$AAs?$AAs?$AAi?$AAo?$AAn?$AAS?$AAt?$AAa?$AAr?$AAt?$AA?$AA@ 1002e188     stdafx.obj
 0002:000081b4       ??_C@_1CO@LGPNPECH@?$AAS?$AAW?$AAI?$AAO?$AAM?$AAA?$AAE?$AAX?$AAS?$AAe?$AAt?$AAE?$AAv?$AAe?$AAn?$AAt?$AAR?$AAe?$AAp?$AAo?$AAr?$AAt?$AA?$AA@ 1002e1b4     stdafx.obj
 0002:000081e4       ??_C@_1CG@NFCINIOE@?$AAG?$AAe?$AAt?$AAI?$AAP?$AAC?$AAo?$AAn?$AAf?$AAi?$AAg?$AAu?$AAr?$AAa?$AAt?$AAi?$AAo?$AAn?$AA?$AA@ 1002e1e4     stdafx.obj
 0002:0000820c       ??_C@_1CG@DMPJHODC@?$AAO?$AAM?$AAA?$AAD?$AAM?$AAS?$AAe?$AAn?$AAd?$AAS?$AAe?$AAl?$AAe?$AAc?$AAt?$AAi?$AAo?$AAn?$AA?$AA@ 1002e20c     stdafx.obj
 0002:00008234       ??_C@_1CG@HKOMINGG@?$AAO?$AAM?$AAA?$AAD?$AAM?$AAG?$AAe?$AAt?$AAP?$AAe?$AAn?$AAd?$AAi?$AAn?$AAg?$AAN?$AAI?$AAA?$AA?$AA@ 1002e234     stdafx.obj
 0002:0000825c       ??_C@_1CG@HPMHKNDG@?$AAO?$AAM?$AAA?$AAD?$AAM?$AAC?$AAa?$AAn?$AAc?$AAe?$AAl?$AAS?$AAe?$AAs?$AAs?$AAi?$AAo?$AAn?$AA?$AA@ 1002e25c     stdafx.obj
 0002:00008284       ??_C@_1CE@NFPGDNPI@?$AAO?$AAM?$AAA?$AAD?$AAM?$AAS?$AAt?$AAa?$AAr?$AAt?$AAS?$AAe?$AAs?$AAs?$AAi?$AAo?$AAn?$AA?$AA@ 1002e284     stdafx.obj
 0002:000082a8       ??_C@_1DC@KHFMANMB@?$AAO?$AAM?$AAA?$AAD?$AAM?$AAS?$AAe?$AAt?$AAP?$AAR?$AAL?$AAU?$AAp?$AAd?$AAa?$AAt?$AAe?$AAF?$AAe?$AAa?$AAt?$AAu?$AAr?$AAe?$AA?$AA@ 1002e2a8     stdafx.obj
 0002:000082dc       ??_C@_1DI@LBKFFHPH@?$AAO?$AAM?$AAA?$AAD?$AAM?$AAS?$AAe?$AAt?$AAP?$AAr?$AAo?$AAv?$AAi?$AAs?$AAi?$AAo?$AAn?$AAi?$AAn?$AAg?$AAF?$AAe?$AAa?$AAt?$AAu?$AAr?$AAe?$AA?$AA@ 1002e2dc     stdafx.obj
 0002:00008314       ??_C@_1CI@JIPGCIG@?$AAO?$AAM?$AAA?$AAD?$AAM?$AAG?$AAe?$AAt?$AAS?$AAe?$AAs?$AAs?$AAi?$AAo?$AAn?$AAI?$AAn?$AAf?$AAo?$AA?$AA@ 1002e314     stdafx.obj
 0002:0000833c       ??_C@_1DA@IDBJEHNH@?$AAO?$AAM?$AAA?$AAD?$AAM?$AAG?$AAe?$AAt?$AAF?$AAe?$AAa?$AAt?$AAu?$AAr?$AAe?$AAS?$AAe?$AAt?$AAt?$AAi?$AAn?$AAg?$AAs?$AA?$AA@ 1002e33c     stdafx.obj
 0002:0000836c       ??_C@_1CG@LJKPPMHK@?$AAG?$AAe?$AAt?$AAA?$AAc?$AAt?$AAi?$AAv?$AAa?$AAt?$AAi?$AAo?$AAn?$AAS?$AAt?$AAa?$AAt?$AAe?$AA?$AA@ 1002e36c     stdafx.obj
 0002:00008394       ??_C@_1CE@HJFAADDN@?$AAA?$AAc?$AAt?$AAi?$AAv?$AAa?$AAt?$AAe?$AAA?$AAu?$AAt?$AAo?$AAm?$AAa?$AAt?$AAi?$AAc?$AA?$AA@ 1002e394     stdafx.obj
 0002:000083b8       ??_C@_1BC@HFJKMGOB@?$AAS?$AAe?$AAt?$AAP?$AAo?$AAw?$AAe?$AAr?$AA?$AA@ 1002e3b8     stdafx.obj
 0002:000083cc       ??_C@_1DI@LOOEAKEM@?$AAS?$AAw?$AAi?$AAS?$AAe?$AAt?$AAD?$AAe?$AAv?$AAi?$AAc?$AAe?$AAR?$AAe?$AAm?$AAo?$AAv?$AAa?$AAl?$AAC?$AAa?$AAl?$AAl?$AAb?$AAa?$AAc?$AAk?$AA?$AA@ 1002e3cc     stdafx.obj
 0002:00008404       ??_C@_1BO@LDFOMHLP@?$AAG?$AAe?$AAt?$AAI?$AAm?$AAa?$AAg?$AAe?$AAS?$AAt?$AAo?$AAr?$AAe?$AAW?$AA?$AA@ 1002e404     stdafx.obj
 0002:00008424       ??_C@_1BM@LMCPNJMJ@?$AAG?$AAe?$AAt?$AAI?$AAm?$AAa?$AAg?$AAe?$AAI?$AAn?$AAf?$AAo?$AAW?$AA?$AA@ 1002e424     stdafx.obj
 0002:00008440       ??_C@_1CG@HGNNBAKA@?$AAU?$AAp?$AAg?$AAr?$AAa?$AAd?$AAe?$AAF?$AAi?$AAr?$AAm?$AAw?$AAa?$AAr?$AAe?$AA2?$AAk?$AAW?$AA?$AA@ 1002e440     stdafx.obj
 0002:00008468       ??_C@_1BA@FDMAHHFC@?$AAG?$AAe?$AAt?$AAI?$AAM?$AAS?$AAI?$AA?$AA@ 1002e468     stdafx.obj
 0002:00008478       ??_C@_1CC@BFFFCEKD@?$AAG?$AAe?$AAt?$AAS?$AAe?$AAr?$AAi?$AAa?$AAl?$AAN?$AAu?$AAm?$AAb?$AAe?$AAr?$AAs?$AA?$AA@ 1002e478     stdafx.obj
 0002:0000849c       ??_C@_1BO@DCEMMFDN@?$AAG?$AAe?$AAt?$AAV?$AAo?$AAi?$AAc?$AAe?$AAN?$AAu?$AAm?$AAb?$AAe?$AAr?$AA?$AA@ 1002e49c     stdafx.obj
 0002:000084bc       ??_C@_1CI@PIMIADNL@?$AAG?$AAe?$AAt?$AAH?$AAa?$AAr?$AAd?$AAw?$AAa?$AAr?$AAe?$AAR?$AAe?$AAv?$AAi?$AAs?$AAi?$AAo?$AAn?$AA?$AA@ 1002e4bc     stdafx.obj
 0002:000084e4       ??_C@_1BG@GEINAGNB@?$AAG?$AAe?$AAt?$AAM?$AAo?$AAd?$AAe?$AAl?$AAI?$AAD?$AA?$AA@ 1002e4e4     stdafx.obj
 0002:000084fc       ??_C@_1CA@PPLNCIKK@?$AAG?$AAe?$AAt?$AAM?$AAa?$AAn?$AAu?$AAf?$AAa?$AAc?$AAt?$AAu?$AAr?$AAe?$AAr?$AA?$AA@ 1002e4fc     stdafx.obj
 0002:0000851c       ??_C@_1CE@OAPGAKBB@?$AAS?$AAw?$AAi?$AAG?$AAe?$AAt?$AAC?$AAw?$AAe?$AAP?$AAk?$AAg?$AAs?$AAI?$AAn?$AAf?$AAo?$AA?$AA@ 1002e51c     stdafx.obj
 0002:00008540       ??_C@_1CA@GLALHLMI@?$AAG?$AAe?$AAt?$AAF?$AAi?$AAr?$AAm?$AAw?$AAa?$AAr?$AAe?$AAI?$AAn?$AAf?$AAo?$AA?$AA@ 1002e540     stdafx.obj
 0002:00008560       ??_C@_1CI@DDKIELDP@?$AAG?$AAe?$AAt?$AAF?$AAi?$AAr?$AAm?$AAw?$AAa?$AAr?$AAe?$AAR?$AAe?$AAv?$AAi?$AAs?$AAi?$AAo?$AAn?$AA?$AA@ 1002e560     stdafx.obj
 0002:00008588       ??_C@_1BO@KDNAPCGO@?$AAG?$AAe?$AAt?$AAH?$AAo?$AAm?$AAe?$AAN?$AAe?$AAt?$AAw?$AAo?$AAr?$AAk?$AA?$AA@ 1002e588     stdafx.obj
 0002:000085a8       ??_C@_1CE@GLLOHEPH@?$AAG?$AAe?$AAt?$AAS?$AAe?$AAr?$AAv?$AAi?$AAn?$AAg?$AAN?$AAe?$AAt?$AAw?$AAo?$AAr?$AAk?$AA?$AA@ 1002e5a8     stdafx.obj
 0002:000085cc       ??_C@_1CE@KOCPNJOP@?$AAG?$AAe?$AAt?$AAC?$AAo?$AAn?$AAn?$AAe?$AAc?$AAt?$AAi?$AAo?$AAn?$AAR?$AAa?$AAt?$AAe?$AA?$AA@ 1002e5cc     stdafx.obj
 0002:000085f0       ??_C@_1DM@IPJHDBDK@?$AAG?$AAe?$AAt?$AAS?$AAe?$AAr?$AAv?$AAi?$AAn?$AAg?$AAN?$AAe?$AAt?$AAw?$AAo?$AAr?$AAk?$AAC?$AAa?$AAp?$AAa?$AAb?$AAi?$AAl?$AAi?$AAt?$AAi?$AAe?$AAs?$AA?$AA@ 1002e5f0     stdafx.obj
 0002:0000862c       ??_C@_1CG@FELIKJGA@?$AAG?$AAe?$AAt?$AAS?$AAi?$AAg?$AAn?$AAa?$AAl?$AAS?$AAt?$AAr?$AAe?$AAn?$AAg?$AAt?$AAh?$AAs?$AA?$AA@ 1002e62c     stdafx.obj
 0002:00008654       ??_C@_1CG@HOIPIAHO@?$AAG?$AAe?$AAt?$AAS?$AAe?$AAs?$AAs?$AAi?$AAo?$AAn?$AAD?$AAu?$AAr?$AAa?$AAt?$AAi?$AAo?$AAn?$AA?$AA@ 1002e654     stdafx.obj
 0002:0000867c       ??_C@_1DA@DKMHBAKK@?$AAG?$AAe?$AAt?$AAD?$AAa?$AAt?$AAa?$AAB?$AAe?$AAa?$AAr?$AAe?$AAr?$AAT?$AAe?$AAc?$AAh?$AAn?$AAo?$AAl?$AAo?$AAg?$AAy?$AA?$AA@ 1002e67c     stdafx.obj
 0002:000086ac       ??_C@_1BO@EKIOKBPL@?$AAG?$AAe?$AAt?$AAD?$AAu?$AAn?$AAC?$AAa?$AAl?$AAl?$AAI?$AAn?$AAf?$AAo?$AA?$AA@ 1002e6ac     stdafx.obj
 0002:000086cc       ??_C@_1CC@NHFMMBGI@?$AAG?$AAe?$AAt?$AAD?$AAo?$AAr?$AAm?$AAa?$AAn?$AAc?$AAy?$AAS?$AAt?$AAa?$AAt?$AAe?$AA?$AA@ 1002e6cc     stdafx.obj
 0002:000086f0       ??_C@_1CK@KIBDCEK@?$AAW?$AAr?$AAi?$AAt?$AAe?$AAP?$AAh?$AAo?$AAn?$AAe?$AAb?$AAo?$AAo?$AAk?$AAR?$AAe?$AAc?$AAo?$AAr?$AAd?$AA?$AA@ 1002e6f0     stdafx.obj
 0002:0000871c       ??_C@_1CM@NEKOPCMI@?$AAD?$AAe?$AAl?$AAe?$AAt?$AAe?$AAP?$AAh?$AAo?$AAn?$AAe?$AAb?$AAo?$AAo?$AAk?$AAR?$AAe?$AAc?$AAo?$AAr?$AAd?$AA?$AA@ 1002e71c     stdafx.obj
 0002:00008748       ??_C@_1CK@DFIMJAHF@?$AAR?$AAe?$AAa?$AAd?$AAP?$AAh?$AAo?$AAn?$AAe?$AAb?$AAo?$AAo?$AAk?$AAR?$AAe?$AAc?$AAo?$AAr?$AAd?$AAs?$AA?$AA@ 1002e748     stdafx.obj
 0002:00008774       ??_C@_1DC@FBPBHONH@?$AAG?$AAe?$AAt?$AAP?$AAh?$AAo?$AAn?$AAe?$AAb?$AAo?$AAo?$AAk?$AAC?$AAa?$AAp?$AAa?$AAb?$AAi?$AAl?$AAi?$AAt?$AAi?$AAe?$AAs?$AA?$AA@ 1002e774     stdafx.obj
 0002:000087a8       ??_C@_1BK@EMHIBMDL@?$AAR?$AAe?$AAs?$AAe?$AAt?$AAP?$AAD?$AAS?$AAD?$AAa?$AAt?$AAa?$AA?$AA@ 1002e7a8     stdafx.obj
 0002:000087c4       ??_C@_1DC@BGGGMCCN@?$AAS?$AAe?$AAt?$AAP?$AAo?$AAr?$AAt?$AAA?$AAu?$AAt?$AAo?$AAm?$AAa?$AAt?$AAi?$AAc?$AAT?$AAr?$AAa?$AAc?$AAk?$AAi?$AAn?$AAg?$AA?$AA@ 1002e7c4     stdafx.obj
 0002:000087f8       ??_C@_1DC@EFBNBNHH@?$AAG?$AAe?$AAt?$AAP?$AAo?$AAr?$AAt?$AAA?$AAu?$AAt?$AAo?$AAm?$AAa?$AAt?$AAi?$AAc?$AAT?$AAr?$AAa?$AAc?$AAk?$AAi?$AAn?$AAg?$AA?$AA@ 1002e7f8     stdafx.obj
 0002:0000882c       ??_C@_1DI@HGHGBMHG@?$AAS?$AAe?$AAt?$AAS?$AAe?$AAr?$AAv?$AAi?$AAc?$AAe?$AAA?$AAu?$AAt?$AAo?$AAm?$AAa?$AAt?$AAi?$AAc?$AAT?$AAr?$AAa?$AAc?$AAk?$AAi?$AAn?$AAg?$AA?$AA@ 1002e82c     stdafx.obj
 0002:00008864       ??_C@_1DI@CACGIBL@?$AAG?$AAe?$AAt?$AAS?$AAe?$AAr?$AAv?$AAi?$AAc?$AAe?$AAA?$AAu?$AAt?$AAo?$AAm?$AAa?$AAt?$AAi?$AAc?$AAT?$AAr?$AAa?$AAc?$AAk?$AAi?$AAn?$AAg?$AA?$AA@ 1002e864     stdafx.obj
 0002:0000889c       ??_C@_1BM@IELCHDP@?$AAS?$AAe?$AAt?$AAA?$AAG?$AAP?$AAS?$AAC?$AAo?$AAn?$AAf?$AAi?$AAg?$AA?$AA@ 1002e89c     stdafx.obj
 0002:000088b8       ??_C@_1BM@BFMDACJL@?$AAG?$AAe?$AAt?$AAA?$AAG?$AAP?$AAS?$AAC?$AAo?$AAn?$AAf?$AAi?$AAg?$AA?$AA@ 1002e8b8     stdafx.obj
 0002:000088d4       ??_C@_1CE@NCLCCBKH@?$AAF?$AAo?$AAr?$AAc?$AAe?$AAX?$AAT?$AAR?$AAA?$AAD?$AAo?$AAw?$AAn?$AAl?$AAo?$AAa?$AAd?$AA?$AA@ 1002e8d4     stdafx.obj
 0002:000088f8       ??_C@_1CM@DDKEFNNN@?$AAS?$AAe?$AAt?$AAX?$AAT?$AAR?$AAA?$AAE?$AAm?$AAb?$AAe?$AAd?$AAd?$AAe?$AAd?$AAC?$AAl?$AAi?$AAe?$AAn?$AAt?$AA?$AA@ 1002e8f8     stdafx.obj
 0002:00008924       ??_C@_1BM@DFJCJMOH@?$AAG?$AAe?$AAt?$AAN?$AAM?$AAE?$AAA?$AAC?$AAo?$AAn?$AAf?$AAi?$AAg?$AA?$AA@ 1002e924     stdafx.obj
 0002:00008940       ??_C@_1BM@CIBKLJED@?$AAS?$AAe?$AAt?$AAN?$AAM?$AAE?$AAA?$AAC?$AAo?$AAn?$AAf?$AAi?$AAg?$AA?$AA@ 1002e940     stdafx.obj
 0002:0000895c       ??_C@_1CA@KMIGBNMK@?$AAS?$AAe?$AAt?$AAX?$AAT?$AAR?$AAA?$AAV?$AAa?$AAl?$AAi?$AAd?$AAi?$AAt?$AAy?$AA?$AA@ 1002e95c     stdafx.obj
 0002:0000897c       ??_C@_1CA@MAFFGJAJ@?$AAG?$AAe?$AAt?$AAX?$AAT?$AAR?$AAA?$AAV?$AAa?$AAl?$AAi?$AAd?$AAi?$AAt?$AAy?$AA?$AA@ 1002e97c     stdafx.obj
 0002:0000899c       ??_C@_1BO@CMMMIKIK@?$AAS?$AAe?$AAt?$AAX?$AAT?$AAR?$AAA?$AAN?$AAe?$AAt?$AAw?$AAo?$AAr?$AAk?$AA?$AA@ 1002e99c     stdafx.obj
 0002:000089bc       ??_C@_1BO@KNKDDKKI@?$AAG?$AAe?$AAt?$AAX?$AAT?$AAR?$AAA?$AAN?$AAe?$AAt?$AAw?$AAo?$AAr?$AAk?$AA?$AA@ 1002e9bc     stdafx.obj
 0002:000089dc       ??_C@_1DC@HPMMEIMG@?$AAS?$AAe?$AAt?$AAX?$AAT?$AAR?$AAA?$AAA?$AAu?$AAt?$AAo?$AAm?$AAa?$AAt?$AAi?$AAc?$AAD?$AAo?$AAw?$AAn?$AAl?$AAo?$AAa?$AAd?$AA?$AA@ 1002e9dc     stdafx.obj
 0002:00008a10       ??_C@_1DC@CMLHJHJM@?$AAG?$AAe?$AAt?$AAX?$AAT?$AAR?$AAA?$AAA?$AAu?$AAt?$AAo?$AAm?$AAa?$AAt?$AAi?$AAc?$AAD?$AAo?$AAw?$AAn?$AAl?$AAo?$AAa?$AAd?$AA?$AA@ 1002ea10     stdafx.obj
 0002:00008a44       ??_C@_1BO@LKBLACJA@?$AAS?$AAe?$AAt?$AAP?$AAD?$AAS?$AAD?$AAe?$AAf?$AAa?$AAu?$AAl?$AAt?$AAs?$AA?$AA@ 1002ea44     stdafx.obj
 0002:00008a64       ??_C@_1BO@DLHELCLC@?$AAG?$AAe?$AAt?$AAP?$AAD?$AAS?$AAD?$AAe?$AAf?$AAa?$AAu?$AAl?$AAt?$AAs?$AA?$AA@ 1002ea64     stdafx.obj
 0002:00008a84       ??_C@_1CO@NGELCAG@?$AAP?$AAD?$AAS?$AAI?$AAn?$AAj?$AAe?$AAc?$AAt?$AAT?$AAi?$AAm?$AAe?$AAR?$AAe?$AAf?$AAe?$AAr?$AAe?$AAn?$AAc?$AAe?$AA?$AA@ 1002ea84     stdafx.obj
 0002:00008ab4       ??_C@_1BI@NEKGNCEE@?$AAS?$AAe?$AAt?$AAP?$AAD?$AAS?$AAS?$AAt?$AAa?$AAt?$AAe?$AA?$AA@ 1002eab4     stdafx.obj
 0002:00008acc       ??_C@_1BI@MCMLDDCG@?$AAG?$AAe?$AAt?$AAP?$AAD?$AAS?$AAS?$AAt?$AAa?$AAt?$AAe?$AA?$AA@ 1002eacc     stdafx.obj
 0002:00008ae4       ??_C@_1CO@KFNELFLK@?$AAR?$AAe?$AAs?$AAe?$AAt?$AAT?$AAo?$AAF?$AAa?$AAc?$AAt?$AAo?$AAr?$AAy?$AAD?$AAe?$AAf?$AAa?$AAu?$AAl?$AAt?$AAs?$AA?$AA@ 1002eae4     stdafx.obj
 0002:00008b14       ??_C@_1BK@GJHIJMBE@?$AAU?$AAI?$AAM?$AAC?$AAh?$AAa?$AAn?$AAg?$AAe?$AAP?$AAI?$AAN?$AA?$AA@ 1002eb14     stdafx.obj
 0002:00008b30       ??_C@_1CI@IDBLGFEF@?$AAU?$AAI?$AAM?$AAS?$AAe?$AAt?$AAP?$AAI?$AAN?$AAP?$AAr?$AAo?$AAt?$AAe?$AAc?$AAt?$AAi?$AAo?$AAn?$AA?$AA@ 1002eb30     stdafx.obj
 0002:00008b58       ??_C@_1BM@KMFJODPI@?$AAU?$AAI?$AAM?$AAU?$AAn?$AAb?$AAl?$AAo?$AAc?$AAk?$AAP?$AAI?$AAN?$AA?$AA@ 1002eb58     stdafx.obj
 0002:00008b74       ??_C@_1BK@FNIKCFGA@?$AAU?$AAI?$AAM?$AAV?$AAe?$AAr?$AAi?$AAf?$AAy?$AAP?$AAI?$AAN?$AA?$AA@ 1002eb74     stdafx.obj
 0002:00008b90       ??_C@_1CC@MAOGAOLF@?$AAU?$AAI?$AAM?$AAG?$AAe?$AAt?$AAC?$AAa?$AAr?$AAd?$AAS?$AAt?$AAa?$AAt?$AAu?$AAs?$AA?$AA@ 1002eb90     stdafx.obj
 0002:00008bb4       ??_C@_1DA@GHLIECNF@?$AAD?$AAM?$AAS?$AAU?$AAI?$AAM?$AAU?$AAn?$AAb?$AAl?$AAo?$AAc?$AAk?$AAC?$AAo?$AAn?$AAt?$AAr?$AAo?$AAl?$AAK?$AAe?$AAy?$AA?$AA@ 1002ebb4     stdafx.obj
 0002:00008be4       ??_C@_1DM@PICNGJDJ@?$AAD?$AAM?$AAS?$AAU?$AAI?$AAM?$AAS?$AAe?$AAt?$AAC?$AAo?$AAn?$AAt?$AAr?$AAo?$AAl?$AAK?$AAe?$AAy?$AAP?$AAr?$AAo?$AAt?$AAe?$AAc?$AAt?$AAi?$AAo?$AAn?$AA?$AA@ 1002ebe4     stdafx.obj
 0002:00008c20       ??_C@_1DE@KJIFEPBC@?$AAD?$AAM?$AAS?$AAU?$AAI?$AAM?$AAG?$AAe?$AAt?$AAC?$AAo?$AAn?$AAt?$AAr?$AAo?$AAl?$AAK?$AAe?$AAy?$AAS?$AAt?$AAa?$AAt?$AAu?$AAs?$AA?$AA@ 1002ec20     stdafx.obj
 0002:00008c54       ??_C@_1BO@BDMAADME@?$AAD?$AAM?$AAS?$AAU?$AAI?$AAM?$AAG?$AAe?$AAt?$AAI?$AAC?$AAC?$AAI?$AAD?$AA?$AA@ 1002ec54     stdafx.obj
 0002:00008c74       ??_C@_1CG@GOOPNCGG@?$AAD?$AAM?$AAS?$AAU?$AAI?$AAM?$AAG?$AAe?$AAt?$AAP?$AAI?$AAN?$AAS?$AAt?$AAa?$AAt?$AAu?$AAs?$AA?$AA@ 1002ec74     stdafx.obj
 0002:00008c9c       ??_C@_1CA@ECNLMANC@?$AAD?$AAM?$AAS?$AAU?$AAI?$AAM?$AAC?$AAh?$AAa?$AAn?$AAg?$AAe?$AAP?$AAI?$AAN?$AA?$AA@ 1002ec9c     stdafx.obj
 0002:00008cbc       ??_C@_1CC@FDCEKFEM@?$AAD?$AAM?$AAS?$AAU?$AAI?$AAM?$AAU?$AAn?$AAb?$AAl?$AAo?$AAc?$AAk?$AAP?$AAI?$AAN?$AA?$AA@ 1002ecbc     stdafx.obj
 0002:00008ce0       ??_C@_1CA@HGCJHJKG@?$AAD?$AAM?$AAS?$AAU?$AAI?$AAM?$AAV?$AAe?$AAr?$AAi?$AAf?$AAy?$AAP?$AAI?$AAN?$AA?$AA@ 1002ece0     stdafx.obj
 0002:00008d00       ??_C@_1CO@IAPGNGBB@?$AAD?$AAM?$AAS?$AAU?$AAI?$AAM?$AAS?$AAe?$AAt?$AAP?$AAI?$AAN?$AAP?$AAr?$AAo?$AAt?$AAe?$AAc?$AAt?$AAi?$AAo?$AAn?$AA?$AA@ 1002ed00     stdafx.obj
 0002:00008d30       ??_C@_1BO@PHBFFHLB@?$AAS?$AAe?$AAt?$AAS?$AAM?$AAS?$AAC?$AAA?$AAd?$AAd?$AAr?$AAe?$AAs?$AAs?$AA?$AA@ 1002ed30     stdafx.obj
 0002:00008d50       ??_C@_1BO@HGHKOHJD@?$AAG?$AAe?$AAt?$AAS?$AAM?$AAS?$AAC?$AAA?$AAd?$AAd?$AAr?$AAe?$AAs?$AAs?$AA?$AA@ 1002ed50     stdafx.obj
 0002:00008d70       ??_C@_1BA@FCBDHPLP@?$AAS?$AAe?$AAn?$AAd?$AAS?$AAM?$AAS?$AA?$AA@ 1002ed70     stdafx.obj
 0002:00008d80       ??_C@_1BA@KOGJAAJI@?$AAS?$AAa?$AAv?$AAe?$AAS?$AAM?$AAS?$AA?$AA@ 1002ed80     stdafx.obj
 0002:00008d90       ??_C@_1CA@JHJDBCGM@?$AAM?$AAo?$AAd?$AAi?$AAf?$AAy?$AAS?$AAM?$AAS?$AAS?$AAt?$AAa?$AAt?$AAu?$AAs?$AA?$AA@ 1002ed90     stdafx.obj
 0002:00008db0       ??_C@_1CO@LFANFNEA@?$AAS?$AAe?$AAt?$AAB?$AAr?$AAo?$AAa?$AAd?$AAc?$AAa?$AAs?$AAt?$AAA?$AAc?$AAt?$AAi?$AAv?$AAa?$AAt?$AAi?$AAo?$AAn?$AA?$AA@ 1002edb0     stdafx.obj
 0002:00008de0       ??_C@_1BE@HLBMIMG@?$AAS?$AAe?$AAt?$AAR?$AAo?$AAu?$AAt?$AAe?$AAs?$AA?$AA@ 1002ede0     stdafx.obj
 0002:00008df4       ??_C@_1BO@MAJBHHDN@?$AAS?$AAe?$AAt?$AAS?$AAM?$AAS?$AAP?$AAr?$AAo?$AAt?$AAo?$AAc?$AAo?$AAl?$AA?$AA@ 1002edf4     stdafx.obj
 0002:00008e14       ??_C@_1O@PELEKICI@?$AAG?$AAe?$AAt?$AAS?$AAM?$AAS?$AA?$AA@ 1002ee14     stdafx.obj
 0002:00008e24       ??_C@_1BG@EAPBFHAO@?$AAG?$AAe?$AAt?$AAS?$AAM?$AAS?$AAL?$AAi?$AAs?$AAt?$AA?$AA@ 1002ee24     stdafx.obj
 0002:00008e3c       ??_C@_1BE@LPEGABOF@?$AAD?$AAe?$AAl?$AAe?$AAt?$AAe?$AAS?$AAM?$AAS?$AA?$AA@ 1002ee3c     stdafx.obj
 0002:00008e50       ??_C@_1BI@LBBBPLGJ@?$AAV?$AAa?$AAl?$AAi?$AAd?$AAa?$AAt?$AAe?$AAS?$AAP?$AAC?$AA?$AA@ 1002ee50     stdafx.obj
 0002:00008e68       ??_C@_1BO@DANEGBA@?$AAG?$AAe?$AAt?$AAN?$AAe?$AAt?$AAw?$AAo?$AAr?$AAk?$AAT?$AAi?$AAm?$AAe?$AA?$AA@ 1002ee68     stdafx.obj
 0002:00008e88       ??_C@_1CC@JNFHEGAK@?$AAG?$AAe?$AAt?$AAO?$AAf?$AAf?$AAl?$AAi?$AAn?$AAe?$AAR?$AAe?$AAa?$AAs?$AAo?$AAn?$AA?$AA@ 1002ee88     stdafx.obj
 0002:00008eac       ??_C@_1BC@FAJBENPP@?$AAG?$AAe?$AAt?$AAP?$AAo?$AAw?$AAe?$AAr?$AA?$AA@ 1002eeac     stdafx.obj
 0002:00008ec0       ??_C@_1BO@EMLBJBFB@?$AAA?$AAc?$AAt?$AAi?$AAv?$AAa?$AAt?$AAe?$AAM?$AAa?$AAn?$AAu?$AAa?$AAl?$AA?$AA@ 1002eec0     stdafx.obj
 0002:00008ee0       ??_C@_1BG@COEJJNAO@?$AAG?$AAe?$AAt?$AAE?$AAR?$AAI?$AAF?$AAi?$AAl?$AAe?$AA?$AA@ 1002eee0     stdafx.obj
 0002:00008ef8       ??_C@_1DC@BLOBPCMC@?$AAG?$AAe?$AAt?$AA3?$AAG?$AAp?$AAp?$AA2?$AAS?$AAu?$AAb?$AAs?$AAc?$AAr?$AAi?$AAp?$AAt?$AAi?$AAo?$AAn?$AAI?$AAn?$AAf?$AAo?$AA?$AA@ 1002eef8     stdafx.obj
 0002:00008f2c       ??_C@_1DC@EIJKCNJI@?$AAS?$AAe?$AAt?$AA3?$AAG?$AAp?$AAp?$AA2?$AAS?$AAu?$AAb?$AAs?$AAc?$AAr?$AAi?$AAp?$AAt?$AAi?$AAo?$AAn?$AAI?$AAn?$AAf?$AAo?$AA?$AA@ 1002ef2c     stdafx.obj
 0002:00008f60       ??_C@_1BM@CPGDMEDL@?$AAG?$AAe?$AAt?$AAP?$AAR?$AAL?$AAV?$AAe?$AAr?$AAs?$AAi?$AAo?$AAn?$AA?$AA@ 1002ef60     stdafx.obj
 0002:00008f7c       ??_C@_1CK@MAFKIOPO@?$AAG?$AAe?$AAt?$AAF?$AAi?$AAr?$AAm?$AAw?$AAa?$AAr?$AAe?$AAR?$AAe?$AAv?$AAi?$AAs?$AAi?$AAo?$AAn?$AAs?$AA?$AA@ 1002ef7c     stdafx.obj
 0002:00008fa8       ??_C@_1CM@EDIJFBLL@?$AAG?$AAe?$AAt?$AAD?$AAe?$AAv?$AAi?$AAc?$AAe?$AAC?$AAa?$AAp?$AAa?$AAb?$AAi?$AAl?$AAi?$AAt?$AAi?$AAe?$AAs?$AA?$AA@ 1002efa8     stdafx.obj
 0002:00008fd4       ??_C@_1DK@FDHAHLGB@?$AAG?$AAe?$AAt?$AAA?$AAN?$AAA?$AAA?$AAA?$AAA?$AAu?$AAt?$AAh?$AAe?$AAn?$AAt?$AAi?$AAc?$AAa?$AAt?$AAi?$AAo?$AAn?$AAS?$AAt?$AAa?$AAt?$AAu?$AAs?$AA?$AA@ 1002efd4     stdafx.obj
 0002:00009010       ??_C@_1BE@GNJLFGAD@?$AAS?$AAe?$AAt?$AAA?$AAC?$AAC?$AAO?$AAL?$AAC?$AA?$AA@ 1002f010     stdafx.obj
 0002:00009024       ??_C@_1BE@MDLABGHP@?$AAG?$AAe?$AAt?$AAA?$AAC?$AAC?$AAO?$AAL?$AAC?$AA?$AA@ 1002f024     stdafx.obj
 0002:00009038       ??_C@_1DC@MGKINNOP@?$AAG?$AAe?$AAt?$AAC?$AAD?$AAM?$AAA?$AAN?$AAe?$AAt?$AAw?$AAo?$AAr?$AAk?$AAP?$AAa?$AAr?$AAa?$AAm?$AAe?$AAt?$AAe?$AAr?$AAs?$AA?$AA@ 1002f038     stdafx.obj
 0002:0000906c       ??_C@_1DC@JFNDACLF@?$AAS?$AAe?$AAt?$AAC?$AAD?$AAM?$AAA?$AAN?$AAe?$AAt?$AAw?$AAo?$AAr?$AAk?$AAP?$AAa?$AAr?$AAa?$AAm?$AAe?$AAt?$AAe?$AAr?$AAs?$AA?$AA@ 1002f06c     stdafx.obj
 0002:000090a0       ??_C@_1CK@EGBLJME@?$AAS?$AAe?$AAt?$AAN?$AAe?$AAt?$AAw?$AAo?$AAr?$AAk?$AAP?$AAr?$AAe?$AAf?$AAe?$AAr?$AAe?$AAn?$AAc?$AAe?$AA?$AA@ 1002f0a0     stdafx.obj
 0002:000090cc       ??_C@_1CK@POCCMJNB@?$AAG?$AAe?$AAt?$AAN?$AAe?$AAt?$AAw?$AAo?$AAr?$AAk?$AAP?$AAr?$AAe?$AAf?$AAe?$AAr?$AAe?$AAn?$AAc?$AAe?$AA?$AA@ 1002f0cc     stdafx.obj
 0002:000090f8       ??_C@_1CK@JIMFDDIE@?$AAI?$AAn?$AAi?$AAt?$AAi?$AAa?$AAt?$AAe?$AAD?$AAo?$AAm?$AAa?$AAi?$AAn?$AAA?$AAt?$AAt?$AAa?$AAc?$AAh?$AA?$AA@ 1002f0f8     stdafx.obj
 0002:00009124       ??_C@_1DI@CIBLKDLK@?$AAI?$AAn?$AAi?$AAt?$AAi?$AAa?$AAt?$AAe?$AAN?$AAe?$AAt?$AAw?$AAo?$AAr?$AAk?$AAR?$AAe?$AAg?$AAi?$AAs?$AAt?$AAr?$AAa?$AAt?$AAi?$AAo?$AAn?$AA?$AA@ 1002f124     stdafx.obj
 0002:0000915c       ??_C@_1CM@KHNJMIGB@?$AAP?$AAe?$AAr?$AAf?$AAo?$AAr?$AAm?$AAN?$AAe?$AAt?$AAw?$AAo?$AAr?$AAk?$AAR?$AAA?$AAT?$AAS?$AAc?$AAa?$AAn?$AA?$AA@ 1002f15c     stdafx.obj
 0002:00009188       ??_C@_1CG@KIPBFHFH@?$AAP?$AAe?$AAr?$AAf?$AAo?$AAr?$AAm?$AAN?$AAe?$AAt?$AAw?$AAo?$AAr?$AAk?$AAS?$AAc?$AAa?$AAn?$AA?$AA@ 1002f188     stdafx.obj
 0002:000091b0       ??_C@_1BE@CPONLMAP@?$AAG?$AAe?$AAt?$AAR?$AAF?$AAI?$AAn?$AAf?$AAo?$AA?$AA@ 1002f1b0     stdafx.obj
 0002:000091c4       ??_C@_1BM@INJOIDEM@?$AAG?$AAe?$AAt?$AAB?$AAy?$AAt?$AAe?$AAT?$AAo?$AAt?$AAa?$AAl?$AAs?$AA?$AA@ 1002f1c4     stdafx.obj
 0002:000091e0       ??_C@_1CE@ENGLIMHE@?$AAG?$AAe?$AAt?$AAD?$AAe?$AAf?$AAa?$AAu?$AAl?$AAt?$AAP?$AAr?$AAo?$AAf?$AAi?$AAl?$AAe?$AA?$AA@ 1002f1e0     stdafx.obj
 0002:00009204       ??_C@_1CE@JEHKLGLP@?$AAS?$AAe?$AAt?$AAD?$AAe?$AAf?$AAa?$AAu?$AAl?$AAt?$AAP?$AAr?$AAo?$AAf?$AAi?$AAl?$AAe?$AA?$AA@ 1002f204     stdafx.obj
 0002:00009228       ??_C@_1BO@PCFFIAAI@?$AAS?$AAe?$AAt?$AAA?$AAu?$AAt?$AAo?$AAC?$AAo?$AAn?$AAn?$AAe?$AAc?$AAt?$AA?$AA@ 1002f228     stdafx.obj
 0002:00009248       ??_C@_1BO@HDDKDACK@?$AAG?$AAe?$AAt?$AAA?$AAu?$AAt?$AAo?$AAC?$AAo?$AAn?$AAn?$AAe?$AAc?$AAt?$AA?$AA@ 1002f248     stdafx.obj
 0002:00009268       ??_C@_1CK@MBMHNBNM@?$AAG?$AAe?$AAt?$AAL?$AAa?$AAs?$AAt?$AAM?$AAo?$AAb?$AAi?$AAl?$AAe?$AAI?$AAP?$AAE?$AAr?$AAr?$AAo?$AAr?$AA?$AA@ 1002f268     stdafx.obj
 0002:00009294       ??_C@_1CM@IGBGPKHE@?$AAG?$AAe?$AAt?$AAM?$AAo?$AAb?$AAi?$AAl?$AAe?$AAI?$AAP?$AAP?$AAa?$AAr?$AAa?$AAm?$AAe?$AAt?$AAe?$AAr?$AAs?$AA?$AA@ 1002f294     stdafx.obj
 0002:000092c0       ??_C@_1CM@OBKGJHBP@?$AAS?$AAe?$AAt?$AAM?$AAo?$AAb?$AAi?$AAl?$AAe?$AAI?$AAP?$AAP?$AAa?$AAr?$AAa?$AAm?$AAe?$AAt?$AAe?$AAr?$AAs?$AA?$AA@ 1002f2c0     stdafx.obj
 0002:000092ec       ??_C@_1CG@COPLLMPK@?$AAG?$AAe?$AAt?$AAM?$AAo?$AAb?$AAi?$AAl?$AAe?$AAI?$AAP?$AAP?$AAr?$AAo?$AAf?$AAi?$AAl?$AAe?$AA?$AA@ 1002f2ec     stdafx.obj
 0002:00009314       ??_C@_1CG@MAPJLCNM@?$AAS?$AAe?$AAt?$AAM?$AAo?$AAb?$AAi?$AAl?$AAe?$AAI?$AAP?$AAP?$AAr?$AAo?$AAf?$AAi?$AAl?$AAe?$AA?$AA@ 1002f314     stdafx.obj
 0002:0000933c       ??_C@_1DC@LKPLPLHN@?$AAG?$AAe?$AAt?$AAA?$AAc?$AAt?$AAi?$AAv?$AAe?$AAM?$AAo?$AAb?$AAi?$AAl?$AAe?$AAI?$AAP?$AAP?$AAr?$AAo?$AAf?$AAi?$AAl?$AAe?$AA?$AA@ 1002f33c     stdafx.obj
 0002:00009370       ??_C@_1DC@OJIACECH@?$AAS?$AAe?$AAt?$AAA?$AAc?$AAt?$AAi?$AAv?$AAe?$AAM?$AAo?$AAb?$AAi?$AAl?$AAe?$AAI?$AAP?$AAP?$AAr?$AAo?$AAf?$AAi?$AAl?$AAe?$AA?$AA@ 1002f370     stdafx.obj
 0002:000093a4       ??_C@_1BI@FFMCFILE@?$AAG?$AAe?$AAt?$AAM?$AAo?$AAb?$AAi?$AAl?$AAe?$AAI?$AAP?$AA?$AA@ 1002f3a4     stdafx.obj
 0002:000093bc       ??_C@_1BI@EDKPLJNG@?$AAS?$AAe?$AAt?$AAM?$AAo?$AAb?$AAi?$AAl?$AAe?$AAI?$AAP?$AA?$AA@ 1002f3bc     stdafx.obj
 0002:000093d4       ??_C@_1CA@EINFGIBA@?$AAG?$AAe?$AAt?$AAP?$AAa?$AAc?$AAk?$AAe?$AAt?$AAS?$AAt?$AAa?$AAt?$AAu?$AAs?$AA?$AA@ 1002f3d4     stdafx.obj
 0002:000093f4       ??_C@_1BK@DCHGBAOJ@?$AAG?$AAe?$AAt?$AAI?$AAP?$AAA?$AAd?$AAd?$AAr?$AAe?$AAs?$AAs?$AA?$AA@ 1002f3f4     stdafx.obj
 0002:00009410       ??_C@_1CA@JMBMOINF@?$AAG?$AAe?$AAt?$AAS?$AAe?$AAs?$AAs?$AAi?$AAo?$AAn?$AAS?$AAt?$AAa?$AAt?$AAe?$AA?$AA@ 1002f410     stdafx.obj
 0002:00009430       ??_C@_1CA@FFLEDDOC@?$AAS?$AAt?$AAo?$AAp?$AAD?$AAa?$AAt?$AAa?$AAS?$AAe?$AAs?$AAs?$AAi?$AAo?$AAn?$AA?$AA@ 1002f430     stdafx.obj
 0002:00009450       ??_C@_1CE@LOHPJLLL@?$AAS?$AAt?$AAa?$AAr?$AAt?$AAD?$AAa?$AAt?$AAa?$AAS?$AAe?$AAs?$AAs?$AAi?$AAo?$AAn?$AA2?$AA?$AA@ 1002f450     stdafx.obj
 0002:00009474       ??_C@_1CI@GFOILFKB@?$AAG?$AAe?$AAt?$AAC?$AAe?$AAl?$AAl?$AAL?$AAo?$AAc?$AAa?$AAt?$AAi?$AAo?$AAn?$AAI?$AAn?$AAf?$AAo?$AA?$AA@ 1002f474     stdafx.obj
 0002:0000949c       ??_C@_1CE@CJHGMCHL@?$AAG?$AAe?$AAt?$AAW?$AAa?$AAi?$AAt?$AAi?$AAn?$AAg?$AAM?$AAs?$AAg?$AAI?$AAn?$AAf?$AAo?$AA?$AA@ 1002f49c     stdafx.obj
 0002:000094c0       ??_C@_1CO@NJMGNGIC@?$AAS?$AAe?$AAt?$AAC?$AAa?$AAl?$AAl?$AAB?$AAa?$AAr?$AAr?$AAi?$AAn?$AAg?$AAP?$AAa?$AAs?$AAs?$AAw?$AAo?$AAr?$AAd?$AA?$AA@ 1002f4c0     stdafx.obj
 0002:000094f0       ??_C@_1BG@JMOHBGIL@?$AAA?$AAb?$AAo?$AAr?$AAt?$AAs?$AAU?$AAS?$AAS?$AAD?$AA?$AA@ 1002f4f0     stdafx.obj
 0002:00009508       ??_C@_1BA@JNDIFGHG@?$AAA?$AAn?$AAs?$AAU?$AAS?$AAS?$AAD?$AA?$AA@ 1002f508     stdafx.obj
 0002:00009518       ??_C@_1BC@OIGJILDE@?$AAO?$AAr?$AAi?$AAg?$AAU?$AAS?$AAS?$AAD?$AA?$AA@ 1002f518     stdafx.obj
 0002:0000952c       ??_C@_1CG@GALIHLLO@?$AAA?$AAu?$AAd?$AAi?$AAo?$AAP?$AAl?$AAa?$AAy?$AAA?$AAu?$AAd?$AAi?$AAo?$AAT?$AAo?$AAn?$AAe?$AA?$AA@ 1002f52c     stdafx.obj
 0002:00009554       ??_C@_1CK@NFNPLDHL@?$AAA?$AAu?$AAd?$AAi?$AAo?$AAS?$AAe?$AAt?$AAV?$AAo?$AAl?$AAT?$AAL?$AAB?$AAC?$AAo?$AAn?$AAf?$AAi?$AAg?$AA?$AA@ 1002f554     stdafx.obj
 0002:00009580       ??_C@_1CM@LIFDNPFB@?$AAA?$AAu?$AAd?$AAi?$AAo?$AAG?$AAe?$AAt?$AAP?$AAa?$AAt?$AAh?$AAP?$AAC?$AAM?$AAF?$AAi?$AAl?$AAt?$AAe?$AAr?$AA?$AA@ 1002f580     stdafx.obj
 0002:000095ac       ??_C@_1CC@KGCLAPBJ@?$AAA?$AAu?$AAd?$AAi?$AAo?$AAG?$AAe?$AAt?$AAP?$AAa?$AAt?$AAh?$AAW?$AAo?$AAr?$AAd?$AA?$AA@ 1002f5ac     stdafx.obj
 0002:000095d0       ??_C@_1CC@LDJNPJGB@?$AAA?$AAu?$AAd?$AAi?$AAo?$AAG?$AAe?$AAt?$AAP?$AAa?$AAt?$AAh?$AAB?$AAy?$AAt?$AAe?$AA?$AA@ 1002f5d0     stdafx.obj
 0002:000095f4       ??_C@_1CE@NEFGGJGB@?$AAA?$AAu?$AAd?$AAi?$AAo?$AAS?$AAe?$AAt?$AAA?$AAu?$AAd?$AAi?$AAo?$AAP?$AAa?$AAt?$AAh?$AA?$AA@ 1002f5f4     stdafx.obj
 0002:00009618       ??_C@_1CA@CJLLLPJJ@?$AAA?$AAu?$AAd?$AAi?$AAo?$AAG?$AAe?$AAt?$AAP?$AAr?$AAo?$AAf?$AAi?$AAl?$AAe?$AA?$AA@ 1002f618     stdafx.obj
 0002:00009638       ??_C@_1CA@NMONGGNI@?$AAA?$AAu?$AAd?$AAi?$AAo?$AAS?$AAe?$AAt?$AAP?$AAr?$AAo?$AAf?$AAi?$AAl?$AAe?$AA?$AA@ 1002f638     stdafx.obj
 0002:00009658       ??_C@_1CI@LOMIGCGI@?$AAS?$AAe?$AAt?$AAI?$AAm?$AAa?$AAg?$AAe?$AAs?$AAP?$AAr?$AAe?$AAf?$AAe?$AAr?$AAe?$AAn?$AAc?$AAe?$AA?$AA@ 1002f658     stdafx.obj
 0002:00009680       ??_C@_1CI@JKKOCCEJ@?$AAG?$AAe?$AAt?$AAI?$AAm?$AAa?$AAg?$AAe?$AAs?$AAP?$AAr?$AAe?$AAf?$AAe?$AAr?$AAe?$AAn?$AAc?$AAe?$AA?$AA@ 1002f680     stdafx.obj
 0002:000096a8       ??_C@_1DC@LEEDOOEP@?$AAS?$AAe?$AAt?$AAS?$AAW?$AAI?$AAO?$AAM?$AAA?$AAE?$AAX?$AAE?$AAv?$AAe?$AAn?$AAt?$AAC?$AAa?$AAl?$AAl?$AAb?$AAa?$AAc?$AAk?$AA?$AA@ 1002f6a8     stdafx.obj
 0002:000096dc       ??_C@_1DO@IOPPEPMM@?$AAS?$AAe?$AAt?$AAS?$AAy?$AAs?$AAt?$AAe?$AAm?$AAS?$AAe?$AAl?$AAe?$AAc?$AAt?$AAi?$AAo?$AAn?$AAP?$AAr?$AAe?$AAf?$AAC?$AAa?$AAl?$AAl?$AAb?$AAa?$AAc?$AAk?$AA?$AA@ 1002f6dc     stdafx.obj
 0002:0000971c       ??_C@_1CO@FGFKLCLK@?$AAS?$AAe?$AAt?$AAN?$AAe?$AAt?$AAw?$AAo?$AAr?$AAk?$AAT?$AAi?$AAm?$AAe?$AAC?$AAa?$AAl?$AAl?$AAb?$AAa?$AAc?$AAk?$AA?$AA@ 1002f71c     stdafx.obj
 0002:0000974c       ??_C@_1DC@MBGELGLO@?$AAS?$AAe?$AAt?$AAE?$AAm?$AAe?$AAr?$AAg?$AAe?$AAn?$AAc?$AAy?$AAL?$AAi?$AAs?$AAt?$AAC?$AAa?$AAl?$AAl?$AAb?$AAa?$AAc?$AAk?$AA?$AA@ 1002f74c     stdafx.obj
 0002:00009780       ??_C@_1EA@INMGDAJH@?$AAS?$AAe?$AAt?$AAA?$AAl?$AAl?$AAP?$AAh?$AAo?$AAn?$AAe?$AAb?$AAo?$AAo?$AAk?$AAI?$AAn?$AAi?$AAt?$AAD?$AAo?$AAn?$AAe?$AAC?$AAa?$AAl?$AAl?$AAb?$AAa?$AAc?$AAk?$AA?$AA@ 1002f780     stdafx.obj
 0002:000097c0       ??_C@_1DO@DLOHKDJD@?$AAS?$AAe?$AAt?$AAP?$AAh?$AAo?$AAn?$AAe?$AAb?$AAo?$AAo?$AAk?$AAR?$AAe?$AAc?$AAo?$AAr?$AAd?$AAR?$AAe?$AAa?$AAd?$AAC?$AAa?$AAl?$AAl?$AAb?$AAa?$AAc?$AAk?$AA?$AA@ 1002f7c0     stdafx.obj
 0002:00009800       ??_C@_1CM@HCOEPPEB@?$AAS?$AAe?$AAt?$AAO?$AAM?$AAA?$AAD?$AAM?$AAA?$AAl?$AAe?$AAr?$AAt?$AAC?$AAa?$AAl?$AAl?$AAb?$AAa?$AAc?$AAk?$AA?$AA@ 1002f800     stdafx.obj
 0002:0000982c       ??_C@_1CM@LPNPGND@?$AAS?$AAe?$AAt?$AAO?$AAM?$AAA?$AAD?$AAM?$AAS?$AAt?$AAa?$AAt?$AAe?$AAC?$AAa?$AAl?$AAl?$AAb?$AAa?$AAc?$AAk?$AA?$AA@ 1002f82c     stdafx.obj
 0002:00009858       ??_C@_1CM@JPEMOGPL@?$AAS?$AAe?$AAt?$AAB?$AAy?$AAt?$AAe?$AAT?$AAo?$AAt?$AAa?$AAl?$AAs?$AAC?$AAa?$AAl?$AAl?$AAb?$AAa?$AAc?$AAk?$AA?$AA@ 1002f858     stdafx.obj
 0002:00009884       ??_C@_1DI@NCMMIEFA@?$AAS?$AAe?$AAt?$AAD?$AAa?$AAt?$AAa?$AAC?$AAa?$AAp?$AAa?$AAb?$AAi?$AAl?$AAi?$AAt?$AAi?$AAe?$AAs?$AAC?$AAa?$AAl?$AAl?$AAb?$AAa?$AAc?$AAk?$AA?$AA@ 1002f884     stdafx.obj
 0002:000098bc       ??_C@_1CM@ODEGDLPB@?$AAS?$AAe?$AAt?$AAM?$AAs?$AAg?$AAW?$AAa?$AAi?$AAt?$AAi?$AAn?$AAg?$AAC?$AAa?$AAl?$AAl?$AAb?$AAa?$AAc?$AAk?$AA?$AA@ 1002f8bc     stdafx.obj
 0002:000098e8       ??_C@_1CI@MKCNFE@?$AAS?$AAe?$AAt?$AAN?$AAe?$AAw?$AAS?$AAM?$AAS?$AAC?$AAB?$AAC?$AAa?$AAl?$AAl?$AAb?$AAa?$AAc?$AAk?$AA?$AA@ 1002f8e8     stdafx.obj
 0002:00009910       ??_C@_1CE@DABFEIP@?$AAS?$AAe?$AAt?$AAN?$AAe?$AAw?$AAS?$AAM?$AAS?$AAC?$AAa?$AAl?$AAl?$AAb?$AAa?$AAc?$AAk?$AA?$AA@ 1002f910     stdafx.obj
 0002:00009934       ??_C@_1CE@FLDCNMCI@?$AAS?$AAe?$AAt?$AAR?$AAF?$AAI?$AAn?$AAf?$AAo?$AAC?$AAa?$AAl?$AAl?$AAb?$AAa?$AAc?$AAk?$AA?$AA@ 1002f934     stdafx.obj
 0002:00009958       ??_C@_1DE@DAEJPNFC@?$AAS?$AAe?$AAt?$AAS?$AAi?$AAg?$AAn?$AAa?$AAl?$AAS?$AAt?$AAr?$AAe?$AAn?$AAg?$AAt?$AAh?$AAC?$AAa?$AAl?$AAl?$AAb?$AAa?$AAc?$AAk?$AA?$AA@ 1002f958     stdafx.obj
 0002:0000998c       ??_C@_1DI@OAEMGPHA@?$AAS?$AAe?$AAt?$AAR?$AAo?$AAa?$AAm?$AAi?$AAn?$AAg?$AAI?$AAn?$AAd?$AAi?$AAc?$AAa?$AAt?$AAo?$AAr?$AAC?$AAa?$AAl?$AAl?$AAb?$AAa?$AAc?$AAk?$AA?$AA@ 1002f98c     stdafx.obj
 0002:000099c4       ??_C@_1CC@BKDJJPFD@?$AAS?$AAe?$AAt?$AAP?$AAo?$AAw?$AAe?$AAr?$AAC?$AAa?$AAl?$AAl?$AAb?$AAa?$AAc?$AAk?$AA?$AA@ 1002f9c4     stdafx.obj
 0002:000099e8       ??_C@_1DI@PLBJFEGC@?$AAS?$AAe?$AAt?$AAA?$AAc?$AAt?$AAi?$AAv?$AAa?$AAt?$AAi?$AAo?$AAn?$AAS?$AAt?$AAa?$AAt?$AAu?$AAs?$AAC?$AAa?$AAl?$AAl?$AAb?$AAa?$AAc?$AAk?$AA?$AA@ 1002f9e8     stdafx.obj
 0002:00009a20       ??_C@_1DE@IIMOCCEI@?$AAS?$AAe?$AAt?$AAM?$AAo?$AAb?$AAi?$AAl?$AAe?$AAI?$AAP?$AAS?$AAt?$AAa?$AAt?$AAu?$AAs?$AAC?$AAa?$AAl?$AAl?$AAb?$AAa?$AAc?$AAk?$AA?$AA@ 1002fa20     stdafx.obj
 0002:00009a54       ??_C@_1DE@NMHAIBGI@?$AAS?$AAe?$AAt?$AAD?$AAo?$AAr?$AAm?$AAa?$AAn?$AAc?$AAy?$AAS?$AAt?$AAa?$AAt?$AAu?$AAs?$AAC?$AAa?$AAl?$AAl?$AAb?$AAa?$AAc?$AAk?$AA?$AA@ 1002fa54     stdafx.obj
 0002:00009a88       ??_C@_1CM@JIDPIPCP@?$AAS?$AAe?$AAt?$AAD?$AAa?$AAt?$AAa?$AAB?$AAe?$AAa?$AAr?$AAe?$AAr?$AAC?$AAa?$AAl?$AAl?$AAb?$AAa?$AAc?$AAk?$AA?$AA@ 1002fa88     stdafx.obj
 0002:00009ab4       ??_C@_1DA@JDCAJDBL@?$AAS?$AAe?$AAt?$AAS?$AAe?$AAs?$AAs?$AAi?$AAo?$AAn?$AAS?$AAt?$AAa?$AAt?$AAe?$AAC?$AAa?$AAl?$AAl?$AAb?$AAa?$AAc?$AAk?$AA?$AA@ 1002fab4     stdafx.obj
 0002:00009ae4       ??_C@_1DG@PCCFMBCH@?$AAQ?$AAC?$AAW?$AAW?$AAA?$AAN?$AAG?$AAe?$AAt?$AAC?$AAo?$AAn?$AAn?$AAe?$AAc?$AAt?$AAe?$AAd?$AAD?$AAe?$AAv?$AAi?$AAc?$AAe?$AAI?$AAD?$AA?$AA@ 1002fae4     stdafx.obj
 0002:00009b1c       ??_C@_1CC@JBHNEBD@?$AAQ?$AAC?$AAW?$AAW?$AAA?$AAN?$AAD?$AAi?$AAs?$AAc?$AAo?$AAn?$AAn?$AAe?$AAc?$AAt?$AA?$AA@ 1002fb1c     stdafx.obj
 0002:00009b40       ??_C@_1BM@ICODGDCC@?$AAQ?$AAC?$AAW?$AAW?$AAA?$AAN?$AAC?$AAo?$AAn?$AAn?$AAe?$AAc?$AAt?$AA?$AA@ 1002fb40     stdafx.obj
 0002:00009b5c       ??_C@_1BM@HKEBDPIM@?$AAG?$AAe?$AAt?$AAR?$AAT?$AAR?$AAE?$AAC?$AAo?$AAn?$AAf?$AAi?$AAg?$AA?$AA@ 1002fb5c     stdafx.obj
 0002:00009b78       ??_C@_1BK@JPAMOEJH@?$AAS?$AAt?$AAo?$AAp?$AAC?$AAo?$AAn?$AAt?$AAD?$AAT?$AAM?$AAF?$AA?$AA@ 1002fb78     stdafx.obj
 0002:00009b94       ??_C@_1BM@BBOAIDPB@?$AAS?$AAt?$AAa?$AAr?$AAt?$AAC?$AAo?$AAn?$AAt?$AAD?$AAT?$AAM?$AAF?$AA?$AA@ 1002fb94     stdafx.obj
 0002:00009bb0       ??_C@_1BE@HONOAGGK@?$AAS?$AAe?$AAn?$AAd?$AAF?$AAl?$AAa?$AAs?$AAh?$AA?$AA@ 1002fbb0     stdafx.obj
 0002:00009bc4       ??_C@_1BO@GPPPCEIO@?$AAG?$AAe?$AAt?$AAA?$AAl?$AAl?$AAC?$AAa?$AAl?$AAl?$AAI?$AAn?$AAf?$AAo?$AA?$AA@ 1002fbc4     stdafx.obj
 0002:00009be4       ??_C@_1BO@NMMIKEEG@?$AAG?$AAe?$AAt?$AAC?$AAa?$AAl?$AAl?$AAW?$AAa?$AAi?$AAt?$AAi?$AAn?$AAg?$AA?$AA@ 1002fbe4     stdafx.obj
 0002:00009c04       ??_C@_1CE@LMIADLLA@?$AAG?$AAe?$AAt?$AAC?$AAa?$AAl?$AAl?$AAF?$AAo?$AAr?$AAw?$AAa?$AAr?$AAd?$AAi?$AAn?$AAg?$AA?$AA@ 1002fc04     stdafx.obj
 0002:00009c28       ??_C@_1BA@KNBNBGGG@?$AAG?$AAe?$AAt?$AAC?$AAL?$AAI?$AAR?$AA?$AA@ 1002fc28     stdafx.obj
 0002:00009c38       ??_C@_1BO@JOMDFNKA@?$AAS?$AAe?$AAt?$AAS?$AAu?$AAp?$AAs?$AAS?$AAe?$AAr?$AAv?$AAi?$AAc?$AAe?$AA?$AA@ 1002fc38     stdafx.obj
 0002:00009c58       ??_C@_1BO@DACCHOHL@?$AAG?$AAe?$AAt?$AAC?$AAa?$AAl?$AAl?$AAB?$AAa?$AAr?$AAr?$AAi?$AAn?$AAg?$AA?$AA@ 1002fc58     stdafx.obj
 0002:00009c78       ??_C@_1BI@BPLGPDPM@?$AAM?$AAa?$AAn?$AAa?$AAg?$AAe?$AAC?$AAa?$AAl?$AAl?$AAs?$AA?$AA@ 1002fc78     stdafx.obj
 0002:00009c90       ??_C@_1DI@LJBDKNNH@?$AAS?$AAe?$AAt?$AAU?$AAS?$AAS?$AAD?$AAN?$AAo?$AAt?$AAi?$AAf?$AAi?$AAc?$AAa?$AAt?$AAi?$AAo?$AAn?$AAC?$AAa?$AAl?$AAl?$AAb?$AAa?$AAc?$AAk?$AA?$AA@ 1002fc90     stdafx.obj
 0002:00009cc8       ??_C@_1CG@JABLONJK@?$AAS?$AAe?$AAt?$AAI?$AAn?$AAf?$AAo?$AAR?$AAe?$AAc?$AAC?$AAa?$AAl?$AAl?$AAb?$AAa?$AAc?$AAk?$AA?$AA@ 1002fcc8     stdafx.obj
 0002:00009cf0       ??_C@_1CI@OOGJCAEL@?$AAS?$AAe?$AAt?$AAC?$AAa?$AAl?$AAl?$AAI?$AAn?$AAf?$AAo?$AAC?$AAa?$AAl?$AAl?$AAb?$AAa?$AAc?$AAk?$AA?$AA@ 1002fcf0     stdafx.obj
 0002:00009d18       ??_C@_1BA@EMHLIJIE@?$AAE?$AAn?$AAd?$AAC?$AAa?$AAl?$AAl?$AA?$AA@ 1002fd18     stdafx.obj
 0002:00009d28       ??_C@_1BG@BKDINFBH@?$AAA?$AAn?$AAs?$AAw?$AAe?$AAr?$AAC?$AAa?$AAl?$AAl?$AA?$AA@ 1002fd28     stdafx.obj
 0002:00009d40       ??_C@_1BC@JGHLMAEH@?$AAD?$AAi?$AAa?$AAl?$AAC?$AAa?$AAl?$AAl?$AA?$AA@ 1002fd40     stdafx.obj
 0002:00009d54       ??_C@_1BI@PLMCJPHK@?$AAG?$AAo?$AAb?$AAi?$AAA?$AAp?$AAi?$AA?4?$AAd?$AAl?$AAl?$AA?$AA@ 1002fd54     stdafx.obj
 0002:00009d6c       ??_C@_1CA@CNOKPCAK@?$AA?4?$AA?2?$AAS?$AAw?$AAi?$AAA?$AAt?$AAP?$AAo?$AAr?$AAt?$AA?4?$AAc?$AAp?$AAp?$AA?$AA@ 1002fd6c     SwiAtPort.obj
 0002:00009d90       ??_C@_1HC@OCJPGFJI@?$AAA?$AAS?$AAS?$AAE?$AAR?$AAT?$AAI?$AAO?$AAN?$AA?5?$AAF?$AAA?$AAI?$AAL?$AAU?$AAR?$AAE?$AA?3?$AA?5?$AA?$DN?$AA?$DN?$AA?$DN?$AA?$DO?$AAm?$AA_?$AAh?$AAA?$AAT?$AAP?$AAo?$AAr?$AAt@ 1002fd90     SwiAtPort.obj
 0002:00009e04       ??_C@_15GANGMFKL@?$AA?$CF?$AAs?$AA?$AA@ 1002fe04     SwiAtPort.obj
 0002:00009e0c       ??_C@_13EBCNDICG@?$AA?3?$AA?$AA@ 1002fe0c     SwiAtPort.obj
 0002:00009e10       ??_C@_1CM@MAELFJAI@?$AAF?$AAi?$AAn?$AAa?$AAl?$AA?5?$AAP?$AAo?$AAr?$AAt?$AAN?$AAa?$AAm?$AAe?$AA?5?$AA?$DN?$AA?5?$AA?5?$AA?$CF?$AAs?$AA?5?$AA?$AA@ 1002fe10     SwiAtPort.obj
 0002:00009e40       ??_C@_1EI@EOCLNEBF@?$AAC?$AAr?$AAe?$AAa?$AAt?$AAe?$AAF?$AAi?$AAl?$AAe?$AA?$CI?$AA?$CJ?$AA?5?$AAo?$AAn?$AA?5?$AA?$CF?$AAs?$AA?5?$AAf?$AAa?$AAi?$AAl?$AAe?$AAd?$AA?0?$AA?5?$AAe?$AAr?$AAr?$AAn?$AAo@ 1002fe40     SwiAtPort.obj
 0002:00009e88       ??_C@_1EG@JDEAECKH@?$AAS?$AAe?$AAt?$AAC?$AAo?$AAm?$AAm?$AAT?$AAi?$AAm?$AAe?$AAo?$AAu?$AAt?$AAs?$AA?$CI?$AA?$CJ?$AA?5?$AAf?$AAa?$AAi?$AAl?$AAe?$AAd?$AA?0?$AA?5?$AAe?$AAr?$AAr?$AAn?$AAo?$AA?5@ 1002fe88     SwiAtPort.obj
 0002:00009ed0       ??_C@_1DK@GHDNLIGJ@?$AAS?$AAe?$AAt?$AAu?$AAp?$AAC?$AAo?$AAm?$AAm?$AA?$CI?$AA?$CJ?$AA?5?$AAf?$AAa?$AAi?$AAl?$AAe?$AAd?$AA?0?$AA?5?$AAe?$AAr?$AAr?$AAn?$AAo?$AA?5?$AA?$CF?$AAd?$AA?$AA@ 1002fed0     SwiAtPort.obj
 0002:00009f0c       ??_C@_1DC@ELDKGAGD@?$AAA?$AAS?$AAS?$AAE?$AAR?$AAT?$AAI?$AAO?$AAN?$AA?5?$AAF?$AAA?$AAI?$AAL?$AAU?$AAR?$AAE?$AA?3?$AA?5?$AA?$DN?$AA?$DN?$AA?$DN?$AA?$DO?$AA0?$AA?$AA@ 1002ff0c     SwiAtPort.obj
 0002:00009f40       ??_C@_1EI@EAPLNMAK@?$AAS?$AAe?$AAt?$AAC?$AAo?$AAm?$AAm?$AAS?$AAt?$AAa?$AAt?$AAe?$AA?5?$AAf?$AAa?$AAi?$AAl?$AAe?$AAd?$AA?0?$AA?5?$AAW?$AAi?$AAn?$AA?5?$AAE?$AAr?$AAr?$AAo?$AAr?$AA?5?$AA?$DN@ 1002ff40     SwiAtPort.obj
 0002:00009f88       ??_C@_1DK@JBCAIHHN@?$AAP?$AAu?$AAr?$AAg?$AAe?$AAC?$AAo?$AAm?$AAm?$AA?$CI?$AA?$CJ?$AA?5?$AAf?$AAa?$AAi?$AAl?$AAe?$AAd?$AA?0?$AA?5?$AAe?$AAr?$AAr?$AAn?$AAo?$AA?5?$AA?$CF?$AAd?$AA?$AA@ 1002ff88     SwiAtPort.obj
 0002:00009fc8       ??_C@_1EA@PDEGNLIG@?$AAR?$AAe?$AAa?$AAd?$AAF?$AAi?$AAl?$AAe?$AA?5?$AAf?$AAa?$AAi?$AAl?$AAe?$AAd?$AA?0?$AA?5?$AAW?$AAi?$AAn?$AA?5?$AAE?$AAr?$AAr?$AAo?$AAr?$AA?5?$AA?$DN?$AA?5?$AA?$CF?$AAd?$AA?$AA@ 1002ffc8     SwiAtPort.obj
 0002:0000a008       ??_C@_05MBDEGLCK@ERROR?$AA@ 10030008     SwiAtPort.obj
 0002:0000a010       ??_C@_1CA@FCALIIKG@?$AAa?$AAt?$AAc?$AAm?$AAd?$AA?5?$AAt?$AAi?$AAm?$AAe?$AAd?$AAo?$AAu?$AAt?$AA?$CB?$AA?$AA@ 10030010     SwiAtPort.obj
 0002:0000a030       ??_C@_06HBBEPAPC@?$AN?6AT?$AN?6?$AA@ 10030030     SwiAtPort.obj
 0002:0000a038       ??_C@_1CI@OKMALDLC@?$AAA?$AAT?$AA?5?$AAR?$AAS?$AAP?$AA?5?$AA?5?$AAs?$AAt?$AAr?$AAi?$AAn?$AAg?$AA?5?$AA?$DN?$AA?5?$AA?$CF?$AAs?$AA?$AA@ 10030038     SwiAtPort.obj
 0002:0000a060       ??_C@_09PJFLLFKF@?$CLPACSP0?$AN?6?$AA@ 10030060     SwiAtPort.obj
 0002:0000a06c       ??_C@_09EBOHNCMA@?$CLPACSP1?$AN?6?$AA@ 1003006c     SwiAtPort.obj
 0002:0000a078       ??_C@_1IA@EBLMMBOK@?$AAN?$AAo?$AAt?$AAi?$AAf?$AAi?$AAc?$AAa?$AAt?$AAi?$AAo?$AAn?$AA?5?$AAf?$AAo?$AAu?$AAn?$AAd?$AA?5?$AAa?$AAt?$AA?5?$AAt?$AAh?$AAe?$AA?5?$AAb?$AAe?$AAg?$AAi?$AAn?$AAn@ 10030078     SwiAtPort.obj
 0002:0000a0f8       ??_C@_1CC@HGBGDAB@?$AAA?$AAT?$AA?5?$AAP?$AAo?$AAr?$AAt?$AA?5?$AAn?$AAo?$AAt?$AA?5?$AAI?$AAN?$AAI?$AAT?$AA?$AA@ 100300f8     SwiAtPort.obj
 0002:0000a11c       ??_C@_1CC@PHDEGBFD@?$AAW?$AAr?$AAi?$AAt?$AAe?$AAF?$AAi?$AAl?$AAe?$AA?5?$AAd?$AAa?$AAt?$AAa?$AA?3?$AA?5?$AA?$AA@ 1003011c     SwiAtPort.obj
 0002:0000a140       ??_C@_1EC@NACHPKAA@?$AAW?$AAr?$AAi?$AAt?$AAe?$AAF?$AAi?$AAl?$AAe?$AA?5?$AAf?$AAa?$AAi?$AAl?$AAe?$AAd?$AA?0?$AA?5?$AAW?$AAi?$AAn?$AA?5?$AAE?$AAr?$AAr?$AAo?$AAr?$AA?5?$AA?$DN?$AA?5?$AA?$CF?$AAd@ 10030140     SwiAtPort.obj
 0002:0000a184       ??_C@_02GIPFHKNO@OK?$AA@   10030184     SwiAtPort.obj
 0002:0000a188       ??_C@_1BO@MDIOANPL@?$AA?4?$AA?2?$AAS?$AAw?$AAi?$AAE?$AAr?$AAr?$AAo?$AAr?$AA?4?$AAc?$AAp?$AAp?$AA?$AA@ 10030188     SwiError.obj
 0002:0000a1a8       ??_C@_1DC@CFJKGJDO@?$AAO?$AAu?$AAt?$AA?5?$AAo?$AAf?$AA?5?$AAr?$AAa?$AAn?$AAg?$AAe?$AA?5?$AAu?$AAE?$AAr?$AAr?$AAo?$AAr?$AA?5?$AA?$DN?$AA?5?$AA?$CF?$AAd?$AA?$AA@ 100301a8     SwiError.obj
 0002:0000a1dc       ??_C@_1DM@MPPFMKOE@?$AAS?$AAe?$AAs?$AAs?$AAi?$AAo?$AAn?$AAT?$AAy?$AAp?$AAe?$AA?5?$AAo?$AAu?$AAt?$AA?5?$AAo?$AAf?$AA?5?$AAr?$AAa?$AAn?$AAg?$AAe?$AA?5?$AA?$DN?$AA?5?$AA?$CF?$AAd?$AA?$AA@ 100301dc     SwiError.obj
 0002:0000a218       ??_C@_1FM@FMIGAALN@?$AAM?$AAa?$AAx?$AAi?$AAm?$AAu?$AAm?$AA?5?$AAD?$AAe?$AAv?$AAi?$AAc?$AAe?$AA?5?$AAI?$AAn?$AAi?$AAt?$AAi?$AAa?$AAt?$AAe?$AAd?$AA?5?$AAO?$AAM?$AAA?$AAD?$AAM?$AA?5?$AAr@ 10030218     SwiError.obj
 0002:0000a278       ??_C@_1EA@IMCBEILA@?$AAO?$AAu?$AAt?$AA?5?$AAo?$AAf?$AA?5?$AAr?$AAa?$AAn?$AAg?$AAe?$AA?5?$AAo?$AAp?$AAe?$AAr?$AAa?$AAt?$AAi?$AAn?$AAg?$AAM?$AAo?$AAd?$AAe?$AA?5?$AA?$DN?$AA?5?$AA?$CF?$AAd?$AA?$AA@ 10030278     SwiError.obj
 0002:0000a2b8       ??_C@_1DE@GGOPAHAM@?$AAU?$AAn?$AAs?$AAu?$AAp?$AAp?$AAo?$AAr?$AAt?$AAe?$AAd?$AA?5?$AAr?$AAe?$AAg?$AAS?$AAt?$AAa?$AAt?$AAe?$AA?5?$AA?$DN?$AA?5?$AA?$CF?$AAd?$AA?$AA@ 100302b8     SwiError.obj
 0002:0000a2f0       ??_C@_1EG@NNGHMPDL@?$AAN?$AAo?$AAt?$AA?5?$AAr?$AAe?$AAc?$AAo?$AAg?$AAn?$AAi?$AAz?$AAe?$AAd?$AA?5?$AAd?$AAa?$AAt?$AAa?$AAB?$AAe?$AAa?$AAr?$AAe?$AAr?$AAT?$AAe?$AAc?$AAh?$AA?5?$AA?$DN?$AA?5@ 100302f0     SwiError.obj
 0002:0000a338       ??_C@_1IA@NKGCIACG@?$AAC?$AAo?$AAn?$AAv?$AAe?$AAr?$AAt?$AAG?$AAo?$AAb?$AAi?$AA2?$AAS?$AAw?$AAi?$AAN?$AAv?$AAP?$AAr?$AAe?$AAf?$AAO?$AAp?$AAM?$AAo?$AAd?$AAe?$AA?5?$AAu?$AAP?$AAr?$AAe@ 10030338     SwiError.obj
 0002:0000a3b8       ??_C@_1FI@NGMGNIAH@?$AAC?$AAo?$AAn?$AAv?$AAe?$AAr?$AAt?$AAG?$AAo?$AAb?$AAi?$AA2?$AAS?$AAw?$AAi?$AAN?$AAv?$AAP?$AAr?$AAe?$AAf?$AAO?$AAp?$AAM?$AAo?$AAd?$AAe?$AA?5?$AAu?$AAP?$AAr?$AAo@ 100303b8     SwiError.obj
 0002:0000a410       ??_C@_1EM@CGEBOGEI@?$AAP?$AAr?$AAe?$AAf?$AA?5?$AAM?$AAo?$AAd?$AAe?$AA?5?$AAp?$AAr?$AAo?$AAt?$AAo?$AAc?$AAo?$AAl?$AA?$DN?$AA?5?$AA?$CF?$AAl?$AAu?$AA?5?$AAN?$AAo?$AAt?$AA?5?$AAs?$AAu?$AAp?$AAp@ 10030410     SwiError.obj
 0002:0000a460       ??_C@_1FC@FMHJFOGL@?$AAP?$AAr?$AAe?$AAf?$AA?5?$AAM?$AAo?$AAd?$AAe?$AA?5?$AAT?$AAe?$AAc?$AAh?$AAn?$AAo?$AAl?$AAo?$AAg?$AAy?$AA?5?$AA?$DN?$AA?5?$AA?$CF?$AAl?$AAu?$AA?5?$AAN?$AAo?$AAt?$AA?5?$AAs@ 10030460     SwiError.obj
 0002:0000a4b8       ??_C@_1EK@PKGIEHCB@?$AAP?$AAr?$AAe?$AAf?$AA?5?$AAm?$AAo?$AAd?$AAe?$AA?5?$AAn?$AAo?$AAt?$AA?5?$AAs?$AAu?$AAp?$AAp?$AAo?$AAr?$AAt?$AAe?$AAd?$AA?5?$AAb?$AAy?$AA?5?$AAG?$AAo?$AAb?$AAi?$AA?5@ 100304b8     SwiError.obj
 0002:0000a504       ??_C@_1CI@JDJEEEIN@?$AAG?$AAo?$AAb?$AAi?$AA?5?$AAP?$AAr?$AAe?$AAf?$AA?5?$AAm?$AAo?$AAd?$AAe?$AA?5?$AA?$DN?$AA?5?$AA?$CF?$AAu?$AA?$AA@ 10030504     SwiError.obj
 0002:0000a530       ??_C@_1GM@OGCDBPAK@?$AAE?$AAx?$AAt?$AAr?$AAa?$AAc?$AAt?$AAE?$AAr?$AAr?$AAo?$AAr?$AAC?$AAo?$AAd?$AAe?$AA?3?$AAM?$AAa?$AAt?$AAc?$AAh?$AAS?$AAt?$AAr?$AAi?$AAn?$AAg?$AAB?$AAe?$AAg?$AAi@ 10030530     SwiError.obj
 0002:0000a59c       ??_C@_0N@JHNBODDK@?$CLCME?5ERROR?3?5?$AA@ 1003059c     SwiError.obj
 0002:0000a5b0       ??_C@_1FM@IOBBOGNI@?$AAE?$AAx?$AAt?$AAr?$AAa?$AAc?$AAt?$AAE?$AAr?$AAr?$AAo?$AAr?$AAC?$AAo?$AAd?$AAe?$AA?3?$AAM?$AAa?$AAt?$AAc?$AAh?$AAS?$AAt?$AAr?$AAi?$AAn?$AAg?$AAB?$AAe?$AAg?$AAi@ 100305b0     SwiError.obj
 0002:0000a610       ??_C@_1EK@IBHGFAIA@?$AAE?$AAx?$AAt?$AAr?$AAa?$AAc?$AAt?$AAE?$AAr?$AAr?$AAo?$AAr?$AAC?$AAo?$AAd?$AAe?$AA?3?$AAP?$AAa?$AAr?$AAs?$AAe?$AAU?$AAI?$AAn?$AAt?$AA?5?$AA1?$AA?5?$AAf?$AAa?$AAi@ 10030610     SwiError.obj
 0002:0000a65c       ??_C@_1CC@NHFAMJFA@?$AA?4?$AA?2?$AAS?$AAw?$AAi?$AAG?$AAo?$AAb?$AAi?$AAD?$AAl?$AAl?$AA?4?$AAc?$AAp?$AAp?$AA?$AA@ 1003065c     SwiGobiDll.obj
 0002:0000a680       ??_C@_1DO@CBACMFO@?$AAG?$AAo?$AAb?$AAi?$AAC?$AAo?$AAn?$AAn?$AAe?$AAc?$AAt?$AA?5?$AAf?$AAa?$AAi?$AAl?$AAe?$AAd?$AA?5?$AAs?$AAt?$AAa?$AAt?$AAu?$AAs?$AA?5?$AA?$DN?$AA?5?$AA?$CF?$AAd?$AA?$AA@ 10030680     SwiGobiDll.obj
 0002:0000a6c0       ??_C@_17INOCEEPC@?$AA1?$AA0?$AA2?$AA?$AA@ 100306c0     SwiGobiDll.obj
 0002:0000a6c8       ??_C@_1EO@OLNFOIFC@?$AAS?$AAe?$AAt?$AAD?$AAe?$AAf?$AAa?$AAu?$AAl?$AAt?$AAP?$AAr?$AAo?$AAf?$AAi?$AAl?$AAe?$AA?5?$AAr?$AAe?$AAt?$AAu?$AAr?$AAn?$AAs?$AA?5?$AAu?$AAS?$AAt?$AAa?$AAt?$AAu@ 100306c8     SwiGobiDll.obj
 0002:0000a718       ??_C@_1EO@HBHDOKFN@?$AAG?$AAe?$AAt?$AAD?$AAe?$AAf?$AAa?$AAu?$AAl?$AAt?$AAP?$AAr?$AAo?$AAf?$AAi?$AAl?$AAe?$AA?5?$AAr?$AAe?$AAt?$AAu?$AAr?$AAn?$AAs?$AA?5?$AAu?$AAS?$AAt?$AAa?$AAt?$AAu@ 10030718     SwiGobiDll.obj
 0002:0000a768       ??_C@_1DE@EKBCEPAI@?$AAS?$AAe?$AAt?$AAS?$AAM?$AAS?$AAB?$AAr?$AAo?$AAa?$AAd?$AAc?$AAa?$AAs?$AAt?$AAA?$AAc?$AAt?$AAi?$AAv?$AAa?$AAt?$AAi?$AAo?$AAn?$AA?$AA@ 10030768     SwiGobiDll.obj
 0002:0000a7a0       ??_C@_1EO@ICGPEANE@?$AAG?$AAe?$AAt?$AAS?$AAi?$AAg?$AAn?$AAa?$AAl?$AAS?$AAt?$AAr?$AAe?$AAn?$AAg?$AAt?$AAh?$AAs?$AA?5?$AAr?$AAe?$AAt?$AAu?$AAr?$AAn?$AAs?$AA?5?$AAs?$AAt?$AAa?$AAt?$AAu@ 100307a0     SwiGobiDll.obj
 0002:0000a7f0       ??_C@_1HA@EFLGNFNI@?$AAC?$AAa?$AAl?$AAl?$AAi?$AAn?$AAg?$AA?5?$AAm?$AAp?$AAF?$AAN?$AAS?$AAe?$AAt?$AAS?$AAe?$AAs?$AAs?$AAi?$AAo?$AAn?$AAS?$AAt?$AAa?$AAt?$AAe?$AAC?$AAB?$AA?5?$AA?$DN?$AA?5@ 100307f0     SwiGobiDll.obj
 0002:0000a860       ??_C@_1CK@BGOLANAA@?$AAS?$AAe?$AAt?$AAV?$AAo?$AAi?$AAc?$AAe?$AAM?$AAe?$AAs?$AAs?$AAa?$AAg?$AAe?$AAC?$AAB?$AA?5?$AA?$CF?$AAd?$AA?$AA@ 10030860     SwiGobiDll.obj
 0002:0000a890       ??_C@_1FK@LLMBFEPE@?$AAS?$AAe?$AAt?$AAD?$AAe?$AAv?$AAi?$AAc?$AAe?$AAR?$AAe?$AAm?$AAo?$AAv?$AAa?$AAl?$AAC?$AAa?$AAl?$AAl?$AAb?$AAa?$AAc?$AAk?$AA?5?$AAr?$AAe?$AAt?$AAu?$AAr?$AAn?$AAs@ 10030890     SwiGobiDll.obj
 0002:0000a8f0       ??_C@_1FI@ONFLAPAG@?$AAS?$AAe?$AAt?$AAP?$AAo?$AAw?$AAe?$AAr?$AA?5?$AAp?$AAo?$AAw?$AAe?$AAr?$AAM?$AAo?$AAd?$AAe?$AA?5?$AA?$DN?$AA?5?$AA?$CF?$AAd?$AA?5?$AAr?$AAe?$AAt?$AAu?$AAr?$AAn?$AAs?$AA?5@ 100308f0     SwiGobiDll.obj
 0002:0000a948       ??_C@_1HG@NDAEJPAH@?$AAA?$AAc?$AAt?$AAi?$AAv?$AAa?$AAt?$AAe?$AAA?$AAu?$AAt?$AAo?$AAm?$AAa?$AAt?$AAi?$AAc?$AA?5?$AAp?$AAA?$AAc?$AAt?$AAi?$AAv?$AAa?$AAt?$AAi?$AAo?$AAn?$AAC?$AAo?$AAd@ 10030948     SwiGobiDll.obj
 0002:0000a9c0       ??_C@_1EO@HKKEBGCC@?$AAG?$AAe?$AAt?$AAA?$AAc?$AAt?$AAi?$AAv?$AAa?$AAt?$AAi?$AAo?$AAn?$AAS?$AAt?$AAa?$AAt?$AAe?$AA?5?$AAr?$AAe?$AAt?$AAu?$AAr?$AAn?$AAs?$AA?5?$AAs?$AAt?$AAa?$AAt?$AAu@ 100309c0     SwiGobiDll.obj
 0002:0000aa10       ??_C@_1FI@MMMLHOOG@?$AAO?$AAM?$AAA?$AAD?$AAM?$AAG?$AAe?$AAt?$AAF?$AAe?$AAa?$AAt?$AAu?$AAr?$AAe?$AAS?$AAe?$AAt?$AAt?$AAi?$AAn?$AAg?$AAs?$AA?5?$AAr?$AAe?$AAt?$AAu?$AAr?$AAn?$AAs?$AA?5@ 10030a10     SwiGobiDll.obj
 0002:0000aa68       ??_C@_1FA@BIDCIGCC@?$AAO?$AAM?$AAA?$AAD?$AAM?$AAG?$AAe?$AAt?$AAS?$AAe?$AAs?$AAs?$AAi?$AAo?$AAn?$AAI?$AAn?$AAf?$AAo?$AA?5?$AAr?$AAe?$AAt?$AAu?$AAr?$AAn?$AAs?$AA?5?$AAs?$AAt?$AAa?$AAt@ 10030a68     SwiGobiDll.obj
 0002:0000aab8       ??_C@_1GA@PFKAIBHB@?$AAO?$AAM?$AAA?$AAD?$AAM?$AAS?$AAe?$AAt?$AAP?$AAr?$AAo?$AAv?$AAi?$AAs?$AAi?$AAo?$AAn?$AAi?$AAn?$AAg?$AAF?$AAe?$AAa?$AAt?$AAu?$AAr?$AAe?$AA?5?$AAr?$AAe?$AAt?$AAu@ 10030ab8     SwiGobiDll.obj
 0002:0000ab18       ??_C@_1FK@OAANMIJC@?$AAO?$AAM?$AAA?$AAD?$AAM?$AAS?$AAe?$AAt?$AAP?$AAR?$AAL?$AAU?$AAp?$AAd?$AAa?$AAt?$AAe?$AAF?$AAe?$AAa?$AAt?$AAu?$AAr?$AAe?$AA?5?$AAr?$AAe?$AAt?$AAu?$AAr?$AAn?$AAs@ 10030b18     SwiGobiDll.obj
 0002:0000ab78       ??_C@_1EM@OCDJPOHJ@?$AAO?$AAM?$AAA?$AAD?$AAM?$AAS?$AAt?$AAa?$AAr?$AAt?$AAS?$AAe?$AAs?$AAs?$AAi?$AAo?$AAn?$AA?5?$AAr?$AAe?$AAt?$AAu?$AAr?$AAn?$AAs?$AA?5?$AAs?$AAt?$AAa?$AAt?$AAu?$AAs@ 10030b78     SwiGobiDll.obj
 0002:0000abc8       ??_C@_1EO@PKKCPBPK@?$AAO?$AAM?$AAA?$AAD?$AAM?$AAC?$AAa?$AAn?$AAc?$AAe?$AAl?$AAS?$AAe?$AAs?$AAs?$AAi?$AAo?$AAn?$AA?5?$AAr?$AAe?$AAt?$AAu?$AAr?$AAn?$AAs?$AA?5?$AAs?$AAt?$AAa?$AAt?$AAu@ 10030bc8     SwiGobiDll.obj
 0002:0000ac18       ??_C@_1EO@KIGIPEJI@?$AAO?$AAM?$AAA?$AAD?$AAM?$AAG?$AAe?$AAt?$AAP?$AAe?$AAn?$AAd?$AAi?$AAn?$AAg?$AAN?$AAI?$AAA?$AA?5?$AAr?$AAe?$AAt?$AAu?$AAr?$AAn?$AAs?$AA?5?$AAs?$AAt?$AAa?$AAt?$AAu@ 10030c18     SwiGobiDll.obj
 0002:0000ac68       ??_C@_1EO@GCOGGBBK@?$AAO?$AAM?$AAA?$AAD?$AAM?$AAS?$AAe?$AAn?$AAd?$AAS?$AAe?$AAl?$AAe?$AAc?$AAt?$AAi?$AAo?$AAn?$AA?5?$AAr?$AAe?$AAt?$AAu?$AAr?$AAn?$AAs?$AA?5?$AAs?$AAt?$AAa?$AAt?$AAu@ 10030c68     SwiGobiDll.obj
 0002:0000acb8       ??_C@_1EO@HDBIMGID@?$AAG?$AAe?$AAt?$AAI?$AAP?$AAC?$AAo?$AAn?$AAf?$AAi?$AAg?$AAu?$AAr?$AAa?$AAt?$AAi?$AAo?$AAn?$AA?5?$AAr?$AAe?$AAt?$AAu?$AAr?$AAn?$AAs?$AA?5?$AAs?$AAt?$AAa?$AAt?$AAu@ 10030cb8     SwiGobiDll.obj
 0002:0000ad08       ??_C@_1FA@JPGOJHBE@?$AAO?$AAM?$AAA?$AAE?$AAX?$AAS?$AAe?$AAt?$AAE?$AAv?$AAe?$AAn?$AAt?$AAR?$AAe?$AAp?$AAo?$AAr?$AAt?$AA?5?$AAr?$AAe?$AAt?$AAu?$AAr?$AAn?$AAs?$AA?5?$AAs?$AAt?$AAa?$AAt@ 10030d08     SwiGobiDll.obj
 0002:0000ad58       ??_C@_1EM@BMEMLAED@?$AAO?$AAM?$AAA?$AAE?$AAX?$AAS?$AAe?$AAs?$AAs?$AAi?$AAo?$AAn?$AAS?$AAt?$AAa?$AAr?$AAt?$AA?5?$AAr?$AAe?$AAt?$AAu?$AAr?$AAn?$AAs?$AA?5?$AAs?$AAt?$AAa?$AAt?$AAu?$AAs@ 10030d58     SwiGobiDll.obj
 0002:0000ada8       ??_C@_1EO@MAAOJNA@?$AAO?$AAM?$AAA?$AAE?$AAX?$AAS?$AAe?$AAs?$AAs?$AAi?$AAo?$AAn?$AAC?$AAa?$AAn?$AAc?$AAe?$AAl?$AA?5?$AAr?$AAe?$AAt?$AAu?$AAr?$AAn?$AAs?$AA?5?$AAs?$AAt?$AAa?$AAt?$AAu@ 10030da8     SwiGobiDll.obj
 0002:0000adf8       ??_C@_1EG@NJLACBAG@?$AAO?$AAM?$AAA?$AAE?$AAX?$AAS?$AAe?$AAl?$AAe?$AAc?$AAt?$AAi?$AAo?$AAn?$AA?5?$AAr?$AAe?$AAt?$AAu?$AAr?$AAn?$AAs?$AA?5?$AAs?$AAt?$AAa?$AAt?$AAu?$AAs?$AA?5?$AA?$DN?$AA?5@ 10030df8     SwiGobiDll.obj
 0002:0000ae40       ??_C@_1EK@GAJNKLCG@?$AAO?$AAM?$AAA?$AAE?$AAX?$AAG?$AAe?$AAt?$AAS?$AAe?$AAt?$AAt?$AAi?$AAn?$AAg?$AAs?$AA?5?$AAr?$AAe?$AAt?$AAu?$AAr?$AAn?$AAs?$AA?5?$AAs?$AAt?$AAa?$AAt?$AAu?$AAs?$AA?5@ 10030e40     SwiGobiDll.obj
 0002:0000ae90       ??_C@_1EK@KPLFODKM@?$AAO?$AAM?$AAA?$AAE?$AAX?$AAS?$AAe?$AAt?$AAS?$AAe?$AAt?$AAt?$AAi?$AAn?$AAg?$AAs?$AA?5?$AAr?$AAe?$AAt?$AAu?$AAr?$AAn?$AAs?$AA?5?$AAs?$AAt?$AAa?$AAt?$AAu?$AAs?$AA?5@ 10030e90     SwiGobiDll.obj
 0002:0000aee0       ??_C@_1FA@LCFOFJFD@?$AAO?$AAM?$AAA?$AAE?$AAX?$AAS?$AAe?$AAs?$AAs?$AAi?$AAo?$AAn?$AAG?$AAe?$AAt?$AAI?$AAn?$AAf?$AAo?$AA?5?$AAr?$AAe?$AAt?$AAu?$AAr?$AAn?$AAs?$AA?5?$AAs?$AAt?$AAa?$AAt@ 10030ee0     SwiGobiDll.obj
 0002:0000af30       ??_C@_1DM@IOCILBCI@?$AAO?$AAM?$AAA?$AAE?$AAX?$AAI?$AAn?$AAi?$AAt?$AA?5?$AAr?$AAe?$AAt?$AAu?$AAr?$AAn?$AAs?$AA?5?$AAs?$AAt?$AAa?$AAt?$AAu?$AAs?$AA?5?$AA?$DN?$AA?5?$AA?$CF?$AAd?$AA?$AA@ 10030f30     SwiGobiDll.obj
 0002:0000af70       ??_C@_1EE@NBKKEGOO@?$AAO?$AAM?$AAA?$AAE?$AAX?$AAS?$AAh?$AAu?$AAt?$AAd?$AAo?$AAw?$AAn?$AA?5?$AAr?$AAe?$AAt?$AAu?$AAr?$AAn?$AAs?$AA?5?$AAs?$AAt?$AAa?$AAt?$AAu?$AAs?$AA?5?$AA?$DN?$AA?5?$AA?$CF@ 10030f70     SwiGobiDll.obj
 0002:0000afb4       ??_C@_1DI@FPOIJINB@?$AAm?$AAp?$AAF?$AAn?$AAG?$AAe?$AAt?$AAA?$AAu?$AAd?$AAi?$AAo?$AAP?$AAr?$AAo?$AAf?$AAi?$AAl?$AAe?$AA?5?$AAf?$AAa?$AAi?$AAl?$AAe?$AAd?$AA?4?$AA?$AA@ 10030fb4     SwiGobiDll.obj
 0002:0000aff0       ??_C@_1EC@LCKLGMMI@?$AAm?$AAp?$AAF?$AAn?$AAG?$AAe?$AAt?$AAA?$AAu?$AAd?$AAi?$AAo?$AAP?$AAr?$AAo?$AAf?$AAi?$AAl?$AAe?$AA?5?$AAf?$AAa?$AAi?$AAl?$AAe?$AAd?$AA?4?$AA?5?$AA0?$AAx?$AA?$CF?$AAx@ 10030ff0     SwiGobiDll.obj
 0002:0000b038       ??_C@_1EO@HCMFABIC@?$AAm?$AAp?$AAF?$AAn?$AAP?$AAl?$AAa?$AAy?$AAA?$AAu?$AAd?$AAi?$AAo?$AAT?$AAo?$AAn?$AAe?$AA?5?$AAf?$AAa?$AAi?$AAl?$AAe?$AAd?$AA?5?$AAp?$AAT?$AAo?$AAn?$AAe?$AA?5?$AA?$DN@ 10031038     SwiGobiDll.obj
 0002:0000b088       ??_C@_1EA@EFHNHGPN@?$AAm?$AAp?$AAF?$AAN?$AAS?$AAe?$AAt?$AAA?$AAl?$AAl?$AAP?$AAb?$AAI?$AAn?$AAi?$AAt?$AAD?$AAo?$AAn?$AAe?$AAC?$AAB?$AA?5?$AAi?$AAs?$AA?5?$AAN?$AAU?$AAL?$AAL?$AA?$CB?$AA?$AA@ 10031088     SwiGobiDll.obj
 0002:0000b0c8       ??_C@_1EA@NKOLKGE@?$AAm?$AAp?$AAF?$AAN?$AAS?$AAe?$AAt?$AAE?$AAm?$AAe?$AAr?$AAg?$AAe?$AAn?$AAc?$AAy?$AAL?$AAi?$AAs?$AAt?$AAC?$AAB?$AA?5?$AAi?$AAs?$AA?5?$AAN?$AAU?$AAL?$AAL?$AA?$CB?$AA?$AA@ 100310c8     SwiGobiDll.obj
 0002:0000b108       ??_C@_1DK@GANCOJLG@?$AAm?$AAp?$AAF?$AAN?$AAS?$AAe?$AAt?$AAO?$AAM?$AAA?$AAE?$AAX?$AAE?$AAv?$AAe?$AAn?$AAt?$AAC?$AAB?$AA?5?$AAi?$AAs?$AA?5?$AAN?$AAU?$AAL?$AAL?$AA?$CB?$AA?$AA@ 10031108     SwiGobiDll.obj
 0002:0000b148       ??_C@_1EE@KMGACLIO@?$AAm?$AAp?$AAF?$AAn?$AAG?$AAe?$AAt?$AAC?$AAe?$AAl?$AAl?$AAL?$AAo?$AAc?$AAa?$AAt?$AAi?$AAo?$AAn?$AAI?$AAn?$AAf?$AAo?$AAM?$AAs?$AAg?$AA?5?$AA?$DN?$AA?5?$AAN?$AAU?$AAL@ 10031148     SwiGobiDll.obj
 0002:0000b18c       ??_C@_1DC@HDKKLFLH@?$AAm?$AAp?$AAF?$AAn?$AAG?$AAe?$AAt?$AAW?$AAa?$AAi?$AAt?$AAi?$AAn?$AAg?$AAM?$AAs?$AAg?$AA?5?$AA?$DN?$AA?5?$AAN?$AAU?$AAL?$AAL?$AA?$AA@ 1003118c     SwiGobiDll.obj
 0002:0000b1c0       ??_C@_1DC@JFFGHCIE@?$AAm?$AAp?$AAF?$AAn?$AAG?$AAe?$AAt?$AAR?$AAT?$AAR?$AAE?$AAC?$AAo?$AAn?$AAf?$AAi?$AAg?$AA?5?$AA?$DN?$AA?5?$AAN?$AAU?$AAL?$AAL?$AA?$AA@ 100311c0     SwiGobiDll.obj
 0002:0000b1f4       ??_C@_1CA@MHAKGOFM@?$AA?4?$AA?2?$AAS?$AAw?$AAi?$AAN?$AAo?$AAt?$AAi?$AAf?$AAy?$AA?4?$AAc?$AAp?$AAp?$AA?$AA@ 100311f4     SwiNotify.obj
 0002:0000b214       ??_C@_1CG@OPIJDBKM@?$AAO?$AAM?$AAA?$AAE?$AAX?$AAE?$AAv?$AAe?$AAn?$AAt?$AAC?$AAa?$AAl?$AAl?$AAb?$AAa?$AAc?$AAk?$AA?$AA@ 10031214     SwiNotify.obj
 0002:0000b23c       ??_C@_1CC@NDKAJLFJ@?$AAC?$AAa?$AAl?$AAl?$AAI?$AAn?$AAf?$AAo?$AAC?$AAa?$AAl?$AAl?$AAb?$AAa?$AAc?$AAk?$AA?$AA@ 1003123c     SwiNotify.obj
 0002:0000b260       ??_C@_1FM@KOCHHDEM@?$AAC?$AAa?$AAl?$AAl?$AAI?$AAn?$AAf?$AAo?$AAC?$AAa?$AAl?$AAl?$AAb?$AAa?$AAc?$AAk?$AA?5?$AA?3?$AA?5?$AAi?$AA?3?$AA?$CF?$AAd?$AA?0?$AA?5?$AAc?$AAa?$AAl?$AAl?$AAi?$AAd?$AA?5@ 10031260     SwiNotify.obj
 0002:0000b2c0       ??_C@_1EC@BGDHDKFB@?$AAs?$AAe?$AAn?$AAd?$AA?5?$AAr?$AAi?$AAn?$AAg?$AA?5?$AA?3?$AA?5?$AAc?$AAa?$AAl?$AAl?$AAi?$AAd?$AA?3?$AA?5?$AA?$CF?$AAd?$AA?0?$AAn?$AAu?$AAm?$AAb?$AAe?$AAr?$AA?3?$AA?$CF?$AAS@ 100312c0     SwiNotify.obj
 0002:0000b304       ??_C@_1BE@GLAMIBKP@?$AAC?$AAo?$AAn?$AAn?$AAe?$AAc?$AAt?$AAe?$AAd?$AA?$AA@ 10031304     SwiNotify.obj
 0002:0000b318       ??_C@_1BK@GGPLAOLF@?$AAD?$AAi?$AAs?$AAc?$AAo?$AAn?$AAn?$AAe?$AAc?$AAt?$AAe?$AAd?$AA?$AA@ 10031318     SwiNotify.obj
 0002:0000b334       ??_C@_1BK@DAKIOGJ@?$AAw?$AAa?$AAi?$AAt?$AAi?$AAn?$AAg?$AA?5?$AAr?$AAi?$AAn?$AAg?$AA?$AA@ 10031334     SwiNotify.obj
 0002:0000b350       ??_C@_1BK@JOPOGKOG@?$AAC?$AAa?$AAl?$AAl?$AA?5?$AAo?$AAn?$AA?5?$AAH?$AAo?$AAl?$AAd?$AA?$AA@ 10031350     SwiNotify.obj
 0002:0000b36c       ??_C@_1CA@LPNFNEEB@?$AAI?$AAn?$AAf?$AAo?$AAR?$AAe?$AAc?$AAC?$AAa?$AAl?$AAl?$AAb?$AAa?$AAc?$AAk?$AA?$AA@ 1003136c     SwiNotify.obj
 0002:0000b38c       ??_C@_1BK@DECJBJPB@?$AAU?$AAS?$AAS?$AAD?$AAC?$AAa?$AAl?$AAl?$AAb?$AAa?$AAc?$AAk?$AA?$AA@ 1003138c     SwiNotify.obj
 0002:0000b3a8       ??_C@_1BM@BEAJPNBG@?$AAb?$AA4?$AA?5?$AAd?$AAu?$AAm?$AAp?$AA?5?$AAp?$AAU?$AAS?$AAS?$AAD?$AA?$AA@ 100313a8     SwiNotify.obj
 0002:0000b3c4       ??_C@_1DK@ICEDHDGB@?$AAb?$AA4?$AA?5?$AAd?$AAu?$AAm?$AAp?$AA?5?$AAs?$AAN?$AAo?$AAt?$AAi?$AAf?$AAy?$AAV?$AAa?$AAr?$AAi?$AAa?$AAn?$AAt?$AA?4?$AA_?$AAU?$AAS?$AAS?$AAD?$AA?$AA@ 100313c4     SwiNotify.obj
 0002:0000b400       ??_C@_1DC@GDIOLDDG@?$AAR?$AAe?$AAa?$AAd?$AAS?$AAI?$AAM?$AAP?$AAh?$AAo?$AAn?$AAe?$AAB?$AAo?$AAo?$AAk?$AAC?$AAa?$AAl?$AAl?$AAb?$AAa?$AAc?$AAk?$AA?$AA@ 10031400     SwiNotify.obj
 0002:0000b434       ??_C@_1BO@MEBMCJHM@?$AAN?$AAU?$AAL?$AAL?$AA?5?$AAP?$AAo?$AAi?$AAn?$AAt?$AAe?$AAr?$AA?$CB?$AA?$CB?$AA?$AA@ 10031434     SwiNotify.obj
 0002:0000b458       ??_C@_1GK@ECHOMPNI@?$AAS?$AAI?$AAM?$AA?5?$AAr?$AAe?$AAc?$AAo?$AAr?$AAd?$AA?5?$AAi?$AAd?$AA?5?$AA?$DN?$AA?5?$AA?$CF?$AAd?$AA?0?$AA?5?$AAt?$AAy?$AAp?$AAe?$AA?$DN?$AA?$CF?$AAd?$AA?0?$AA?5?$AAN?$AAu?$AAm@ 10031458     SwiNotify.obj
 0002:0000b4c8       ??_C@_1EA@JDGCJENP@?$AAA?$AAl?$AAl?$AAS?$AAI?$AAM?$AAP?$AAh?$AAo?$AAn?$AAe?$AAb?$AAo?$AAo?$AAk?$AAI?$AAn?$AAi?$AAt?$AAD?$AAo?$AAn?$AAe?$AAC?$AAa?$AAl?$AAl?$AAb?$AAa?$AAc?$AAk?$AA?$AA@ 100314c8     SwiNotify.obj
 0002:0000b508       ??_C@_1MA@DGJKNJFP@?$AAE?$AAm?$AAe?$AAr?$AAg?$AAe?$AAn?$AAc?$AAy?$AAL?$AAi?$AAs?$AAt?$AAC?$AAa?$AAl?$AAl?$AAb?$AAa?$AAc?$AAk?$AA?3?$AA?5?$AAn?$AAo?$AAO?$AAf?$AAI?$AAn?$AAs?$AAt?$AAa@ 10031508     SwiNotify.obj
 0002:0000b5c8       ??_C@_1IM@JENBIICK@?$AAE?$AAm?$AAe?$AAr?$AAg?$AAe?$AAn?$AAc?$AAy?$AAL?$AAi?$AAs?$AAt?$AAC?$AAa?$AAl?$AAl?$AAb?$AAa?$AAc?$AAk?$AA?3?$AA?5?$AAn?$AAo?$AAO?$AAf?$AAI?$AAn?$AAs?$AAt?$AAa@ 100315c8     SwiNotify.obj
 0002:0000b654       ??_C@_1DA@NDIKHLKN@?$AAE?$AAm?$AAe?$AAr?$AAg?$AAe?$AAn?$AAc?$AAy?$AA?5?$AAM?$AAo?$AAd?$AAe?$AA?5?$AAC?$AAa?$AAl?$AAl?$AAb?$AAa?$AAc?$AAk?$AA?$AA@ 10031654     SwiNotify.obj
 0002:0000b688       ??_C@_1II@PJNJPLA@?$AAG?$AAo?$AAb?$AAi?$AA?5?$AAS?$AAM?$AAS?$AA?5?$AAC?$AAA?$AAL?$AAL?$AAB?$AAA?$AAC?$AAK?$AA?5?$AAR?$AAe?$AAc?$AAe?$AAi?$AAv?$AAe?$AAd?$AA?0?$AA?5?$AAs?$AAt?$AAo?$AAr@ 10031688     SwiNotify.obj
 0002:0000b710       ??_C@_1FO@HIHBNAMO@?$AAG?$AAo?$AAb?$AAi?$AA?5?$AAS?$AAM?$AAS?$AA?5?$AAC?$AAA?$AAL?$AAL?$AAB?$AAA?$AAC?$AAK?$AA?5?$AAR?$AAe?$AAc?$AAe?$AAi?$AAv?$AAe?$AAd?$AA?0?$AA?5?$AAs?$AAt?$AAo?$AAr@ 10031710     SwiNotify.obj
 0002:0000b770       ??_C@_1CK@BJJGDKKL@?$AAV?$AAo?$AAi?$AAc?$AAe?$AAM?$AAe?$AAs?$AAs?$AAa?$AAg?$AAe?$AAC?$AAa?$AAl?$AAl?$AAb?$AAa?$AAc?$AAk?$AA?$AA@ 10031770     SwiNotify.obj
 0002:0000b7a0       ??_C@_1FG@CHIFKBHL@?$AAV?$AAo?$AAi?$AAc?$AAe?$AAM?$AAe?$AAs?$AAs?$AAa?$AAg?$AAe?$AAC?$AAa?$AAl?$AAl?$AAb?$AAa?$AAc?$AAk?$AA?5?$AAw?$AAi?$AAt?$AAh?$AA?5?$AAN?$AAU?$AAL?$AAL?$AA?5?$AAp@ 100317a0     SwiNotify.obj
 0002:0000b7f8       ??_C@_1FA@FEJBGKMC@?$AAA?$AAS?$AAS?$AAE?$AAR?$AAT?$AAI?$AAO?$AAN?$AA?5?$AAF?$AAA?$AAI?$AAL?$AAU?$AAR?$AAE?$AA?3?$AA?5?$AA?$DN?$AA?$DN?$AA?$DN?$AA?$DO?$AAg?$AA_?$AAs?$AAe?$AAs?$AAs?$AAi?$AAo?$AAn@ 100317f8     SwiNotify.obj
 0002:0000b848       ??_C@_1JO@MBKALBHM@?$AAS?$AAw?$AAi?$AAN?$AAo?$AAt?$AAi?$AAf?$AAy?$AA?5?$AA?$DN?$AA?5?$AA?$CF?$AAd?$AA?5?$AAh?$AAa?$AAs?$AA?5?$AAn?$AAe?$AAv?$AAe?$AAr?$AA?5?$AAb?$AAe?$AAe?$AAn?$AA?5?$AAe?$AAn@ 10031848     SwiNotify.obj
 0002:0000b8e8       ??_C@_1GO@GHBCAKOF@?$AAA?$AAS?$AAS?$AAE?$AAR?$AAT?$AAI?$AAO?$AAN?$AA?5?$AAF?$AAA?$AAI?$AAL?$AAU?$AAR?$AAE?$AA?3?$AA?5?$AA?$DN?$AA?$DN?$AA?$DN?$AA?$DO?$AAb?$AAL?$AAa?$AAs?$AAt?$AAC?$AAo?$AAu?$AAn@ 100318e8     SwiNotify.obj
 0002:0000b958       ??_C@_1EI@NMMEPNJO@?$AAS?$AAe?$AAt?$AAN?$AAI?$AAT?$AAZ?$AAC?$AAB?$AA?5?$AAe?$AAn?$AAa?$AAb?$AAl?$AAe?$AAd?$AA?0?$AA?5?$AAs?$AAe?$AAt?$AAC?$AAB?$AAR?$AAe?$AAs?$AAu?$AAl?$AAt?$AA?5?$AA?$DN@ 10031958     SwiNotify.obj
 0002:0000b9a0       ??_C@_1FK@NOFJBMIG@?$AAS?$AAe?$AAt?$AAE?$AAm?$AAe?$AAr?$AAg?$AAe?$AAn?$AAc?$AAy?$AAM?$AAo?$AAd?$AAe?$AAC?$AAB?$AA?5?$AAe?$AAn?$AAa?$AAb?$AAl?$AAe?$AAd?$AA?0?$AA?5?$AAs?$AAe?$AAt?$AAC@ 100319a0     SwiNotify.obj
 0002:0000ba00       ??_C@_1FK@PJIJJPIL@?$AAS?$AAe?$AAt?$AAA?$AAl?$AAl?$AAP?$AAb?$AAI?$AAn?$AAi?$AAt?$AAD?$AAo?$AAn?$AAe?$AAC?$AAB?$AA?5?$AAe?$AAn?$AAa?$AAb?$AAl?$AAe?$AAd?$AA?0?$AA?5?$AAs?$AAe?$AAt?$AAC@ 10031a00     SwiNotify.obj
 0002:0000ba60       ??_C@_1GG@MDGECNJN@?$AAS?$AAe?$AAt?$AAP?$AAh?$AAo?$AAn?$AAe?$AAb?$AAo?$AAo?$AAk?$AAR?$AAe?$AAc?$AAo?$AAr?$AAd?$AAR?$AAe?$AAa?$AAd?$AAC?$AAB?$AA?5?$AAe?$AAn?$AAa?$AAb?$AAl?$AAe?$AAd@ 10031a60     SwiNotify.obj
 0002:0000bac8       ??_C@_1FC@EGHJOMJH@?$AAS?$AAe?$AAt?$AAN?$AAe?$AAw?$AAS?$AAM?$AAS?$AAC?$AAB?$AAC?$AAB?$AA?5?$AAf?$AAa?$AAi?$AAl?$AAe?$AAd?$AA?0?$AA?5?$AAs?$AAe?$AAt?$AAC?$AAB?$AAR?$AAe?$AAs?$AAu?$AAl@ 10031ac8     SwiNotify.obj
 0002:0000bb20       ??_C@_1EO@HJKFOFD@?$AAS?$AAe?$AAt?$AAN?$AAe?$AAw?$AAS?$AAM?$AAS?$AAC?$AAB?$AA?5?$AAf?$AAa?$AAi?$AAl?$AAe?$AAd?$AA?0?$AA?5?$AAs?$AAe?$AAt?$AAC?$AAB?$AAR?$AAe?$AAs?$AAu?$AAl?$AAt?$AA?5@ 10031b20     SwiNotify.obj
 0002:0000bb70       ??_C@_1FK@MDFOODMB@?$AAS?$AAe?$AAt?$AAV?$AAo?$AAi?$AAc?$AAe?$AAM?$AAe?$AAs?$AAs?$AAa?$AAg?$AAe?$AAC?$AAB?$AA?5?$AAf?$AAa?$AAi?$AAl?$AAe?$AAd?$AA?0?$AA?5?$AAs?$AAe?$AAt?$AAC?$AAB?$AAR@ 10031b70     SwiNotify.obj
 0002:0000bbd0       ??_C@_1FM@BKOCBMLK@?$AAS?$AAe?$AAt?$AAE?$AAm?$AAe?$AAr?$AAg?$AAe?$AAn?$AAc?$AAy?$AAL?$AAi?$AAs?$AAt?$AAC?$AAB?$AA?5?$AAf?$AAa?$AAi?$AAl?$AAe?$AAd?$AA?0?$AA?5?$AAs?$AAe?$AAt?$AAC?$AAB@ 10031bd0     SwiNotify.obj
 0002:0000bc30       ??_C@_1GK@CLBONFLA@?$AAS?$AAe?$AAt?$AAS?$AAe?$AAs?$AAs?$AAi?$AAo?$AAn?$AAS?$AAt?$AAa?$AAt?$AAe?$AAC?$AAB?$AA?5?$AAf?$AAo?$AAr?$AA?5?$AAa?$AAN?$AAo?$AAt?$AAi?$AAf?$AAy?$AA?5?$AA?$DN?$AA?5@ 10031c30     SwiNotify.obj
 0002:0000bca0       ??_C@_1HI@GGNFLLKG@?$AAS?$AAW?$AAI?$AA_?$AAN?$AAO?$AAT?$AAI?$AAF?$AAY?$AA_?$AAC?$AAa?$AAl?$AAl?$AAN?$AAo?$AAt?$AAi?$AAf?$AAi?$AAc?$AAa?$AAt?$AAi?$AAo?$AAn?$AAS?$AAt?$AAa?$AAt?$AAu@ 10031ca0     SwiNotify.obj
 0002:0000bd18       ??_C@_1FE@IBLGJFOF@?$AAS?$AAe?$AAt?$AAO?$AAM?$AAA?$AAE?$AAX?$AAE?$AAv?$AAe?$AAn?$AAt?$AAC?$AAB?$AA?5?$AAe?$AAn?$AAa?$AAb?$AAl?$AAe?$AAd?$AA?0?$AA?5?$AAs?$AAe?$AAt?$AAC?$AAB?$AAR?$AAe@ 10031d18     SwiNotify.obj
 0002:0000bd70       ??_C@_1EC@DEMNNGPP@?$AAS?$AAW?$AAI?$AA_?$AAN?$AAO?$AAT?$AAI?$AAF?$AAY?$AA?5?$AA?$DN?$AA?5?$AA?$CF?$AAd?$AA?5?$AAi?$AAs?$AA?5?$AAN?$AAO?$AAT?$AA?5?$AAs?$AAu?$AAp?$AAp?$AAo?$AAr?$AAt?$AAe?$AAd@ 10031d70     SwiNotify.obj
 0002:0000bdb8       ??_C@_1IO@HAPBEGKP@?$AAC?$AAS?$AAw?$AAi?$AAN?$AAo?$AAt?$AAi?$AAf?$AAy?$AA?3?$AA?3?$AAR?$AAe?$AAm?$AAo?$AAv?$AAe?$AA?5?$AAS?$AAe?$AAt?$AAP?$AAh?$AAo?$AAn?$AAe?$AAb?$AAo?$AAo?$AAk?$AAR@ 10031db8     SwiNotify.obj
 0002:0000be48       ??_C@_1IC@IJLDIBNJ@?$AAC?$AAS?$AAw?$AAi?$AAN?$AAo?$AAt?$AAi?$AAf?$AAy?$AA?3?$AA?3?$AAR?$AAe?$AAm?$AAo?$AAv?$AAe?$AA?5?$AAS?$AAe?$AAt?$AAA?$AAl?$AAl?$AAP?$AAb?$AAI?$AAn?$AAi?$AAt?$AAD@ 10031e48     SwiNotify.obj
 0002:0000bed0       ??_C@_1HI@IBFCDNKN@?$AAC?$AAS?$AAw?$AAi?$AAN?$AAo?$AAt?$AAi?$AAf?$AAy?$AA?3?$AA?3?$AAR?$AAe?$AAm?$AAo?$AAv?$AAe?$AA?5?$AAS?$AAe?$AAt?$AAN?$AAe?$AAw?$AAS?$AAM?$AAS?$AAC?$AAB?$AAC?$AAB@ 10031ed0     SwiNotify.obj
 0002:0000bf48       ??_C@_1IA@OMLJGFLL@?$AAC?$AAS?$AAw?$AAi?$AAN?$AAo?$AAt?$AAi?$AAf?$AAy?$AA?3?$AA?3?$AAR?$AAe?$AAm?$AAo?$AAv?$AAe?$AA?5?$AAS?$AAe?$AAt?$AAV?$AAo?$AAi?$AAc?$AAe?$AAM?$AAe?$AAs?$AAs?$AAa@ 10031f48     SwiNotify.obj
 0002:0000bfc8       ??_C@_1HE@KOPDLOC@?$AAC?$AAS?$AAw?$AAi?$AAN?$AAo?$AAt?$AAi?$AAf?$AAy?$AA?3?$AA?3?$AAR?$AAe?$AAm?$AAo?$AAv?$AAe?$AA?5?$AAS?$AAe?$AAt?$AAN?$AAe?$AAw?$AAS?$AAM?$AAS?$AAC?$AAB?$AA?5?$AAf@ 10031fc8     SwiNotify.obj
 0002:0000c040       ??_C@_1IC@BEEDGJJJ@?$AAC?$AAa?$AAl?$AAl?$AAb?$AAa?$AAc?$AAk?$AAL?$AAi?$AAs?$AAt?$AA?5?$AAo?$AAf?$AA?5?$AAn?$AAo?$AAt?$AAi?$AAf?$AAi?$AAc?$AAa?$AAt?$AAi?$AAo?$AAn?$AA?5?$AAi?$AAs?$AA?5@ 10032040     SwiNotify.obj
 0002:0000c0c4       ??_C@_1DE@KMKICGHM@?$AAm?$AA_?$AAp?$AAG?$AAo?$AAb?$AAi?$AA?5?$AAi?$AAs?$AA?5?$AAN?$AAU?$AAL?$AAL?$AA?4?$AA?5?$AAR?$AAE?$AAT?$AAU?$AAR?$AAN?$AA?$CB?$AA?$CB?$AA?$AA@ 100320c4     SwiNotify.obj
 0002:0000c0f8       ??_C@_1HO@LKGDDIMM@?$AAA?$AAS?$AAS?$AAE?$AAR?$AAT?$AAI?$AAO?$AAN?$AA?5?$AAF?$AAA?$AAI?$AAL?$AAU?$AAR?$AAE?$AA?3?$AA?5?$AA?$DN?$AA?$DN?$AA?$DN?$AA?$DO?$AAg?$AA_?$AAD?$AAa?$AAt?$AAa?$AAC?$AAa?$AAp@ 100320f8     SwiNotify.obj
 0002:0000c178       ??_C@_1FE@IPEGAMEK@?$AAG?$AAe?$AAt?$AAS?$AAe?$AAr?$AAv?$AAi?$AAn?$AAg?$AAN?$AAe?$AAt?$AAw?$AAo?$AAr?$AAk?$AAC?$AAa?$AAp?$AAs?$AA?5?$AAr?$AAe?$AAt?$AAu?$AAr?$AAn?$AAs?$AA?5?$AAs?$AAt@ 10032178     SwiNotify.obj
 0002:0000c1d0       ??_C@_1LO@JDCBBKHC@?$AAR?$AAe?$AAc?$AAe?$AAi?$AAv?$AAe?$AAd?$AA?5?$AAr?$AAa?$AAd?$AAi?$AAo?$AAI?$AAn?$AAt?$AAe?$AAr?$AAf?$AAa?$AAc?$AAe?$AA?5?$AA?$DN?$AA?5?$AA?$CF?$AAd?$AA?0?$AA?5?$AAS?$AAS@ 100321d0     SwiNotify.obj
 0002:0000c290       ??_C@_1BI@CBJPPGGF@?$AAG?$AAo?$AAb?$AAi?$AA?5?$AAN?$AAu?$AAm?$AAb?$AAe?$AAr?$AA?$AA@ 10032290     SwiNotify.obj
 0002:0000c2a8       ??_C@_1FI@ONNGIGOK@?$AAR?$AAI?$AAC?$AAB?$AA?3?$AA?5?$AAG?$AAe?$AAt?$AAS?$AAe?$AAr?$AAv?$AAi?$AAn?$AAg?$AAN?$AAe?$AAt?$AAw?$AAo?$AAr?$AAk?$AA?5?$AAf?$AAa?$AAi?$AAl?$AAe?$AAd?$AA?0?$AA?5@ 100322a8     SwiNotify.obj
 0002:0000c300       ??_C@_1IE@DDOLPIPG@?$AAF?$AAa?$AAi?$AAl?$AA?5?$AAt?$AAo?$AA?5?$AAd?$AAi?$AAs?$AAa?$AAb?$AAl?$AAe?$AA?5?$AAc?$AAa?$AAl?$AAl?$AAb?$AAa?$AAc?$AAk?$AA?5?$AAf?$AAo?$AAr?$AA?5?$AAt?$AAh?$AAe@ 10032300     SwiNotify.obj
 0002:0000c384       ??_C@_0BB@MOGOBHAF@list?$DMT?$DO?5too?5long?$AA@ 10032384     SwiNotify.obj
 0002:0000c398       ??_C@_1BG@FEAIPEDD@?$AA?4?$AA?2?$AAu?$AAt?$AAi?$AAl?$AA?4?$AAc?$AAp?$AAp?$AA?$AA@ 10032398     util.obj
 0002:0000c3b0       ??_C@_1FA@NLCMAGGI@?$AAA?$AAS?$AAS?$AAE?$AAR?$AAT?$AAI?$AAO?$AAN?$AA?5?$AAF?$AAA?$AAI?$AAL?$AAU?$AAR?$AAE?$AA?3?$AA?5?$AA?$DN?$AA?$DN?$AA?$DN?$AA?$DO?$AA0?$AAx?$AA1?$AA0?$AA?5?$AA?$DO?$AA?5?$AAb?$AAS@ 100323b0     util.obj
 0002:0000c400       ??_C@_1FA@BAEIDPMH@?$AAA?$AAS?$AAS?$AAE?$AAR?$AAT?$AAI?$AAO?$AAN?$AA?5?$AAF?$AAA?$AAI?$AAL?$AAU?$AAR?$AAE?$AA?3?$AA?5?$AA?$DN?$AA?$DN?$AA?$DN?$AA?$DO?$AAN?$AAU?$AAL?$AAL?$AA?5?$AA?$CB?$AA?$DN?$AA?5?$AAs@ 10032400     util.obj
 0002:0000c450       ??_C@_1FC@JMMKGCOD@?$AAA?$AAS?$AAS?$AAE?$AAR?$AAT?$AAI?$AAO?$AAN?$AA?5?$AAF?$AAA?$AAI?$AAL?$AAU?$AAR?$AAE?$AA?3?$AA?5?$AA?$DN?$AA?$DN?$AA?$DN?$AA?$DO?$AAN?$AAU?$AAL?$AAL?$AA?5?$AA?$CB?$AA?$DN?$AA?5?$AAs@ 10032450     util.obj
 0002:0000c4a8       ??_C@_1HI@CCJJJII@?$AAA?$AAS?$AAS?$AAE?$AAR?$AAT?$AAI?$AAO?$AAN?$AA?5?$AAF?$AAA?$AAI?$AAL?$AAU?$AAR?$AAE?$AA?3?$AA?5?$AA?$DN?$AA?$DN?$AA?$DN?$AA?$DO?$AAc?$AAb?$AAC?$AAm?$AAd?$AA?5?$AA?$DO?$AA?$DN?$AA?5@ 100324a8     util.obj
 0002:0000c520       ??_C@_1KK@HDNBDLCH@?$AAA?$AAS?$AAS?$AAE?$AAR?$AAT?$AAI?$AAO?$AAN?$AA?5?$AAF?$AAA?$AAI?$AAL?$AAU?$AAR?$AAE?$AA?3?$AA?5?$AA?$DN?$AA?$DN?$AA?$DN?$AA?$DO?$AAp?$AAr?$AAg?$AAr?$AAD?$AAa?$AAt?$AAa?$AA?5@ 10032520     util.obj
 0002:0000c5d0       ??_C@_1FC@OJNKDJBH@?$AA?9?$AA?9?$AA?9?$AA?9?$AA?9?$AA?9?$AA?9?$AA?9?$AA?9?$AA?9?$AA?9?$AA?9?$AA?9?$AA?9?$AA?9?$AA?9?$AA?9?$AA?9?$AA?9?$AA?9?$AA?9?$AA?9?$AA?9?$AA?9?$AA?9?$AA?9?$AA?9?$AA?9?$AA?9?$AA?9?$AA?9?$AA?9@ 100325d0     util.obj
 0002:0000c624       ??_C@_1CM@HPIFCGNF@?$AAd?$AAu?$AAm?$AAp?$AAi?$AAn?$AAg?$AA?5?$AA0?$AAx?$AA?$CF?$AAx?$AA?5?$AA?$CF?$AAd?$AA?5?$AAb?$AAy?$AAt?$AAe?$AAs?$AA?$AA@ 10032624     util.obj
 0002:0000c650       ??_C@_1KI@OKJGOAHE@?$AA?$CF?$AA4?$AAx?$AA?3?$AA?5?$AA?$CF?$AA2?$AAx?$AA?0?$AA?5?$AA?$CF?$AA2?$AAx?$AA?0?$AA?5?$AA?$CF?$AA2?$AAx?$AA?0?$AA?5?$AA?$CF?$AA2?$AAx?$AA?0?$AA?5?$AA?$CF?$AA2?$AAx?$AA?0?$AA?5?$AA?$CF?$AA2@ 10032650     util.obj
 0002:0000c6f8       ??_C@_1JO@GODFMKGC@?$AA?$CF?$AA4?$AAx?$AA?3?$AA?5?$AA?$CF?$AA2?$AAx?$AA?0?$AA?5?$AA?$CF?$AA2?$AAx?$AA?0?$AA?5?$AA?$CF?$AA2?$AAx?$AA?0?$AA?5?$AA?$CF?$AA2?$AAx?$AA?0?$AA?5?$AA?$CF?$AA2?$AAx?$AA?0?$AA?5?$AA?$CF?$AA2@ 100326f8     util.obj
 0002:0000c798       ??_C@_1JE@CEJEFJOI@?$AA?$CF?$AA4?$AAx?$AA?3?$AA?5?$AA?$CF?$AA2?$AAx?$AA?0?$AA?5?$AA?$CF?$AA2?$AAx?$AA?0?$AA?5?$AA?$CF?$AA2?$AAx?$AA?0?$AA?5?$AA?$CF?$AA2?$AAx?$AA?0?$AA?5?$AA?$CF?$AA2?$AAx?$AA?0?$AA?5?$AA?$CF?$AA2@ 10032798     util.obj
 0002:0000c830       ??_C@_1IK@HCKKAFBG@?$AA?$CF?$AA4?$AAx?$AA?3?$AA?5?$AA?$CF?$AA2?$AAx?$AA?0?$AA?5?$AA?$CF?$AA2?$AAx?$AA?0?$AA?5?$AA?$CF?$AA2?$AAx?$AA?0?$AA?5?$AA?$CF?$AA2?$AAx?$AA?0?$AA?5?$AA?$CF?$AA2?$AAx?$AA?0?$AA?5?$AA?$CF?$AA2@ 10032830     util.obj
 0002:0000c8c0       ??_C@_1IA@FJDLOKKO@?$AA?$CF?$AA4?$AAx?$AA?3?$AA?5?$AA?$CF?$AA2?$AAx?$AA?0?$AA?5?$AA?$CF?$AA2?$AAx?$AA?0?$AA?5?$AA?$CF?$AA2?$AAx?$AA?0?$AA?5?$AA?$CF?$AA2?$AAx?$AA?0?$AA?5?$AA?$CF?$AA2?$AAx?$AA?0?$AA?5?$AA?$CF?$AA2@ 100328c0     util.obj
 0002:0000c940       ??_C@_1HG@EKODKFIL@?$AA?$CF?$AA4?$AAx?$AA?3?$AA?5?$AA?$CF?$AA2?$AAx?$AA?0?$AA?5?$AA?$CF?$AA2?$AAx?$AA?0?$AA?5?$AA?$CF?$AA2?$AAx?$AA?0?$AA?5?$AA?$CF?$AA2?$AAx?$AA?0?$AA?5?$AA?$CF?$AA2?$AAx?$AA?0?$AA?5?$AA?$CF?$AA2@ 10032940     util.obj
 0002:0000c9b8       ??_C@_1GM@JBCNBELM@?$AA?$CF?$AA4?$AAx?$AA?3?$AA?5?$AA?$CF?$AA2?$AAx?$AA?0?$AA?5?$AA?$CF?$AA2?$AAx?$AA?0?$AA?5?$AA?$CF?$AA2?$AAx?$AA?0?$AA?5?$AA?$CF?$AA2?$AAx?$AA?0?$AA?5?$AA?$CF?$AA2?$AAx?$AA?0?$AA?5?$AA?$CF?$AA2@ 100329b8     util.obj
 0002:0000ca28       ??_C@_1GC@HEMALIIH@?$AA?$CF?$AA4?$AAx?$AA?3?$AA?5?$AA?$CF?$AA2?$AAx?$AA?0?$AA?5?$AA?$CF?$AA2?$AAx?$AA?0?$AA?5?$AA?$CF?$AA2?$AAx?$AA?0?$AA?5?$AA?$CF?$AA2?$AAx?$AA?0?$AA?5?$AA?$CF?$AA2?$AAx?$AA?0?$AA?5?$AA?$CF?$AA2@ 10032a28     util.obj
 0002:0000ca90       ??_C@_1FI@GAMHCDJP@?$AA?$CF?$AA4?$AAx?$AA?3?$AA?5?$AA?$CF?$AA2?$AAx?$AA?0?$AA?5?$AA?$CF?$AA2?$AAx?$AA?0?$AA?5?$AA?$CF?$AA2?$AAx?$AA?0?$AA?5?$AA?$CF?$AA2?$AAx?$AA?0?$AA?5?$AA?$CF?$AA2?$AAx?$AA?0?$AA?5?$AA?$CF?$AA2@ 10032a90     util.obj
 0002:0000cae8       ??_C@_1EO@HNCMBCJC@?$AA?$CF?$AA4?$AAx?$AA?3?$AA?5?$AA?$CF?$AA2?$AAx?$AA?0?$AA?5?$AA?$CF?$AA2?$AAx?$AA?0?$AA?5?$AA?$CF?$AA2?$AAx?$AA?0?$AA?5?$AA?$CF?$AA2?$AAx?$AA?0?$AA?5?$AA?$CF?$AA2?$AAx?$AA?0?$AA?5?$AA?$CF?$AA2@ 10032ae8     util.obj
 0002:0000cb38       ??_C@_1EE@GLGEACLC@?$AA?$CF?$AA4?$AAx?$AA?3?$AA?5?$AA?$CF?$AA2?$AAx?$AA?0?$AA?5?$AA?$CF?$AA2?$AAx?$AA?0?$AA?5?$AA?$CF?$AA2?$AAx?$AA?0?$AA?5?$AA?$CF?$AA2?$AAx?$AA?0?$AA?5?$AA?$CF?$AA2?$AAx?$AA?0?$AA?5?$AA?$CF?$AA2@ 10032b38     util.obj
 0002:0000cb7c       ??_C@_1DK@JHILCJLD@?$AA?$CF?$AA4?$AAx?$AA?3?$AA?5?$AA?$CF?$AA2?$AAx?$AA?0?$AA?5?$AA?$CF?$AA2?$AAx?$AA?0?$AA?5?$AA?$CF?$AA2?$AAx?$AA?0?$AA?5?$AA?$CF?$AA2?$AAx?$AA?0?$AA?5?$AA?$CF?$AA2?$AAx?$AA?$AA@ 10032b7c     util.obj
 0002:0000cbb8       ??_C@_1DA@HMAJKJAB@?$AA?$CF?$AA4?$AAx?$AA?3?$AA?5?$AA?$CF?$AA2?$AAx?$AA?0?$AA?5?$AA?$CF?$AA2?$AAx?$AA?0?$AA?5?$AA?$CF?$AA2?$AAx?$AA?0?$AA?5?$AA?$CF?$AA2?$AAx?$AA?$AA@ 10032bb8     util.obj
 0002:0000cbe8       ??_C@_1CG@MKENLECL@?$AA?$CF?$AA4?$AAx?$AA?3?$AA?5?$AA?$CF?$AA2?$AAx?$AA?0?$AA?5?$AA?$CF?$AA2?$AAx?$AA?0?$AA?5?$AA?$CF?$AA2?$AAx?$AA?$AA@ 10032be8     util.obj
 0002:0000cc10       ??_C@_1BM@IKFBLMOH@?$AA?$CF?$AA4?$AAx?$AA?3?$AA?5?$AA?$CF?$AA2?$AAx?$AA?0?$AA?5?$AA?$CF?$AA2?$AAx?$AA?$AA@ 10032c10     util.obj
 0002:0000cc2c       ??_C@_1BC@DKKLNCCA@?$AA?$CF?$AA4?$AAx?$AA?3?$AA?5?$AA?$CF?$AA2?$AAx?$AA?$AA@ 10032c2c     util.obj
 0002:0000d26c       ??_R4bad_alloc@std@@6B@    1003326c     libcpmt:string.obj
 0002:0000d280       ??_R3bad_alloc@std@@8      10033280     libcpmt:string.obj
 0002:0000d290       ??_R2bad_alloc@std@@8      10033290     libcpmt:string.obj
 0002:0000d29c       ??_R1A@?0A@EA@bad_alloc@std@@8 1003329c     libcpmt:string.obj
 0002:0000d2b8       ??_R1A@?0A@EA@exception@std@@8 100332b8     libcpmt:string.obj
 0002:0000d2d4       ??_R3exception@std@@8      100332d4     libcpmt:string.obj
 0002:0000d2e4       ??_R2exception@std@@8      100332e4     libcpmt:string.obj
 0002:0000d2ec       ??_R4logic_error@std@@6B@  100332ec     libcpmt:string.obj
 0002:0000d300       ??_R3logic_error@std@@8    10033300     libcpmt:string.obj
 0002:0000d310       ??_R2logic_error@std@@8    10033310     libcpmt:string.obj
 0002:0000d31c       ??_R1A@?0A@EA@logic_error@std@@8 1003331c     libcpmt:string.obj
 0002:0000d338       ??_R4length_error@std@@6B@ 10033338     libcpmt:string.obj
 0002:0000d34c       ??_R3length_error@std@@8   1003334c     libcpmt:string.obj
 0002:0000d35c       ??_R2length_error@std@@8   1003335c     libcpmt:string.obj
 0002:0000d36c       ??_R1A@?0A@EA@length_error@std@@8 1003336c     libcpmt:string.obj
 0002:0000d388       ??_R4out_of_range@std@@6B@ 10033388     libcpmt:string.obj
 0002:0000d39c       ??_R3out_of_range@std@@8   1003339c     libcpmt:string.obj
 0002:0000d3ac       ??_R2out_of_range@std@@8   100333ac     libcpmt:string.obj
 0002:0000d3bc       ??_R1A@?0A@EA@out_of_range@std@@8 100333bc     libcpmt:string.obj
 0002:0000d468       _TI3?AVout_of_range@std@@  10033468     libcpmt:string.obj
 0002:0000d478       _CTA3?AVout_of_range@std@@ 10033478     libcpmt:string.obj
 0002:0000d488       _CT??_R0?AVout_of_range@std@@@8??0out_of_range@std@@QAA@ABV01@@Z40 10033488     libcpmt:string.obj
 0002:0000d4a4       _CT??_R0?AVlength_error@std@@@8??0length_error@std@@QAA@ABV01@@Z40 100334a4     SwiNotify.obj
 0002:0000d4c0       _CT??_R0?AVlogic_error@std@@@8??0logic_error@std@@QAA@ABV01@@Z40 100334c0     SwiNotify.obj
 0002:0000d4dc       _CT??_R0?AVexception@std@@@8??0exception@std@@QAA@ABV01@@Z12 100334dc     SwiNotify.obj
 0002:0000d4f8       _CTA3?AVlength_error@std@@ 100334f8     SwiNotify.obj
 0002:0000d508       _TI3?AVlength_error@std@@  10033508     SwiNotify.obj
 0002:0000d518       _CT??_R0?AVbad_alloc@std@@@8??0bad_alloc@std@@QAA@ABV01@@Z12 10033518     SwiNotify.obj
 0002:0000d534       _CTA2?AVbad_alloc@std@@    10033534     SwiNotify.obj
 0002:0000d540       _TI2?AVbad_alloc@std@@     10033540     SwiNotify.obj
 0002:0000d550       __IMPORT_DESCRIPTOR_WS2    10033550     ws2:WS2.dll
 0002:0000d564       __IMPORT_DESCRIPTOR_sw_utilityG 10033564     sw_utilityG:sw_utilityG.dll
 0002:0000d578       __IMPORT_DESCRIPTOR_COREDLL 10033578     coredll:COREDLL.dll
 0002:0000d58c       __NULL_IMPORT_DESCRIPTOR   1003358c     ccoreutl:ccoreutl.dll
 0003:00000000       __imp_??_7type_info@@6B@   1003a000     coredll:COREDLL.dll
 0003:00000004       __imp_wcscat               1003a004     coredll:COREDLL.dll
 0003:00000008       __imp_strcat               1003a008     coredll:COREDLL.dll
 0003:0000000c       __imp_strcpy               1003a00c     coredll:COREDLL.dll
 0003:00000010       __imp_InterlockedCompareExchange 1003a010     coredll:COREDLL.dll
 0003:00000014       __imp_TlsGetValue          1003a014     coredll:COREDLL.dll
 0003:00000018       __imp_TlsSetValue          1003a018     coredll:COREDLL.dll
 0003:0000001c       __imp_TlsCall              1003a01c     coredll:COREDLL.dll
 0003:00000020       __imp_?terminate@std@@YAXXZ 1003a020     coredll:COREDLL.dll
 0003:00000024       __imp_strcmp               1003a024     coredll:COREDLL.dll
 0003:00000028       __imp___CxxThrowException  1003a028     coredll:COREDLL.dll
 0003:0000002c       __imp___rt_udiv            1003a02c     coredll:COREDLL.dll
 0003:00000030       __imp_RaiseException       1003a030     coredll:COREDLL.dll
 0003:00000034       __imp_memset               1003a034     coredll:COREDLL.dll
 0003:00000038       __imp_strspn               1003a038     coredll:COREDLL.dll
 0003:0000003c       __imp_??3@YAXPAX@Z         1003a03c     coredll:COREDLL.dll
 0003:00000040       __imp_strstr               1003a040     coredll:COREDLL.dll
 0003:00000044       __imp_LocalAlloc           1003a044     coredll:COREDLL.dll
 0003:00000048       __imp_LocalFree            1003a048     coredll:COREDLL.dll
 0003:0000004c       __imp_strchr               1003a04c     coredll:COREDLL.dll
 0003:00000050       __imp_??2@YAPAXI@Z         1003a050     coredll:COREDLL.dll
 0003:00000054       __imp_InitializeCriticalSection 1003a054     coredll:COREDLL.dll
 0003:00000058       __imp_DeleteCriticalSection 1003a058     coredll:COREDLL.dll
 0003:0000005c       __imp_EnterCriticalSection 1003a05c     coredll:COREDLL.dll
 0003:00000060       __imp_LeaveCriticalSection 1003a060     coredll:COREDLL.dll
 0003:00000064       __imp_NKDbgPrintfW         1003a064     coredll:COREDLL.dll
 0003:00000068       __imp_swscanf              1003a068     coredll:COREDLL.dll
 0003:0000006c       __imp_GetLastError         1003a06c     coredll:COREDLL.dll
 0003:00000070       __imp__snprintf            1003a070     coredll:COREDLL.dll
 0003:00000074       __imp_??_U@YAPAXI@Z        1003a074     coredll:COREDLL.dll
 0003:00000078       __imp_??_V@YAXPAX@Z        1003a078     coredll:COREDLL.dll
 0003:0000007c       __imp_sscanf               1003a07c     coredll:COREDLL.dll
 0003:00000080       __imp_malloc               1003a080     coredll:COREDLL.dll
 0003:00000084       __imp_free                 1003a084     coredll:COREDLL.dll
 0003:00000088       __imp_CloseHandle          1003a088     coredll:COREDLL.dll
 0003:0000008c       __imp_CreateThread         1003a08c     coredll:COREDLL.dll
 0003:00000090       __imp_wcsstr               1003a090     coredll:COREDLL.dll
 0003:00000094       __imp_Sleep                1003a094     coredll:COREDLL.dll
 0003:00000098       __imp_strtoul              1003a098     coredll:COREDLL.dll
 0003:0000009c       __imp_MultiByteToWideChar  1003a09c     coredll:COREDLL.dll
 0003:000000a0       __imp_sprintf              1003a0a0     coredll:COREDLL.dll
 0003:000000a4       __imp_atol                 1003a0a4     coredll:COREDLL.dll
 0003:000000a8       __imp_swprintf             1003a0a8     coredll:COREDLL.dll
 0003:000000ac       __imp__wtol                1003a0ac     coredll:COREDLL.dll
 0003:000000b0       __imp_CreateFileW          1003a0b0     coredll:COREDLL.dll
 0003:000000b4       __imp_SetLastError         1003a0b4     coredll:COREDLL.dll
 0003:000000b8       __imp_GetCommState         1003a0b8     coredll:COREDLL.dll
 0003:000000bc       __imp_SetCommTimeouts      1003a0bc     coredll:COREDLL.dll
 0003:000000c0       __imp_SetupComm            1003a0c0     coredll:COREDLL.dll
 0003:000000c4       __imp_toupper              1003a0c4     coredll:COREDLL.dll
 0003:000000c8       __imp_SetCommState         1003a0c8     coredll:COREDLL.dll
 0003:000000cc       __imp_PurgeComm            1003a0cc     coredll:COREDLL.dll
 0003:000000d0       __imp_GetTickCount         1003a0d0     coredll:COREDLL.dll
 0003:000000d4       __imp_ReadFile             1003a0d4     coredll:COREDLL.dll
 0003:000000d8       __imp_WriteFile            1003a0d8     coredll:COREDLL.dll
 0003:000000dc       __imp_GetProcAddressW      1003a0dc     coredll:COREDLL.dll
 0003:000000e0       __imp_FreeLibrary          1003a0e0     coredll:COREDLL.dll
 0003:000000e4       __imp_LoadLibraryW         1003a0e4     coredll:COREDLL.dll
 0003:000000e8       __imp_??1exception@std@@UAA@XZ 1003a0e8     coredll:COREDLL.dll
 0003:000000ec       __imp_??0exception@std@@QAA@PBD@Z 1003a0ec     coredll:COREDLL.dll
 0003:000000f0       __imp_??0exception@std@@QAA@XZ 1003a0f0     coredll:COREDLL.dll
 0003:000000f4       __imp___rt_udiv64by64      1003a0f4     coredll:COREDLL.dll
 0003:000000f8       __imp_??0exception@std@@QAA@ABV01@@Z 1003a0f8     coredll:COREDLL.dll
 0003:000000fc       __imp_?what@exception@std@@UBAPBDXZ 1003a0fc     coredll:COREDLL.dll
 0003:00000100       __imp___report_gsfailure   1003a100     coredll:COREDLL.dll
 0003:00000104       __imp_LocalReAlloc         1003a104     coredll:COREDLL.dll
 0003:00000108       __imp_LocalSize            1003a108     coredll:COREDLL.dll
 0003:0000010c       __imp___security_gen_cookie 1003a10c     coredll:COREDLL.dll
 0003:00000110       __imp_wcsncpy              1003a110     coredll:COREDLL.dll
 0003:00000114       __imp_wcslen               1003a114     coredll:COREDLL.dll
 0003:00000118       __imp_strncpy              1003a118     coredll:COREDLL.dll
 0003:0000011c       __imp_strlen               1003a11c     coredll:COREDLL.dll
 0003:00000120       __imp_wcscpy               1003a120     coredll:COREDLL.dll
 0003:00000124       __imp___C_specific_handler 1003a124     coredll:COREDLL.dll
 0003:00000128       __imp_memmove              1003a128     coredll:COREDLL.dll
 0003:0000012c       __imp_memcpy               1003a12c     coredll:COREDLL.dll
 0003:00000130       __imp_wcscmp               1003a130     coredll:COREDLL.dll
 0003:00000134       \177COREDLL_NULL_THUNK_DATA 1003a134     coredll:COREDLL.dll
 0003:00000138       __imp_ntohl                1003a138     ws2:WS2.dll
 0003:0000013c       __imp_inet_ntoa            1003a13c     ws2:WS2.dll
 0003:00000140       \177WS2_NULL_THUNK_DATA    1003a140     ws2:WS2.dll
 0003:00000144       __imp_?TBD_Output@@YAXW4TBD_CLASS_TYPE@@W4TBD_OUTPUT_LEVEL@@QBGZZ 1003a144     sw_utilityG:sw_utilityG.dll
 0003:00000148       __imp_?LogStoreFileLine@@YAXPAGH@Z 1003a148     sw_utilityG:sw_utilityG.dll
 0003:0000014c       __imp_?TBD_Assert@@YA_N_NQBG1H@Z 1003a14c     sw_utilityG:sw_utilityG.dll
 0003:00000150       __imp_?SW_AtoT@@YAPAGPAGPADK@Z 1003a150     sw_utilityG:sw_utilityG.dll
 0003:00000154       __imp_?SW_TtoA@@YAPADPADPAGK@Z 1003a154     sw_utilityG:sw_utilityG.dll
 0003:00000158       __imp_?DisplayRawData@@YAXIPAEHPBG@Z 1003a158     sw_utilityG:sw_utilityG.dll
 0003:0000015c       __imp_?LogC@@YAXPBGZZ      1003a15c     sw_utilityG:sw_utilityG.dll
 0003:00000160       __imp_?GetRegValue@@YAJPAUHKEY__@@PBG1PAGPAK@Z 1003a160     sw_utilityG:sw_utilityG.dll
 0003:00000164       \177sw_utilityG_NULL_THUNK_DATA 1003a164     sw_utilityG:sw_utilityG.dll
 0003:00000168       __xc_a                     1003a168     corelibc:crt0init.obj
 0003:00000180       __xc_z                     1003a180     corelibc:crt0init.obj
 0003:00000184       __xi_a                     1003a184     corelibc:crt0init.obj
 0003:00000188       __xi_z                     1003a188     corelibc:crt0init.obj
 0003:0000018c       __xp_a                     1003a18c     corelibc:crt0init.obj
 0003:00000190       __xp_z                     1003a190     corelibc:crt0init.obj
 0003:00000194       __xt_a                     1003a194     corelibc:crt0init.obj
 0003:00000198       __xt_z                     1003a198     corelibc:crt0init.obj
 0003:000001a0       __security_cookie_complement 1003a1a0     corelibc:seccook.obj
 0003:000001a4       __security_cookie          1003a1a4     corelibc:seccook.obj
 0003:000001ac       ??_R0?AVout_of_range@std@@@8 1003a1ac     libcpmt:string.obj
 0003:000001d4       ?g_CB_SignalStrength@@3CA  1003a1d4     SwiNotify.obj
 0003:000001d8       ?g_iCdmaRssi@@3HA          1003a1d8     SwiNotify.obj
 0003:000001dc       ?g_iCdmaEcio@@3HA          1003a1dc     SwiNotify.obj
 0003:000001e0       ?g_iHdrRssi@@3HA           1003a1e0     SwiNotify.obj
 0003:000001e4       ?g_iHdrEcio@@3HA           1003a1e4     SwiNotify.obj
 0003:000001e8       ?GOBI2SWIOTASPState@@3PAW4SWI_TYPE_OTASPState@@A 1003a1e8     SwiNotify.obj
 0003:00000588       ?errGobiAPI@@3PAW4SWI_RCODE@@A 1003a588     SwiError.obj
 0003:00000600       ?errGobiModule1@@3PAW4SWI_RCODE@@A 1003a600     SwiError.obj
 0003:0000074c       ?errGobiModule2@@3PAW4SWI_RCODE@@A 1003a74c     SwiError.obj
 0003:00000760       ?GOBI2SWIPowerMode@@3PAW4SWI_TYPE_Power@@A 1003a760     SwiError.obj
 0003:00000784       ?GOBI2SWIRoam@@3PAGA       1003a784     SDKRILCdma.obj
 0003:00000790       ?GOBI2SWICDMACarrierID@@3PAW4SWI_TYPE_CarrierID@@A 1003a790     SDKRILCdma.obj
 0003:000007d8       ?GOBI2SWICDMACarrierName@@3PAPAGA 1003a7d8     SDKRILCdma.obj
 0003:00000820       ?SWI2GOBIOMADMSessionType@@3PAJA 1003a820     SDKRILCdma.obj
 0003:00000838       ?g_ATPortInstance@@3VCSwiATPort@@A 1003a838     SDKRIL.obj
 0003:00000a84       ?theSWICR@@3VCriticalSection@@A 1003aa84     SDKRIL.obj
 0003:00000a9c       ??_R0?AVlength_error@std@@@8 1003aa9c     SwiNotify.obj
 0003:00000abc       ??_R0?AVlogic_error@std@@@8 1003aabc     SwiNotify.obj
 0003:00000adc       ??_R0?AVexception@std@@@8  1003aadc     SwiNotify.obj
 0003:00000af8       ??_R0?AVbad_alloc@std@@@8  1003aaf8     SwiNotify.obj
 0003:00000b18       ?g_MSLSet@@3UMSLData@@A    1003ab18     SDKRILCdma.obj
 0003:00000b5c       ?g_SPCStr@@3PADA           1003ab5c     SDKRILCdma.obj
 0003:00000b68       ?g_msgListArray@@3PAUMSG_LIST_ENTRY@@A 1003ab68     SDKRILCdma.obj
 0003:00002aa8       ?g_StoreRawSms@@3USWI_STRUCT_RawSms@@A 1003caa8     SDKRILCdma.obj
 0003:00002eb8       ?g_sAirServerList@@3USWI_STRUCT_AirServerList@@A 1003ceb8     SDKRILGsm.obj
 0003:000032a8       ?g_RATInfoList@@3URATINFOList@@A 1003d2a8     SDKRILGsm.obj
 0003:0000343c       __@@_PchSym_@00@UluurxzoPyfrowUirotlyrUdrmwldhLnlyrovLGLkiluvhhrlmzoLhwpLSzineErTUivovzhvPdnGOFUhwpiroUhgwzucOlyq@ 1003d43c     stdafx.obj
 0003:00003440       ?g_PlmnList@@3UNWINFOList@@A 1003d440     SDKRILGsm.obj
 0003:00006a2c       ?g_WirelessTech@@3W4SWI_TYPE_WirelessTech@@A 10040a2c     SDKRIL.obj
 0003:00006a30       ?g_IsRUIM@@3EA             10040a30     SDKRIL.obj
 0003:00006a31       ?g_bSCM@@3EA               10040a31     SDKRILCdma.obj
 0003:00006a32       ?g_bSCI@@3EA               10040a32     SDKRILCdma.obj
 0003:00006a33       ?g_bRegHomeSID@@3EA        10040a33     SDKRILCdma.obj
 0003:00006a34       ?g_NotifyCallback@@3P6AXPAUSwiNotifyVariant@@@ZA 10040a34     SDKRIL.obj
 0003:00006a38       ?g_StrFirmwareVersion@@3PADA 10040a38     SDKRIL.obj
 0003:00006a8d       ?g_bRegForSID@@3EA         10040a8d     SDKRILCdma.obj
 0003:00006a8e       ?g_bRegForNID@@3EA         10040a8e     SDKRILCdma.obj
 0003:00006a8f       ?g_bForceRev0@@3EA         10040a8f     SDKRILCdma.obj
 0003:00006a90       ?g_StrBootVersion@@3PADA   10040a90     SDKRIL.obj
 0003:00006ae5       ?g_bCustomSCP@@3EA         10040ae5     SDKRILCdma.obj
 0003:00006ae8       ?g_StrPRIVersion@@3PADA    10040ae8     SDKRIL.obj
 0003:00006b40       ?g_bIsCMEErrNumeric@@3HA   10040b40     SDKRIL.obj
 0003:00006b44       ?g_hSmsSendNotifyThread@@3PAXA 10040b44     SDKRILCdma.obj
 0003:00006b48       ?g_DataSessionID@@3KA      10040b48     SDKRILCdma.obj
 0003:00006b4c       ?g_OMADMPRLsessionID@@3GA  10040b4c     SDKRILCdma.obj
 0003:00006b50       ?g_OMADMDCsessionID@@3GA   10040b50     SDKRILCdma.obj
 0003:00006b54       ?g_ulProtocol@@3KA         10040b54     SDKRILCdma.obj
 0003:00006b58       ?g_ulBroadCast@@3KA        10040b58     SDKRILCdma.obj
 0003:00006b5c       ?g_ulApp@@3KA              10040b5c     SDKRILCdma.obj
 0003:00006b60       ?g_ulRoaming@@3KA          10040b60     SDKRILCdma.obj
 0003:00006b64       ?g_PlmnMode@@3W4SWI_TYPE_PLMN_Mode@@A 10040b64     SDKRILGsm.obj
 0003:00006b68       ?g_ulDataSessionId@@3KA    10040b68     SDKRILGsm.obj
 0003:00006b6c       ?g_GsmSmsSource@@3KA       10040b6c     SDKRILGsm.obj
 0003:00006b70       ?g_GsmPinType@@3KA         10040b70     SDKRILGsm.obj
 0003:00006b74       ?mpFNSetSessionStateCB@CSwiGobiDll@@1P6AKP6AXKK@Z@ZA 10040b74     SwiGobiDll.obj
 0003:00006b78       ?mpFNSetDataBearerCB@CSwiGobiDll@@1P6AKP6AXK@Z@ZA 10040b78     SwiGobiDll.obj
 0003:00006b7c       ?mpFNSetDormancyStatusCB@CSwiGobiDll@@1P6AKP6AXK@Z@ZA 10040b7c     SwiGobiDll.obj
 0003:00006b80       ?mpFNSetMobileIPStatusCB@CSwiGobiDll@@1P6AKP6AXK@Z@ZA 10040b80     SwiGobiDll.obj
 0003:00006b84       ?mpFNSetActivationStatusCB@CSwiGobiDll@@1P6AKP6AXK@Z@ZA 10040b84     SwiGobiDll.obj
 0003:00006b88       ?mpFNSetPowerCB@CSwiGobiDll@@1P6AKP6AXK@Z@ZA 10040b88     SwiGobiDll.obj
 0003:00006b8c       ?mpFNSetRoamingIndicatorCB@CSwiGobiDll@@1P6AKP6AXK@Z@ZA 10040b8c     SwiGobiDll.obj
 0003:00006b90       ?mpFNSetSignalStrengthCB@CSwiGobiDll@@1P6AKP6AXCK@ZEPAC@ZA 10040b90     SwiGobiDll.obj
 0003:00006b94       ?mpFNSetRFInfoCB@CSwiGobiDll@@1P6AKP6AXKKK@Z@ZA 10040b94     SwiGobiDll.obj
 0003:00006b98       ?mpFNSetNewSMSCB@CSwiGobiDll@@1P6AKP6AXKK@Z@ZA 10040b98     SwiGobiDll.obj
 0003:00006b9c       ?mpFNSetNewSMSCBCB@CSwiGobiDll@@1P6AKP6AXEKEGPAE@Z@ZA 10040b9c     SwiGobiDll.obj
 0003:00006ba0       ?mpFNSetVoiceMsgCB@CSwiGobiDll@@1P6AKP6AXEPAE00@Z@ZA 10040ba0     SwiGobiDll.obj
 0003:00006ba4       ?mpFNSetDataCapabilitiesCB@CSwiGobiDll@@1P6AKP6AXEPAE@Z@ZA 10040ba4     SwiGobiDll.obj
 0003:00006ba8       ?mpFNSetByteTotalsCB@CSwiGobiDll@@1P6AKP6AX_K0@ZE@ZA 10040ba8     SwiGobiDll.obj
 0003:00006bac       ?mpFNSetOMADMStateCB@CSwiGobiDll@@1P6AKP6AXKK@Z@ZA 10040bac     SwiGobiDll.obj
 0003:00006bb0       ?mpFNSetOMADMNIAlertCB@CSwiGobiDll@@1P6AKP6AXKG@Z@ZA 10040bb0     SwiGobiDll.obj
 0003:00006bb4       ?mpFNSetCallInfoCB@CSwiGobiDll@@1P6AKP6AXPAUarrCallInfo@@PAUarrRemotePartyNum@@PAUarrRemotePartyName@@PAUarrAlertingType@@PAUarrSvcOption@@PAUarrCallEndReason@@PAUarrAlphaIDInfo@@PAUarrPeerNumInfo@@PAUarrDiagInfo@@77PAUarrAlertingPattern@@@Z@ZA 10040bb4     SwiGobiDll.obj
 0003:00006bb8       ?mpFNSetInfoRecCB@CSwiGobiDll@@1P6AKP6AXPAEPAUsignalInfo@@PAUcallerIDInfo@@PAD330PAUpeerNumInfo@@44PAUredirectNumInfo@@0000PAUlineCtlInfo@@PAUextDisplayInfo@@@Z@ZA 10040bb8     SwiGobiDll.obj
 0003:00006bbc       ?mpFNSetUSSDInfoCB@CSwiGobiDll@@1P6AKP6AXPAEPAUUSSInfo@@@Z@ZA 10040bbc     SwiGobiDll.obj
 0003:00006bc0       ?mpFNSetPhonebookRecordReadCB@CSwiGobiDll@@1P6AKP6AXEGPAUarrPBInfo@@@Z@ZA 10040bc0     SwiGobiDll.obj
 0003:00006bc4       ?mpFNSetAllPbInitDoneCB@CSwiGobiDll@@1P6AKP6AXEPAEPAG@Z@ZA 10040bc4     SwiGobiDll.obj
 0003:00006bc8       ?mpFNSetEmergencyListCB@CSwiGobiDll@@1P6AKP6AXEPAUemergencyNumberEntry@@@Z@ZA 10040bc8     SwiGobiDll.obj
 0003:00006bcc       ?mpFNSetNITZCB@CSwiGobiDll@@1P6AKP6AXGEEEEEEEE@Z@ZA 10040bcc     SwiGobiDll.obj
 0003:00006bd0       ?mpFNSetEmergencyModeCB@CSwiGobiDll@@1P6AKP6AXPAE@Z@ZA 10040bd0     SwiGobiDll.obj
 0003:00006bd4       ?mpFNSetOMAEXEventCB@CSwiGobiDll@@1P6AKP6AXPAUFUMOInfo@@PAUOMAInfo@@@Z@ZA 10040bd4     SwiGobiDll.obj
 0003:00006bd8       ?m_NotifyCallback@CSwiNotify@@2P6AXPAUSwiNotifyVariant@@@ZA 10040bd8     SwiNotify.obj
 0003:00006bdc       ?m_pGobi@CSwiNotify@@0PAVCSwiGobiDll@@A 10040bdc     SwiNotify.obj
 0003:00006be0       ?m_pSwiNotify@CSwiNotify@@0PAV1@A 10040be0     SwiNotify.obj
 0003:00006be4       ?g_CB_RadioInterface@@3KA  10040be4     SwiNotify.obj
 0003:00006be8       ?g_DataCapsMask@@3W4eDataCaps@@A 10040be8     SwiNotify.obj
 0003:00006bec       ?g_OMADMsessionType@@3KA   10040bec     SwiNotify.obj
 0003:00006bf0       ?g_sessionID@@3GA          10040bf0     SwiNotify.obj
 0003:00006bf8       ?g_GobiInstance@@3VCSwiGobiDll@@A 10040bf8     SDKRIL.obj
 0003:00006f20       ?g_Notify@@3VCSwiNotify@@A 10040f20     SDKRIL.obj
 0003:00006f30       __onexitend                10040f30     <common>
 0003:00006f34       __onexitbegin              10040f34     <common>
 0003:00006f38       _exitflag                  10040f38     <common>
 0003:00006f3c       _pRawDllMain               10040f3c     <common>

 entry point at        0001:0002214c

 Static symbols

 0001:0001b708       __unwind$85781             1001c708 f i  CIL library: CIL module
 0001:0001c890       __unwind$85685             1001d890 f    CIL library: CIL module
 0001:0001c918       __unwind$85629             1001d918 f    CIL library: CIL module
 0001:0001c9dc       __unwind$85573             1001d9dc f    CIL library: CIL module
 0001:0001caa0       __unwind$85517             1001daa0 f    CIL library: CIL module
 0001:0001cb80       __unwind$85447             1001db80 f    CIL library: CIL module
 0001:0001cc48       __unwind$85380             1001dc48 f    CIL library: CIL module
 0001:0001d0e8       __unwind$85321             1001e0e8 f    CIL library: CIL module
 0001:0001d24c       __unwind$85233             1001e24c f    CIL library: CIL module
 0001:0001d2cc       __unwind$85178             1001e2cc f    CIL library: CIL module
 0001:0001d3f4       __unwind$87877             1001e3f4 f    CIL library: CIL module
 0001:0001da28       __unwind$91100             1001ea28 f    CIL library: CIL module
 0001:0001da38       __unwind$91101             1001ea38 f    CIL library: CIL module
 0001:0001da48       __unwind$91482             1001ea48 f    CIL library: CIL module
 0001:00020b24       __unwind$89606             10021b24 f i  CIL library: CIL module
 0001:00020d74       __catch$90510              10021d74 f i  CIL library: CIL module
 0001:00020d8c       __unwind$90610             10021d8c f i  CIL library: CIL module
 0001:00020e24       __unwind$86198             10021e24 f i  CIL library: CIL module
 0001:00020f68       __catch$80162              10021f68 f i  CIL library: CIL module
 0001:00020f94       __catch$80160              10021f94 f i  CIL library: CIL module
 0001:000211b0       __catch$90083              100221b0 f i  CIL library: CIL module
 0001:000212c4       __catch$89894              100222c4 f i  CIL library: CIL module
 0001:00022250       doexit                     10023250 f   corelibc:crt0dat.obj
 0001:00022bf0       __unwind$17778             10023bf0 f   libcpmt:string.obj
 0001:00022c80       __unwind$17968             10023c80 f   libcpmt:string.obj
 0001:00022f04       ?CanThisExceptionObjectBeDestructed@@YAEPAUEHExceptionRecord@@E@Z 10023f04 f   LIBCMT:frame_ce.obj
 0001:00023250       ?CallCatchBlock@@YAPAXPAUEHExceptionRecord@@PAKPAU_CONTEXT@@PBU_s_FuncInfo@@PAXHK@Z 10024250 f   LIBCMT:frame_ce.obj
 0001:000235e8       ?BuildCatchObject@@YAXPAUEHExceptionRecord@@PAKPBU_s_HandlerType@@PBU_s_CatchableType@@@Z 100245e8 f   LIBCMT:frame_ce.obj
 0001:000237bc       ?FindHandler@@YAEPAUEHExceptionRecord@@PAKPAU_CONTEXT@@PAU_DISPATCHER_CONTEXT@@PBU_s_FuncInfo@@H@Z 100247bc f   LIBCMT:frame_ce.obj
 0001:0002413c       ??__Eg_GobiInstance@@YAXXZ 1002513c f    CIL library: CIL module
 0001:0002415c       ??__Eg_ATPortInstance@@YAXXZ 1002515c f    CIL library: CIL module
 0001:00024168       ??__Eg_Notify@@YAXXZ       10025168 f    CIL library: CIL module
 0001:000241bc       ??__EtheSWICR@@YAXXZ       100251bc f    CIL library: CIL module
 0001:000241e0       ??__Fg_GobiInstance@@YAXXZ 100251e0 f    CIL library: CIL module
 0001:000241ec       ??__Fg_ATPortInstance@@YAXXZ 100251ec f    CIL library: CIL module
 0001:00024258       ??__Fg_Notify@@YAXXZ       10025258 f    CIL library: CIL module
 0001:0002427c       __unwind$93674             1002527c f    CIL library: CIL module
 0001:00024290       ??__FtheSWICR@@YAXXZ       10025290 f    CIL library: CIL module

 Exports

  ordinal    name

        1    ??0CSwiGobiDll@@QAA@XZ (public: __cdecl CSwiGobiDll::CSwiGobiDll(void))
        2    ??1CSwiGobiDll@@QAA@XZ (public: __cdecl CSwiGobiDll::~CSwiGobiDll(void))
        3    ??4CSwiGobiDll@@QAAAAV0@ABV0@@Z (public: class CSwiGobiDll & __cdecl CSwiGobiDll::operator=(class CSwiGobiDll const &))
        4    ?ActivateAutomatic@CSwiGobiDll@@QAAKPAD@Z (public: unsigned long __cdecl CSwiGobiDll::ActivateAutomatic(char *))
        5    ?ActivateManual@CSwiGobiDll@@QAAKPADG00KPAE00@Z (public: unsigned long __cdecl CSwiGobiDll::ActivateManual(char *,unsigned short,char *,char *,unsigned long,unsigned char *,char *,char *))
        6    ?AnserCall@CSwiGobiDll@@QAAKPAE0@Z (public: unsigned long __cdecl CSwiGobiDll::AnserCall(unsigned char *,unsigned char *))
        7    ?AnswerUSSD@CSwiGobiDll@@QAAKPAUUSSInfo@@@Z (public: unsigned long __cdecl CSwiGobiDll::AnswerUSSD(struct USSInfo *))
        8    ?CancelUSSD@CSwiGobiDll@@QAAKXZ (public: unsigned long __cdecl CSwiGobiDll::CancelUSSD(void))
        9    ?ChangeBarringPwd@CSwiGobiDll@@QAAKPAUcallBarringPwd@@PAGPAUalphaIDInfo@@PAE3PAUccSUPSType@@@Z (public: unsigned long __cdecl CSwiGobiDll::ChangeBarringPwd(struct callBarringPwd *,unsigned short *,struct alphaIDInfo *,unsigned char *,unsigned char *,struct ccSUPSType *))
       10    ?Cleanup@CSwiGobiDll@@IAAXXZ (protected: void __cdecl CSwiGobiDll::Cleanup(void))
       11    ?Connect@CSwiGobiDll@@QAAKXZ (public: unsigned long __cdecl CSwiGobiDll::Connect(void))
       12    ?DMSUIMChangePIN@CSwiGobiDll@@QAAKKPAD0PAK1@Z (public: unsigned long __cdecl CSwiGobiDll::DMSUIMChangePIN(unsigned long,char *,char *,unsigned long *,unsigned long *))
       13    ?DMSUIMGetControlKeyStatus@CSwiGobiDll@@QAAKKPAK00@Z (public: unsigned long __cdecl CSwiGobiDll::DMSUIMGetControlKeyStatus(unsigned long,unsigned long *,unsigned long *,unsigned long *))
       14    ?DMSUIMGetICCID@CSwiGobiDll@@QAAKEPAD@Z (public: unsigned long __cdecl CSwiGobiDll::DMSUIMGetICCID(unsigned char,char *))
       15    ?DMSUIMGetPINStatus@CSwiGobiDll@@QAAKKPAK00@Z (public: unsigned long __cdecl CSwiGobiDll::DMSUIMGetPINStatus(unsigned long,unsigned long *,unsigned long *,unsigned long *))
       16    ?DMSUIMSetControlKeyProtection@CSwiGobiDll@@QAAKKKPADPAK@Z (public: unsigned long __cdecl CSwiGobiDll::DMSUIMSetControlKeyProtection(unsigned long,unsigned long,char *,unsigned long *))
       17    ?DMSUIMSetPINProtection@CSwiGobiDll@@QAAKKKPADPAK1@Z (public: unsigned long __cdecl CSwiGobiDll::DMSUIMSetPINProtection(unsigned long,unsigned long,char *,unsigned long *,unsigned long *))
       18    ?DMSUIMUnblockControlKey@CSwiGobiDll@@QAAKKPADPAK@Z (public: unsigned long __cdecl CSwiGobiDll::DMSUIMUnblockControlKey(unsigned long,char *,unsigned long *))
       19    ?DMSUIMUnblockPIN@CSwiGobiDll@@QAAKKPAD0PAK1@Z (public: unsigned long __cdecl CSwiGobiDll::DMSUIMUnblockPIN(unsigned long,char *,char *,unsigned long *,unsigned long *))
       20    ?DMSUIMVerifyPIN@CSwiGobiDll@@QAAKKPADPAK1@Z (public: unsigned long __cdecl CSwiGobiDll::DMSUIMVerifyPIN(unsigned long,char *,unsigned long *,unsigned long *))
       21    ?DeletePhonebookRecord@CSwiGobiDll@@QAAKPAEPAG1@Z (public: unsigned long __cdecl CSwiGobiDll::DeletePhonebookRecord(unsigned char *,unsigned short *,unsigned short *))
       22    ?DeleteSMS@CSwiGobiDll@@QAAKKPAK0@Z (public: unsigned long __cdecl CSwiGobiDll::DeleteSMS(unsigned long,unsigned long *,unsigned long *))
       23    ?DialCall@CSwiGobiDll@@QAAKPAUtDialReqParam@@PAEPAUalphaIDInfo@@1PAUccSUPSType@@@Z (public: unsigned long __cdecl CSwiGobiDll::DialCall(struct tDialReqParam *,unsigned char *,struct alphaIDInfo *,unsigned char *,struct ccSUPSType *))
       24    ?DisableCallbacks@CSwiGobiDll@@QAAXXZ (public: void __cdecl CSwiGobiDll::DisableCallbacks(void))
       25    ?Disconnect@CSwiGobiDll@@QAAKXZ (public: unsigned long __cdecl CSwiGobiDll::Disconnect(void))
       26    ?EndCall@CSwiGobiDll@@QAAKPAE0@Z (public: unsigned long __cdecl CSwiGobiDll::EndCall(unsigned char *,unsigned char *))
       27    ?ForceXTRADownload@CSwiGobiDll@@QAAKXZ (public: unsigned long __cdecl CSwiGobiDll::ForceXTRADownload(void))
       28    ?Get3Gpp2SubscriptionInfo@CSwiGobiDll@@QAAKPAEPAUMinBasedImsi@@PAUTrueImsi@@00@Z (public: unsigned long __cdecl CSwiGobiDll::Get3Gpp2SubscriptionInfo(unsigned char *,struct MinBasedImsi *,struct TrueImsi *,unsigned char *,unsigned char *))
       29    ?GetACCOLC@CSwiGobiDll@@QAAKPAE@Z (public: unsigned long __cdecl CSwiGobiDll::GetACCOLC(unsigned char *))
       30    ?GetAGPSConfig@CSwiGobiDll@@QAAKPAK0@Z (public: unsigned long __cdecl CSwiGobiDll::GetAGPSConfig(unsigned long *,unsigned long *))
       31    ?GetANAAAAuthenticationStatus@CSwiGobiDll@@QAAKPAK@Z (public: unsigned long __cdecl CSwiGobiDll::GetANAAAAuthenticationStatus(unsigned long *))
       32    ?GetActivationState@CSwiGobiDll@@QAAKPAK@Z (public: unsigned long __cdecl CSwiGobiDll::GetActivationState(unsigned long *))
       33    ?GetActiveMobileIPProfile@CSwiGobiDll@@QAAKPAE@Z (public: unsigned long __cdecl CSwiGobiDll::GetActiveMobileIPProfile(unsigned char *))
       34    ?GetAllCallInfo@CSwiGobiDll@@QAAKPAUarrCallInfo@@PAUarrRemotePartyNum@@PAUarrRemotePartyName@@PAUarrAlertingType@@PAUarrUUSInfo@@PAUarrSvcOption@@PAE6PAUarrCallEndReason@@PAUarrAlphaIDInfo@@PAUarrPeerNumInfo@@PAUarrDiagInfo@@99PAUarrAlertingPattern@@@Z (public: unsigned long __cdecl CSwiGobiDll::GetAllCallInfo(struct arrCallInfo *,struct arrRemotePartyNum *,struct arrRemotePartyName *,struct arrAlertingType *,struct arrUUSInfo *,struct arrSvcOption *,unsigned char *,unsigned char *,struct arrCallEndReason *,struct arrAlphaIDInfo *,struct arrPeerNumInfo *,struct arrDiagInfo *,struct arrPeerNumInfo *,struct arrPeerNumInfo *,struct arrAlertingPattern *))
       35    ?GetAudioProfile@CSwiGobiDll@@QAAKPAE@Z (public: unsigned long __cdecl CSwiGobiDll::GetAudioProfile(unsigned char *))
       36    ?GetAutoInputGain@CSwiGobiDll@@QAAKPAE@Z (public: unsigned long __cdecl CSwiGobiDll::GetAutoInputGain(unsigned char *))
       37    ?GetAutoOutputGain@CSwiGobiDll@@QAAKPAE@Z (public: unsigned long __cdecl CSwiGobiDll::GetAutoOutputGain(unsigned char *))
       38    ?GetAutoconnect@CSwiGobiDll@@QAAKPAK@Z (public: unsigned long __cdecl CSwiGobiDll::GetAutoconnect(unsigned long *))
       39    ?GetByteTotals@CSwiGobiDll@@QAAKPAK0@Z (public: unsigned long __cdecl CSwiGobiDll::GetByteTotals(unsigned long *,unsigned long *))
       40    ?GetCDMANetworkParameters@CSwiGobiDll@@QAAKPAE000000PAK111@Z (public: unsigned long __cdecl CSwiGobiDll::GetCDMANetworkParameters(unsigned char *,unsigned char *,unsigned char *,unsigned char *,unsigned char *,unsigned char *,unsigned char *,unsigned long *,unsigned long *,unsigned long *,unsigned long *))
       41    ?GetCLIR@CSwiGobiDll@@QAAKPAUstatusResp@@PAGPAUalphaIDInfo@@PAE3PAUccSUPSType@@@Z (public: unsigned long __cdecl CSwiGobiDll::GetCLIR(struct statusResp *,unsigned short *,struct alphaIDInfo *,unsigned char *,unsigned char *,struct ccSUPSType *))
       42    ?GetCallBarring@CSwiGobiDll@@QAAKPAE00PAGPAUalphaIDInfo@@00PAUccSUPSType@@@Z (public: unsigned long __cdecl CSwiGobiDll::GetCallBarring(unsigned char *,unsigned char *,unsigned char *,unsigned short *,struct alphaIDInfo *,unsigned char *,unsigned char *,struct ccSUPSType *))
       43    ?GetCallForwarding@CSwiGobiDll@@QAAKPAE0PAUgetCallFWInfo@@0PAUalphaIDInfo@@00PAUccSUPSType@@PAUgetExtCallFWInfo@@@Z (public: unsigned long __cdecl CSwiGobiDll::GetCallForwarding(unsigned char *,unsigned char *,struct getCallFWInfo *,unsigned char *,struct alphaIDInfo *,unsigned char *,unsigned char *,struct ccSUPSType *,struct getExtCallFWInfo *))
       44    ?GetCallWaiting@CSwiGobiDll@@QAAKPAE0PAGPAUalphaIDInfo@@00PAUccSUPSType@@@Z (public: unsigned long __cdecl CSwiGobiDll::GetCallWaiting(unsigned char *,unsigned char *,unsigned short *,struct alphaIDInfo *,unsigned char *,unsigned char *,struct ccSUPSType *))
       45    ?GetCellLocationInfo@CSwiGobiDll@@QAAKPAUgeranCellInfo@@PAUumtsCellInfo@@PAUcdmaCellInfo@@PAK@Z (public: unsigned long __cdecl CSwiGobiDll::GetCellLocationInfo(struct geranCellInfo *,struct umtsCellInfo *,struct cdmaCellInfo *,unsigned long *))
       46    ?GetConnectedDeviceID@CSwiGobiDll@@QAAKKPAD@Z (public: unsigned long __cdecl CSwiGobiDll::GetConnectedDeviceID(unsigned long,char *))
       47    ?GetConnectionRate@CSwiGobiDll@@QAAKPAK000@Z (public: unsigned long __cdecl CSwiGobiDll::GetConnectionRate(unsigned long *,unsigned long *,unsigned long *,unsigned long *))
       48    ?GetCwePkgsInfo@CSwiGobiDll@@QAAKPAGPAE010101010101@Z (public: unsigned long __cdecl CSwiGobiDll::GetCwePkgsInfo(unsigned short *,unsigned char *,unsigned short *,unsigned char *,unsigned short *,unsigned char *,unsigned short *,unsigned char *,unsigned short *,unsigned char *,unsigned short *,unsigned char *,unsigned short *,unsigned char *))
       49    ?GetDLLVersion@CSwiGobiDll@@QAAKXZ (public: unsigned long __cdecl CSwiGobiDll::GetDLLVersion(void))
       50    ?GetDataBearerTechnology@CSwiGobiDll@@QAAKPAK@Z (public: unsigned long __cdecl CSwiGobiDll::GetDataBearerTechnology(unsigned long *))
       51    ?GetDefaultProfile@CSwiGobiDll@@QAAKKPAK0000EPADE1E1@Z (public: unsigned long __cdecl CSwiGobiDll::GetDefaultProfile(unsigned long,unsigned long *,unsigned long *,unsigned long *,unsigned long *,unsigned long *,unsigned char,char *,unsigned char,char *,unsigned char,char *))
       52    ?GetDeviceCapabilities@CSwiGobiDll@@QAAKPAK0000PAE@Z (public: unsigned long __cdecl CSwiGobiDll::GetDeviceCapabilities(unsigned long *,unsigned long *,unsigned long *,unsigned long *,unsigned long *,unsigned char *))
       53    ?GetDormancyState@CSwiGobiDll@@QAAKPAK@Z (public: unsigned long __cdecl CSwiGobiDll::GetDormancyState(unsigned long *))
       54    ?GetDunCallInfo@CSwiGobiDll@@QAAKPAKPAE101111PA_KPAG221100002221@Z (public: unsigned long __cdecl CSwiGobiDll::GetDunCallInfo(unsigned long *,unsigned char *,unsigned char *,unsigned long *,unsigned char *,unsigned char *,unsigned char *,unsigned char *,unsigned __int64 *,unsigned short *,unsigned __int64 *,unsigned __int64 *,unsigned char *,unsigned char *,unsigned long *,unsigned long *,unsigned long *,unsigned long *,unsigned __int64 *,unsigned __int64 *,unsigned __int64 *,unsigned char *))
       55    ?GetERIFile@CSwiGobiDll@@QAAKPAKPAE@Z (public: unsigned long __cdecl CSwiGobiDll::GetERIFile(unsigned long *,unsigned char *))
       56    ?GetEchoCancelMode@CSwiGobiDll@@QAAKPAE@Z (public: unsigned long __cdecl CSwiGobiDll::GetEchoCancelMode(unsigned char *))
       57    ?GetFirmwareInfo@CSwiGobiDll@@QAAKPAK0000@Z (public: unsigned long __cdecl CSwiGobiDll::GetFirmwareInfo(unsigned long *,unsigned long *,unsigned long *,unsigned long *,unsigned long *))
       58    ?GetFirmwareRevision@CSwiGobiDll@@QAAKEPAD@Z (public: unsigned long __cdecl CSwiGobiDll::GetFirmwareRevision(unsigned char,char *))
       59    ?GetFirmwareRevisions@CSwiGobiDll@@QAAKEPADE0E0@Z (public: unsigned long __cdecl CSwiGobiDll::GetFirmwareRevisions(unsigned char,char *,unsigned char,char *,unsigned char,char *))
       60    ?GetHardwareRevision@CSwiGobiDll@@QAAKEPAD@Z (public: unsigned long __cdecl CSwiGobiDll::GetHardwareRevision(unsigned char,char *))
       61    ?GetHomeNetwork@CSwiGobiDll@@QAAKPAG0EPAD00@Z (public: unsigned long __cdecl CSwiGobiDll::GetHomeNetwork(unsigned short *,unsigned short *,unsigned char,char *,unsigned short *,unsigned short *))
       62    ?GetIMSI@CSwiGobiDll@@QAAKEPAD@Z (public: unsigned long __cdecl CSwiGobiDll::GetIMSI(unsigned char,char *))
       63    ?GetIPAddress@CSwiGobiDll@@QAAKPAK@Z (public: unsigned long __cdecl CSwiGobiDll::GetIPAddress(unsigned long *))
       64    ?GetIPConfiguration@CSwiGobiDll@@QAAKPAK0000@Z (public: unsigned long __cdecl CSwiGobiDll::GetIPConfiguration(unsigned long *,unsigned long *,unsigned long *,unsigned long *,unsigned long *))
       65    ?GetImageInfoW@CSwiGobiDll@@QAAKPBGPAK1111@Z (public: unsigned long __cdecl CSwiGobiDll::GetImageInfoW(unsigned short const *,unsigned long *,unsigned long *,unsigned long *,unsigned long *,unsigned long *))
       66    ?GetImagePreference@CSwiGobiDll@@QAAKPAKPAE@Z (public: unsigned long __cdecl CSwiGobiDll::GetImagePreference(unsigned long *,unsigned char *))
       67    ?GetImageStoreW@CSwiGobiDll@@QAAKGPAG@Z (public: unsigned long __cdecl CSwiGobiDll::GetImageStoreW(unsigned short,unsigned short *))
       68    ?GetLastMobileIPError@CSwiGobiDll@@QAAKPAK@Z (public: unsigned long __cdecl CSwiGobiDll::GetLastMobileIPError(unsigned long *))
       69    ?GetManufacturer@CSwiGobiDll@@QAAKEPAD@Z (public: unsigned long __cdecl CSwiGobiDll::GetManufacturer(unsigned char,char *))
       70    ?GetMicVolume@CSwiGobiDll@@QAAKPAG@Z (public: unsigned long __cdecl CSwiGobiDll::GetMicVolume(unsigned short *))
       71    ?GetMobileIP@CSwiGobiDll@@QAAKPAK@Z (public: unsigned long __cdecl CSwiGobiDll::GetMobileIP(unsigned long *))
       72    ?GetMobileIPParameters@CSwiGobiDll@@QAAKPAKPAE11111@Z (public: unsigned long __cdecl CSwiGobiDll::GetMobileIPParameters(unsigned long *,unsigned char *,unsigned char *,unsigned char *,unsigned char *,unsigned char *,unsigned char *))
       73    ?GetMobileIPProfile@CSwiGobiDll@@QAAKEPAEPAK110EPAD11@Z (public: unsigned long __cdecl CSwiGobiDll::GetMobileIPProfile(unsigned char,unsigned char *,unsigned long *,unsigned long *,unsigned long *,unsigned char *,unsigned char,char *,unsigned long *,unsigned long *))
       74    ?GetModelID@CSwiGobiDll@@QAAKEPAD@Z (public: unsigned long __cdecl CSwiGobiDll::GetModelID(unsigned char,char *))
       75    ?GetNMEAConfig@CSwiGobiDll@@QAAKPAE00PAG@Z (public: unsigned long __cdecl CSwiGobiDll::GetNMEAConfig(unsigned char *,unsigned char *,unsigned char *,unsigned short *))
       76    ?GetNetworkPreference@CSwiGobiDll@@QAAKPAK00@Z (public: unsigned long __cdecl CSwiGobiDll::GetNetworkPreference(unsigned long *,unsigned long *,unsigned long *))
       77    ?GetNetworkTime@CSwiGobiDll@@QAAKPA_KPAK@Z (public: unsigned long __cdecl CSwiGobiDll::GetNetworkTime(unsigned __int64 *,unsigned long *))
       78    ?GetNoiseSuppression@CSwiGobiDll@@QAAKPAE@Z (public: unsigned long __cdecl CSwiGobiDll::GetNoiseSuppression(unsigned char *))
       79    ?GetOfflineReason@CSwiGobiDll@@QAAKPAK0@Z (public: unsigned long __cdecl CSwiGobiDll::GetOfflineReason(unsigned long *,unsigned long *))
       80    ?GetPDSDefaults@CSwiGobiDll@@QAAKPAKPAE00@Z (public: unsigned long __cdecl CSwiGobiDll::GetPDSDefaults(unsigned long *,unsigned char *,unsigned long *,unsigned long *))
       81    ?GetPDSState@CSwiGobiDll@@QAAKPAK0@Z (public: unsigned long __cdecl CSwiGobiDll::GetPDSState(unsigned long *,unsigned long *))
       82    ?GetPRLVersion@CSwiGobiDll@@QAAKPAG@Z (public: unsigned long __cdecl CSwiGobiDll::GetPRLVersion(unsigned short *))
       83    ?GetPacketStatus@CSwiGobiDll@@QAAKPAK00000@Z (public: unsigned long __cdecl CSwiGobiDll::GetPacketStatus(unsigned long *,unsigned long *,unsigned long *,unsigned long *,unsigned long *,unsigned long *))
       84    ?GetPhonebookCapabilities@CSwiGobiDll@@QAAKPAEPAG1100@Z (public: unsigned long __cdecl CSwiGobiDll::GetPhonebookCapabilities(unsigned char *,unsigned short *,unsigned short *,unsigned short *,unsigned char *,unsigned char *))
       85    ?GetPortAutomaticTracking@CSwiGobiDll@@QAAKPAK@Z (public: unsigned long __cdecl CSwiGobiDll::GetPortAutomaticTracking(unsigned long *))
       86    ?GetPower@CSwiGobiDll@@QAAKPAK@Z (public: unsigned long __cdecl CSwiGobiDll::GetPower(unsigned long *))
       87    ?GetRFInfo@CSwiGobiDll@@QAAKPAE0@Z (public: unsigned long __cdecl CSwiGobiDll::GetRFInfo(unsigned char *,unsigned char *))
       88    ?GetRTREConfig@CSwiGobiDll@@QAAKPAE0@Z (public: unsigned long __cdecl CSwiGobiDll::GetRTREConfig(unsigned char *,unsigned char *))
       89    ?GetRXPCMFilter@CSwiGobiDll@@QAAKPAG0PAK0@Z (public: unsigned long __cdecl CSwiGobiDll::GetRXPCMFilter(unsigned short *,unsigned short *,unsigned long *,unsigned short *))
       90    ?GetSMS@CSwiGobiDll@@QAAKKKPAK00PAE@Z (public: unsigned long __cdecl CSwiGobiDll::GetSMS(unsigned long,unsigned long,unsigned long *,unsigned long *,unsigned long *,unsigned char *))
       91    ?GetSMSCAddress@CSwiGobiDll@@QAAKEPADE0@Z (public: unsigned long __cdecl CSwiGobiDll::GetSMSCAddress(unsigned char,char *,unsigned char,char *))
       92    ?GetSMSList@CSwiGobiDll@@QAAKKPAK0PAE@Z (public: unsigned long __cdecl CSwiGobiDll::GetSMSList(unsigned long,unsigned long *,unsigned long *,unsigned char *))
       93    ?GetSerialNumbers@CSwiGobiDll@@QAAKEPADE0E0@Z (public: unsigned long __cdecl CSwiGobiDll::GetSerialNumbers(unsigned char,char *,unsigned char,char *,unsigned char,char *))
       94    ?GetServiceAutomaticTracking@CSwiGobiDll@@QAAKPAK@Z (public: unsigned long __cdecl CSwiGobiDll::GetServiceAutomaticTracking(unsigned long *))
       95    ?GetServingNetwork@CSwiGobiDll@@QAAKPAK000PAE10PAG2EPAD@Z (public: unsigned long __cdecl CSwiGobiDll::GetServingNetwork(unsigned long *,unsigned long *,unsigned long *,unsigned long *,unsigned char *,unsigned char *,unsigned long *,unsigned short *,unsigned short *,unsigned char,char *))
       96    ?GetServingNetworkCaps@CSwiGobiDll@@QAAKPAE0@Z (public: unsigned long __cdecl CSwiGobiDll::GetServingNetworkCaps(unsigned char *,unsigned char *))
       97    ?GetSessionDuration@CSwiGobiDll@@QAAKPA_K@Z (public: unsigned long __cdecl CSwiGobiDll::GetSessionDuration(unsigned __int64 *))
       98    ?GetSessionState@CSwiGobiDll@@QAAKPAK@Z (public: unsigned long __cdecl CSwiGobiDll::GetSessionState(unsigned long *))
       99    ?GetSideToneGain@CSwiGobiDll@@QAAKPAG@Z (public: unsigned long __cdecl CSwiGobiDll::GetSideToneGain(unsigned short *))
      100    ?GetSignalStrengths@CSwiGobiDll@@QAAKPAKPAC0@Z (public: unsigned long __cdecl CSwiGobiDll::GetSignalStrengths(unsigned long *,signed char *,unsigned long *))
      101    ?GetTXPCMFilter@CSwiGobiDll@@QAAKPAG0PAK0@Z (public: unsigned long __cdecl CSwiGobiDll::GetTXPCMFilter(unsigned short *,unsigned short *,unsigned long *,unsigned short *))
      102    ?GetVoiceNumber@CSwiGobiDll@@QAAKEPADE0@Z (public: unsigned long __cdecl CSwiGobiDll::GetVoiceNumber(unsigned char,char *,unsigned char,char *))
      103    ?GetWaitingMessage@CSwiGobiDll@@QAAKPAUwaitingMsgInfo@@@Z (public: unsigned long __cdecl CSwiGobiDll::GetWaitingMessage(struct waitingMsgInfo *))
      104    ?GetWirelessTech@CSwiGobiDll@@QAA?AW4SWI_TYPE_WirelessTech@@XZ (public: enum SWI_TYPE_WirelessTech __cdecl CSwiGobiDll::GetWirelessTech(void))
      105    ?GetXTRAAutomaticDownload@CSwiGobiDll@@QAAKPAKPAG@Z (public: unsigned long __cdecl CSwiGobiDll::GetXTRAAutomaticDownload(unsigned long *,unsigned short *))
      106    ?GetXTRANetwork@CSwiGobiDll@@QAAKPAK@Z (public: unsigned long __cdecl CSwiGobiDll::GetXTRANetwork(unsigned long *))
      107    ?GetXTRAValidity@CSwiGobiDll@@QAAKPAG00@Z (public: unsigned long __cdecl CSwiGobiDll::GetXTRAValidity(unsigned short *,unsigned short *,unsigned short *))
      108    ?Initialize@CSwiGobiDll@@QAA_NXZ (public: bool __cdecl CSwiGobiDll::Initialize(void))
      109    ?InitiateDomainAttach@CSwiGobiDll@@QAAKK@Z (public: unsigned long __cdecl CSwiGobiDll::InitiateDomainAttach(unsigned long))
      110    ?InitiateNetworkRegistration@CSwiGobiDll@@QAAKKGGK@Z (public: unsigned long __cdecl CSwiGobiDll::InitiateNetworkRegistration(unsigned long,unsigned short,unsigned short,unsigned long))
      111    ?IsInitialized@CSwiGobiDll@@QAA_NXZ (public: bool __cdecl CSwiGobiDll::IsInitialized(void))
      112    ?ManageCalls@CSwiGobiDll@@QAAKPAE0PAG@Z (public: unsigned long __cdecl CSwiGobiDll::ManageCalls(unsigned char *,unsigned char *,unsigned short *))
      113    ?ModifySMSStatus@CSwiGobiDll@@QAAKKKK@Z (public: unsigned long __cdecl CSwiGobiDll::ModifySMSStatus(unsigned long,unsigned long,unsigned long))
      114    ?OMADMCancelSession@CSwiGobiDll@@QAAKXZ (public: unsigned long __cdecl CSwiGobiDll::OMADMCancelSession(void))
      115    ?OMADMGetFeatureSettings@CSwiGobiDll@@QAAKPAK0@Z (public: unsigned long __cdecl CSwiGobiDll::OMADMGetFeatureSettings(unsigned long *,unsigned long *))
      116    ?OMADMGetPendingNIA@CSwiGobiDll@@QAAKPAKPAG@Z (public: unsigned long __cdecl CSwiGobiDll::OMADMGetPendingNIA(unsigned long *,unsigned short *))
      117    ?OMADMGetSessionInfo@CSwiGobiDll@@QAAKPAK00PAEPAG2@Z (public: unsigned long __cdecl CSwiGobiDll::OMADMGetSessionInfo(unsigned long *,unsigned long *,unsigned long *,unsigned char *,unsigned short *,unsigned short *))
      118    ?OMADMSendSelection@CSwiGobiDll@@QAAKKG@Z (public: unsigned long __cdecl CSwiGobiDll::OMADMSendSelection(unsigned long,unsigned short))
      119    ?OMADMSetPRLUpdateFeature@CSwiGobiDll@@QAAKK@Z (public: unsigned long __cdecl CSwiGobiDll::OMADMSetPRLUpdateFeature(unsigned long))
      120    ?OMADMSetProvisioningFeature@CSwiGobiDll@@QAAKK@Z (public: unsigned long __cdecl CSwiGobiDll::OMADMSetProvisioningFeature(unsigned long))
      121    ?OMADMStartSession@CSwiGobiDll@@QAAKK@Z (public: unsigned long __cdecl CSwiGobiDll::OMADMStartSession(unsigned long))
      122    ?OMAEXGetSettings@CSwiGobiDll@@QAAKPAE00000@Z (public: unsigned long __cdecl CSwiGobiDll::OMAEXGetSettings(unsigned char *,unsigned char *,unsigned char *,unsigned char *,unsigned char *,unsigned char *))
      123    ?OMAEXInit@CSwiGobiDll@@QAAKXZ (public: unsigned long __cdecl CSwiGobiDll::OMAEXInit(void))
      124    ?OMAEXSelection@CSwiGobiDll@@QAAKPAE@Z (public: unsigned long __cdecl CSwiGobiDll::OMAEXSelection(unsigned char *))
      125    ?OMAEXSessionCancel@CSwiGobiDll@@QAAKXZ (public: unsigned long __cdecl CSwiGobiDll::OMAEXSessionCancel(void))
      126    ?OMAEXSessionGetInfo@CSwiGobiDll@@QAAKPAUomaSessionInfo@@@Z (public: unsigned long __cdecl CSwiGobiDll::OMAEXSessionGetInfo(struct omaSessionInfo *))
      127    ?OMAEXSessionStart@CSwiGobiDll@@QAAKPAE@Z (public: unsigned long __cdecl CSwiGobiDll::OMAEXSessionStart(unsigned char *))
      128    ?OMAEXSetEventReport@CSwiGobiDll@@QAAKXZ (public: unsigned long __cdecl CSwiGobiDll::OMAEXSetEventReport(void))
      129    ?OMAEXSetSettings@CSwiGobiDll@@QAAKPAE00000@Z (public: unsigned long __cdecl CSwiGobiDll::OMAEXSetSettings(unsigned char *,unsigned char *,unsigned char *,unsigned char *,unsigned char *,unsigned char *))
      130    ?OMAEXShutdown@CSwiGobiDll@@QAAKXZ (public: unsigned long __cdecl CSwiGobiDll::OMAEXShutdown(void))
      131    ?OrigUSSD@CSwiGobiDll@@QAAKPAUUSSInfo@@PAGPAUalphaIDInfo@@0PAE3PAUccSUPSType@@@Z (public: unsigned long __cdecl CSwiGobiDll::OrigUSSD(struct USSInfo *,unsigned short *,struct alphaIDInfo *,struct USSInfo *,unsigned char *,unsigned char *,struct ccSUPSType *))
      132    ?PDSInjectTimeReference@CSwiGobiDll@@QAAK_KG@Z (public: unsigned long __cdecl CSwiGobiDll::PDSInjectTimeReference(unsigned __int64,unsigned short))
      133    ?PerformNetworkRATScan@CSwiGobiDll@@QAAKPAE000@Z (public: unsigned long __cdecl CSwiGobiDll::PerformNetworkRATScan(unsigned char *,unsigned char *,unsigned char *,unsigned char *))
      134    ?PerformNetworkScan@CSwiGobiDll@@QAAKPAE0@Z (public: unsigned long __cdecl CSwiGobiDll::PerformNetworkScan(unsigned char *,unsigned char *))
      135    ?PlayAudioTone@CSwiGobiDll@@QAAKPAE@Z (public: unsigned long __cdecl CSwiGobiDll::PlayAudioTone(unsigned char *))
      136    ?ReadPhonebookRecords@CSwiGobiDll@@QAAKPAEPAG111@Z (public: unsigned long __cdecl CSwiGobiDll::ReadPhonebookRecords(unsigned char *,unsigned short *,unsigned short *,unsigned short *,unsigned short *))
      137    ?ResetPDSData@CSwiGobiDll@@QAAKPAK0@Z (public: unsigned long __cdecl CSwiGobiDll::ResetPDSData(unsigned long *,unsigned long *))
      138    ?ResetToFactoryDefaults@CSwiGobiDll@@QAAKPAD@Z (public: unsigned long __cdecl CSwiGobiDll::ResetToFactoryDefaults(char *))
      139    ?SaveSMS@CSwiGobiDll@@QAAKKKKPAEPAK@Z (public: unsigned long __cdecl CSwiGobiDll::SaveSMS(unsigned long,unsigned long,unsigned long,unsigned char *,unsigned long *))
      140    ?SendFlash@CSwiGobiDll@@QAAKPAEPAD00@Z (public: unsigned long __cdecl CSwiGobiDll::SendFlash(unsigned char *,char *,unsigned char *,unsigned char *))
      141    ?SendSMS@CSwiGobiDll@@QAAKKKPAEEPAK@Z (public: unsigned long __cdecl CSwiGobiDll::SendSMS(unsigned long,unsigned long,unsigned char *,unsigned char,unsigned long *))
      142    ?Set3Gpp2SubscriptionInfo@CSwiGobiDll@@QAAKPAEPAUMinBasedImsi@@PAUTrueImsi@@00@Z (public: unsigned long __cdecl CSwiGobiDll::Set3Gpp2SubscriptionInfo(unsigned char *,struct MinBasedImsi *,struct TrueImsi *,unsigned char *,unsigned char *))
      143    ?SetACCOLC@CSwiGobiDll@@QAAKPADE@Z (public: unsigned long __cdecl CSwiGobiDll::SetACCOLC(char *,unsigned char))
      144    ?SetAGPSConfig@CSwiGobiDll@@QAAKKK@Z (public: unsigned long __cdecl CSwiGobiDll::SetAGPSConfig(unsigned long,unsigned long))
      145    ?SetActivationStatusCB@CSwiGobiDll@@SAKP6AXK@Z@Z (public: static unsigned long __cdecl CSwiGobiDll::SetActivationStatusCB(void (__cdecl*)(unsigned long)))
      146    ?SetActiveMobileIPProfile@CSwiGobiDll@@QAAKPADE@Z (public: unsigned long __cdecl CSwiGobiDll::SetActiveMobileIPProfile(char *,unsigned char))
      147    ?SetAllPbInitDoneCB@CSwiGobiDll@@SAKP6AXEPAEPAG@Z@Z (public: static unsigned long __cdecl CSwiGobiDll::SetAllPbInitDoneCB(void (__cdecl*)(unsigned char,unsigned char *,unsigned short *)))
      148    ?SetAudioProfile@CSwiGobiDll@@QAAKPAE@Z (public: unsigned long __cdecl CSwiGobiDll::SetAudioProfile(unsigned char *))
      149    ?SetAutoInputGain@CSwiGobiDll@@QAAKPAE@Z (public: unsigned long __cdecl CSwiGobiDll::SetAutoInputGain(unsigned char *))
      150    ?SetAutoOutputGain@CSwiGobiDll@@QAAKPAE@Z (public: unsigned long __cdecl CSwiGobiDll::SetAutoOutputGain(unsigned char *))
      151    ?SetAutoconnect@CSwiGobiDll@@QAAKK@Z (public: unsigned long __cdecl CSwiGobiDll::SetAutoconnect(unsigned long))
      152    ?SetByteTotalsCB@CSwiGobiDll@@SAKP6AX_K0@ZE@Z (public: static unsigned long __cdecl CSwiGobiDll::SetByteTotalsCB(void (__cdecl*)(unsigned __int64,unsigned __int64),unsigned char))
      153    ?SetCDMANetworkParameters@CSwiGobiDll@@QAAKPADPAE1PAK222@Z (public: unsigned long __cdecl CSwiGobiDll::SetCDMANetworkParameters(char *,unsigned char *,unsigned char *,unsigned long *,unsigned long *,unsigned long *,unsigned long *))
      154    ?SetCallInfoCB@CSwiGobiDll@@SAKP6AXPAUarrCallInfo@@PAUarrRemotePartyNum@@PAUarrRemotePartyName@@PAUarrAlertingType@@PAUarrSvcOption@@PAUarrCallEndReason@@PAUarrAlphaIDInfo@@PAUarrPeerNumInfo@@PAUarrDiagInfo@@77PAUarrAlertingPattern@@@Z@Z (public: static unsigned long __cdecl CSwiGobiDll::SetCallInfoCB(void (__cdecl*)(struct arrCallInfo *,struct arrRemotePartyNum *,struct arrRemotePartyName *,struct arrAlertingType *,struct arrSvcOption *,struct arrCallEndReason *,struct arrAlphaIDInfo *,struct arrPeerNumInfo *,struct arrDiagInfo *,struct arrPeerNumInfo *,struct arrPeerNumInfo *,struct arrAlertingPattern *)))
      155    ?SetDataBearerCB@CSwiGobiDll@@SAKP6AXK@Z@Z (public: static unsigned long __cdecl CSwiGobiDll::SetDataBearerCB(void (__cdecl*)(unsigned long)))
      156    ?SetDataCapsCB@CSwiGobiDll@@SAKP6AXEPAE@Z@Z (public: static unsigned long __cdecl CSwiGobiDll::SetDataCapsCB(void (__cdecl*)(unsigned char,unsigned char *)))
      157    ?SetDefaultProfile@CSwiGobiDll@@QAAKKPAK0000PAD111@Z (public: unsigned long __cdecl CSwiGobiDll::SetDefaultProfile(unsigned long,unsigned long *,unsigned long *,unsigned long *,unsigned long *,unsigned long *,char *,char *,char *,char *))
      158    ?SetDeviceRemovalCallback@CSwiGobiDll@@QAAKP6AXK@Z@Z (public: unsigned long __cdecl CSwiGobiDll::SetDeviceRemovalCallback(void (__cdecl*)(unsigned long)))
      159    ?SetDormancyStatusCB@CSwiGobiDll@@SAKP6AXK@Z@Z (public: static unsigned long __cdecl CSwiGobiDll::SetDormancyStatusCB(void (__cdecl*)(unsigned long)))
      160    ?SetEchoCancelMode@CSwiGobiDll@@QAAKPAE@Z (public: unsigned long __cdecl CSwiGobiDll::SetEchoCancelMode(unsigned char *))
      161    ?SetEmergencyListCB@CSwiGobiDll@@SAKP6AXEPAUemergencyNumberEntry@@@Z@Z (public: static unsigned long __cdecl CSwiGobiDll::SetEmergencyListCB(void (__cdecl*)(unsigned char,struct emergencyNumberEntry *)))
      162    ?SetEmergencyModeCB@CSwiGobiDll@@SAKP6AXPAE@Z@Z (public: static unsigned long __cdecl CSwiGobiDll::SetEmergencyModeCB(void (__cdecl*)(unsigned char *)))
      163    ?SetImagePreference@CSwiGobiDll@@QAAKKPAEKEPAK0@Z (public: unsigned long __cdecl CSwiGobiDll::SetImagePreference(unsigned long,unsigned char *,unsigned long,unsigned char,unsigned long *,unsigned char *))
      164    ?SetInfoRecCB@CSwiGobiDll@@SAKP6AXPAEPAUsignalInfo@@PAUcallerIDInfo@@PAD330PAUpeerNumInfo@@44PAUredirectNumInfo@@0000PAUlineCtlInfo@@PAUextDisplayInfo@@@Z@Z (public: static unsigned long __cdecl CSwiGobiDll::SetInfoRecCB(void (__cdecl*)(unsigned char *,struct signalInfo *,struct callerIDInfo *,char *,char *,char *,unsigned char *,struct peerNumInfo *,struct peerNumInfo *,struct peerNumInfo *,struct redirectNumInfo *,unsigned char *,unsigned char *,unsigned char *,unsigned char *,struct lineCtlInfo *,struct extDisplayInfo *)))
      165    ?SetMICMuteStatus@CSwiGobiDll@@QAAKPAE@Z (public: unsigned long __cdecl CSwiGobiDll::SetMICMuteStatus(unsigned char *))
      166    ?SetMicVolume@CSwiGobiDll@@QAAKPAG@Z (public: unsigned long __cdecl CSwiGobiDll::SetMicVolume(unsigned short *))
      167    ?SetMobileIP@CSwiGobiDll@@QAAKK@Z (public: unsigned long __cdecl CSwiGobiDll::SetMobileIP(unsigned long))
      168    ?SetMobileIPParameters@CSwiGobiDll@@QAAKPADPAKPAE22222@Z (public: unsigned long __cdecl CSwiGobiDll::SetMobileIPParameters(char *,unsigned long *,unsigned char *,unsigned char *,unsigned char *,unsigned char *,unsigned char *,unsigned char *))
      169    ?SetMobileIPProfile@CSwiGobiDll@@QAAKPADEPAEPAK22102200@Z (public: unsigned long __cdecl CSwiGobiDll::SetMobileIPProfile(char *,unsigned char,unsigned char *,unsigned long *,unsigned long *,unsigned long *,unsigned char *,char *,unsigned long *,unsigned long *,char *,char *))
      170    ?SetMobileIPStatusCB@CSwiGobiDll@@SAKP6AXK@Z@Z (public: static unsigned long __cdecl CSwiGobiDll::SetMobileIPStatusCB(void (__cdecl*)(unsigned long)))
      171    ?SetNITZCB@CSwiGobiDll@@SAKP6AXGEEEEEEEE@Z@Z (public: static unsigned long __cdecl CSwiGobiDll::SetNITZCB(void (__cdecl*)(unsigned short,unsigned char,unsigned char,unsigned char,unsigned char,unsigned char,unsigned char,unsigned char,unsigned char)))
      172    ?SetNMEAConfig@CSwiGobiDll@@QAAKEEEPAG@Z (public: unsigned long __cdecl CSwiGobiDll::SetNMEAConfig(unsigned char,unsigned char,unsigned char,unsigned short *))
      173    ?SetNetworkPreference@CSwiGobiDll@@QAAKKK@Z (public: unsigned long __cdecl CSwiGobiDll::SetNetworkPreference(unsigned long,unsigned long))
      174    ?SetNewSMSCB@CSwiGobiDll@@SAKP6AXKK@Z@Z (public: static unsigned long __cdecl CSwiGobiDll::SetNewSMSCB(void (__cdecl*)(unsigned long,unsigned long)))
      175    ?SetNewSMSCBCB@CSwiGobiDll@@SAKP6AXEKEGPAE@Z@Z (public: static unsigned long __cdecl CSwiGobiDll::SetNewSMSCBCB(void (__cdecl*)(unsigned char,unsigned long,unsigned char,unsigned short,unsigned char *)))
      176    ?SetNoiseSuppression@CSwiGobiDll@@QAAKPAE@Z (public: unsigned long __cdecl CSwiGobiDll::SetNoiseSuppression(unsigned char *))
      177    ?SetOMADMAlertCB@CSwiGobiDll@@SAKP6AXKG@Z@Z (public: static unsigned long __cdecl CSwiGobiDll::SetOMADMAlertCB(void (__cdecl*)(unsigned long,unsigned short)))
      178    ?SetOMADMStateCB@CSwiGobiDll@@SAKP6AXKK@Z@Z (public: static unsigned long __cdecl CSwiGobiDll::SetOMADMStateCB(void (__cdecl*)(unsigned long,unsigned long)))
      179    ?SetOMAEXEventCB@CSwiGobiDll@@SAKP6AXPAUFUMOInfo@@PAUOMAInfo@@@Z@Z (public: static unsigned long __cdecl CSwiGobiDll::SetOMAEXEventCB(void (__cdecl*)(struct FUMOInfo *,struct OMAInfo *)))
      180    ?SetPDSDefaults@CSwiGobiDll@@QAAKKEKK@Z (public: unsigned long __cdecl CSwiGobiDll::SetPDSDefaults(unsigned long,unsigned char,unsigned long,unsigned long))
      181    ?SetPDSState@CSwiGobiDll@@QAAKK@Z (public: unsigned long __cdecl CSwiGobiDll::SetPDSState(unsigned long))
      182    ?SetPhonebookRecordReadCB@CSwiGobiDll@@SAKP6AXEGPAUarrPBInfo@@@Z@Z (public: static unsigned long __cdecl CSwiGobiDll::SetPhonebookRecordReadCB(void (__cdecl*)(unsigned char,unsigned short,struct arrPBInfo *)))
      183    ?SetPortAutomaticTracking@CSwiGobiDll@@QAAKK@Z (public: unsigned long __cdecl CSwiGobiDll::SetPortAutomaticTracking(unsigned long))
      184    ?SetPower@CSwiGobiDll@@QAAKK@Z (public: unsigned long __cdecl CSwiGobiDll::SetPower(unsigned long))
      185    ?SetPowerCB@CSwiGobiDll@@SAKP6AXK@Z@Z (public: static unsigned long __cdecl CSwiGobiDll::SetPowerCB(void (__cdecl*)(unsigned long)))
      186    ?SetRFInfoCB@CSwiGobiDll@@SAKP6AXKKK@Z@Z (public: static unsigned long __cdecl CSwiGobiDll::SetRFInfoCB(void (__cdecl*)(unsigned long,unsigned long,unsigned long)))
      187    ?SetRXGainLevel@CSwiGobiDll@@QAAKPAEPAG1@Z (public: unsigned long __cdecl CSwiGobiDll::SetRXGainLevel(unsigned char *,unsigned short *,unsigned short *))
      188    ?SetRXPCMFilter@CSwiGobiDll@@QAAKPAG0PAK0@Z (public: unsigned long __cdecl CSwiGobiDll::SetRXPCMFilter(unsigned short *,unsigned short *,unsigned long *,unsigned short *))
      189    ?SetReceiverVolume@CSwiGobiDll@@QAAKPAE@Z (public: unsigned long __cdecl CSwiGobiDll::SetReceiverVolume(unsigned char *))
      190    ?SetRoamingIndicatorCB@CSwiGobiDll@@SAKP6AXK@Z@Z (public: static unsigned long __cdecl CSwiGobiDll::SetRoamingIndicatorCB(void (__cdecl*)(unsigned long)))
      191    ?SetSMSBroadcastActivation@CSwiGobiDll@@QAAKEE@Z (public: unsigned long __cdecl CSwiGobiDll::SetSMSBroadcastActivation(unsigned char,unsigned char))
      192    ?SetSMSCAddress@CSwiGobiDll@@QAAKPAD0@Z (public: unsigned long __cdecl CSwiGobiDll::SetSMSCAddress(char *,char *))
      193    ?SetSMSProtocol@CSwiGobiDll@@QAAKE@Z (public: unsigned long __cdecl CSwiGobiDll::SetSMSProtocol(unsigned char))
      194    ?SetSMSRoute@CSwiGobiDll@@QAAKKPAE@Z (public: unsigned long __cdecl CSwiGobiDll::SetSMSRoute(unsigned long,unsigned char *))
      195    ?SetSUPS@CSwiGobiDll@@QAAKPAUvoiceSetSUPSServiceReq@@PAGPAUalphaIDInfo@@PAE3PAUccSUPSType@@@Z (public: unsigned long __cdecl CSwiGobiDll::SetSUPS(struct voiceSetSUPSServiceReq *,unsigned short *,struct alphaIDInfo *,unsigned char *,unsigned char *,struct ccSUPSType *))
      196    ?SetServiceAutomaticTracking@CSwiGobiDll@@QAAKK@Z (public: unsigned long __cdecl CSwiGobiDll::SetServiceAutomaticTracking(unsigned long))
      197    ?SetSessionStateCB@CSwiGobiDll@@SAKP6AXKK@Z@Z (public: static unsigned long __cdecl CSwiGobiDll::SetSessionStateCB(void (__cdecl*)(unsigned long,unsigned long)))
      198    ?SetSideToneGain@CSwiGobiDll@@QAAKPAG@Z (public: unsigned long __cdecl CSwiGobiDll::SetSideToneGain(unsigned short *))
      199    ?SetSignalStrengthCB@CSwiGobiDll@@SAKP6AXCK@ZEPAC@Z (public: static unsigned long __cdecl CSwiGobiDll::SetSignalStrengthCB(void (__cdecl*)(signed char,unsigned long),unsigned char,signed char *))
      200    ?SetSpeakerMuteStatus@CSwiGobiDll@@QAAKPAE@Z (public: unsigned long __cdecl CSwiGobiDll::SetSpeakerMuteStatus(unsigned char *))
      201    ?SetTXPCMFilter@CSwiGobiDll@@QAAKPAG0PAK0@Z (public: unsigned long __cdecl CSwiGobiDll::SetTXPCMFilter(unsigned short *,unsigned short *,unsigned long *,unsigned short *))
      202    ?SetUSSDInfoCB@CSwiGobiDll@@SAKP6AXPAEPAUUSSInfo@@@Z@Z (public: static unsigned long __cdecl CSwiGobiDll::SetUSSDInfoCB(void (__cdecl*)(unsigned char *,struct USSInfo *)))
      203    ?SetVoiceMessageCB@CSwiGobiDll@@SAKP6AXEPAE00@Z@Z (public: static unsigned long __cdecl CSwiGobiDll::SetVoiceMessageCB(void (__cdecl*)(unsigned char,unsigned char *,unsigned char *,unsigned char *)))
      204    ?SetXTRAAutomaticDownload@CSwiGobiDll@@QAAKKG@Z (public: unsigned long __cdecl CSwiGobiDll::SetXTRAAutomaticDownload(unsigned long,unsigned short))
      205    ?SetXTRAEmbeddedClient@CSwiGobiDll@@QAAKEE@Z (public: unsigned long __cdecl CSwiGobiDll::SetXTRAEmbeddedClient(unsigned char,unsigned char))
      206    ?SetXTRANetwork@CSwiGobiDll@@QAAKK@Z (public: unsigned long __cdecl CSwiGobiDll::SetXTRANetwork(unsigned long))
      207    ?SetXTRAValidity@CSwiGobiDll@@QAAKGGG@Z (public: unsigned long __cdecl CSwiGobiDll::SetXTRAValidity(unsigned short,unsigned short,unsigned short))
      208    ?StartDTMF@CSwiGobiDll@@QAAKPAE00@Z (public: unsigned long __cdecl CSwiGobiDll::StartDTMF(unsigned char *,unsigned char *,unsigned char *))
      209    ?StartDataSession@CSwiGobiDll@@QAAKPAD00PAK1@Z (public: unsigned long __cdecl CSwiGobiDll::StartDataSession(char *,char *,char *,unsigned long *,unsigned long *))
      210    ?StopDTMF@CSwiGobiDll@@QAAKPAE0@Z (public: unsigned long __cdecl CSwiGobiDll::StopDTMF(unsigned char *,unsigned char *))
      211    ?StopDataSession@CSwiGobiDll@@QAAKK@Z (public: unsigned long __cdecl CSwiGobiDll::StopDataSession(unsigned long))
      212    ?SwiGetAudioMode@@YA?AW4SWI_RCODE@@PAGK@Z (enum SWI_RCODE __cdecl SwiGetAudioMode(unsigned short *,unsigned long))
      213    ?SwiM2MAV_AudioGetAVCFG@CSwiGobiDll@@QAAKPAUAudioConfig@@PAE@Z (public: unsigned long __cdecl CSwiGobiDll::SwiM2MAV_AudioGetAVCFG(struct AudioConfig *,unsigned char *))
      214    ?SwiM2MAV_AudioGetAVEC@CSwiGobiDll@@QAAKPAE0@Z (public: unsigned long __cdecl CSwiGobiDll::SwiM2MAV_AudioGetAVEC(unsigned char *,unsigned char *))
      215    ?SwiM2MAV_AudioGetAVMute@CSwiGobiDll@@QAAKPAE000@Z (public: unsigned long __cdecl CSwiGobiDll::SwiM2MAV_AudioGetAVMute(unsigned char *,unsigned char *,unsigned char *,unsigned char *))
      216    ?SwiM2MAV_AudioGetAVNS@CSwiGobiDll@@QAAKPAE0@Z (public: unsigned long __cdecl CSwiGobiDll::SwiM2MAV_AudioGetAVNS(unsigned char *,unsigned char *))
      217    ?SwiM2MAV_AudioGetAVRXG@CSwiGobiDll@@QAAKPAEPAG@Z (public: unsigned long __cdecl CSwiGobiDll::SwiM2MAV_AudioGetAVRXG(unsigned char *,unsigned short *))
      218    ?SwiM2MAV_AudioGetAVTXG@CSwiGobiDll@@QAAKPAEPAG@Z (public: unsigned long __cdecl CSwiGobiDll::SwiM2MAV_AudioGetAVTXG(unsigned char *,unsigned short *))
      219    ?SwiM2MAV_AudioGetMicGain@CSwiGobiDll@@QAAKPAEPAG@Z (public: unsigned long __cdecl CSwiGobiDll::SwiM2MAV_AudioGetMicGain(unsigned char *,unsigned short *))
      220    ?SwiM2MAV_AudioGetProfile@CSwiGobiDll@@QAAKPAE000000@Z (public: unsigned long __cdecl CSwiGobiDll::SwiM2MAV_AudioGetProfile(unsigned char *,unsigned char *,unsigned char *,unsigned char *,unsigned char *,unsigned char *,unsigned char *))
      221    ?SwiM2MAV_AudioGetSTG@CSwiGobiDll@@QAAKPAEPAG@Z (public: unsigned long __cdecl CSwiGobiDll::SwiM2MAV_AudioGetSTG(unsigned char *,unsigned short *))
      222    ?SwiM2MAV_AudioGetSpeakerGain@CSwiGobiDll@@QAAKPAEPAG@Z (public: unsigned long __cdecl CSwiGobiDll::SwiM2MAV_AudioGetSpeakerGain(unsigned char *,unsigned short *))
      223    ?SwiM2MAV_AudioGetTxVolume@CSwiGobiDll@@QAAKPAEPAG@Z (public: unsigned long __cdecl CSwiGobiDll::SwiM2MAV_AudioGetTxVolume(unsigned char *,unsigned short *))
      224    ?SwiM2MAV_AudioGetVolDB@CSwiGobiDll@@QAAKPAE00PAG@Z (public: unsigned long __cdecl CSwiGobiDll::SwiM2MAV_AudioGetVolDB(unsigned char *,unsigned char *,unsigned char *,unsigned short *))
      225    ?SwiM2MAV_AudioGetVolume@CSwiGobiDll@@QAAKPAE00@Z (public: unsigned long __cdecl CSwiGobiDll::SwiM2MAV_AudioGetVolume(unsigned char *,unsigned char *,unsigned char *))
      226    ?SwiM2MAV_AudioNVDef@CSwiGobiDll@@QAAKXZ (public: unsigned long __cdecl CSwiGobiDll::SwiM2MAV_AudioNVDef(void))
      227    ?SwiM2MAV_AudioPlayTone@CSwiGobiDll@@QAAKPAE0PAG@Z (public: unsigned long __cdecl CSwiGobiDll::SwiM2MAV_AudioPlayTone(unsigned char *,unsigned char *,unsigned short *))
      228    ?SwiM2MAV_AudioSetAVCFG@CSwiGobiDll@@QAAKPAE00PAUPIFACETable@@@Z (public: unsigned long __cdecl CSwiGobiDll::SwiM2MAV_AudioSetAVCFG(unsigned char *,unsigned char *,unsigned char *,struct PIFACETable *))
      229    ?SwiM2MAV_AudioSetAVEC@CSwiGobiDll@@QAAKPAE0@Z (public: unsigned long __cdecl CSwiGobiDll::SwiM2MAV_AudioSetAVEC(unsigned char *,unsigned char *))
      230    ?SwiM2MAV_AudioSetAVMute@CSwiGobiDll@@QAAKPAE000@Z (public: unsigned long __cdecl CSwiGobiDll::SwiM2MAV_AudioSetAVMute(unsigned char *,unsigned char *,unsigned char *,unsigned char *))
      231    ?SwiM2MAV_AudioSetAVNS@CSwiGobiDll@@QAAKPAE0@Z (public: unsigned long __cdecl CSwiGobiDll::SwiM2MAV_AudioSetAVNS(unsigned char *,unsigned char *))
      232    ?SwiM2MAV_AudioSetAVRXG@CSwiGobiDll@@QAAKPAEPAG@Z (public: unsigned long __cdecl CSwiGobiDll::SwiM2MAV_AudioSetAVRXG(unsigned char *,unsigned short *))
      233    ?SwiM2MAV_AudioSetAVTXG@CSwiGobiDll@@QAAKPAEPAG@Z (public: unsigned long __cdecl CSwiGobiDll::SwiM2MAV_AudioSetAVTXG(unsigned char *,unsigned short *))
      234    ?SwiM2MAV_AudioSetLPBK@CSwiGobiDll@@QAAKPAE@Z (public: unsigned long __cdecl CSwiGobiDll::SwiM2MAV_AudioSetLPBK(unsigned char *))
      235    ?SwiM2MAV_AudioSetMicGain@CSwiGobiDll@@QAAKPAEPAG@Z (public: unsigned long __cdecl CSwiGobiDll::SwiM2MAV_AudioSetMicGain(unsigned char *,unsigned short *))
      236    ?SwiM2MAV_AudioSetProfile@CSwiGobiDll@@QAAKPAE00000@Z (public: unsigned long __cdecl CSwiGobiDll::SwiM2MAV_AudioSetProfile(unsigned char *,unsigned char *,unsigned char *,unsigned char *,unsigned char *,unsigned char *))
      237    ?SwiM2MAV_AudioSetSTG@CSwiGobiDll@@QAAKPAEPAG@Z (public: unsigned long __cdecl CSwiGobiDll::SwiM2MAV_AudioSetSTG(unsigned char *,unsigned short *))
      238    ?SwiM2MAV_AudioSetSpeakerGain@CSwiGobiDll@@QAAKPAEPAG@Z (public: unsigned long __cdecl CSwiGobiDll::SwiM2MAV_AudioSetSpeakerGain(unsigned char *,unsigned short *))
      239    ?SwiM2MAV_AudioSetTxVolume@CSwiGobiDll@@QAAKPAEPAG@Z (public: unsigned long __cdecl CSwiGobiDll::SwiM2MAV_AudioSetTxVolume(unsigned char *,unsigned short *))
      240    ?SwiM2MAV_AudioSetVolDB@CSwiGobiDll@@QAAKPAE00PAG@Z (public: unsigned long __cdecl CSwiGobiDll::SwiM2MAV_AudioSetVolDB(unsigned char *,unsigned char *,unsigned char *,unsigned short *))
      241    ?SwiM2MAV_AudioSetVolume@CSwiGobiDll@@QAAKPAE00@Z (public: unsigned long __cdecl CSwiGobiDll::SwiM2MAV_AudioSetVolume(unsigned char *,unsigned char *,unsigned char *))
      242    ?SwiSetAudioMode@@YA?AW4SWI_RCODE@@GK@Z (enum SWI_RCODE __cdecl SwiSetAudioMode(unsigned short,unsigned long))
      243    ?UIMChangePIN@CSwiGobiDll@@QAAKPAUQMI_UIM_CHANGE_PIN_REQ_SESSION_INFORMATION@@PAUQMI_UIM_CHANGE_PIN_REQ_CHANGE_PIN@@PAUQMI_UIM_CHANGE_PIN_RESP_RETRIES_REMAINING@@@Z (public: unsigned long __cdecl CSwiGobiDll::UIMChangePIN(struct QMI_UIM_CHANGE_PIN_REQ_SESSION_INFORMATION *,struct QMI_UIM_CHANGE_PIN_REQ_CHANGE_PIN *,struct QMI_UIM_CHANGE_PIN_RESP_RETRIES_REMAINING *))
      244    ?UIMGetCardStatus@CSwiGobiDll@@QAAKPAHPAUQMI_UIM_GET_CARD_STATUS_RESP@@@Z (public: unsigned long __cdecl CSwiGobiDll::UIMGetCardStatus(int *,struct QMI_UIM_GET_CARD_STATUS_RESP *))
      245    ?UIMSetPINProtection@CSwiGobiDll@@QAAKPAUQMI_UIM_SET_PIN_PROTECTION_REQ_SESSION_INFORMATION@@PAUQMI_UIM_SET_PIN_PROTECTION_REQ_SET_PIN_PROTECTION@@PAUQMI_UIM_SET_PIN_PROTECTION_RESP_RETRIES_REMAINING@@@Z (public: unsigned long __cdecl CSwiGobiDll::UIMSetPINProtection(struct QMI_UIM_SET_PIN_PROTECTION_REQ_SESSION_INFORMATION *,struct QMI_UIM_SET_PIN_PROTECTION_REQ_SET_PIN_PROTECTION *,struct QMI_UIM_SET_PIN_PROTECTION_RESP_RETRIES_REMAINING *))
      246    ?UIMUnblockPIN@CSwiGobiDll@@QAAKPAUQMI_UIM_UNBLOCK_PIN_REQ_SESSION_INFORMATION@@PAUQMI_UIM_UNBLOCK_PIN_REQ_UNBLOCK_PIN@@PAUQMI_UIM_UNBLOCK_PIN_RESP_RETRIES_REMAINING@@@Z (public: unsigned long __cdecl CSwiGobiDll::UIMUnblockPIN(struct QMI_UIM_UNBLOCK_PIN_REQ_SESSION_INFORMATION *,struct QMI_UIM_UNBLOCK_PIN_REQ_UNBLOCK_PIN *,struct QMI_UIM_UNBLOCK_PIN_RESP_RETRIES_REMAINING *))
      247    ?UIMVerifyPIN@CSwiGobiDll@@QAAKPAUQMI_UIM_VERIFY_PIN_REQ_SESSION_INFORMATION@@PAUQMI_UIM_VERIFY_PIN_REQ_VERIFY_PIN@@PAUQMI_UIM_VERIFY_PIN_RESP_RETRIES_REMAINING@@@Z (public: unsigned long __cdecl CSwiGobiDll::UIMVerifyPIN(struct QMI_UIM_VERIFY_PIN_REQ_SESSION_INFORMATION *,struct QMI_UIM_VERIFY_PIN_REQ_VERIFY_PIN *,struct QMI_UIM_VERIFY_PIN_RESP_RETRIES_REMAINING *))
      248    ?UpgradeFirmwareW@CSwiGobiDll@@QAAKPAG@Z (public: unsigned long __cdecl CSwiGobiDll::UpgradeFirmwareW(unsigned short *))
      249    ?ValidateSPC@CSwiGobiDll@@QAAKPAD@Z (public: unsigned long __cdecl CSwiGobiDll::ValidateSPC(char *))
      250    ?WritePhonebookRecord@CSwiGobiDll@@QAAKPAEPAG1000000@Z (public: unsigned long __cdecl CSwiGobiDll::WritePhonebookRecord(unsigned char *,unsigned short *,unsigned short *,unsigned char *,unsigned char *,unsigned char *,unsigned char *,unsigned char *,unsigned char *))
      251    ?mpFNSetActivationStatusCB@CSwiGobiDll@@1P6AKP6AXK@Z@ZA (protected: static unsigned long (__cdecl* CSwiGobiDll::mpFNSetActivationStatusCB)(void (__cdecl*)(unsigned long)))
      252    ?mpFNSetAllPbInitDoneCB@CSwiGobiDll@@1P6AKP6AXEPAEPAG@Z@ZA (protected: static unsigned long (__cdecl* CSwiGobiDll::mpFNSetAllPbInitDoneCB)(void (__cdecl*)(unsigned char,unsigned char *,unsigned short *)))
      253    ?mpFNSetByteTotalsCB@CSwiGobiDll@@1P6AKP6AX_K0@ZE@ZA (protected: static unsigned long (__cdecl* CSwiGobiDll::mpFNSetByteTotalsCB)(void (__cdecl*)(unsigned __int64,unsigned __int64),unsigned char))
      254    ?mpFNSetCallInfoCB@CSwiGobiDll@@1P6AKP6AXPAUarrCallInfo@@PAUarrRemotePartyNum@@PAUarrRemotePartyName@@PAUarrAlertingType@@PAUarrSvcOption@@PAUarrCallEndReason@@PAUarrAlphaIDInfo@@PAUarrPeerNumInfo@@PAUarrDiagInfo@@77PAUarrAlertingPattern@@@Z@ZA (protected: static unsigned long (__cdecl* CSwiGobiDll::mpFNSetCallInfoCB)(void (__cdecl*)(struct arrCallInfo *,struct arrRemotePartyNum *,struct arrRemotePartyName *,struct arrAlertingType *,struct arrSvcOption *,struct arrCallEndReason *,struct arrAlphaIDInfo *,struct arrPeerNumInfo *,struct arrDiagInfo *,struct arrPeerNumInfo *,struct arrPeerNumInfo *,struct arrAlertingPattern *)))
      255    ?mpFNSetDataBearerCB@CSwiGobiDll@@1P6AKP6AXK@Z@ZA (protected: static unsigned long (__cdecl* CSwiGobiDll::mpFNSetDataBearerCB)(void (__cdecl*)(unsigned long)))
      256    ?mpFNSetDataCapabilitiesCB@CSwiGobiDll@@1P6AKP6AXEPAE@Z@ZA (protected: static unsigned long (__cdecl* CSwiGobiDll::mpFNSetDataCapabilitiesCB)(void (__cdecl*)(unsigned char,unsigned char *)))
      257    ?mpFNSetDormancyStatusCB@CSwiGobiDll@@1P6AKP6AXK@Z@ZA (protected: static unsigned long (__cdecl* CSwiGobiDll::mpFNSetDormancyStatusCB)(void (__cdecl*)(unsigned long)))
      258    ?mpFNSetEmergencyListCB@CSwiGobiDll@@1P6AKP6AXEPAUemergencyNumberEntry@@@Z@ZA (protected: static unsigned long (__cdecl* CSwiGobiDll::mpFNSetEmergencyListCB)(void (__cdecl*)(unsigned char,struct emergencyNumberEntry *)))
      259    ?mpFNSetEmergencyModeCB@CSwiGobiDll@@1P6AKP6AXPAE@Z@ZA (protected: static unsigned long (__cdecl* CSwiGobiDll::mpFNSetEmergencyModeCB)(void (__cdecl*)(unsigned char *)))
      260    ?mpFNSetInfoRecCB@CSwiGobiDll@@1P6AKP6AXPAEPAUsignalInfo@@PAUcallerIDInfo@@PAD330PAUpeerNumInfo@@44PAUredirectNumInfo@@0000PAUlineCtlInfo@@PAUextDisplayInfo@@@Z@ZA (protected: static unsigned long (__cdecl* CSwiGobiDll::mpFNSetInfoRecCB)(void (__cdecl*)(unsigned char *,struct signalInfo *,struct callerIDInfo *,char *,char *,char *,unsigned char *,struct peerNumInfo *,struct peerNumInfo *,struct peerNumInfo *,struct redirectNumInfo *,unsigned char *,unsigned char *,unsigned char *,unsigned char *,struct lineCtlInfo *,struct extDisplayInfo *)))
      261    ?mpFNSetMobileIPStatusCB@CSwiGobiDll@@1P6AKP6AXK@Z@ZA (protected: static unsigned long (__cdecl* CSwiGobiDll::mpFNSetMobileIPStatusCB)(void (__cdecl*)(unsigned long)))
      262    ?mpFNSetNITZCB@CSwiGobiDll@@1P6AKP6AXGEEEEEEEE@Z@ZA (protected: static unsigned long (__cdecl* CSwiGobiDll::mpFNSetNITZCB)(void (__cdecl*)(unsigned short,unsigned char,unsigned char,unsigned char,unsigned char,unsigned char,unsigned char,unsigned char,unsigned char)))
      263    ?mpFNSetNewSMSCB@CSwiGobiDll@@1P6AKP6AXKK@Z@ZA (protected: static unsigned long (__cdecl* CSwiGobiDll::mpFNSetNewSMSCB)(void (__cdecl*)(unsigned long,unsigned long)))
      264    ?mpFNSetNewSMSCBCB@CSwiGobiDll@@1P6AKP6AXEKEGPAE@Z@ZA (protected: static unsigned long (__cdecl* CSwiGobiDll::mpFNSetNewSMSCBCB)(void (__cdecl*)(unsigned char,unsigned long,unsigned char,unsigned short,unsigned char *)))
      265    ?mpFNSetOMADMNIAlertCB@CSwiGobiDll@@1P6AKP6AXKG@Z@ZA (protected: static unsigned long (__cdecl* CSwiGobiDll::mpFNSetOMADMNIAlertCB)(void (__cdecl*)(unsigned long,unsigned short)))
      266    ?mpFNSetOMADMStateCB@CSwiGobiDll@@1P6AKP6AXKK@Z@ZA (protected: static unsigned long (__cdecl* CSwiGobiDll::mpFNSetOMADMStateCB)(void (__cdecl*)(unsigned long,unsigned long)))
      267    ?mpFNSetOMAEXEventCB@CSwiGobiDll@@1P6AKP6AXPAUFUMOInfo@@PAUOMAInfo@@@Z@ZA (protected: static unsigned long (__cdecl* CSwiGobiDll::mpFNSetOMAEXEventCB)(void (__cdecl*)(struct FUMOInfo *,struct OMAInfo *)))
      268    ?mpFNSetPhonebookRecordReadCB@CSwiGobiDll@@1P6AKP6AXEGPAUarrPBInfo@@@Z@ZA (protected: static unsigned long (__cdecl* CSwiGobiDll::mpFNSetPhonebookRecordReadCB)(void (__cdecl*)(unsigned char,unsigned short,struct arrPBInfo *)))
      269    ?mpFNSetPowerCB@CSwiGobiDll@@1P6AKP6AXK@Z@ZA (protected: static unsigned long (__cdecl* CSwiGobiDll::mpFNSetPowerCB)(void (__cdecl*)(unsigned long)))
      270    ?mpFNSetRFInfoCB@CSwiGobiDll@@1P6AKP6AXKKK@Z@ZA (protected: static unsigned long (__cdecl* CSwiGobiDll::mpFNSetRFInfoCB)(void (__cdecl*)(unsigned long,unsigned long,unsigned long)))
      271    ?mpFNSetRoamingIndicatorCB@CSwiGobiDll@@1P6AKP6AXK@Z@ZA (protected: static unsigned long (__cdecl* CSwiGobiDll::mpFNSetRoamingIndicatorCB)(void (__cdecl*)(unsigned long)))
      272    ?mpFNSetSessionStateCB@CSwiGobiDll@@1P6AKP6AXKK@Z@ZA (protected: static unsigned long (__cdecl* CSwiGobiDll::mpFNSetSessionStateCB)(void (__cdecl*)(unsigned long,unsigned long)))
      273    ?mpFNSetSignalStrengthCB@CSwiGobiDll@@1P6AKP6AXCK@ZEPAC@ZA (protected: static unsigned long (__cdecl* CSwiGobiDll::mpFNSetSignalStrengthCB)(void (__cdecl*)(signed char,unsigned long),unsigned char,signed char *))
      274    ?mpFNSetUSSDInfoCB@CSwiGobiDll@@1P6AKP6AXPAEPAUUSSInfo@@@Z@ZA (protected: static unsigned long (__cdecl* CSwiGobiDll::mpFNSetUSSDInfoCB)(void (__cdecl*)(unsigned char *,struct USSInfo *)))
      275    ?mpFNSetVoiceMsgCB@CSwiGobiDll@@1P6AKP6AXEPAE00@Z@ZA (protected: static unsigned long (__cdecl* CSwiGobiDll::mpFNSetVoiceMsgCB)(void (__cdecl*)(unsigned char,unsigned char *,unsigned char *,unsigned char *)))
      276    SwiATGetCLIP
      277    SwiATGetCLIR
      278    SwiATGetCOLP
      279    SwiATGetCOLR
      280    SwiATGetProvisionStatus
      281    SwiATReleaseCall
      282    SwiATReset
      283    SwiATRtnReset
      284    SwiATSetCLIP
      285    SwiATSetCLIR
      286    SwiATSetCOLP
      287    SwiATSetCOLR
      288    SwiATSetEnum
      289    SwiATSetSideToneGain
      290    SwiActivateAutomatic
      291    SwiActivateProfile
      292    SwiAddPreferredOperatorGobi
      293    SwiAnserCall
      294    SwiApiShutdown
      295    SwiApiStartup
      296    SwiCancelOMADMSession
      297    SwiDeRegisterCallback
      298    SwiDialCall
      299    SwiEndCall
      300    SwiGetActivationStatus
      301    SwiGetActiveNam
      302    SwiGetAirServerInfo
      303    SwiGetAvailAirServers
      304    SwiGetBootVersion
      305    SwiGetByteCounter
      306    SwiGetCDMANetworkParameters
      307    SwiGetCallConnectionState
      308    SwiGetCarrierID
      309    SwiGetCdmaIMSI
      310    SwiGetCdmaSMSMessageStatus
      311    SwiGetChannelNumber
      312    SwiGetCurrentBaseStation
      313    SwiGetECIO
      314    SwiGetEFile
      315    SwiGetEFileInfo
      316    SwiGetESN
      317    SwiGetESNGobi
      318    SwiGetFirmwareVersion
      319    SwiGetGeneralFeatureSupport
      320    SwiGetGsmIMSI
      321    SwiGetGsmProfileBasic
      322    SwiGetGsmProfileSummary
      323    SwiGetGsmSMSCAddr
      324    SwiGetGsmSystemStatus
      325    SwiGetHardwareVersion
      326    SwiGetHdrHybrPref
      327    SwiGetHdrRoamStatus
      328    SwiGetHdrSrvState
      329    SwiGetIOTADisable
      330    SwiGetIPAddress
      331    SwiGetIPConfigurationGobi
      332    SwiGetImagePreference
      333    SwiGetImei
      334    SwiGetMEIDESN
      335    SwiGetMipErrCode
      336    SwiGetMobileIPProfile
      337    SwiGetModelID
      338    SwiGetNDISMode
      339    SwiGetNetworkProviderID
      340    SwiGetOMADMConfig
      341    SwiGetOMADMNIAlert
      342    SwiGetOMADMSessionState
      343    SwiGetPLMNMode
      344    SwiGetPLMNSelection
      345    SwiGetPRLVersion
      346    SwiGetPhoneNumber
      347    SwiGetPhonebookEntry
      348    SwiGetPinStatus
      349    SwiGetPktSessionStatus
      350    SwiGetPktSessionStatusEx
      351    SwiGetPower
      352    SwiGetPreferredOperatorListGobi
      353    SwiGetPriInfo
      354    SwiGetPriVersion
      355    SwiGetProfile
      356    SwiGetProfileSummary
      357    SwiGetRadioPower
      358    SwiGetRoamingStatus
      359    SwiGetRssi
      360    SwiGetRssiEcio
      361    SwiGetSIMRecordStatus
      362    SwiGetSMSMessageStatus
      363    SwiGetServiceIndication
      364    SwiGetServingNetworkGobi
      365    SwiGetSimLock
      366    SwiGetSimLockGobi
      367    SwiGetSimVerifyGobi
      368    SwiGetSystemTime
      369    SwiGetTechBandClass
      370    SwiGetTechHardwareVersion
      371    SwiGetTechNID
      372    SwiGetTechPowersaveMode
      373    SwiGetTechSID
      374    SwiGetTrafficStatistics
      375    SwiHandleResume
      376    SwiHandleSuspend
      377    SwiIsModemReady
      378    SwiManageCalls
      379    SwiModemReset
      380    SwiNotify
      381    SwiOMAEXGetSessionInfo
      382    SwiOMAEXGetSettings
      383    SwiOMAEXInit
      384    SwiOMAEXSelection
      385    SwiOMAEXSessionCancel
      386    SwiOMAEXSessionStart
      387    SwiOMAEXSetSettings
      388    SwiOMAEXShutdown
      389    SwiPowerSaveExit
      390    SwiPriGetActivationMask
      391    SwiPriGetMDNLength
      392    SwiPriGetMaxMosmsLen
      393    SwiPstGetAccolc
      394    SwiPstGetDisplayBannerName
      395    SwiPstGetDsMipActiveProf
      396    SwiPstGetDsMipEnableProf
      397    SwiPstGetDsMipGenUser
      398    SwiPstGetDsMipSsUserProf
      399    SwiPstGetDsQcMip
      400    SwiPstGetHdrPassword
      401    SwiPstGetHdrUserId
      402    SwiPstGetHomeSidNid
      403    SwiPstGetImsi1112
      404    SwiPstGetImsiMcc
      405    SwiPstGetPrefMode
      406    SwiPstGetSci
      407    SwiPstGetSystemPref
      408    SwiPstGetTermHome
      409    SwiPstGetTermNid
      410    SwiPstGetTermSid
      411    SwiPstLock
      412    SwiPstSetAccolc
      413    SwiPstSetCurrentNam
      414    SwiPstSetDsMipActiveProf
      415    SwiPstSetDsMipGenUser
      416    SwiPstSetDsMipSsUserProf
      417    SwiPstSetDsQcMip
      418    SwiPstSetHdrPassword
      419    SwiPstSetHdrUserId
      420    SwiPstSetHomeSidNid
      421    SwiPstSetImsi1112
      422    SwiPstSetImsiMcc
      423    SwiPstSetPrefMode
      424    SwiPstSetSci
      425    SwiPstUnlock
      426    SwiRegisterCallback
      427    SwiRemovePreferredOperatorGobi
      428    SwiResetByteCounter
      429    SwiResetModem
      430    SwiRetrieveCBSMSMessageGobi
      431    SwiRetrieveCdmaSMSMessage
      432    SwiRetrieveSMSMessageGobi
      433    SwiRtnReset
      434    SwiSelectAirServer
      435    SwiSendCdmaSMS
      436    SwiSendGenericSimCommand
      437    SwiSendRestrictedSIMCmd
      438    SwiSendSMS
      439    SwiSetAKey
      440    SwiSetCallDisconnectCmd
      441    SwiSetCallOriginateCmd
      442    SwiSetDormant
      443    SwiSetGsmProfileBasic
      444    SwiSetGsmSMSCAddr
      445    SwiSetHdrHybrPref
      446    SwiSetHostStartup
      447    SwiSetIMSI
      448    SwiSetImagePreference
      449    SwiSetMobileDirNum
      450    SwiSetMobileIPProfile
      451    SwiSetNDISPrefMode
      452    SwiSetNetworkPreferenceGobi
      453    SwiSetOMADMConfig
      454    SwiSetOMADMNIAlertResponse
      455    SwiSetOMAEXEventReport
      456    SwiSetPLMNMode
      457    SwiSetPower
      458    SwiSetPowerDown
      459    SwiSetProfile
      460    SwiSetRadioPower
      461    SwiSetSimLock
      462    SwiSetSimLockGobi
      463    SwiSetSimPassword
      464    SwiSetSimPasswordGobi
      465    SwiSetSimVerifyGobi
      466    SwiSetTempModePref
      467    SwiStartDataSession
      468    SwiStartOMADMSession
      469    SwiStartPLMNSearch
      470    SwiStopDataSession
      471    SwiStopNotify
      472    SwiStoreCdmaSMSMessage
      473    SwiStoreSMSMessageGobi
      474    SwiUpgradeFirmware
